 fontmanager

 Timestamp is 68fa9000 (Thu Oct 23 20:28:48 2025)

 Preferred load address is 10000000

 Start         Length     Name                   Class
 0001:00000000 00070055H .text$mn                CODE
 0002:00000000 000001d4H .idata$5                DATA
 0002:000001d4 00000008H .00cfg                  DATA
 0002:000001dc 00000004H .CRT$XCA                DATA
 0002:000001e0 00000004H .CRT$XCZ                DATA
 0002:000001e4 00000004H .CRT$XIA                DATA
 0002:000001e8 00000004H .CRT$XIZ                DATA
 0002:000001ec 00000004H .CRT$XPA                DATA
 0002:000001f0 00000004H .CRT$XPZ                DATA
 0002:000001f4 00000004H .CRT$XTA                DATA
 0002:000001f8 00000008H .CRT$XTZ                DATA
 0002:000001fc 00000000H .gfids$y                DATA
 0002:00000200 000295c0H .rdata                  DATA
 0002:000297c0 00000000H .rdata$CastGuardVftablesA DATA
 0002:000297c0 00000000H .rdata$CastGuardVftablesC DATA
 0002:000297c0 000011b8H .rdata$r                DATA
 0002:0002a978 00000004H .rdata$sxdata           DATA
 0002:0002a97c 000002d4H .rdata$voltmd           DATA
 0002:0002ac50 0000032cH .rdata$zzzdbg           DATA
 0002:0002af7c 00000004H .rtc$IAA                DATA
 0002:0002af80 00000004H .rtc$IZZ                DATA
 0002:0002af84 00000004H .rtc$TAA                DATA
 0002:0002af88 00000008H .rtc$TZZ                DATA
 0002:0002af90 00000120H .xdata$x                DATA
 0002:0002b0b0 00000930H .edata                  DATA
 0002:0002b9e0 0000012cH .idata$2                DATA
 0002:0002bb0c 00000014H .idata$3                DATA
 0002:0002bb20 000001d4H .idata$4                DATA
 0002:0002bcf4 000008beH .idata$6                DATA
 0003:00000000 00000234H .data                   DATA
 0003:00000234 00000060H .data$r                 DATA
 0003:00000294 000007ecH .data$rs                DATA
 0003:00000a80 00000b0cH .bss                    DATA
 0004:00000000 00000060H .rsrc$01                DATA
 0004:00000060 00000348H .rsrc$02                DATA

  Address         Publics by Value              Rva+Base       Lib:Object

 0000:00000000       ___AbsoluteZero            00000000     <absolute>
 0000:00000000       ___arm64x_extra_rfe_table  00000000     <absolute>
 0000:00000000       ___arm64x_extra_rfe_table_size 00000000     <absolute>
 0000:00000000       ___arm64x_native_entrypoint 00000000     <absolute>
 0000:00000000       ___arm64x_redirection_metadata 00000000     <absolute>
 0000:00000000       ___arm64x_redirection_metadata_count 00000000     <absolute>
 0000:00000000       ___dynamic_value_reloc_table 00000000     <absolute>
 0000:00000000       ___enclave_config          00000000     <absolute>
 0000:00000000       ___guard_check_icall_a64n_fptr 00000000     <absolute>
 0000:00000000       ___guard_eh_cont_count     00000000     <absolute>
 0000:00000000       ___guard_eh_cont_table     00000000     <absolute>
 0000:00000000       ___guard_fids_count        00000000     <absolute>
 0000:00000000       ___guard_fids_table        00000000     <absolute>
 0000:00000000       ___guard_iat_count         00000000     <absolute>
 0000:00000000       ___guard_iat_table         00000000     <absolute>
 0000:00000000       ___guard_longjmp_count     00000000     <absolute>
 0000:00000000       ___guard_longjmp_table     00000000     <absolute>
 0000:00000000       ___hybrid_auxiliary_delayload_iat 00000000     <absolute>
 0000:00000000       ___hybrid_auxiliary_delayload_iat_copy 00000000     <absolute>
 0000:00000000       ___hybrid_auxiliary_iat    00000000     <absolute>
 0000:00000000       ___hybrid_auxiliary_iat_copy 00000000     <absolute>
 0000:00000000       ___hybrid_code_map         00000000     <absolute>
 0000:00000000       ___hybrid_code_map_count   00000000     <absolute>
 0000:00000000       ___hybrid_image_info_bitfield 00000000     <absolute>
 0000:00000000       ___x64_code_ranges_to_entry_points 00000000     <absolute>
 0000:00000000       ___x64_code_ranges_to_entry_points_count 00000000     <absolute>
 0000:00000001       ___safe_se_handler_count   00000001     <absolute>
 0000:00000100       ___guard_flags             00000100     <absolute>
 0000:00000000       ___ImageBase               10000000     <linker-defined>
 0001:00000000       ??0?$LEReferenceTo@ULookupSubtable@@@@QAE@ABVLETableReference@@AAW4LEErrorCode@@PBX@Z 10001000 f i AlternateSubstSubtables.obj
 0001:000000e0       ??0?$LEReferenceToArrayOf@F@@QAE@ABVLETableReference@@AAW4LEErrorCode@@PBFK@Z 100010e0 f i ContextualGlyphSubstProc2.obj
 0001:000000e0       ??0?$LEReferenceToArrayOf@G@@QAE@ABVLETableReference@@AAW4LEErrorCode@@PBGK@Z 100010e0 f i AlternateSubstSubtables.obj
 0001:00000200       ?getGlyphCoverage@LookupSubtable@@QBEJABVLETableReference@@KAAW4LEErrorCode@@@Z 10001200 f i AlternateSubstSubtables.obj
 0001:00000300       ?isEmpty@LETableReference@@QBEDXZ 10001300 f i AlternateSubstSubtables.obj
 0001:00000320       ?isValid@LETableReference@@QBEDXZ 10001320 f i AlternateSubstSubtables.obj
 0001:00000340       ?process@AlternateSubstitutionSubtable@@QBEKABV?$LEReferenceTo@UAlternateSubstitutionSubtable@@@@PAVGlyphIterator@@AAW4LEErrorCode@@PBVLEGlyphFilter@@@Z 10001340 f   AlternateSubstSubtables.obj
 0001:00000650       ??0?$LEReferenceTo@UDeviceTable@@@@QAE@ABVLETableReference@@AAW4LEErrorCode@@I@Z 10001650 f i AnchorTables.obj
 0001:00000720       ??0?$LEReferenceTo@UClassDefFormat1Table@@@@QAE@ABVLETableReference@@AAW4LEErrorCode@@@Z 10001720 f i ClassDefinitionTables.obj
 0001:00000720       ??0?$LEReferenceTo@UFormat1AnchorTable@@@@QAE@ABVLETableReference@@AAW4LEErrorCode@@@Z 10001720 f i AnchorTables.obj
 0001:000007c0       ?getAnchor@AnchorTable@@QBEXABVLETableReference@@KPBVLEFontInstance@@AAULEPoint@@AAW4LEErrorCode@@@Z 100017c0 f   AnchorTables.obj
 0001:00000c80       ?getAnchor@Format1AnchorTable@@QBEXABV?$LEReferenceTo@UFormat1AnchorTable@@@@PBVLEFontInstance@@AAULEPoint@@AAW4LEErrorCode@@@Z 10001c80 f   AnchorTables.obj
 0001:00000ce0       ??0ArabicOpenTypeLayoutEngine@@QAE@PBVLEFontInstance@@JJJABV?$LEReferenceTo@UGlyphSubstitutionTableHeader@@@@AAW4LEErrorCode@@@Z 10001ce0 f   ArabicLayoutEngine.obj
 0001:00000d20       ??0UnicodeArabicOpenTypeLayoutEngine@@QAE@PBVLEFontInstance@@JJJAAW4LEErrorCode@@@Z 10001d20 f   ArabicLayoutEngine.obj
 0001:00000db0       ??_EArabicOpenTypeLayoutEngine@@UAEPAXI@Z 10001db0 f i ArabicLayoutEngine.obj
 0001:00000db0       ??_EUnicodeArabicOpenTypeLayoutEngine@@UAEPAXI@Z 10001db0 f i ArabicLayoutEngine.obj
 0001:00000db0       ??_GArabicOpenTypeLayoutEngine@@UAEPAXI@Z 10001db0 f i ArabicLayoutEngine.obj
 0001:00000db0       ??_GUnicodeArabicOpenTypeLayoutEngine@@UAEPAXI@Z 10001db0 f i ArabicLayoutEngine.obj
 0001:00000de0       ?accept@CharSubstitutionFilter@@UBEDKAAW4LEErrorCode@@@Z 10001de0 f   ArabicLayoutEngine.obj
 0001:00000e00       ?adjustGlyphPositions@ArabicOpenTypeLayoutEngine@@MAEXQBGJJDAAVLEGlyphStorage@@AAW4LEErrorCode@@@Z 10001e00 f   ArabicLayoutEngine.obj
 0001:00000f20       ?adjustGlyphPositions@UnicodeArabicOpenTypeLayoutEngine@@MAEXQBGJJDAAVLEGlyphStorage@@AAW4LEErrorCode@@@Z 10001f20 f   ArabicLayoutEngine.obj
 0001:00000fa0       ?characterProcessing@ArabicOpenTypeLayoutEngine@@MAEJQBGJJJDAAPAGAAVLEGlyphStorage@@AAW4LEErrorCode@@@Z 10001fa0 f   ArabicLayoutEngine.obj
 0001:000010c0       ?getDynamicClassID@ArabicOpenTypeLayoutEngine@@UBEPBDXZ 100020c0 f   ArabicLayoutEngine.obj
 0001:000010d0       ?getFontTable@LayoutEngine@@MBEPBXK@Z 100020d0 f i ArabicLayoutEngine.obj
 0001:000010f0       ?glyphPostProcessing@UnicodeArabicOpenTypeLayoutEngine@@MAEJAAVLEGlyphStorage@@0AAW4LEErrorCode@@@Z 100020f0 f   ArabicLayoutEngine.obj
 0001:00001190       ?mapCharsToGlyphs@UnicodeArabicOpenTypeLayoutEngine@@MAEXQBGJJDDAAVLEGlyphStorage@@AAW4LEErrorCode@@@Z 10002190 f   ArabicLayoutEngine.obj
 0001:00001220       ?getFeatureMap@ArabicShaping@@SAPBUFeatureMap@@AAJ@Z 10002220 f   ArabicShaping.obj
 0001:00001230       ?shape@ArabicShaping@@SAXPBGJJJDAAVLEGlyphStorage@@@Z 10002230 f   ArabicShaping.obj
 0001:00001580       ?reorderMarks@CanonShaping@@SAXPBGJDPAGAAVLEGlyphStorage@@@Z 10002580 f   CanonShaping.obj
 0001:00001760       ??0?$LEReferenceTo@UClassDefFormat2Table@@@@QAE@ABVLETableReference@@AAW4LEErrorCode@@@Z 10002760 f i ClassDefinitionTables.obj
 0001:00001800       ??0?$LEReferenceTo@UClassDefinitionTable@@@@QAE@ABVLETableReference@@AAW4LEErrorCode@@@Z 10002800 f i ClassDefinitionTables.obj
 0001:000018a0       ??0?$LEReferenceToArrayOf@UFeatureRecord@@@@QAE@ABVLETableReference@@AAW4LEErrorCode@@PBUFeatureRecord@@K@Z 100028a0 f i Features.obj
 0001:000018a0       ??0?$LEReferenceToArrayOf@UGlyphRangeRecord@@@@QAE@ABVLETableReference@@AAW4LEErrorCode@@PBUGlyphRangeRecord@@K@Z 100028a0 f i ClassDefinitionTables.obj
 0001:000018a0       ??0?$LEReferenceToArrayOf@UTagAndOffsetRecord@@@@QAE@ABVLETableReference@@AAW4LEErrorCode@@PBUTagAndOffsetRecord@@K@Z 100028a0 f i ScriptAndLanguage.obj
 0001:000019d0       ??R?$LEReferenceToArrayOf@G@@QBEABGKAAW4LEErrorCode@@@Z 100029d0 f i ClassDefinitionTables.obj
 0001:00001a00       ?getGlyphClass@ClassDefinitionTable@@QBEJABVLETableReference@@KAAW4LEErrorCode@@@Z 10002a00 f   ClassDefinitionTables.obj
 0001:00001b70       ?hasGlyphClass@ClassDefinitionTable@@QBEDABVLETableReference@@JAAW4LEErrorCode@@@Z 10002b70 f   ClassDefinitionTables.obj
 0001:00001da0       ??0?$LEReferenceToArrayOf@G@@QAE@ABVLETableReference@@AAW4LEErrorCode@@IK@Z 10002da0 f i ContextualGlyphInsertionProc2.obj
 0001:00001e90       ??0ContextualGlyphInsertionProcessor2@@QAE@ABV?$LEReferenceTo@UMorphSubtableHeader2@@@@AAW4LEErrorCode@@@Z 10002e90 f   ContextualGlyphInsertionProc2.obj
 0001:000021c0       ??_EContextualGlyphInsertionProcessor2@@UAEPAXI@Z 100031c0 f i ContextualGlyphInsertionProc2.obj
 0001:000021c0       ??_GContextualGlyphInsertionProcessor2@@UAEPAXI@Z 100031c0 f i ContextualGlyphInsertionProc2.obj
 0001:00002210       ?beginStateTable@ContextualGlyphInsertionProcessor2@@UAEXXZ 10003210 f   ContextualGlyphInsertionProc2.obj
 0001:00002220       ?endStateTable@ContextualGlyphInsertionProcessor2@@UAEXXZ 10003220 f   ContextualGlyphInsertionProc2.obj
 0001:00002220       ?endStateTable@ContextualGlyphSubstitutionProcessor2@@UAEXXZ 10003220 f   ContextualGlyphSubstProc2.obj
 0001:00002220       ?endStateTable@ContextualGlyphSubstitutionProcessor@@UAEXXZ 10003220 f   ContextualGlyphSubstProc.obj
 0001:00002220       ?endStateTable@IndicRearrangementProcessor2@@UAEXXZ 10003220 f   IndicRearrangementProcessor2.obj
 0001:00002220       ?endStateTable@IndicRearrangementProcessor@@UAEXXZ 10003220 f   IndicRearrangementProcessor.obj
 0001:00002220       ?endStateTable@LigatureSubstitutionProcessor2@@UAEXXZ 10003220 f   LigatureSubstProc2.obj
 0001:00002220       ?endStateTable@LigatureSubstitutionProcessor@@UAEXXZ 10003220 f   LigatureSubstProc.obj
 0001:00002220       @_guard_check_icall_nop@4  10003220 f   MSVCRT:guard_support.obj
 0001:00002230       ?getDynamicClassID@ContextualGlyphInsertionProcessor2@@UBEPBDXZ 10003230 f   ContextualGlyphInsertionProc2.obj
 0001:00002240       ?processStateEntry@ContextualGlyphInsertionProcessor2@@UAEGAAVLEGlyphStorage@@AAJGAAW4LEErrorCode@@@Z 10003240 f   ContextualGlyphInsertionProc2.obj
 0001:00002440       ?swapLong@LESwaps@@SAKK@Z  10003440 f i ContextualGlyphInsertionProc2.obj
 0001:00002460       ??0ContextualGlyphSubstitutionProcessor@@QAE@ABV?$LEReferenceTo@UMorphSubtableHeader@@@@AAW4LEErrorCode@@@Z 10003460 f   ContextualGlyphSubstProc.obj
 0001:000027c0       ??_EContextualGlyphSubstitutionProcessor@@UAEPAXI@Z 100037c0 f i ContextualGlyphSubstProc.obj
 0001:000027c0       ??_GContextualGlyphSubstitutionProcessor@@UAEPAXI@Z 100037c0 f i ContextualGlyphSubstProc.obj
 0001:00002810       ?beginStateTable@ContextualGlyphSubstitutionProcessor@@UAEXXZ 10003810 f   ContextualGlyphSubstProc.obj
 0001:00002820       ?getDynamicClassID@ContextualGlyphSubstitutionProcessor@@UBEPBDXZ 10003820 f   ContextualGlyphSubstProc.obj
 0001:00002830       ?processStateEntry@ContextualGlyphSubstitutionProcessor@@UAEFAAVLEGlyphStorage@@AAJEAAW4LEErrorCode@@@Z 10003830 f   ContextualGlyphSubstProc.obj
 0001:00002a00       ??0ContextualGlyphSubstitutionProcessor2@@QAE@ABV?$LEReferenceTo@UMorphSubtableHeader2@@@@AAW4LEErrorCode@@@Z 10003a00 f   ContextualGlyphSubstProc2.obj
 0001:00002d20       ??_EContextualGlyphSubstitutionProcessor2@@UAEPAXI@Z 10003d20 f i ContextualGlyphSubstProc2.obj
 0001:00002d20       ??_GContextualGlyphSubstitutionProcessor2@@UAEPAXI@Z 10003d20 f i ContextualGlyphSubstProc2.obj
 0001:00002d70       ?beginStateTable@ContextualGlyphSubstitutionProcessor2@@UAEXXZ 10003d70 f   ContextualGlyphSubstProc2.obj
 0001:00002d80       ?getDynamicClassID@ContextualGlyphSubstitutionProcessor2@@UBEPBDXZ 10003d80 f   ContextualGlyphSubstProc2.obj
 0001:00002d90       ?processStateEntry@ContextualGlyphSubstitutionProcessor2@@UAEGAAVLEGlyphStorage@@AAJGAAW4LEErrorCode@@@Z 10003d90 f   ContextualGlyphSubstProc2.obj
 0001:000033a0       ??0?$LEReferenceTo@UClassDefinitionTable@@@@QAE@ABVLETableReference@@AAW4LEErrorCode@@I@Z 100043a0 f i ContextualSubstSubtables.obj
 0001:000033a0       ??0?$LEReferenceTo@UScriptListTable@@@@QAE@ABVLETableReference@@AAW4LEErrorCode@@I@Z 100043a0 f i GlyphLookupTables.obj
 0001:00003470       ?matchGlyphCoverages@ContextualSubstitutionBase@@SADABV?$LEReferenceToArrayOf@G@@GPAVGlyphIterator@@ABVLETableReference@@AAW4LEErrorCode@@D@Z 10004470 f   ContextualSubstSubtables.obj
 0001:000035c0       ?matchGlyphIDs@ContextualSubstitutionBase@@SADABV?$LEReferenceToArrayOf@G@@GPAVGlyphIterator@@D@Z 100045c0 f   ContextualSubstSubtables.obj
 0001:00003650       ?process@ChainingContextualSubstitutionFormat1Subtable@@QBEKABVLETableReference@@PBVLookupProcessor@@PAVGlyphIterator@@PBVLEFontInstance@@AAW4LEErrorCode@@@Z 10004650 f   ContextualSubstSubtables.obj
 0001:00004360       ?process@ChainingContextualSubstitutionFormat2Subtable@@QBEKABVLETableReference@@PBVLookupProcessor@@PAVGlyphIterator@@PBVLEFontInstance@@AAW4LEErrorCode@@@Z 10005360 f   ContextualSubstSubtables.obj
 0001:00005310       ?process@ChainingContextualSubstitutionFormat3Subtable@@QBEKABVLETableReference@@PBVLookupProcessor@@PAVGlyphIterator@@PBVLEFontInstance@@AAW4LEErrorCode@@@Z 10006310 f   ContextualSubstSubtables.obj
 0001:00005850       ?process@ChainingContextualSubstitutionSubtable@@QBEKABV?$LEReferenceTo@UChainingContextualSubstitutionSubtable@@@@PBVLookupProcessor@@PAVGlyphIterator@@PBVLEFontInstance@@AAW4LEErrorCode@@@Z 10006850 f   ContextualSubstSubtables.obj
 0001:00005b40       ?process@ContextualSubstitutionFormat1Subtable@@QBEKABVLETableReference@@PBVLookupProcessor@@PAVGlyphIterator@@PBVLEFontInstance@@AAW4LEErrorCode@@@Z 10006b40 f   ContextualSubstSubtables.obj
 0001:000061d0       ?process@ContextualSubstitutionFormat2Subtable@@QBEKABVLETableReference@@PBVLookupProcessor@@PAVGlyphIterator@@PBVLEFontInstance@@AAW4LEErrorCode@@@Z 100071d0 f   ContextualSubstSubtables.obj
 0001:00006a40       ?process@ContextualSubstitutionSubtable@@QBEKABVLETableReference@@PBVLookupProcessor@@PAVGlyphIterator@@PBVLEFontInstance@@AAW4LEErrorCode@@@Z 10007a40 f   ContextualSubstSubtables.obj
 0001:00007030       ?getGlyphCoverage@CoverageTable@@QBEJABVLETableReference@@KAAW4LEErrorCode@@@Z 10008030 f   CoverageTables.obj
 0001:00007450       ?process@CursiveAttachmentSubtable@@QBEKABV?$LEReferenceTo@UCursiveAttachmentSubtable@@@@PAVGlyphIterator@@PBVLEFontInstance@@AAW4LEErrorCode@@@Z 10008450 f   CursiveAttachmentSubtables.obj
 0001:00007800       ?getAdjustment@DeviceTable@@QBEFABV?$LEReferenceTo@UDeviceTable@@@@GAAW4LEErrorCode@@@Z 10008800 f   DeviceTables.obj
 0001:00007910       _Java_sun_java2d_loops_DrawGlyphListAA_DrawGlyphListAA@20 10008910 f   DrawGlyphList.obj
 0001:00007910       _Java_sun_java2d_loops_DrawGlyphList_DrawGlyphList@20 10008910 f   DrawGlyphList.obj
 0001:00007980       _Java_sun_java2d_loops_DrawGlyphListLCD_DrawGlyphListLCD@20 10008980 f   DrawGlyphList.obj
 0001:00007a30       _RefineBounds              10008a30 f   DrawGlyphList.obj
 0001:00007ee0       _initLCDGammaTables        10008ee0 f   DrawGlyphList.obj
 0001:00007f30       _initLUT                   10008f30 f   DrawGlyphList.obj
 0001:00008060       _setupBlitVector           10009060 f   DrawGlyphList.obj
 0001:00008420       _setupLCDBlitVector        10009420 f   DrawGlyphList.obj
 0001:000089e0       ?process@ExtensionSubtable@@QBEKABV?$LEReferenceTo@UExtensionSubtable@@@@PBVLookupProcessor@@GPAVGlyphIterator@@PBVLEFontInstance@@AAW4LEErrorCode@@@Z 100099e0 f   ExtensionSubtables.obj
 0001:00008ad0       ??0?$LEReferenceTo@UFeatureTable@@@@QAE@XZ 10009ad0 f i Features.obj
 0001:00008ad0       ??0?$LEReferenceTo@UPairValueRecord@@@@QAE@XZ 10009ad0 f i PairPositioningSubtables.obj
 0001:00008b00       ?getFeatureTable@FeatureListTable@@QBE?AV?$LEReferenceTo@UFeatureTable@@@@ABVLETableReference@@GPAKAAW4LEErrorCode@@@Z 10009b00 f   Features.obj
 0001:00008c80       ??0FontInstanceAdapter@@QAE@PAUJNIEnv_@@PAV_jobject@@1PAMJJJPAUTTLayoutTableCache@@@Z 10009c80 f   FontInstanceAdapter.obj
 0001:00008f40       ??_EFontInstanceAdapter@@UAEPAXI@Z 10009f40 f i FontInstanceAdapter.obj
 0001:00008f40       ??_GFontInstanceAdapter@@UAEPAXI@Z 10009f40 f i FontInstanceAdapter.obj
 0001:00008f70       ??_ELEFontInstance@@UAEPAXI@Z 10009f70 f i FontInstanceAdapter.obj
 0001:00008f70       ??_GLEFontInstance@@UAEPAXI@Z 10009f70 f i FontInstanceAdapter.obj
 0001:00008f90       ?CallBooleanMethod@JNIEnv_@@QAAEPAV_jobject@@PAU_jmethodID@@ZZ 10009f90 f i FontInstanceAdapter.obj
 0001:00008fb0       ?CallIntMethod@JNIEnv_@@QAAJPAV_jobject@@PAU_jmethodID@@ZZ 10009fb0 f i FontInstanceAdapter.obj
 0001:00008fd0       ?CallObjectMethod@JNIEnv_@@QAAPAV_jobject@@PAV2@PAU_jmethodID@@ZZ 10009fd0 f i FontInstanceAdapter.obj
 0001:00008ff0       ?NewObject@JNIEnv_@@QAAPAV_jobject@@PAV_jclass@@PAU_jmethodID@@ZZ 10009ff0 f i FontInstanceAdapter.obj
 0001:00009010       ?canDisplay@FontInstanceAdapter@@UBEDK@Z 1000a010 f i FontInstanceAdapter.obj
 0001:00009030       ?getAscent@FontInstanceAdapter@@UBEJXZ 1000a030 f i FontInstanceAdapter.obj
 0001:00009030       ?getDescent@FontInstanceAdapter@@UBEJXZ 1000a030 f i FontInstanceAdapter.obj
 0001:00009030       ?getLeading@FontInstanceAdapter@@UBEJXZ 1000a030 f i FontInstanceAdapter.obj
 0001:00009030       ___scrt_stub_for_is_c_termination_complete 1000a030 f i MSVCRT:ucrt_stubs.obj
 0001:00009030       __is_c_termination_complete 1000a030 f i MSVCRT:ucrt_stubs.obj
 0001:00009040       ?getFontTable@FontInstanceAdapter@@UBEPBXK@Z 1000a040 f   FontInstanceAdapter.obj
 0001:00009060       ?getFontTable@FontInstanceAdapter@@UBEPBXKAAI@Z 1000a060 f   FontInstanceAdapter.obj
 0001:00009130       ?getFontTable@LEFontInstance@@UBEPBXKAAI@Z 1000a130 f i FontInstanceAdapter.obj
 0001:00009150       ?getGlyphAdvance@FontInstanceAdapter@@UBEXKAAULEPoint@@@Z 1000a150 f   FontInstanceAdapter.obj
 0001:00009160       ?getGlyphPoint@FontInstanceAdapter@@UBEDKJAAULEPoint@@@Z 1000a160 f   FontInstanceAdapter.obj
 0001:000091e0       ?getKernPairs@FontInstanceAdapter@@UBEPAXXZ 1000a1e0 f i FontInstanceAdapter.obj
 0001:000091f0       ?getKerningAdjustment@FontInstanceAdapter@@UBEXAAULEPoint@@@Z 1000a1f0 f   FontInstanceAdapter.obj
 0001:00009320       ?getScaleFactorX@FontInstanceAdapter@@UBEMXZ 1000a320 f i FontInstanceAdapter.obj
 0001:00009330       ?getScaleFactorY@FontInstanceAdapter@@UBEMXZ 1000a330 f i FontInstanceAdapter.obj
 0001:00009340       ?getSubFont@FontInstanceAdapter@@UBEPBVLEFontInstance@@QBGPAJJJAAW4LEErrorCode@@@Z 1000a340 f i FontInstanceAdapter.obj
 0001:00009350       ?getUnitsPerEM@FontInstanceAdapter@@UBEJXZ 1000a350 f i FontInstanceAdapter.obj
 0001:00009360       ?getWideGlyphAdvance@FontInstanceAdapter@@UBEXKAAULEPoint@@@Z 1000a360 f   FontInstanceAdapter.obj
 0001:000093f0       ?getXPixelsPerEm@FontInstanceAdapter@@UBEMXZ 1000a3f0 f i FontInstanceAdapter.obj
 0001:00009400       ?getYPixelsPerEm@FontInstanceAdapter@@UBEMXZ 1000a400 f i FontInstanceAdapter.obj
 0001:00009410       ?mapCharToGlyph@FontInstanceAdapter@@UBEKK@Z 1000a410 f   FontInstanceAdapter.obj
 0001:00009440       ?mapCharToGlyph@FontInstanceAdapter@@UBEKKPBVLECharMapper@@@Z 1000a440 f   FontInstanceAdapter.obj
 0001:000094a0       ?mapCharToWideGlyph@FontInstanceAdapter@@UBEKKPBVLECharMapper@@@Z 1000a4a0 f   FontInstanceAdapter.obj
 0001:00009500       ?mapCharsToWideGlyphs@FontInstanceAdapter@@UBEXQBGJJDPBVLECharMapper@@QAK@Z 1000a500 f   FontInstanceAdapter.obj
 0001:000095c0       ?pixelsToUnits@FontInstanceAdapter@@UBEXAAULEPoint@@0@Z 1000a5c0 f i FontInstanceAdapter.obj
 0001:000095c0       ?pixelsToUnits@LEFontInstance@@UBEXAAULEPoint@@0@Z 1000a5c0 f i LEFontInstance.obj
 0001:00009600       ?setKernPairs@FontInstanceAdapter@@UBEXPAX@Z 1000a600 f i FontInstanceAdapter.obj
 0001:00009610       ?transformFunits@FontInstanceAdapter@@UBEXMMAAULEPoint@@@Z 1000a610 f   FontInstanceAdapter.obj
 0001:000096b0       ?unitsToPoints@FontInstanceAdapter@@UBEXAAULEPoint@@0@Z 1000a6b0 f i FontInstanceAdapter.obj
 0001:000096b0       ?unitsToPoints@LEFontInstance@@UBEXAAULEPoint@@0@Z 1000a6b0 f i LEFontInstance.obj
 0001:000096f0       ?xPixelsToUnits@FontInstanceAdapter@@UBEMM@Z 1000a6f0 f i FontInstanceAdapter.obj
 0001:00009700       ?xUnitsToPoints@FontInstanceAdapter@@UBEMM@Z 1000a700 f i FontInstanceAdapter.obj
 0001:00009710       ?yPixelsToUnits@FontInstanceAdapter@@UBEMM@Z 1000a710 f i FontInstanceAdapter.obj
 0001:00009720       ?yUnitsToPoints@FontInstanceAdapter@@UBEMM@Z 1000a720 f i FontInstanceAdapter.obj
 0001:00009730       ??0GDEFMarkFilter@@QAE@ABV?$LEReferenceTo@UGlyphDefinitionTableHeader@@@@AAW4LEErrorCode@@@Z 1000a730 f   GDEFMarkFilter.obj
 0001:00009770       ??1GDEFMarkFilter@@UAE@XZ  1000a770 f   GDEFMarkFilter.obj
 0001:00009790       ??_EGDEFMarkFilter@@UAEPAXI@Z 1000a790 f i GDEFMarkFilter.obj
 0001:00009790       ??_GGDEFMarkFilter@@UAEPAXI@Z 1000a790 f i GDEFMarkFilter.obj
 0001:000097c0       ??_ELEGlyphFilter@@UAEPAXI@Z 1000a7c0 f i GDEFMarkFilter.obj
 0001:000097c0       ??_GLEGlyphFilter@@UAEPAXI@Z 1000a7c0 f i GDEFMarkFilter.obj
 0001:000097e0       ?accept@GDEFMarkFilter@@UBEDKAAW4LEErrorCode@@@Z 1000a7e0 f   GDEFMarkFilter.obj
 0001:00009800       ??0GXLayoutEngine@@QAE@PBVLEFontInstance@@JJABV?$LEReferenceTo@UMorphTableHeader@@@@AAW4LEErrorCode@@@Z 1000a800 f   GXLayoutEngine.obj
 0001:00009840       ??_EGXLayoutEngine@@UAEPAXI@Z 1000a840 f i GXLayoutEngine.obj
 0001:00009840       ??_GGXLayoutEngine@@UAEPAXI@Z 1000a840 f i GXLayoutEngine.obj
 0001:00009880       ?adjustGlyphPositions@GXLayoutEngine2@@MAEXQBGJJDAAVLEGlyphStorage@@AAW4LEErrorCode@@@Z 1000a880 f   GXLayoutEngine2.obj
 0001:00009880       ?adjustGlyphPositions@GXLayoutEngine@@MAEXQBGJJDAAVLEGlyphStorage@@AAW4LEErrorCode@@@Z 1000a880 f   GXLayoutEngine.obj
 0001:000098b0       ?computeGlyphs@GXLayoutEngine@@MAEJQBGJJJDAAVLEGlyphStorage@@AAW4LEErrorCode@@@Z 1000a8b0 f   GXLayoutEngine.obj
 0001:00009930       ?getDynamicClassID@GXLayoutEngine@@UBEPBDXZ 1000a930 f   GXLayoutEngine.obj
 0001:00009940       ??0GXLayoutEngine2@@QAE@PBVLEFontInstance@@JJABV?$LEReferenceTo@UMorphTableHeader2@@@@JAAW4LEErrorCode@@@Z 1000a940 f   GXLayoutEngine2.obj
 0001:00009980       ??_EGXLayoutEngine2@@UAEPAXI@Z 1000a980 f i GXLayoutEngine2.obj
 0001:00009980       ??_GGXLayoutEngine2@@UAEPAXI@Z 1000a980 f i GXLayoutEngine2.obj
 0001:000099c0       ?computeGlyphs@GXLayoutEngine2@@MAEJQBGJJJDAAVLEGlyphStorage@@AAW4LEErrorCode@@@Z 1000a9c0 f   GXLayoutEngine2.obj
 0001:00009a50       ?getDynamicClassID@GXLayoutEngine2@@UBEPBDXZ 1000aa50 f   GXLayoutEngine2.obj
 0001:00009a60       ?getGlyphClassDefinitionTable@GlyphDefinitionTableHeader@@QBE?BV?$LEReferenceTo@UClassDefinitionTable@@@@ABV?$LEReferenceTo@UGlyphDefinitionTableHeader@@@@AAW4LEErrorCode@@@Z 1000aa60 f   GlyphDefinitionTables.obj
 0001:00009ac0       ?getMarkAttachClassDefinitionTable@GlyphDefinitionTableHeader@@QBE?BV?$LEReferenceTo@UClassDefinitionTable@@@@ABV?$LEReferenceTo@UGlyphDefinitionTableHeader@@@@AAW4LEErrorCode@@@Z 1000aac0 f   GlyphDefinitionTables.obj
 0001:00009b20       ??0GlyphIterator@@QAE@AAV0@@Z 1000ab20 f   GlyphIterator.obj
 0001:00009be0       ??0GlyphIterator@@QAE@AAV0@G@Z 1000abe0 f   GlyphIterator.obj
 0001:00009ca0       ??0GlyphIterator@@QAE@AAV0@K@Z 1000aca0 f   GlyphIterator.obj
 0001:00009d60       ??0GlyphIterator@@QAE@AAVLEGlyphStorage@@PAVGlyphPositionAdjustments@@DGKABV?$LEReferenceTo@UGlyphDefinitionTableHeader@@@@AAW4LEErrorCode@@@Z 1000ad60 f   GlyphIterator.obj
 0001:00009e90       ??1GlyphIterator@@UAE@XZ   1000ae90 f   GlyphIterator.obj
 0001:00009eb0       ??_EGlyphIterator@@UAEPAXI@Z 1000aeb0 f i GlyphIterator.obj
 0001:00009eb0       ??_GGlyphIterator@@UAEPAXI@Z 1000aeb0 f i GlyphIterator.obj
 0001:00009ee0       ?adjustCurrGlyphPositionAdjustment@GlyphIterator@@QAEXMMMM@Z 1000aee0 f   GlyphIterator.obj
 0001:00009f80       ?applyInsertions@GlyphIterator@@QAEJXZ 1000af80 f   GlyphIterator.obj
 0001:00009fa0       ?findFeatureTag@GlyphIterator@@QAEDXZ 1000afa0 f   GlyphIterator.obj
 0001:0000a020       ?findMark2Glyph@GlyphIterator@@QAEDXZ 1000b020 f   GlyphIterator.obj
 0001:0000a140       ?getCurrGlyphID@GlyphIterator@@QBEKXZ 1000b140 f   GlyphIterator.obj
 0001:0000a170       ?getCurrStreamPosition@GlyphIterator@@QBEJXZ 1000b170 f   GlyphIterator.obj
 0001:0000a180       ?getMarkComponent@GlyphIterator@@QBEJJ@Z 1000b180 f   GlyphIterator.obj
 0001:0000a1d0       ?ignoresMarks@GlyphIterator@@QBEDXZ 1000b1d0 f   GlyphIterator.obj
 0001:0000a1e0       ?insertGlyphs@GlyphIterator@@QAEPAKJAAW4LEErrorCode@@@Z 1000b1e0 f   GlyphIterator.obj
 0001:0000a200       ?isRightToLeft@GlyphIterator@@QBEDXZ 1000b200 f   GlyphIterator.obj
 0001:0000a210       ?next@GlyphIterator@@QAEDK@Z 1000b210 f   GlyphIterator.obj
 0001:0000a260       ?nextInternal@GlyphIterator@@AAEDK@Z 1000b260 f   GlyphIterator.obj
 0001:0000a3b0       ?prev@GlyphIterator@@QAEDK@Z 1000b3b0 f   GlyphIterator.obj
 0001:0000a400       ?prevInternal@GlyphIterator@@AAEDK@Z 1000b400 f   GlyphIterator.obj
 0001:0000a550       ?reset@GlyphIterator@@QAEXGK@Z 1000b550 f   GlyphIterator.obj
 0001:0000a580       ?setCurrGlyphBaseOffset@GlyphIterator@@QAEXJ@Z 1000b580 f   GlyphIterator.obj
 0001:0000a5c0       ?setCurrGlyphID@GlyphIterator@@QAEXG@Z 1000b5c0 f   GlyphIterator.obj
 0001:0000a600       ?setCurrGlyphPositionAdjustment@GlyphIterator@@QAEXMMMM@Z 1000b600 f   GlyphIterator.obj
 0001:0000a690       ?setCurrStreamPosition@GlyphIterator@@QAEXJ@Z 1000b690 f   GlyphIterator.obj
 0001:0000a700       ?setCursiveEntryPoint@GlyphIterator@@QAEXAAULEPoint@@@Z 1000b700 f   GlyphIterator.obj
 0001:0000a740       ?setCursiveExitPoint@GlyphIterator@@QAEXAAULEPoint@@@Z 1000b740 f   GlyphIterator.obj
 0001:0000a780       ?setCursiveGlyph@GlyphIterator@@QAEXXZ 1000b780 f   GlyphIterator.obj
 0001:0000a7c0       ?coversScript@GlyphLookupTableHeader@@QBEDABVLETableReference@@KAAW4LEErrorCode@@@Z 1000b7c0 f   GlyphLookupTables.obj
 0001:0000a830       ?coversScriptAndLanguage@GlyphLookupTableHeader@@QBEDABVLETableReference@@KKAAW4LEErrorCode@@D@Z 1000b830 f   GlyphLookupTables.obj
 0001:0000a8a0       ??0GlyphPositionAdjustments@@QAE@J@Z 1000b8a0 f   GlyphPositionAdjustments.obj
 0001:0000a940       ??1GlyphPositionAdjustments@@QAE@XZ 1000b940 f   GlyphPositionAdjustments.obj
 0001:0000a990       ?applyCursiveAdjustments@GlyphPositionAdjustments@@QAEXAAVLEGlyphStorage@@DPBVLEFontInstance@@@Z 1000b990 f   GlyphPositionAdjustments.obj
 0001:0000ac90       ?setCursiveGlyph@GlyphPositionAdjustments@@QAEXJD@Z 1000bc90 f   GlyphPositionAdjustments.obj
 0001:0000ad40       ?setEntryPoint@GlyphPositionAdjustments@@QAEXJAAULEPoint@@D@Z 1000bd40 f   GlyphPositionAdjustments.obj
 0001:0000ae00       ?setExitPoint@GlyphPositionAdjustments@@QAEXJAAULEPoint@@D@Z 1000be00 f   GlyphPositionAdjustments.obj
 0001:0000aec0       ?process@GlyphPositioningTableHeader@@QBEXABV?$LEReferenceTo@UGlyphPositioningTableHeader@@@@AAVLEGlyphStorage@@PAVGlyphPositionAdjustments@@DKKABV?$LEReferenceTo@UGlyphDefinitionTableHeader@@@@AAW4LEErrorCode@@PBVLEFontInstance@@PBUFeatureMap@@JD@Z 1000bec0 f   GlyphPositioningTables.obj
 0001:0000af40       ??0GlyphPositioningLookupProcessor@@QAE@ABV?$LEReferenceTo@UGlyphPositioningTableHeader@@@@KKPBUFeatureMap@@JDAAW4LEErrorCode@@@Z 1000bf40 f   GlyphPosnLookupProc.obj
 0001:0000afa0       ??1GlyphPositioningLookupProcessor@@UAE@XZ 1000bfa0 f   GlyphPosnLookupProc.obj
 0001:0000afb0       ??_EGlyphPositioningLookupProcessor@@UAEPAXI@Z 1000bfb0 f i GlyphPosnLookupProc.obj
 0001:0000afb0       ??_GGlyphPositioningLookupProcessor@@UAEPAXI@Z 1000bfb0 f i GlyphPosnLookupProc.obj
 0001:0000afe0       ?applySubtable@GlyphPositioningLookupProcessor@@UBEKABV?$LEReferenceTo@ULookupSubtable@@@@GPAVGlyphIterator@@PBVLEFontInstance@@AAW4LEErrorCode@@@Z 1000bfe0 f   GlyphPosnLookupProc.obj
 0001:0000b5a0       ??0GlyphSubstitutionLookupProcessor@@QAE@ABV?$LEReferenceTo@UGlyphSubstitutionTableHeader@@@@KKPBVLEGlyphFilter@@PBUFeatureMap@@JDAAW4LEErrorCode@@@Z 1000c5a0 f   GlyphSubstLookupProc.obj
 0001:0000b610       ??1GlyphSubstitutionLookupProcessor@@UAE@XZ 1000c610 f   GlyphSubstLookupProc.obj
 0001:0000b620       ??_EGlyphSubstitutionLookupProcessor@@UAEPAXI@Z 1000c620 f i GlyphSubstLookupProc.obj
 0001:0000b620       ??_GGlyphSubstitutionLookupProcessor@@UAEPAXI@Z 1000c620 f i GlyphSubstLookupProc.obj
 0001:0000b650       ?applySubtable@GlyphSubstitutionLookupProcessor@@UBEKABV?$LEReferenceTo@ULookupSubtable@@@@GPAVGlyphIterator@@PBVLEFontInstance@@AAW4LEErrorCode@@@Z 1000c650 f   GlyphSubstLookupProc.obj
 0001:0000bae0       ?process@GlyphSubstitutionTableHeader@@QBEJABV?$LEReferenceTo@UGlyphSubstitutionTableHeader@@@@AAVLEGlyphStorage@@DKKABV?$LEReferenceTo@UGlyphDefinitionTableHeader@@@@PBVLEGlyphFilter@@PBUFeatureMap@@JDAAW4LEErrorCode@@@Z 1000cae0 f   GlyphSubstitutionTables.obj
 0001:0000bb60       ??0HanOpenTypeLayoutEngine@@QAE@PBVLEFontInstance@@JJJABV?$LEReferenceTo@UGlyphSubstitutionTableHeader@@@@AAW4LEErrorCode@@@Z 1000cb60 f   HanLayoutEngine.obj
 0001:0000bba0       ??_EHanOpenTypeLayoutEngine@@UAEPAXI@Z 1000cba0 f i HanLayoutEngine.obj
 0001:0000bba0       ??_GHanOpenTypeLayoutEngine@@UAEPAXI@Z 1000cba0 f i HanLayoutEngine.obj
 0001:0000bbd0       ?characterProcessing@HanOpenTypeLayoutEngine@@MAEJQBGJJJDAAPAGAAVLEGlyphStorage@@AAW4LEErrorCode@@@Z 1000cbd0 f   HanLayoutEngine.obj
 0001:0000bc60       ?getDynamicClassID@HanOpenTypeLayoutEngine@@UBEPBDXZ 1000cc60 f   HanLayoutEngine.obj
 0001:0000bc70       ??0HangulOpenTypeLayoutEngine@@QAE@PBVLEFontInstance@@JJJAAW4LEErrorCode@@@Z 1000cc70 f   HangulLayoutEngine.obj
 0001:0000bcb0       ??0HangulOpenTypeLayoutEngine@@QAE@PBVLEFontInstance@@JJJABV?$LEReferenceTo@UGlyphSubstitutionTableHeader@@@@AAW4LEErrorCode@@@Z 1000ccb0 f   HangulLayoutEngine.obj
 0001:0000bcf0       ??_EHangulOpenTypeLayoutEngine@@UAEPAXI@Z 1000ccf0 f i HangulLayoutEngine.obj
 0001:0000bcf0       ??_GHangulOpenTypeLayoutEngine@@UAEPAXI@Z 1000ccf0 f i HangulLayoutEngine.obj
 0001:0000bd20       ?characterProcessing@HangulOpenTypeLayoutEngine@@MAEJQBGJJJDAAPAGAAVLEGlyphStorage@@AAW4LEErrorCode@@@Z 1000cd20 f   HangulLayoutEngine.obj
 0001:0000c260       ?getDynamicClassID@HangulOpenTypeLayoutEngine@@UBEPBDXZ 1000d260 f   HangulLayoutEngine.obj
 0001:0000c270       ?getCharClass@IndicClassTable@@QBEKG@Z 1000d270 f   IndicClassTables.obj
 0001:0000c2d0       ?getFilterZeroWidth@IndicReordering@@SADJ@Z 1000d2d0 f   IndicClassTables.obj
 0001:0000c300       ?getScriptClassTable@IndicClassTable@@SAPBU1@J@Z 1000d300 f   IndicClassTables.obj
 0001:0000c320       ?getWorstCaseExpansion@IndicReordering@@SAJJ@Z 1000d320 f   IndicClassTables.obj
 0001:0000c340       ??0IndicOpenTypeLayoutEngine@@QAE@PBVLEFontInstance@@JJJAAW4LEErrorCode@@@Z 1000d340 f   IndicLayoutEngine.obj
 0001:0000c390       ??0IndicOpenTypeLayoutEngine@@QAE@PBVLEFontInstance@@JJJDABV?$LEReferenceTo@UGlyphSubstitutionTableHeader@@@@AAW4LEErrorCode@@@Z 1000d390 f   IndicLayoutEngine.obj
 0001:0000c400       ??_EIndicOpenTypeLayoutEngine@@UAEPAXI@Z 1000d400 f i IndicLayoutEngine.obj
 0001:0000c400       ??_GIndicOpenTypeLayoutEngine@@UAEPAXI@Z 1000d400 f i IndicLayoutEngine.obj
 0001:0000c430       ?characterProcessing@IndicOpenTypeLayoutEngine@@MAEJQBGJJJDAAPAGAAVLEGlyphStorage@@AAW4LEErrorCode@@@Z 1000d430 f   IndicLayoutEngine.obj
 0001:0000c580       ?getDynamicClassID@IndicOpenTypeLayoutEngine@@UBEPBDXZ 1000d580 f   IndicLayoutEngine.obj
 0001:0000c590       ?glyphProcessing@IndicOpenTypeLayoutEngine@@MAEJQBGJJJDAAVLEGlyphStorage@@AAW4LEErrorCode@@@Z 1000d590 f   IndicLayoutEngine.obj
 0001:0000c660       ??0IndicRearrangementProcessor@@QAE@ABV?$LEReferenceTo@UMorphSubtableHeader@@@@AAW4LEErrorCode@@@Z 1000d660 f   IndicRearrangementProcessor.obj
 0001:0000c960       ??_EIndicRearrangementProcessor@@UAEPAXI@Z 1000d960 f i IndicRearrangementProcessor.obj
 0001:0000c960       ??_GIndicRearrangementProcessor@@UAEPAXI@Z 1000d960 f i IndicRearrangementProcessor.obj
 0001:0000c9b0       ?beginStateTable@IndicRearrangementProcessor@@UAEXXZ 1000d9b0 f   IndicRearrangementProcessor.obj
 0001:0000c9c0       ?doRearrangementAction@IndicRearrangementProcessor@@QBEXAAVLEGlyphStorage@@W4IndicRearrangementVerb@@AAW4LEErrorCode@@@Z 1000d9c0 f   IndicRearrangementProcessor.obj
 0001:0000d4b0       ?getDynamicClassID@IndicRearrangementProcessor@@UBEPBDXZ 1000e4b0 f   IndicRearrangementProcessor.obj
 0001:0000d4c0       ?processStateEntry@IndicRearrangementProcessor@@UAEFAAVLEGlyphStorage@@AAJEAAW4LEErrorCode@@@Z 1000e4c0 f   IndicRearrangementProcessor.obj
 0001:0000d570       ??0?$LEReferenceToArrayOf@UIndicRearrangementStateEntry2@@@@QAE@ABVLETableReference@@AAW4LEErrorCode@@IK@Z 1000e570 f i IndicRearrangementProcessor2.obj
 0001:0000d660       ??0IndicRearrangementProcessor2@@QAE@ABV?$LEReferenceTo@UMorphSubtableHeader2@@@@AAW4LEErrorCode@@@Z 1000e660 f   IndicRearrangementProcessor2.obj
 0001:0000d750       ??_EIndicRearrangementProcessor2@@UAEPAXI@Z 1000e750 f i IndicRearrangementProcessor2.obj
 0001:0000d750       ??_GIndicRearrangementProcessor2@@UAEPAXI@Z 1000e750 f i IndicRearrangementProcessor2.obj
 0001:0000d790       ?beginStateTable@IndicRearrangementProcessor2@@UAEXXZ 1000e790 f   IndicRearrangementProcessor2.obj
 0001:0000d7b0       ?doRearrangementAction@IndicRearrangementProcessor2@@QBEXAAVLEGlyphStorage@@W4IndicRearrangementVerb@@AAW4LEErrorCode@@@Z 1000e7b0 f   IndicRearrangementProcessor2.obj
 0001:0000e3a0       ?getDynamicClassID@IndicRearrangementProcessor2@@UBEPBDXZ 1000f3a0 f   IndicRearrangementProcessor2.obj
 0001:0000e3b0       ?processStateEntry@IndicRearrangementProcessor2@@UAEGAAVLEGlyphStorage@@AAJGAAW4LEErrorCode@@@Z 1000f3b0 f   IndicRearrangementProcessor2.obj
 0001:0000e470       ??0IndicReorderingOutput@@QAE@PAGAAVLEGlyphStorage@@PAVMPreFixups@@@Z 1000f470 f i IndicReordering.obj
 0001:0000e4f0       ?adjustMPres@IndicReordering@@SAXPAVMPreFixups@@AAVLEGlyphStorage@@AAW4LEErrorCode@@@Z 1000f4f0 f   IndicReordering.obj
 0001:0000e520       ?applyPresentationForms@IndicReordering@@SAXAAVLEGlyphStorage@@J@Z 1000f520 f   IndicReordering.obj
 0001:0000e560       ?decomposeReorderMatras@IndicReorderingOutput@@QAEXPBUIndicClassTable@@JJJ@Z 1000f560 f i IndicReordering.obj
 0001:0000e8b0       ?finalReordering@IndicReordering@@SAXAAVLEGlyphStorage@@J@Z 1000f8b0 f   IndicReordering.obj
 0001:0000e9b0       ?findSyllable@IndicReordering@@CAJPBUIndicClassTable@@PBGJJ@Z 1000f9b0 f   IndicReordering.obj
 0001:0000ea20       ?getFeatureMap@IndicReordering@@SAPBUFeatureMap@@AAJ@Z 1000fa20 f   IndicReordering.obj
 0001:0000ea30       ?getv2FeatureMap@IndicReordering@@SAPBUFeatureMap@@AAJ@Z 1000fa30 f   IndicReordering.obj
 0001:0000ea40       ?reorder@IndicReordering@@SAJPBGJJPAGAAVLEGlyphStorage@@PAPAVMPreFixups@@AAW4LEErrorCode@@@Z 1000fa40 f   IndicReordering.obj
 0001:00010220       ?saveMatra@IndicReorderingOutput@@AAEXGJK@Z 10011220 f i IndicReordering.obj
 0001:000102d0       ?v2process@IndicReordering@@SAJPBGJJPAGAAVLEGlyphStorage@@AAW4LEErrorCode@@@Z 100112d0 f   IndicReordering.obj
 0001:00010840       ?writeMpre@IndicReorderingOutput@@QAEXXZ 10011840 f i IndicReordering.obj
 0001:000108a0       ??0KernTable@@QAE@ABVLETableReference@@AAW4LEErrorCode@@@Z 100118a0 f   KernTable.obj
 0001:00010c70       ?process@KernTable@@QAEXAAVLEGlyphStorage@@AAW4LEErrorCode@@@Z 10011c70 f   KernTable.obj
 0001:00010dd0       ??0KhmerOpenTypeLayoutEngine@@QAE@PBVLEFontInstance@@JJJABV?$LEReferenceTo@UGlyphSubstitutionTableHeader@@@@AAW4LEErrorCode@@@Z 10011dd0 f   KhmerLayoutEngine.obj
 0001:00010e10       ??_EKhmerOpenTypeLayoutEngine@@UAEPAXI@Z 10011e10 f i KhmerLayoutEngine.obj
 0001:00010e10       ??_GKhmerOpenTypeLayoutEngine@@UAEPAXI@Z 10011e10 f i KhmerLayoutEngine.obj
 0001:00010e40       ?characterProcessing@KhmerOpenTypeLayoutEngine@@MAEJQBGJJJDAAPAGAAVLEGlyphStorage@@AAW4LEErrorCode@@@Z 10011e40 f   KhmerLayoutEngine.obj
 0001:00010f60       ?getDynamicClassID@KhmerOpenTypeLayoutEngine@@UBEPBDXZ 10011f60 f   KhmerLayoutEngine.obj
 0001:00010f70       ?getFeatureMap@KhmerReordering@@SAPBUFeatureMap@@AAJ@Z 10011f70 f   KhmerReordering.obj
 0001:00010f80       ?reorder@KhmerReordering@@SAJPBGJJPAGAAVLEGlyphStorage@@@Z 10011f80 f   KhmerReordering.obj
 0001:00011750       ??1LECharMapper@@UAE@XZ    10012750 f   LEFontInstance.obj
 0001:00011760       ??1LEFontInstance@@UAE@XZ  10012760 f   LEFontInstance.obj
 0001:00011770       ??_ELECharMapper@@UAEPAXI@Z 10012770 f i LEFontInstance.obj
 0001:00011770       ??_GLECharMapper@@UAEPAXI@Z 10012770 f i LEFontInstance.obj
 0001:000117a0       ?canDisplay@LEFontInstance@@UBEDK@Z 100127a0 f   LEFontInstance.obj
 0001:000117c0       ?getDynamicClassID@LEFontInstance@@UBEPBDXZ 100127c0 f   LEFontInstance.obj
 0001:000117d0       ?getLineHeight@LEFontInstance@@UBEJXZ 100127d0 f   LEFontInstance.obj
 0001:000117f0       ?getSubFont@LEFontInstance@@UBEPBV1@QBGPAJJJAAW4LEErrorCode@@@Z 100127f0 f   LEFontInstance.obj
 0001:00011840       ?mapCharToGlyph@LEFontInstance@@UBEKKPBVLECharMapper@@@Z 10012840 f   LEFontInstance.obj
 0001:00011860       ?mapCharToGlyph@LEFontInstance@@UBEKKPBVLECharMapper@@D@Z 10012860 f   LEFontInstance.obj
 0001:000118d0       ?mapCharsToGlyphs@LEFontInstance@@UBEXQBGJJDPBVLECharMapper@@DAAVLEGlyphStorage@@@Z 100128d0 f   LEFontInstance.obj
 0001:000119b0       ?transformFunits@LEFontInstance@@UBEXMMAAULEPoint@@@Z 100129b0 f   LEFontInstance.obj
 0001:00011a10       ?xPixelsToUnits@LEFontInstance@@UBEMM@Z 10012a10 f   LEFontInstance.obj
 0001:00011a40       ?xUnitsToPoints@LEFontInstance@@UBEMM@Z 10012a40 f   LEFontInstance.obj
 0001:00011a80       ?yPixelsToUnits@LEFontInstance@@UBEMM@Z 10012a80 f   LEFontInstance.obj
 0001:00011ab0       ?yUnitsToPoints@LEFontInstance@@UBEMM@Z 10012ab0 f   LEFontInstance.obj
 0001:00011af0       ??0LEGlyphStorage@@QAE@XZ  10012af0 f   LEGlyphStorage.obj
 0001:00011b40       ??1LEGlyphStorage@@UAE@XZ  10012b40 f   LEGlyphStorage.obj
 0001:00011be0       ??_ELEGlyphStorage@@UAEPAXI@Z 10012be0 f i LEGlyphStorage.obj
 0001:00011be0       ??_GLEGlyphStorage@@UAEPAXI@Z 10012be0 f i LEGlyphStorage.obj
 0001:00011c90       ??_ELEInsertionCallback@@UAEPAXI@Z 10012c90 f i LEGlyphStorage.obj
 0001:00011c90       ??_GLEInsertionCallback@@UAEPAXI@Z 10012c90 f i LEGlyphStorage.obj
 0001:00011cc0       ?adjustPosition@LEGlyphStorage@@QAEXJMMAAW4LEErrorCode@@@Z 10012cc0 f   LEGlyphStorage.obj
 0001:00011d10       ?adoptAuxDataArray@LEGlyphStorage@@QAEXAAV1@@Z 10012d10 f   LEGlyphStorage.obj
 0001:00011d40       ?adoptCharIndicesArray@LEGlyphStorage@@QAEXAAV1@@Z 10012d40 f   LEGlyphStorage.obj
 0001:00011d70       ?adoptGlyphArray@LEGlyphStorage@@QAEXAAV1@@Z 10012d70 f   LEGlyphStorage.obj
 0001:00011dd0       ?adoptGlyphCount@LEGlyphStorage@@QAEXAAV1@@Z 10012dd0 f   LEGlyphStorage.obj
 0001:00011de0       ?adoptGlyphCount@LEGlyphStorage@@QAEXJ@Z 10012de0 f   LEGlyphStorage.obj
 0001:00011df0       ?allocateAuxData@LEGlyphStorage@@QAEJAAW4LEErrorCode@@@Z 10012df0 f   LEGlyphStorage.obj
 0001:00011e60       ?allocateGlyphArray@LEGlyphStorage@@QAEXJDAAW4LEErrorCode@@@Z 10012e60 f   LEGlyphStorage.obj
 0001:00011fc0       ?allocatePositions@LEGlyphStorage@@QAEJAAW4LEErrorCode@@@Z 10012fc0 f   LEGlyphStorage.obj
 0001:00012040       ?applyInsertion@LEGlyphStorage@@MAEDJJQAK@Z 10013040 f   LEGlyphStorage.obj
 0001:00012130       ?applyInsertions@LEGlyphStorage@@QAEJXZ 10013130 f   LEGlyphStorage.obj
 0001:000121c0       ?getAuxData@LEGlyphStorage@@QBEKJAAW4LEErrorCode@@@Z 100131c0 f   LEGlyphStorage.obj
 0001:00012200       ?getCharIndex@LEGlyphStorage@@QBEJJAAW4LEErrorCode@@@Z 10013200 f   LEGlyphStorage.obj
 0001:00012250       ?getCharIndices@LEGlyphStorage@@QBEXQAJJAAW4LEErrorCode@@@Z 10013250 f   LEGlyphStorage.obj
 0001:000122b0       ?getDynamicClassID@LEGlyphStorage@@UBEPBDXZ 100132b0 f   LEGlyphStorage.obj
 0001:000122c0       ?getGlyphID@LEGlyphStorage@@QBEKJAAW4LEErrorCode@@@Z 100132c0 f   LEGlyphStorage.obj
 0001:00012310       ?getGlyphPosition@LEGlyphStorage@@QBEXJAAM0AAW4LEErrorCode@@@Z 10013310 f   LEGlyphStorage.obj
 0001:00012360       ?getGlyphPositions@LEGlyphStorage@@QBEXQAMAAW4LEErrorCode@@@Z 10013360 f   LEGlyphStorage.obj
 0001:000123b0       ?getGlyphs@LEGlyphStorage@@QBEXQAKKAAW4LEErrorCode@@@Z 100133b0 f   LEGlyphStorage.obj
 0001:00012410       ?insertGlyphs@LEGlyphStorage@@QAEPAKJJAAW4LEErrorCode@@@Z 10013410 f   LEGlyphStorage.obj
 0001:00012420       ?moveGlyph@LEGlyphStorage@@QAEXJJK@Z 10013420 f   LEGlyphStorage.obj
 0001:00012670       ?reset@LEGlyphStorage@@QAEXXZ 10013670 f   LEGlyphStorage.obj
 0001:00012700       ?setAuxData@LEGlyphStorage@@QAEXJKAAW4LEErrorCode@@@Z 10013700 f   LEGlyphStorage.obj
 0001:00012740       ?setCharIndex@LEGlyphStorage@@QAEXJJAAW4LEErrorCode@@@Z 10013740 f   LEGlyphStorage.obj
 0001:00012780       ?setPosition@LEGlyphStorage@@QAEXJMMAAW4LEErrorCode@@@Z 10013780 f   LEGlyphStorage.obj
 0001:000127c0       ??0LEInsertionList@@QAE@D@Z 100137c0 f   LEInsertionList.obj
 0001:000127f0       ??1LEInsertionList@@QAE@XZ 100137f0 f   LEInsertionList.obj
 0001:00012830       ?applyInsertions@LEInsertionList@@QAEDPAVLEInsertionCallback@@@Z 10013830 f   LEInsertionList.obj
 0001:00012870       ?getDynamicClassID@LEInsertionList@@UBEPBDXZ 10013870 f   LEInsertionList.obj
 0001:00012880       ?getGrowAmount@LEInsertionList@@QAEJXZ 10013880 f   LEInsertionList.obj
 0001:00012890       ?insert@LEInsertionList@@QAEPAKJJAAW4LEErrorCode@@@Z 10013890 f   LEInsertionList.obj
 0001:00012910       ?reset@LEInsertionList@@QAEXXZ 10013910 f   LEInsertionList.obj
 0001:00012950       ??0CharSubstitutionFilter@@QAE@PBVLEFontInstance@@@Z 10013950 f   LayoutEngine.obj
 0001:00012970       ??0LayoutEngine@@IAE@PBVLEFontInstance@@JJJAAW4LEErrorCode@@@Z 10013970 f   LayoutEngine.obj
 0001:000129f0       ??1LEGlyphFilter@@UAE@XZ   100139f0 f   LayoutEngine.obj
 0001:00012a00       ??1LayoutEngine@@UAE@XZ    10013a00 f   LayoutEngine.obj
 0001:00012a20       ??_ECanonMarkFilter@@UAEPAXI@Z 10013a20 f i LayoutEngine.obj
 0001:00012a20       ??_GCanonMarkFilter@@UAEPAXI@Z 10013a20 f i LayoutEngine.obj
 0001:00012a50       ??_ECharSubstitutionFilter@@UAEPAXI@Z 10013a50 f i LayoutEngine.obj
 0001:00012a50       ??_GCharSubstitutionFilter@@UAEPAXI@Z 10013a50 f i LayoutEngine.obj
 0001:00012a80       ??_EDefaultCharMapper@@UAEPAXI@Z 10013a80 f i LayoutEngine.obj
 0001:00012a80       ??_GDefaultCharMapper@@UAEPAXI@Z 10013a80 f i LayoutEngine.obj
 0001:00012ab0       ??_ELayoutEngine@@UAEPAXI@Z 10013ab0 f i LayoutEngine.obj
 0001:00012ab0       ??_GLayoutEngine@@UAEPAXI@Z 10013ab0 f i LayoutEngine.obj
 0001:00012ae0       ?accept@CanonMarkFilter@@UBEDKAAW4LEErrorCode@@@Z 10013ae0 f   LayoutEngine.obj
 0001:00012b10       ?adjustGlyphPositions@LayoutEngine@@MAEXQBGJJDAAVLEGlyphStorage@@AAW4LEErrorCode@@@Z 10013b10 f   LayoutEngine.obj
 0001:00012d90       ?adjustMarkGlyphs@LayoutEngine@@KAXAAVLEGlyphStorage@@PAVLEGlyphFilter@@AAW4LEErrorCode@@@Z 10013d90 f   LayoutEngine.obj
 0001:00012ea0       ?adjustMarkGlyphs@LayoutEngine@@KAXQBGJDAAVLEGlyphStorage@@PAVLEGlyphFilter@@AAW4LEErrorCode@@@Z 10013ea0 f   LayoutEngine.obj
 0001:00012ff0       ?characterProcessing@LayoutEngine@@MAEJQBGJJJDAAPAGAAVLEGlyphStorage@@AAW4LEErrorCode@@@Z 10013ff0 f   LayoutEngine.obj
 0001:00013390       ?computeGlyphs@LayoutEngine@@MAEJQBGJJJDAAVLEGlyphStorage@@AAW4LEErrorCode@@@Z 10014390 f   LayoutEngine.obj
 0001:00013480       ?getCharIndices@LayoutEngine@@QBEXQAJJAAW4LEErrorCode@@@Z 10014480 f   LayoutEngine.obj
 0001:00013490       ?getDynamicClassID@LayoutEngine@@UBEPBDXZ 10014490 f   LayoutEngine.obj
 0001:000134a0       ?getFontTable@LayoutEngine@@MBEPBXKAAI@Z 100144a0 f   LayoutEngine.obj
 0001:000134b0       ?getGlyphPosition@LayoutEngine@@QBEXJAAM0AAW4LEErrorCode@@@Z 100144b0 f   LayoutEngine.obj
 0001:000134c0       ?getGlyphPositions@LayoutEngine@@QBEXQAMAAW4LEErrorCode@@@Z 100144c0 f   LayoutEngine.obj
 0001:000134d0       ?getGlyphs@LayoutEngine@@UBEXQAKKAAW4LEErrorCode@@@Z 100144d0 f   LayoutEngine.obj
 0001:000134e0       ?layoutChars@LayoutEngine@@UAEJQBGJJJDMMAAW4LEErrorCode@@@Z 100144e0 f   LayoutEngine.obj
 0001:000135c0       ?layoutEngineFactory@LayoutEngine@@SAPAV1@PBVLEFontInstance@@JJJAAW4LEErrorCode@@@Z 100145c0 f   LayoutEngine.obj
 0001:00013cd0       ?mapChar@DefaultCharMapper@@UBEKK@Z 10014cd0 f   LayoutEngine.obj
 0001:00013d80       ?mapCharsToGlyphs@LayoutEngine@@MAEXQBGJJDDAAVLEGlyphStorage@@AAW4LEErrorCode@@@Z 10014d80 f   LayoutEngine.obj
 0001:00013e00       ?positionGlyphs@LayoutEngine@@MAEXAAVLEGlyphStorage@@MMAAW4LEErrorCode@@@Z 10014e00 f   LayoutEngine.obj
 0001:00013ed0       ?reset@LayoutEngine@@UAEXXZ 10014ed0 f   LayoutEngine.obj
 0001:00013ee0       ??0LigatureSubstitutionProcessor@@QAE@ABV?$LEReferenceTo@UMorphSubtableHeader@@@@AAW4LEErrorCode@@@Z 10014ee0 f   LigatureSubstProc.obj
 0001:000140e0       ??_ELigatureSubstitutionProcessor@@UAEPAXI@Z 100150e0 f i LigatureSubstProc.obj
 0001:000140e0       ??_GLigatureSubstitutionProcessor@@UAEPAXI@Z 100150e0 f i LigatureSubstProc.obj
 0001:00014120       ?beginStateTable@LigatureSubstitutionProcessor@@UAEXXZ 10015120 f   LigatureSubstProc.obj
 0001:00014130       ?getDynamicClassID@LigatureSubstitutionProcessor@@UBEPBDXZ 10015130 f   LigatureSubstProc.obj
 0001:00014140       ?processStateEntry@LigatureSubstitutionProcessor@@UAEFAAVLEGlyphStorage@@AAJEAAW4LEErrorCode@@@Z 10015140 f   LigatureSubstProc.obj
 0001:000145e0       ??0LigatureSubstitutionProcessor2@@QAE@ABV?$LEReferenceTo@UMorphSubtableHeader2@@@@AAW4LEErrorCode@@@Z 100155e0 f   LigatureSubstProc2.obj
 0001:00014860       ??_ELigatureSubstitutionProcessor2@@UAEPAXI@Z 10015860 f i LigatureSubstProc2.obj
 0001:00014860       ??_GLigatureSubstitutionProcessor2@@UAEPAXI@Z 10015860 f i LigatureSubstProc2.obj
 0001:000148a0       ?beginStateTable@LigatureSubstitutionProcessor2@@UAEXXZ 100158a0 f   LigatureSubstProc2.obj
 0001:000148b0       ?getDynamicClassID@LigatureSubstitutionProcessor2@@UBEPBDXZ 100158b0 f   LigatureSubstProc2.obj
 0001:000148c0       ?processStateEntry@LigatureSubstitutionProcessor2@@UAEGAAVLEGlyphStorage@@AAJGAAW4LEErrorCode@@@Z 100158c0 f   LigatureSubstProc2.obj
 0001:00015070       ?process@LigatureSubstitutionSubtable@@QBEKABVLETableReference@@PAVGlyphIterator@@AAW4LEErrorCode@@PBVLEGlyphFilter@@@Z 10016070 f   LigatureSubstSubtables.obj
 0001:00015960       ??0LookupProcessor@@IAE@ABVLETableReference@@GGGKKPBUFeatureMap@@JDAAW4LEErrorCode@@@Z 10016960 f   LookupProcessor.obj
 0001:000164a0       ??1LookupProcessor@@UAE@XZ 100174a0 f   LookupProcessor.obj
 0001:000164e0       ??_ELookupProcessor@@UAEPAXI@Z 100174e0 f i LookupProcessor.obj
 0001:000164e0       ??_GLookupProcessor@@UAEPAXI@Z 100174e0 f i LookupProcessor.obj
 0001:00016530       ?applyLookupTable@LookupProcessor@@QBEKABV?$LEReferenceTo@ULookupTable@@@@PAVGlyphIterator@@PBVLEFontInstance@@AAW4LEErrorCode@@@Z 10017530 f   LookupProcessor.obj
 0001:000165f0       ?applySingleLookup@LookupProcessor@@QBEKGPAVGlyphIterator@@PBVLEFontInstance@@AAW4LEErrorCode@@@Z 100175f0 f   LookupProcessor.obj
 0001:00016740       ?process@LookupProcessor@@QBEJAAVLEGlyphStorage@@PAVGlyphPositionAdjustments@@DABV?$LEReferenceTo@UGlyphDefinitionTableHeader@@@@PBVLEFontInstance@@AAW4LEErrorCode@@@Z 10017740 f   LookupProcessor.obj
 0001:00016890       ?selectLookups@LookupProcessor@@IAEJABV?$LEReferenceTo@UFeatureTable@@@@KJAAW4LEErrorCode@@@Z 10017890 f   LookupProcessor.obj
 0001:00016970       ?lookupSegment@BinarySearchLookupTable@@QBEPBULookupSegment@@ABVLETableReference@@PBU2@KAAW4LEErrorCode@@@Z 10017970 f   LookupTables.obj
 0001:00016c30       ?lookupSingle@BinarySearchLookupTable@@QBEPBULookupSingle@@ABVLETableReference@@PBU2@KAAW4LEErrorCode@@@Z 10017c30 f   LookupTables.obj
 0001:00016ef0       ?getGlyphCoverage@LookupSubtable@@QBEJABV?$LEReferenceTo@ULookupSubtable@@@@GKAAW4LEErrorCode@@@Z 10017ef0 f   Lookups.obj
 0001:00016fc0       ?getLookupSubtable@LookupTable@@QBE?BV?$LEReferenceTo@ULookupSubtable@@@@ABV?$LEReferenceTo@ULookupTable@@@@GAAW4LEErrorCode@@@Z 10017fc0 f   Lookups.obj
 0001:00017130       ?getLookupTable@LookupListTable@@QBE?BV?$LEReferenceTo@ULookupTable@@@@ABV?$LEReferenceTo@ULookupListTable@@@@GAAW4LEErrorCode@@@Z 10018130 f   Lookups.obj
 0001:000172a0       ??0MPreFixups@@QAE@J@Z     100182a0 f   MPreFixups.obj
 0001:000172e0       ??1MPreFixups@@QAE@XZ      100182e0 f   MPreFixups.obj
 0001:00017300       ?add@MPreFixups@@QAEXJJ@Z  10018300 f   MPreFixups.obj
 0001:00017330       ?apply@MPreFixups@@QAEXAAVLEGlyphStorage@@AAW4LEErrorCode@@@Z 10018330 f   MPreFixups.obj
 0001:000175a0       ??0?$LEReferenceToArrayOf@UMarkRecord@@@@QAE@ABVLETableReference@@AAW4LEErrorCode@@PBUMarkRecord@@K@Z 100185a0 f i MarkArrays.obj
 0001:000176c0       ?getMarkClass@MarkArray@@QBEJABVLETableReference@@KJPBVLEFontInstance@@AAULEPoint@@AAW4LEErrorCode@@@Z 100186c0 f   MarkArrays.obj
 0001:000177d0       ?process@MarkToBasePositioningSubtable@@QBEJABVLETableReference@@PAVGlyphIterator@@PBVLEFontInstance@@AAW4LEErrorCode@@@Z 100187d0 f   MarkToBasePosnSubtables.obj
 0001:000182f0       ?process@MarkToLigaturePositioningSubtable@@QBEJABVLETableReference@@PAVGlyphIterator@@PBVLEFontInstance@@AAW4LEErrorCode@@@Z 100192f0 f   MarkToLigaturePosnSubtables.obj
 0001:00018d40       ?process@MarkToMarkPositioningSubtable@@QBEJABVLETableReference@@PAVGlyphIterator@@PBVLEFontInstance@@AAW4LEErrorCode@@@Z 10019d40 f   MarkToMarkPosnSubtables.obj
 0001:000195a0       ?process@MorphTableHeader@@QBEXABVLETableReference@@AAVLEGlyphStorage@@AAW4LEErrorCode@@@Z 1001a5a0 f   MorphTables.obj
 0001:00019b70       ?process@MorphTableHeader2@@QBEXABV?$LEReferenceTo@UMorphTableHeader2@@@@AAVLEGlyphStorage@@JAAW4LEErrorCode@@@Z 1001ab70 f   MorphTables2.obj
 0001:0001a4a0       ?process@MultipleSubstitutionSubtable@@QBEKABVLETableReference@@PAVGlyphIterator@@AAW4LEErrorCode@@PBVLEGlyphFilter@@@Z 1001b4a0 f   MultipleSubstSubtables.obj
 0001:0001a8f0       ??0NonContextualGlyphSubstitutionProcessor@@IAE@ABV?$LEReferenceTo@UMorphSubtableHeader@@@@AAW4LEErrorCode@@@Z 1001b8f0 f   NonContextualGlyphSubstProc.obj
 0001:0001a910       ??1NonContextualGlyphSubstitutionProcessor@@MAE@XZ 1001b910 f   NonContextualGlyphSubstProc.obj
 0001:0001a920       ??_ENonContextualGlyphSubstitutionProcessor@@MAEPAXI@Z 1001b920 f i NonContextualGlyphSubstProc.obj
 0001:0001a920       ??_GNonContextualGlyphSubstitutionProcessor@@MAEPAXI@Z 1001b920 f i NonContextualGlyphSubstProc.obj
 0001:0001a950       ?createInstance@NonContextualGlyphSubstitutionProcessor@@SAPAVSubtableProcessor@@ABV?$LEReferenceTo@UMorphSubtableHeader@@@@AAW4LEErrorCode@@@Z 1001b950 f   NonContextualGlyphSubstProc.obj
 0001:0001aa90       ??0NonContextualGlyphSubstitutionProcessor2@@IAE@ABV?$LEReferenceTo@UMorphSubtableHeader2@@@@AAW4LEErrorCode@@@Z 1001ba90 f   NonContextualGlyphSubstProc2.obj
 0001:0001aab0       ??1NonContextualGlyphSubstitutionProcessor2@@MAE@XZ 1001bab0 f   NonContextualGlyphSubstProc2.obj
 0001:0001aac0       ??_ENonContextualGlyphSubstitutionProcessor2@@MAEPAXI@Z 1001bac0 f i NonContextualGlyphSubstProc2.obj
 0001:0001aac0       ??_GNonContextualGlyphSubstitutionProcessor2@@MAEPAXI@Z 1001bac0 f i NonContextualGlyphSubstProc2.obj
 0001:0001aaf0       ?createInstance@NonContextualGlyphSubstitutionProcessor2@@SAPAVSubtableProcessor2@@ABV?$LEReferenceTo@UMorphSubtableHeader2@@@@AAW4LEErrorCode@@@Z 1001baf0 f   NonContextualGlyphSubstProc2.obj
 0001:0001ac30       ??0OpenTypeLayoutEngine@@QAE@PBVLEFontInstance@@JJJAAW4LEErrorCode@@@Z 1001bc30 f   OpenTypeLayoutEngine.obj
 0001:0001ace0       ??0OpenTypeLayoutEngine@@QAE@PBVLEFontInstance@@JJJABV?$LEReferenceTo@UGlyphSubstitutionTableHeader@@@@AAW4LEErrorCode@@@Z 1001bce0 f   OpenTypeLayoutEngine.obj
 0001:0001ae90       ??1OpenTypeLayoutEngine@@UAE@XZ 1001be90 f   OpenTypeLayoutEngine.obj
 0001:0001aee0       ??_EOpenTypeLayoutEngine@@UAEPAXI@Z 1001bee0 f i OpenTypeLayoutEngine.obj
 0001:0001aee0       ??_GOpenTypeLayoutEngine@@UAEPAXI@Z 1001bee0 f i OpenTypeLayoutEngine.obj
 0001:0001af40       ?adjustGlyphPositions@OpenTypeLayoutEngine@@MAEXQBGJJDAAVLEGlyphStorage@@AAW4LEErrorCode@@@Z 1001bf40 f   OpenTypeLayoutEngine.obj
 0001:0001b2e0       ?applyTypoFlags@OpenTypeLayoutEngine@@AAEXXZ 1001c2e0 f   OpenTypeLayoutEngine.obj
 0001:0001b460       ?characterProcessing@OpenTypeLayoutEngine@@MAEJQBGJJJDAAPAGAAVLEGlyphStorage@@AAW4LEErrorCode@@@Z 1001c460 f   OpenTypeLayoutEngine.obj
 0001:0001b580       ?computeGlyphs@OpenTypeLayoutEngine@@MAEJQBGJJJDAAVLEGlyphStorage@@AAW4LEErrorCode@@@Z 1001c580 f   OpenTypeLayoutEngine.obj
 0001:0001b6a0       ?getDynamicClassID@OpenTypeLayoutEngine@@UBEPBDXZ 1001c6a0 f   OpenTypeLayoutEngine.obj
 0001:0001b6b0       ?getLangSysTag@OpenTypeLayoutEngine@@SAKJ@Z 1001c6b0 f   OpenTypeLayoutEngine.obj
 0001:0001b6d0       ?getScriptTag@OpenTypeLayoutEngine@@SAKJ@Z 1001c6d0 f   OpenTypeLayoutEngine.obj
 0001:0001b6f0       ?getV2ScriptTag@OpenTypeLayoutEngine@@SAKJ@Z 1001c6f0 f   OpenTypeLayoutEngine.obj
 0001:0001b790       ?glyphPostProcessing@OpenTypeLayoutEngine@@MAEJAAVLEGlyphStorage@@0AAW4LEErrorCode@@@Z 1001c790 f   OpenTypeLayoutEngine.obj
 0001:0001b7d0       ?glyphProcessing@OpenTypeLayoutEngine@@MAEJQBGJJJDAAVLEGlyphStorage@@AAW4LEErrorCode@@@Z 1001c7d0 f   OpenTypeLayoutEngine.obj
 0001:0001b8d0       ?glyphSubstitution@OpenTypeLayoutEngine@@MAEJJJDAAVLEGlyphStorage@@AAW4LEErrorCode@@@Z 1001c8d0 f   OpenTypeLayoutEngine.obj
 0001:0001b980       ?reset@OpenTypeLayoutEngine@@MAEXXZ 1001c980 f   OpenTypeLayoutEngine.obj
 0001:0001b990       ?setScriptAndLanguageTags@OpenTypeLayoutEngine@@AAEXXZ 1001c990 f   OpenTypeLayoutEngine.obj
 0001:0001ba70       ?getGlyphRangeIndex@OpenTypeUtilities@@SAJGABV?$LEReferenceToArrayOf@UGlyphRangeRecord@@@@AAW4LEErrorCode@@@Z 1001ca70 f   OpenTypeUtilities.obj
 0001:0001bb90       ?getTagOffset@OpenTypeUtilities@@SAGKABV?$LEReferenceToArrayOf@UTagAndOffsetRecord@@@@AAW4LEErrorCode@@@Z 1001cb90 f   OpenTypeUtilities.obj
 0001:0001bc80       ?highBit@OpenTypeUtilities@@SACJ@Z 1001cc80 f   OpenTypeUtilities.obj
 0001:0001bd00       ?search@OpenTypeUtilities@@SAJKQBKJ@Z 1001cd00 f   OpenTypeUtilities.obj
 0001:0001bd50       ?sort@OpenTypeUtilities@@SAXPAGJ@Z 1001cd50 f   OpenTypeUtilities.obj
 0001:0001bdb0       ?process@PairPositioningFormat2Subtable@@QBEKABV?$LEReferenceTo@UPairPositioningFormat2Subtable@@@@PAVGlyphIterator@@PBVLEFontInstance@@AAW4LEErrorCode@@@Z 1001cdb0 f   PairPositioningSubtables.obj
 0001:0001c240       ?process@PairPositioningSubtable@@QBEKABV?$LEReferenceTo@UPairPositioningSubtable@@@@PAVGlyphIterator@@PBVLEFontInstance@@AAW4LEErrorCode@@@Z 1001d240 f   PairPositioningSubtables.obj
 0001:0001ca60       ?findLanguage@ScriptListTable@@QBE?AV?$LEReferenceTo@ULangSysTable@@@@ABVLETableReference@@KKAAW4LEErrorCode@@D@Z 1001da60 f   ScriptAndLanguage.obj
 0001:0001caf0       ?findLanguage@ScriptTable@@QBE?AV?$LEReferenceTo@ULangSysTable@@@@ABVLETableReference@@KAAW4LEErrorCode@@D@Z 1001daf0 f   ScriptAndLanguage.obj
 0001:0001ccd0       ?findScript@ScriptListTable@@QBE?AV?$LEReferenceTo@UScriptTable@@@@ABVLETableReference@@KAAW4LEErrorCode@@@Z 1001dcd0 f   ScriptAndLanguage.obj
 0001:0001d1d0       ??0SegmentArrayProcessor@@QAE@ABV?$LEReferenceTo@UMorphSubtableHeader@@@@AAW4LEErrorCode@@@Z 1001e1d0 f   SegmentArrayProcessor.obj
 0001:0001d340       ??_ESegmentArrayProcessor@@UAEPAXI@Z 1001e340 f i SegmentArrayProcessor.obj
 0001:0001d340       ??_GSegmentArrayProcessor@@UAEPAXI@Z 1001e340 f i SegmentArrayProcessor.obj
 0001:0001d370       ?getDynamicClassID@SegmentArrayProcessor@@UBEPBDXZ 1001e370 f   SegmentArrayProcessor.obj
 0001:0001d380       ?process@SegmentArrayProcessor@@UAEXAAVLEGlyphStorage@@AAW4LEErrorCode@@@Z 1001e380 f   SegmentArrayProcessor.obj
 0001:0001d470       ??0SegmentArrayProcessor2@@QAE@ABV?$LEReferenceTo@UMorphSubtableHeader2@@@@AAW4LEErrorCode@@@Z 1001e470 f   SegmentArrayProcessor2.obj
 0001:0001d5e0       ??_ESegmentArrayProcessor2@@UAEPAXI@Z 1001e5e0 f i SegmentArrayProcessor2.obj
 0001:0001d5e0       ??_GSegmentArrayProcessor2@@UAEPAXI@Z 1001e5e0 f i SegmentArrayProcessor2.obj
 0001:0001d610       ?getDynamicClassID@SegmentArrayProcessor2@@UBEPBDXZ 1001e610 f   SegmentArrayProcessor2.obj
 0001:0001d620       ?process@SegmentArrayProcessor2@@UAEXAAVLEGlyphStorage@@AAW4LEErrorCode@@@Z 1001e620 f   SegmentArrayProcessor2.obj
 0001:0001d750       ??0SegmentSingleProcessor@@QAE@ABV?$LEReferenceTo@UMorphSubtableHeader@@@@AAW4LEErrorCode@@@Z 1001e750 f   SegmentSingleProcessor.obj
 0001:0001d8c0       ??_ESegmentSingleProcessor@@UAEPAXI@Z 1001e8c0 f i SegmentSingleProcessor.obj
 0001:0001d8c0       ??_GSegmentSingleProcessor@@UAEPAXI@Z 1001e8c0 f i SegmentSingleProcessor.obj
 0001:0001d8f0       ?getDynamicClassID@SegmentSingleProcessor@@UBEPBDXZ 1001e8f0 f   SegmentSingleProcessor.obj
 0001:0001d900       ?process@SegmentSingleProcessor@@UAEXAAVLEGlyphStorage@@AAW4LEErrorCode@@@Z 1001e900 f   SegmentSingleProcessor.obj
 0001:0001d990       ??0SegmentSingleProcessor2@@QAE@ABV?$LEReferenceTo@UMorphSubtableHeader2@@@@AAW4LEErrorCode@@@Z 1001e990 f   SegmentSingleProcessor2.obj
 0001:0001db00       ??_ESegmentSingleProcessor2@@UAEPAXI@Z 1001eb00 f i SegmentSingleProcessor2.obj
 0001:0001db00       ??_GSegmentSingleProcessor2@@UAEPAXI@Z 1001eb00 f i SegmentSingleProcessor2.obj
 0001:0001db30       ?getDynamicClassID@SegmentSingleProcessor2@@UBEPBDXZ 1001eb30 f   SegmentSingleProcessor2.obj
 0001:0001db40       ?process@SegmentSingleProcessor2@@UAEXAAVLEGlyphStorage@@AAW4LEErrorCode@@@Z 1001eb40 f   SegmentSingleProcessor2.obj
 0001:0001dbd0       ??0SimpleArrayProcessor@@QAE@ABV?$LEReferenceTo@UMorphSubtableHeader@@@@AAW4LEErrorCode@@@Z 1001ebd0 f   SimpleArrayProcessor.obj
 0001:0001dd40       ??_ESimpleArrayProcessor@@UAEPAXI@Z 1001ed40 f i SimpleArrayProcessor.obj
 0001:0001dd40       ??_GSimpleArrayProcessor@@UAEPAXI@Z 1001ed40 f i SimpleArrayProcessor.obj
 0001:0001dd70       ?getDynamicClassID@SimpleArrayProcessor@@UBEPBDXZ 1001ed70 f   SimpleArrayProcessor.obj
 0001:0001dd80       ?process@SimpleArrayProcessor@@UAEXAAVLEGlyphStorage@@AAW4LEErrorCode@@@Z 1001ed80 f   SimpleArrayProcessor.obj
 0001:0001de40       ??0SimpleArrayProcessor2@@QAE@ABV?$LEReferenceTo@UMorphSubtableHeader2@@@@AAW4LEErrorCode@@@Z 1001ee40 f   SimpleArrayProcessor2.obj
 0001:0001e0c0       ??_ESimpleArrayProcessor2@@UAEPAXI@Z 1001f0c0 f i SimpleArrayProcessor2.obj
 0001:0001e0c0       ??_GSimpleArrayProcessor2@@UAEPAXI@Z 1001f0c0 f i SimpleArrayProcessor2.obj
 0001:0001e100       ?getDynamicClassID@SimpleArrayProcessor2@@UBEPBDXZ 1001f100 f   SimpleArrayProcessor2.obj
 0001:0001e110       ?process@SimpleArrayProcessor2@@UAEXAAVLEGlyphStorage@@AAW4LEErrorCode@@@Z 1001f110 f   SimpleArrayProcessor2.obj
 0001:0001e190       ?process@SinglePositioningSubtable@@QBEKABV?$LEReferenceTo@USinglePositioningSubtable@@@@PAVGlyphIterator@@PBVLEFontInstance@@AAW4LEErrorCode@@@Z 1001f190 f   SinglePositioningSubtables.obj
 0001:0001e620       ?process@SingleSubstitutionSubtable@@QBEKABV?$LEReferenceTo@USingleSubstitutionSubtable@@@@PAVGlyphIterator@@AAW4LEErrorCode@@PBVLEGlyphFilter@@@Z 1001f620 f   SingleSubstitutionSubtables.obj
 0001:0001eb90       ??0SingleTableProcessor@@QAE@ABV?$LEReferenceTo@UMorphSubtableHeader@@@@AAW4LEErrorCode@@@Z 1001fb90 f   SingleTableProcessor.obj
 0001:0001ed00       ??_ESingleTableProcessor@@UAEPAXI@Z 1001fd00 f i SingleTableProcessor.obj
 0001:0001ed00       ??_GSingleTableProcessor@@UAEPAXI@Z 1001fd00 f i SingleTableProcessor.obj
 0001:0001ed30       ?getDynamicClassID@SingleTableProcessor@@UBEPBDXZ 1001fd30 f   SingleTableProcessor.obj
 0001:0001ed40       ?process@SingleTableProcessor@@UAEXAAVLEGlyphStorage@@AAW4LEErrorCode@@@Z 1001fd40 f   SingleTableProcessor.obj
 0001:0001edc0       ??0SingleTableProcessor2@@QAE@ABV?$LEReferenceTo@UMorphSubtableHeader2@@@@AAW4LEErrorCode@@@Z 1001fdc0 f   SingleTableProcessor2.obj
 0001:0001ef30       ??_ESingleTableProcessor2@@UAEPAXI@Z 1001ff30 f i SingleTableProcessor2.obj
 0001:0001ef30       ??_GSingleTableProcessor2@@UAEPAXI@Z 1001ff30 f i SingleTableProcessor2.obj
 0001:0001ef60       ?getDynamicClassID@SingleTableProcessor2@@UBEPBDXZ 1001ff60 f   SingleTableProcessor2.obj
 0001:0001ef70       ?process@SingleTableProcessor2@@UAEXAAVLEGlyphStorage@@AAW4LEErrorCode@@@Z 1001ff70 f   SingleTableProcessor2.obj
 0001:0001eff0       ??0StateTableProcessor@@IAE@ABV?$LEReferenceTo@UMorphSubtableHeader@@@@AAW4LEErrorCode@@@Z 1001fff0 f   StateTableProcessor.obj
 0001:0001f2c0       ??1StateTableProcessor@@MAE@XZ 100202c0 f   StateTableProcessor.obj
 0001:0001f2e0       ??_EStateTableProcessor@@MAEPAXI@Z 100202e0 f i StateTableProcessor.obj
 0001:0001f2e0       ??_GStateTableProcessor@@MAEPAXI@Z 100202e0 f i StateTableProcessor.obj
 0001:0001f320       ?process@StateTableProcessor@@UAEXAAVLEGlyphStorage@@AAW4LEErrorCode@@@Z 10020320 f   StateTableProcessor.obj
 0001:0001f4a0       ??0StateTableProcessor2@@IAE@ABV?$LEReferenceTo@UMorphSubtableHeader2@@@@AAW4LEErrorCode@@@Z 100204a0 f   StateTableProcessor2.obj
 0001:0001f850       ??1StateTableProcessor2@@MAE@XZ 10020850 f   StateTableProcessor2.obj
 0001:0001f880       ??_EStateTableProcessor2@@MAEPAXI@Z 10020880 f i StateTableProcessor2.obj
 0001:0001f880       ??_GStateTableProcessor2@@MAEPAXI@Z 10020880 f i StateTableProcessor2.obj
 0001:0001f8d0       ?process@StateTableProcessor2@@UAEXAAVLEGlyphStorage@@AAW4LEErrorCode@@@Z 100208d0 f   StateTableProcessor2.obj
 0001:0001fe40       ??0SubtableProcessor@@IAE@ABV?$LEReferenceTo@UMorphSubtableHeader@@@@AAW4LEErrorCode@@@Z 10020e40 f   SubtableProcessor.obj
 0001:0001feb0       ??1SubtableProcessor@@UAE@XZ 10020eb0 f   SubtableProcessor.obj
 0001:0001fec0       ??_ESubtableProcessor@@UAEPAXI@Z 10020ec0 f i SubtableProcessor.obj
 0001:0001fec0       ??_GSubtableProcessor@@UAEPAXI@Z 10020ec0 f i SubtableProcessor.obj
 0001:0001fef0       ??0SubtableProcessor2@@IAE@ABV?$LEReferenceTo@UMorphSubtableHeader2@@@@AAW4LEErrorCode@@@Z 10020ef0 f   SubtableProcessor2.obj
 0001:00020010       ??1SubtableProcessor2@@UAE@XZ 10021010 f   SubtableProcessor2.obj
 0001:00020020       ??_ESubtableProcessor2@@UAEPAXI@Z 10021020 f i SubtableProcessor2.obj
 0001:00020020       ??_GSubtableProcessor2@@UAEPAXI@Z 10021020 f i SubtableProcessor2.obj
 0001:00020050       ?SetIntField@JNIEnv_@@QAEXPAV_jobject@@PAU_jfieldID@@J@Z 10021050 f i SunLayoutEngine.obj
 0001:00020070       ?putGV@@YAHPAUJNIEnv_@@JJPAV_jobject@@PBVLayoutEngine@@H@Z 10021070 f   SunLayoutEngine.obj
 0001:00020270       _Java_sun_font_SunLayoutEngine_initGVIDs@8 10021270 f   SunLayoutEngine.obj
 0001:00020360       _Java_sun_font_SunLayoutEngine_nativeLayout@84 10021360 f   SunLayoutEngine.obj
 0001:00020660       ??0ThaiLayoutEngine@@QAE@PBVLEFontInstance@@JJJAAW4LEErrorCode@@@Z 10021660 f   ThaiLayoutEngine.obj
 0001:00020720       ??_EThaiLayoutEngine@@UAEPAXI@Z 10021720 f i ThaiLayoutEngine.obj
 0001:00020720       ??_GThaiLayoutEngine@@UAEPAXI@Z 10021720 f i ThaiLayoutEngine.obj
 0001:00020750       ?adjustGlyphPositions@ThaiLayoutEngine@@MAEXQBGJJDAAVLEGlyphStorage@@AAW4LEErrorCode@@@Z 10021750 f   ThaiLayoutEngine.obj
 0001:000207f0       ?computeGlyphs@ThaiLayoutEngine@@MAEJQBGJJJDAAVLEGlyphStorage@@AAW4LEErrorCode@@@Z 100217f0 f   ThaiLayoutEngine.obj
 0001:00020910       ?getDynamicClassID@ThaiLayoutEngine@@UBEPBDXZ 10021910 f   ThaiLayoutEngine.obj
 0001:00020920       ?compose@ThaiShaping@@SAJPBGJJEGPAGAAVLEGlyphStorage@@@Z 10021920 f   ThaiShaping.obj
 0001:00020b30       ?doTransition@ThaiShaping@@CAEUStateTransition@1@GJEGPAGAAVLEGlyphStorage@@AAJ@Z 10021b30 f   ThaiShaping.obj
 0001:00020ec0       ??0TibetanOpenTypeLayoutEngine@@QAE@PBVLEFontInstance@@JJJABV?$LEReferenceTo@UGlyphSubstitutionTableHeader@@@@AAW4LEErrorCode@@@Z 10021ec0 f   TibetanLayoutEngine.obj
 0001:00020f00       ??_ETibetanOpenTypeLayoutEngine@@UAEPAXI@Z 10021f00 f i TibetanLayoutEngine.obj
 0001:00020f00       ??_GTibetanOpenTypeLayoutEngine@@UAEPAXI@Z 10021f00 f i TibetanLayoutEngine.obj
 0001:00020f30       ?characterProcessing@TibetanOpenTypeLayoutEngine@@MAEJQBGJJJDAAPAGAAVLEGlyphStorage@@AAW4LEErrorCode@@@Z 10021f30 f   TibetanLayoutEngine.obj
 0001:00021050       ?getDynamicClassID@TibetanOpenTypeLayoutEngine@@UBEPBDXZ 10022050 f   TibetanLayoutEngine.obj
 0001:00021060       ?getFeatureMap@TibetanReordering@@SAPBUFeatureMap@@AAJ@Z 10022060 f   TibetanReordering.obj
 0001:00021070       ?reorder@TibetanReordering@@SAJPBGJJPAGAAVLEGlyphStorage@@@Z 10022070 f   TibetanReordering.obj
 0001:000213a0       ??0TrimmedArrayProcessor@@QAE@ABV?$LEReferenceTo@UMorphSubtableHeader@@@@AAW4LEErrorCode@@@Z 100223a0 f   TrimmedArrayProcessor.obj
 0001:00021550       ??_ETrimmedArrayProcessor@@UAEPAXI@Z 10022550 f i TrimmedArrayProcessor.obj
 0001:00021550       ??_GTrimmedArrayProcessor@@UAEPAXI@Z 10022550 f i TrimmedArrayProcessor.obj
 0001:00021580       ?getDynamicClassID@TrimmedArrayProcessor@@UBEPBDXZ 10022580 f   TrimmedArrayProcessor.obj
 0001:00021590       ?process@TrimmedArrayProcessor@@UAEXAAVLEGlyphStorage@@AAW4LEErrorCode@@@Z 10022590 f   TrimmedArrayProcessor.obj
 0001:00021600       ??0TrimmedArrayProcessor2@@QAE@ABV?$LEReferenceTo@UMorphSubtableHeader2@@@@AAW4LEErrorCode@@@Z 10022600 f   TrimmedArrayProcessor2.obj
 0001:000218a0       ??_ETrimmedArrayProcessor2@@UAEPAXI@Z 100228a0 f i TrimmedArrayProcessor2.obj
 0001:000218a0       ??_GTrimmedArrayProcessor2@@UAEPAXI@Z 100228a0 f i TrimmedArrayProcessor2.obj
 0001:000218e0       ?getDynamicClassID@TrimmedArrayProcessor2@@UBEPBDXZ 100228e0 f   TrimmedArrayProcessor2.obj
 0001:000218f0       ?process@TrimmedArrayProcessor2@@UAEXAAVLEGlyphStorage@@AAW4LEErrorCode@@@Z 100228f0 f   TrimmedArrayProcessor2.obj
 0001:00021970       ?adjustPosition@ValueRecord@@QBEXFGABVLETableReference@@AAVGlyphIterator@@PBVLEFontInstance@@AAW4LEErrorCode@@@Z 10022970 f   ValueRecords.obj
 0001:00021e70       ?adjustPosition@ValueRecord@@QBEXGABVLETableReference@@AAVGlyphIterator@@PBVLEFontInstance@@AAW4LEErrorCode@@@Z 10022e70 f   ValueRecords.obj
 0001:000222f0       ?getFieldValue@ValueRecord@@QBEFFGF@Z 100232f0 f   ValueRecords.obj
 0001:00022360       ?getSize@ValueRecord@@SAFG@Z 10023360 f   ValueRecords.obj
 0001:00022910       _Java_sun_awt_Win32FontManager_getFontPath@12 10023910 f   fontpath.obj
 0001:00022a90       _Java_sun_awt_Win32FontManager_populateFontFileNameMap0@24 10023a90 f   fontpath.obj
 0001:00023250       _StringCchCatA@12          10024250 f i fontpath.obj
 0001:000236d0       _Java_sun_font_FreetypeFontScaler_createScalerContextNative@36 100246d0 f   freetypeScaler.obj
 0001:000238d0       _Java_sun_font_FreetypeFontScaler_disposeNativeScaler@20 100248d0 f   freetypeScaler.obj
 0001:00023940       _Java_sun_font_FreetypeFontScaler_getFontMetricsNative@28 10024940 f   freetypeScaler.obj
 0001:00023c90       _Java_sun_font_FreetypeFontScaler_getGlyphAdvanceNative@32 10024c90 f   freetypeScaler.obj
 0001:00023cf0       _Java_sun_font_FreetypeFontScaler_getGlyphCodeNative@24 10024cf0 f   freetypeScaler.obj
 0001:00023da0       _Java_sun_font_FreetypeFontScaler_getGlyphImageNative@32 10024da0 f   freetypeScaler.obj
 0001:00023dd0       _Java_sun_font_FreetypeFontScaler_getGlyphMetricsNative@36 10024dd0 f   freetypeScaler.obj
 0001:00023e90       _Java_sun_font_FreetypeFontScaler_getGlyphOutlineBoundsNative@32 10024e90 f   freetypeScaler.obj
 0001:00024010       _Java_sun_font_FreetypeFontScaler_getGlyphOutlineNative@40 10025010 f   freetypeScaler.obj
 0001:00024070       _Java_sun_font_FreetypeFontScaler_getGlyphPointNative@36 10025070 f   freetypeScaler.obj
 0001:00024140       _Java_sun_font_FreetypeFontScaler_getGlyphVectorOutlineNative@44 10025140 f   freetypeScaler.obj
 0001:00024390       _Java_sun_font_FreetypeFontScaler_getLayoutTableCacheNative@16 10025390 f   freetypeScaler.obj
 0001:000243e0       _Java_sun_font_FreetypeFontScaler_getMissingGlyphCodeNative@16 100253e0 f   freetypeScaler.obj
 0001:000243f0       _Java_sun_font_FreetypeFontScaler_getNumGlyphsNative@16 100253f0 f   freetypeScaler.obj
 0001:00024480       _Java_sun_font_FreetypeFontScaler_getUnitsPerEMNative@16 10025480 f   freetypeScaler.obj
 0001:000244a0       _Java_sun_font_FreetypeFontScaler_initIDs@12 100254a0 f   freetypeScaler.obj
 0001:000244d0       _Java_sun_font_FreetypeFontScaler_initNativeScaler@28 100254d0 f   freetypeScaler.obj
 0001:000252a0       _Java_sun_font_FileFontStrike__1getGlyphImageFromWindows@32 100262a0 f   lcdglyph.obj
 0001:00025c30       _Java_sun_font_FileFontStrike_initNative@8 10026c30 f   lcdglyph.obj
 0001:00025c60       _Java_sun_font_NullFontScaler_getGlyphImage@20 10026c60 f   sunFont.obj
 0001:00025c80       _Java_sun_font_NullFontScaler_getNullScalerContext@8 10026c80 f   sunFont.obj
 0001:00025ca0       _Java_sun_font_StrikeCache_freeIntMemory@20 10026ca0 f   sunFont.obj
 0001:00025d50       _Java_sun_font_StrikeCache_freeIntPointer@12 10026d50 f   sunFont.obj
 0001:00025d70       _Java_sun_font_StrikeCache_freeLongMemory@20 10026d70 f   sunFont.obj
 0001:00025e20       _Java_sun_font_StrikeCache_freeLongPointer@16 10026e20 f   sunFont.obj
 0001:00025e40       _Java_sun_font_StrikeCache_getGlyphCacheDescription@12 10026e40 f   sunFont.obj
 0001:00025f60       _Java_sun_font_SunFontManager_initIDs@8 10026f60 f   sunFont.obj
 0001:00025f70       _freeLayoutTableCache      10026f70 f   sunFont.obj
 0001:00025fb0       _getSunFontIDs             10026fb0 f   sunFont.obj
 0001:000265b0       _isNullScalerContext       100275b0 f   sunFont.obj
 0001:000265c0       _newLayoutTableCache       100275c0 f   sunFont.obj
 0001:00026600       _FT_Add_Default_Modules    10027600 f   freetype:ftinit.obj
 0001:00026630       _FT_Done_FreeType          10027630 f   freetype:ftinit.obj
 0001:00026660       _FT_Init_FreeType          10027660 f   freetype:ftinit.obj
 0001:00026a40       _FT_Activate_Size          10027a40 f   freetype:ftbase.obj
 0001:00026aa0       _FT_Add_Module             10027aa0 f   freetype:ftbase.obj
 0001:00026c80       _FT_CMap_New               10027c80 f   freetype:ftbase.obj
 0001:00026d60       _FT_DivFix                 10027d60 f   freetype:ftbase.obj
 0001:00026e00       _FT_Done_Face              10027e00 f   freetype:ftbase.obj
 0001:00026e90       _FT_Done_GlyphSlot         10027e90 f   freetype:ftbase.obj
 0001:00026f00       _FT_Done_Library           10027f00 f   freetype:ftbase.obj
 0001:00027040       _FT_Done_Size              10028040 f   freetype:ftbase.obj
 0001:000270f0       _FT_Get_Advance            100280f0 f   freetype:ftbase.obj
 0001:00027180       _FT_Get_Advances           10028180 f   freetype:ftbase.obj
 0001:00027280       _FT_Get_CMap_Format        10028280 f   freetype:ftbase.obj
 0001:000272d0       _FT_Get_Char_Index         100282d0 f   freetype:ftbase.obj
 0001:00027300       _FT_Get_Glyph_Name         10028300 f   freetype:ftbase.obj
 0001:00027390       _FT_Get_Module             10028390 f   freetype:ftbase.obj
 0001:00027400       _FT_Get_Module_Interface   10028400 f   freetype:ftbase.obj
 0001:00027420       _FT_Get_Next_Char          10028420 f   freetype:ftbase.obj
 0001:00027470       _FT_GlyphLoader_Add        10028470 f   freetype:ftbase.obj
 0001:000275d0       _FT_GlyphLoader_CheckPoints 100285d0 f   freetype:ftbase.obj
 0001:00027750       _FT_GlyphLoader_CheckSubGlyphs 10028750 f   freetype:ftbase.obj
 0001:000277b0       _FT_GlyphLoader_CopyPoints 100287b0 f   freetype:ftbase.obj
 0001:00027880       _FT_GlyphLoader_CreateExtra 10028880 f   freetype:ftbase.obj
 0001:000278d0       _FT_GlyphLoader_Done       100288d0 f   freetype:ftbase.obj
 0001:00027900       _FT_GlyphLoader_New        10028900 f   freetype:ftbase.obj
 0001:00027930       _FT_GlyphLoader_Prepare    10028930 f   freetype:ftbase.obj
 0001:00027960       _FT_GlyphLoader_Reset      10028960 f   freetype:ftbase.obj
 0001:000279f0       _FT_GlyphLoader_Rewind     100289f0 f   freetype:ftbase.obj
 0001:00027a20       _FT_Hypot                  10028a20 f   freetype:ftbase.obj
 0001:00027a50       _FT_List_Add               10028a50 f   freetype:ftbase.obj
 0001:00027a80       _FT_List_Finalize          10028a80 f   freetype:ftbase.obj
 0001:00027ae0       _FT_List_Find              10028ae0 f   freetype:ftbase.obj
 0001:00027b00       _FT_List_Remove            10028b00 f   freetype:ftbase.obj
 0001:00027b30       _FT_List_Up                10028b30 f   freetype:ftbase.obj
 0001:00027b80       _FT_Load_Glyph             10028b80 f   freetype:ftbase.obj
 0001:00027e90       _FT_Lookup_Renderer        10028e90 f   freetype:ftbase.obj
 0001:00027ef0       _FT_MSB                    10028ef0 f   freetype:ftbase.obj
 0001:00027f50       _FT_Match_Size             10028f50 f   freetype:ftbase.obj
 0001:00028040       _FT_Matrix_Invert          10029040 f   freetype:ftbase.obj
 0001:000280c0       _FT_Matrix_Multiply        100290c0 f   freetype:ftbase.obj
 0001:00028170       _FT_Matrix_Multiply_Scaled 10029170 f   freetype:ftbase.obj
 0001:00028260       _FT_MulDiv                 10029260 f   freetype:ftbase.obj
 0001:00028350       _FT_MulDiv_No_Round        10029350 f   freetype:ftbase.obj
 0001:00028410       _FT_MulFix                 10029410 f   freetype:ftbase.obj
 0001:00028440       _FT_New_GlyphSlot          10029440 f   freetype:ftbase.obj
 0001:000284f0       _FT_New_Library            100294f0 f   freetype:ftbase.obj
 0001:00028590       _FT_New_Memory_Face        10029590 f   freetype:ftbase.obj
 0001:000285e0       _FT_New_Size               100295e0 f   freetype:ftbase.obj
 0001:000286c0       _FT_Open_Face              100296c0 f   freetype:ftbase.obj
 0001:00028a70       _FT_Outline_Check          10029a70 f   freetype:ftbase.obj
 0001:00028ae0       _FT_Outline_Decompose      10029ae0 f   freetype:ftbase.obj
 0001:00028e40       _FT_Outline_EmboldenXY     10029e40 f   freetype:ftbase.obj
 0001:00029110       _FT_Outline_Get_CBox       1002a110 f   freetype:ftbase.obj
 0001:000291c0       _FT_Outline_Get_Orientation 1002a1c0 f   freetype:ftbase.obj
 0001:00029380       _FT_Outline_Transform      1002a380 f   freetype:ftbase.obj
 0001:000293c0       _FT_Outline_Translate      1002a3c0 f   freetype:ftbase.obj
 0001:00029400       _FT_Property_Set           1002a400 f   freetype:ftbase.obj
 0001:00029420       _FT_Raccess_Get_DataOffsets 1002a420 f   freetype:ftbase.obj
 0001:00029640       _FT_Raccess_Get_HeaderInfo 1002a640 f   freetype:ftbase.obj
 0001:00029840       _FT_Raccess_Guess          1002a840 f   freetype:ftbase.obj
 0001:000298d0       _FT_Remove_Module          1002a8d0 f   freetype:ftbase.obj
 0001:00029940       _FT_Render_Glyph           1002a940 f   freetype:ftbase.obj
 0001:00029970       _FT_Render_Glyph_Internal  1002a970 f   freetype:ftbase.obj
 0001:00029a40       _FT_Request_Metrics        1002aa40 f   freetype:ftbase.obj
 0001:00029c70       _FT_Request_Size           1002ac70 f   freetype:ftbase.obj
 0001:00029d00       _FT_RoundFix               1002ad00 f   freetype:ftbase.obj
 0001:00029d30       _FT_Select_Charmap         1002ad30 f   freetype:ftbase.obj
 0001:00029da0       _FT_Select_Metrics         1002ada0 f   freetype:ftbase.obj
 0001:00029e40       _FT_Select_Size            1002ae40 f   freetype:ftbase.obj
 0001:00029e90       _FT_Set_Char_Size          1002ae90 f   freetype:ftbase.obj
 0001:00029f20       _FT_Set_Charmap            1002af20 f   freetype:ftbase.obj
 0001:00029f90       _FT_Set_Renderer           1002af90 f   freetype:ftbase.obj
 0001:0002a030       _FT_Set_Transform          1002b030 f   freetype:ftbase.obj
 0001:0002a0d0       _FT_Stream_Close           1002b0d0 f   freetype:ftbase.obj
 0001:0002a0f0       _FT_Stream_EnterFrame      1002b0f0 f   freetype:ftbase.obj
 0001:0002a1b0       _FT_Stream_ExitFrame       1002b1b0 f   freetype:ftbase.obj
 0001:0002a1f0       _FT_Stream_ExtractFrame    1002b1f0 f   freetype:ftbase.obj
 0001:0002a220       _FT_Stream_Free            1002b220 f   freetype:ftbase.obj
 0001:0002a250       _FT_Stream_GetChar         1002b250 f   freetype:ftbase.obj
 0001:0002a270       _FT_Stream_GetULong        1002b270 f   freetype:ftbase.obj
 0001:0002a2c0       _FT_Stream_GetULongLE      1002b2c0 f   freetype:ftbase.obj
 0001:0002a310       _FT_Stream_GetUShort       1002b310 f   freetype:ftbase.obj
 0001:0002a350       _FT_Stream_GetUShortLE     1002b350 f   freetype:ftbase.obj
 0001:0002a390       _FT_Stream_New             1002b390 f   freetype:ftbase.obj
 0001:0002a470       _FT_Stream_OpenMemory      1002b470 f   freetype:ftbase.obj
 0001:0002a4a0       _FT_Stream_Pos             1002b4a0 f   freetype:ftbase.obj
 0001:0002a4b0       _FT_Stream_Read            1002b4b0 f   freetype:ftbase.obj
 0001:0002a4d0       _FT_Stream_ReadAt          1002b4d0 f   freetype:ftbase.obj
 0001:0002a550       _FT_Stream_ReadChar        1002b550 f   freetype:ftbase.obj
 0001:0002a5b0       _FT_Stream_ReadFields      1002b5b0 f   freetype:ftbase.obj
 0001:0002a7d0       _FT_Stream_ReadULong       1002b7d0 f   freetype:ftbase.obj
 0001:0002a850       _FT_Stream_ReadULongLE     1002b850 f   freetype:ftbase.obj
 0001:0002a8d0       _FT_Stream_ReadUOffset     1002b8d0 f   freetype:ftbase.obj
 0001:0002a950       _FT_Stream_ReadUShort      1002b950 f   freetype:ftbase.obj
 0001:0002a9d0       _FT_Stream_ReadUShortLE    1002b9d0 f   freetype:ftbase.obj
 0001:0002aa50       _FT_Stream_ReleaseFrame    1002ba50 f   freetype:ftbase.obj
 0001:0002aa90       _FT_Stream_Seek            1002ba90 f   freetype:ftbase.obj
 0001:0002aad0       _FT_Stream_Skip            1002bad0 f   freetype:ftbase.obj
 0001:0002ab00       _FT_Stream_TryRead         1002bb00 f   freetype:ftbase.obj
 0001:0002ab60       _FT_Vector_Length          1002bb60 f   freetype:ftbase.obj
 0001:0002abd0       _FT_Vector_Transform       1002bbd0 f   freetype:ftbase.obj
 0001:0002ac30       _FT_Vector_Transform_Scaled 1002bc30 f   freetype:ftbase.obj
 0001:0002b580       _ft_corner_is_flat         1002c580 f   freetype:ftbase.obj
 0001:0002b5f0       _ft_corner_orientation     1002c5f0 f   freetype:ftbase.obj
 0001:0002b710       _ft_glyphslot_alloc_bitmap 1002c710 f   freetype:ftbase.obj
 0001:0002b890       _ft_glyphslot_free_bitmap  1002c890 f   freetype:ftbase.obj
 0001:0002ba10       _ft_glyphslot_set_bitmap   1002ca10 f   freetype:ftbase.obj
 0001:0002ba30       _ft_highpow2               1002ca30 f   freetype:ftbase.obj
 0001:0002bc20       _ft_mem_alloc              1002cc20 f   freetype:ftbase.obj
 0001:0002bc60       _ft_mem_dup                1002cc60 f   freetype:ftbase.obj
 0001:0002bcb0       _ft_mem_free               1002ccb0 f   freetype:ftbase.obj
 0001:0002bcd0       _ft_mem_qalloc             1002ccd0 f   freetype:ftbase.obj
 0001:0002bd20       _ft_mem_qrealloc           1002cd20 f   freetype:ftbase.obj
 0001:0002be20       _ft_mem_realloc            1002ce20 f   freetype:ftbase.obj
 0001:0002be90       _ft_mem_strcpyn            1002ce90 f   freetype:ftbase.obj
 0001:0002bec0       _ft_mem_strdup             1002cec0 f   freetype:ftbase.obj
 0001:0002bf10       _ft_module_get_service     1002cf10 f   freetype:ftbase.obj
 0001:0002c220       _ft_service_list_lookup    1002d220 f   freetype:ftbase.obj
 0001:0002c2b0       _ft_synthesize_vertical_metrics 1002d2b0 f   freetype:ftbase.obj
 0001:0002c4c0       _ft_validator_error        1002d4c0 f   freetype:ftbase.obj
 0001:0002c4e0       _ft_validator_init         1002d4e0 f   freetype:ftbase.obj
 0001:0002cf10       _FT_Outline_Get_BBox       1002df10 f   freetype:ftbbox.obj
 0001:0002d1c0       _FT_GlyphSlot_Embolden     1002e1c0 f   freetype:ftsynth.obj
 0001:0002d2c0       _FT_Library_SetLcdFilter   1002e2c0 f   freetype:ftlcdfil.obj
 0001:0002f9e0       _af_get_char_index         100309e0 f   freetype:autofit.obj
 0001:00038720       _TT_New_Context            10039720 f   freetype:truetype.obj
 0001:00038e00       _TT_RunIns                 10039e00 f   freetype:truetype.obj
 0001:00059150       _ps_hints_apply            1005a150 f   freetype:pshinter.obj
 0001:000681e0       ___local_stdio_printf_options 100691e0 f i freetype:bdf.obj
 0001:0006af40       _sprintf                   1006bf40 f i freetype:bdf.obj
 0001:0006af80       _FT_Done_Memory            1006bf80 f   freetype:ftsystem.obj
 0001:0006af90       _FT_New_Memory             1006bf90 f   freetype:ftsystem.obj
 0001:0006afc0       _FT_Stream_Open            1006bfc0 f   freetype:ftsystem.obj
 0001:0006b130       _FT_Bitmap_Convert         1006c130 f   freetype:ftbitmap.obj
 0001:0006b550       _FT_Bitmap_Copy            1006c550 f   freetype:ftbitmap.obj
 0001:0006b610       _FT_Bitmap_Done            1006c610 f   freetype:ftbitmap.obj
 0001:0006b660       _FT_Bitmap_Embolden        1006c660 f   freetype:ftbitmap.obj
 0001:0006b930       _FT_Bitmap_New             1006c930 f   freetype:ftbitmap.obj
 0001:0006b950       _FT_GlyphSlot_Own_Bitmap   1006c950 f   freetype:ftbitmap.obj
 0001:0006bd70       _FT_Gzip_Uncompress        1006cd70 f   freetype:ftgzip.obj
 0001:0006be40       _FT_Stream_OpenGzip        1006ce40 f   freetype:ftgzip.obj
 0001:0006e5f0       _FT_Stream_OpenLZW         1006f5f0 f   freetype:ftlzw.obj
 0001:0006e9b0       _ft_lzwstate_done          1006f9b0 f   freetype:ftlzw.obj
 0001:0006eae0       _ft_lzwstate_init          1006fae0 f   freetype:ftlzw.obj
 0001:0006eb40       _ft_lzwstate_io            1006fb40 f   freetype:ftlzw.obj
 0001:0006eeb0       _ft_lzwstate_reset         1006feb0 f   freetype:ftlzw.obj
 0001:0006ef5f       _JNU_ThrowArrayIndexOutOfBoundsException@8 1006ff5f f   java:java.dll
 0001:0006ef65       _JNU_ThrowInternalError@8  1006ff65 f   java:java.dll
 0001:0006ef6b       _JNU_NewStringPlatform@8   1006ff6b f   java:java.dll
 0001:0006ef71       _SurfaceData_GetOps@8      1006ff71 f   awt:awt.dll
 0001:0006ef77       _SurfaceData_IntersectBounds@8 1006ff77 f   awt:awt.dll
 0001:0006ef7d       _GetNativePrim@8           1006ff7d f   awt:awt.dll
 0001:0006ef83       _GrPrim_Sg2dGetCompInfo@16 1006ff83 f   awt:awt.dll
 0001:0006ef89       _GrPrim_Sg2dGetClip@12     1006ff89 f   awt:awt.dll
 0001:0006ef8f       _GrPrim_Sg2dGetPixel@8     1006ff8f f   awt:awt.dll
 0001:0006ef95       _GrPrim_Sg2dGetEaRGB@8     1006ff95 f   awt:awt.dll
 0001:0006ef9b       _GrPrim_Sg2dGetLCDTextContrast@8 1006ff9b f   awt:awt.dll
 0001:0006efa1       _AccelGlyphCache_RemoveAllCellInfos 1006ffa1 f   awt:awt.dll
 0001:0006efa7       ??2@YAPAXI@Z               1006ffa7 f   MSVCRT:new_scalar.obj
 0001:0006efe0       __ftol2_sse                1006ffe0 f   MSVCRT:ftol2.obj
 0001:0006eff0       __ftoi2                    1006fff0 f   MSVCRT:ftol2.obj
 0001:0006f06c       ??3@YAXPAXI@Z              1007006c f   MSVCRT:delete_scalar_size.obj
 0001:0006f07a       ??_Etype_info@@UAEPAXI@Z   1007007a f i MSVCRT:std_type_info_static.obj
 0001:0006f07a       ??_Gtype_info@@UAEPAXI@Z   1007007a f i MSVCRT:std_type_info_static.obj
 0001:0006f09d       @__security_check_cookie@4 1007009d f   MSVCRT:secchk.obj
 0001:0006f0ab       ??_U@YAPAXI@Z              100700ab f   MSVCRT:new_array.obj
 0001:0006f0b4       ??_V@YAXPAXI@Z             100700b4 f   MSVCRT:delete_array_size.obj
 0001:0006f0d0       __ftol3                    100700d0 f   MSVCRT:ftol3.obj
 0001:0006f140       __alloca_probe_16          10070140 f   MSVCRT:alloca16.obj
 0001:0006f156       __alloca_probe_8           10070156     MSVCRT:alloca16.obj
 0001:0006f4ac       __DllMainCRTStartup@12     100704ac f   MSVCRT:dll_dllmain.obj
 0001:0006f4d0       __alloca_probe             100704d0 f   MSVCRT:chkstk.obj
 0001:0006f4d0       __chkstk                   100704d0 f   MSVCRT:chkstk.obj
 0001:0006f4fb       ___isa_available_init      100704fb f   MSVCRT:cpu_disp.obj
 0001:0006f6cf       ??0bad_alloc@std@@QAE@ABV01@@Z 100706cf f i MSVCRT:throw_bad_alloc.obj
 0001:0006f6ea       ??0bad_alloc@std@@QAE@XZ   100706ea f i MSVCRT:throw_bad_alloc.obj
 0001:0006f702       ??0bad_array_new_length@std@@QAE@ABV01@@Z 10070702 f i MSVCRT:throw_bad_alloc.obj
 0001:0006f71d       ??0bad_array_new_length@std@@QAE@XZ 1007071d f i MSVCRT:throw_bad_alloc.obj
 0001:0006f735       ??0exception@std@@QAE@ABV01@@Z 10070735 f i MSVCRT:throw_bad_alloc.obj
 0001:0006f761       ??1bad_alloc@std@@UAE@XZ   10070761 f i MSVCRT:throw_bad_alloc.obj
 0001:0006f761       ??1bad_array_new_length@std@@UAE@XZ 10070761 f i MSVCRT:throw_bad_alloc.obj
 0001:0006f772       ??_Ebad_alloc@std@@UAEPAXI@Z 10070772 f i MSVCRT:throw_bad_alloc.obj
 0001:0006f772       ??_Ebad_array_new_length@std@@UAEPAXI@Z 10070772 f i MSVCRT:throw_bad_alloc.obj
 0001:0006f772       ??_Eexception@std@@UAEPAXI@Z 10070772 f i MSVCRT:throw_bad_alloc.obj
 0001:0006f772       ??_Gbad_alloc@std@@UAEPAXI@Z 10070772 f i MSVCRT:throw_bad_alloc.obj
 0001:0006f772       ??_Gbad_array_new_length@std@@UAEPAXI@Z 10070772 f i MSVCRT:throw_bad_alloc.obj
 0001:0006f772       ??_Gexception@std@@UAEPAXI@Z 10070772 f i MSVCRT:throw_bad_alloc.obj
 0001:0006f79f       ?__scrt_throw_std_bad_alloc@@YAXXZ 1007079f f   MSVCRT:throw_bad_alloc.obj
 0001:0006f7bc       ?__scrt_throw_std_bad_array_new_length@@YAXXZ 100707bc f   MSVCRT:throw_bad_alloc.obj
 0001:0006f7d9       ?what@exception@std@@UBEPBDXZ 100707d9 f i MSVCRT:throw_bad_alloc.obj
 0001:0006f7e6       ??3@YAXPAX@Z               100707e6 f   MSVCRT:delete_scalar.obj
 0001:0006f7eb       ___raise_securityfailure   100707eb f   MSVCRT:gs_report.obj
 0001:0006f813       ___report_gsfailure        10070813 f   MSVCRT:gs_report.obj
 0001:0006f90d       ??_V@YAXPAX@Z              1007090d f   MSVCRT:delete_array.obj
 0001:0006f95f       ___security_init_cookie    1007095f f   MSVCRT:gs_support.obj
 0001:0006f9aa       _DllMain@12                100709aa f   MSVCRT:dll_dllmain_stub.obj
 0001:0006f9cc       ?__scrt_initialize_type_info@@YAXXZ 100709cc f   MSVCRT:tncleanup.obj
 0001:0006f9d8       ?__scrt_uninitialize_type_info@@YAXXZ 100709d8 f   MSVCRT:tncleanup.obj
 0001:0006f9e4       ___local_stdio_scanf_options 100709e4 f i MSVCRT:default_local_stdio_options.obj
 0001:0006f9ea       ___scrt_initialize_default_local_stdio_options 100709ea f   MSVCRT:default_local_stdio_options.obj
 0001:0006fa4b       ___scrt_acquire_startup_lock 10070a4b f   MSVCRT:utility.obj
 0001:0006fa7d       ___scrt_dllmain_after_initialize_c 10070a7d f   MSVCRT:utility.obj
 0001:0006faa8       ___scrt_dllmain_before_initialize_c 10070aa8 f   MSVCRT:utility.obj
 0001:0006fab6       ___scrt_dllmain_crt_thread_attach 10070ab6 f   MSVCRT:utility.obj
 0001:0006fad5       ___scrt_dllmain_crt_thread_detach 10070ad5 f   MSVCRT:utility.obj
 0001:0006fae2       ___scrt_dllmain_exception_filter 10070ae2 f   MSVCRT:utility.obj
 0001:0006fb16       ___scrt_dllmain_uninitialize_c 10070b16 f   MSVCRT:utility.obj
 0001:0006fb39       ___scrt_dllmain_uninitialize_critical 10070b39 f   MSVCRT:utility.obj
 0001:0006fb46       ___scrt_initialize_crt     10070b46 f   MSVCRT:utility.obj
 0001:0006fb7f       ___scrt_initialize_onexit_tables 10070b7f f   MSVCRT:utility.obj
 0001:0006fc06       ___scrt_is_nonwritable_in_current_image 10070c06 f   MSVCRT:utility.obj
 0001:0006fc9a       ___scrt_release_startup_lock 10070c9a f   MSVCRT:utility.obj
 0001:0006fcb7       ___scrt_uninitialize_crt   10070cb7 f   MSVCRT:utility.obj
 0001:0006fcdf       ___scrt_get_dyn_tls_init_callback 10070cdf f   MSVCRT:dyn_tls_init.obj
 0001:0006fce5       ___scrt_fastfail           10070ce5 f   MSVCRT:utility_desktop.obj
 0001:0006fe00       __crt_debugger_hook        10070e00 f   MSVCRT:utility_desktop.obj
 0001:0006fe08       __RTC_Initialize           10070e08 f   MSVCRT:initsect.obj
 0001:0006fe34       __RTC_Terminate            10070e34 f   MSVCRT:initsect.obj
 0001:0006fe60       __SEH_prolog4              10070e60 f   MSVCRT:sehprolg4.obj
 0001:0006fea5       __except_handler4          10070ea5 f   MSVCRT:chandler4gs.obj
 0001:0006fed4       __get_startup_argv_mode    10070ed4 f   MSVCRT:argv_mode.obj
 0001:0006fed8       ___scrt_is_ucrt_dll_in_use 10070ed8 f   MSVCRT:ucrt_detection.obj
 0001:0006fee4       _memset                    10070ee4 f   vcruntime:VCRUNTIME140.dll
 0001:0006feea       __purecall                 10070eea f   vcruntime:VCRUNTIME140.dll
 0001:0006fef0       _memcpy                    10070ef0 f   vcruntime:VCRUNTIME140.dll
 0001:0006fef6       _strrchr                   10070ef6 f   vcruntime:VCRUNTIME140.dll
 0001:0006fefc       _strstr                    10070efc f   vcruntime:VCRUNTIME140.dll
 0001:0006ff02       _wcsrchr                   10070f02 f   vcruntime:VCRUNTIME140.dll
 0001:0006ff08       _wcsstr                    10070f08 f   vcruntime:VCRUNTIME140.dll
 0001:0006ff0e       _longjmp                   10070f0e f   vcruntime:VCRUNTIME140.dll
 0001:0006ff14       _memmove                   10070f14 f   vcruntime:VCRUNTIME140.dll
 0001:0006ff1a       _memchr                    10070f1a f   vcruntime:VCRUNTIME140.dll
 0001:0006ff20       __setjmp3                  10070f20 f   vcruntime:VCRUNTIME140.dll
 0001:0006ff26       ___std_exception_copy      10070f26 f   vcruntime:VCRUNTIME140.dll
 0001:0006ff2c       ___std_exception_destroy   10070f2c f   vcruntime:VCRUNTIME140.dll
 0001:0006ff32       __CxxThrowException@8      10070f32 f   vcruntime:VCRUNTIME140.dll
 0001:0006ff38       ___std_type_info_destroy_list 10070f38 f   vcruntime:VCRUNTIME140.dll
 0001:0006ff3e       __except_handler4_common   10070f3e f   vcruntime:VCRUNTIME140.dll
 0001:0006ff44       _free                      10070f44 f   ucrt:api-ms-win-crt-heap-l1-1-0.dll
 0001:0006ff4a       _malloc                    10070f4a f   ucrt:api-ms-win-crt-heap-l1-1-0.dll
 0001:0006ff50       __libm_sse2_pow_precise    10070f50 f   ucrt:api-ms-win-crt-math-l1-1-0.dll
 0001:0006ff56       _floor                     10070f56 f   ucrt:api-ms-win-crt-math-l1-1-0.dll
 0001:0006ff5c       _realloc                   10070f5c f   ucrt:api-ms-win-crt-heap-l1-1-0.dll
 0001:0006ff62       __libm_sse2_sqrt_precise   10070f62 f   ucrt:api-ms-win-crt-math-l1-1-0.dll
 0001:0006ff68       _strncpy                   10070f68 f   ucrt:api-ms-win-crt-string-l1-1-0.dll
 0001:0006ff6e       _qsort                     10070f6e f   ucrt:api-ms-win-crt-utility-l1-1-0.dll
 0001:0006ff74       _strncmp                   10070f74 f   ucrt:api-ms-win-crt-string-l1-1-0.dll
 0001:0006ff7a       _atol                      10070f7a f   ucrt:api-ms-win-crt-convert-l1-1-0.dll
 0001:0006ff80       ___stdio_common_vsprintf   10070f80 f   ucrt:api-ms-win-crt-stdio-l1-1-0.dll
 0001:0006ff86       _fclose                    10070f86 f   ucrt:api-ms-win-crt-stdio-l1-1-0.dll
 0001:0006ff8c       _fopen                     10070f8c f   ucrt:api-ms-win-crt-stdio-l1-1-0.dll
 0001:0006ff92       _fread                     10070f92 f   ucrt:api-ms-win-crt-stdio-l1-1-0.dll
 0001:0006ff98       _fseek                     10070f98 f   ucrt:api-ms-win-crt-stdio-l1-1-0.dll
 0001:0006ff9e       _ftell                     10070f9e f   ucrt:api-ms-win-crt-stdio-l1-1-0.dll
 0001:0006ffa4       __callnewh                 10070fa4 f   ucrt:api-ms-win-crt-heap-l1-1-0.dll
 0001:0006ffaa       __initterm                 10070faa f   ucrt:api-ms-win-crt-runtime-l1-1-0.dll
 0001:0006ffb0       __initterm_e               10070fb0 f   ucrt:api-ms-win-crt-runtime-l1-1-0.dll
 0001:0006ffb6       __seh_filter_dll           10070fb6 f   ucrt:api-ms-win-crt-runtime-l1-1-0.dll
 0001:0006ffbc       __configure_narrow_argv    10070fbc f   ucrt:api-ms-win-crt-runtime-l1-1-0.dll
 0001:0006ffc2       __initialize_narrow_environment 10070fc2 f   ucrt:api-ms-win-crt-runtime-l1-1-0.dll
 0001:0006ffc8       __initialize_onexit_table  10070fc8 f   ucrt:api-ms-win-crt-runtime-l1-1-0.dll
 0001:0006ffce       __execute_onexit_table     10070fce f   ucrt:api-ms-win-crt-runtime-l1-1-0.dll
 0001:0006ffd4       __cexit                    10070fd4 f   ucrt:api-ms-win-crt-runtime-l1-1-0.dll
 0001:0006ffda       ___acrt_initialize         10070fda f   MSVCRT:ucrt_stubs.obj
 0001:0006ffda       ___acrt_thread_attach      10070fda f   MSVCRT:ucrt_stubs.obj
 0001:0006ffda       ___acrt_thread_detach      10070fda f   MSVCRT:ucrt_stubs.obj
 0001:0006ffda       ___acrt_uninitialize       10070fda f   MSVCRT:ucrt_stubs.obj
 0001:0006ffda       ___acrt_uninitialize_critical 10070fda f   MSVCRT:ucrt_stubs.obj
 0001:0006ffda       ___scrt_stub_for_acrt_initialize 10070fda f   MSVCRT:ucrt_stubs.obj
 0001:0006ffda       ___scrt_stub_for_acrt_thread_attach 10070fda f   MSVCRT:ucrt_stubs.obj
 0001:0006ffda       ___scrt_stub_for_acrt_thread_detach 10070fda f   MSVCRT:ucrt_stubs.obj
 0001:0006ffda       ___scrt_stub_for_acrt_uninitialize 10070fda f   MSVCRT:ucrt_stubs.obj
 0001:0006ffda       ___scrt_stub_for_acrt_uninitialize_critical 10070fda f   MSVCRT:ucrt_stubs.obj
 0001:0006ffda       ___vcrt_initialize         10070fda f   MSVCRT:ucrt_stubs.obj
 0001:0006ffda       ___vcrt_thread_attach      10070fda f   MSVCRT:ucrt_stubs.obj
 0001:0006ffda       ___vcrt_thread_detach      10070fda f   MSVCRT:ucrt_stubs.obj
 0001:0006ffda       ___vcrt_uninitialize       10070fda f   MSVCRT:ucrt_stubs.obj
 0001:0006ffda       ___vcrt_uninitialize_critical 10070fda f   MSVCRT:ucrt_stubs.obj
 0001:0006ffdd       __filter_x86_sse2_floating_point_exception 10070fdd f   MSVCRT:x86_exception_filter.obj
 0001:0006ffdd       __filter_x86_sse2_floating_point_exception_default 10070fdd f   MSVCRT:x86_exception_filter.obj
 0002:00000000       __imp__RegQueryInfoKeyW@48 10072000     advapi32:ADVAPI32.dll
 0002:00000004       __imp__RegQueryInfoKeyA@48 10072004     advapi32:ADVAPI32.dll
 0002:00000008       __imp__RegOpenKeyExA@20    10072008     advapi32:ADVAPI32.dll
 0002:0000000c       __imp__RegCloseKey@4       1007200c     advapi32:ADVAPI32.dll
 0002:00000010       __imp__RegEnumValueW@32    10072010     advapi32:ADVAPI32.dll
 0002:00000014       __imp__RegEnumValueA@32    10072014     advapi32:ADVAPI32.dll
 0002:00000018       \177ADVAPI32_NULL_THUNK_DATA 10072018     advapi32:ADVAPI32.dll
 0002:0000001c       __imp__GetTextMetricsA@8   1007201c     gdi32:GDI32.dll
 0002:00000020       __imp__ExtTextOutW@32      10072020     gdi32:GDI32.dll
 0002:00000024       __imp__EnumFontFamiliesExA@20 10072024     gdi32:GDI32.dll
 0002:00000028       __imp__SetTextColor@8      10072028     gdi32:GDI32.dll
 0002:0000002c       __imp__SetMapMode@8        1007202c     gdi32:GDI32.dll
 0002:00000030       __imp__SetBkColor@8        10072030     gdi32:GDI32.dll
 0002:00000034       __imp__SelectObject@8      10072034     gdi32:GDI32.dll
 0002:00000038       __imp__GetStockObject@4    10072038     gdi32:GDI32.dll
 0002:0000003c       __imp__GetGlyphOutlineA@28 1007203c     gdi32:GDI32.dll
 0002:00000040       __imp__GetFontData@20      10072040     gdi32:GDI32.dll
 0002:00000044       __imp__GetDIBits@28        10072044     gdi32:GDI32.dll
 0002:00000048       __imp__DeleteObject@4      10072048     gdi32:GDI32.dll
 0002:0000004c       __imp__EnumFontFamiliesExW@20 1007204c     gdi32:GDI32.dll
 0002:00000050       __imp__CreateCompatibleBitmap@12 10072050     gdi32:GDI32.dll
 0002:00000054       __imp__CreateCompatibleDC@4 10072054     gdi32:GDI32.dll
 0002:00000058       __imp__CreateFontIndirectW@4 10072058     gdi32:GDI32.dll
 0002:0000005c       __imp__GetDeviceCaps@8     1007205c     gdi32:GDI32.dll
 0002:00000060       \177GDI32_NULL_THUNK_DATA  10072060     gdi32:GDI32.dll
 0002:00000064       __imp__GetCurrentProcess@0 10072064     kernel32:KERNEL32.dll
 0002:00000068       __imp__TerminateProcess@8  10072068     kernel32:KERNEL32.dll
 0002:0000006c       __imp__QueryPerformanceCounter@4 1007206c     kernel32:KERNEL32.dll
 0002:00000070       __imp__GetCurrentProcessId@0 10072070     kernel32:KERNEL32.dll
 0002:00000074       __imp__GetCurrentThreadId@0 10072074     kernel32:KERNEL32.dll
 0002:00000078       __imp__GetSystemTimeAsFileTime@4 10072078     kernel32:KERNEL32.dll
 0002:0000007c       __imp__DisableThreadLibraryCalls@4 1007207c     kernel32:KERNEL32.dll
 0002:00000080       __imp__InitializeSListHead@4 10072080     kernel32:KERNEL32.dll
 0002:00000084       __imp__IsDebuggerPresent@0 10072084     kernel32:KERNEL32.dll
 0002:00000088       __imp__SetUnhandledExceptionFilter@4 10072088     kernel32:KERNEL32.dll
 0002:0000008c       __imp__UnhandledExceptionFilter@4 1007208c     kernel32:KERNEL32.dll
 0002:00000090       __imp__IsProcessorFeaturePresent@4 10072090     kernel32:KERNEL32.dll
 0002:00000094       __imp__GetVersion@0        10072094     kernel32:KERNEL32.dll
 0002:00000098       __imp__GetVersionExA@4     10072098     kernel32:KERNEL32.dll
 0002:0000009c       __imp__GetWindowsDirectoryA@8 1007209c     kernel32:KERNEL32.dll
 0002:000000a0       __imp__GetSystemDirectoryA@8 100720a0     kernel32:KERNEL32.dll
 0002:000000a4       \177KERNEL32_NULL_THUNK_DATA 100720a4     kernel32:KERNEL32.dll
 0002:000000a8       __imp__GetDC@4             100720a8     user32:USER32.dll
 0002:000000ac       __imp__ReleaseDC@8         100720ac     user32:USER32.dll
 0002:000000b0       __imp__GetWindowDC@4       100720b0     user32:USER32.dll
 0002:000000b4       __imp__FillRect@12         100720b4     user32:USER32.dll
 0002:000000b8       __imp__GetDesktopWindow@0  100720b8     user32:USER32.dll
 0002:000000bc       __imp__SystemParametersInfoA@16 100720bc     user32:USER32.dll
 0002:000000c0       \177USER32_NULL_THUNK_DATA 100720c0     user32:USER32.dll
 0002:000000c4       __imp___except_handler4_common 100720c4     vcruntime:VCRUNTIME140.dll
 0002:000000c8       __imp__wcsstr              100720c8     vcruntime:VCRUNTIME140.dll
 0002:000000cc       __imp__longjmp             100720cc     vcruntime:VCRUNTIME140.dll
 0002:000000d0       __imp__memmove             100720d0     vcruntime:VCRUNTIME140.dll
 0002:000000d4       __imp__memchr              100720d4     vcruntime:VCRUNTIME140.dll
 0002:000000d8       __imp___setjmp3            100720d8     vcruntime:VCRUNTIME140.dll
 0002:000000dc       __imp____std_exception_copy 100720dc     vcruntime:VCRUNTIME140.dll
 0002:000000e0       __imp____std_exception_destroy 100720e0     vcruntime:VCRUNTIME140.dll
 0002:000000e4       __imp___CxxThrowException@8 100720e4     vcruntime:VCRUNTIME140.dll
 0002:000000e8       __imp__strstr              100720e8     vcruntime:VCRUNTIME140.dll
 0002:000000ec       __imp____std_type_info_destroy_list 100720ec     vcruntime:VCRUNTIME140.dll
 0002:000000f0       __imp__wcsrchr             100720f0     vcruntime:VCRUNTIME140.dll
 0002:000000f4       __imp__memset              100720f4     vcruntime:VCRUNTIME140.dll
 0002:000000f8       __imp___purecall           100720f8     vcruntime:VCRUNTIME140.dll
 0002:000000fc       __imp__memcpy              100720fc     vcruntime:VCRUNTIME140.dll
 0002:00000100       __imp__strrchr             10072100     vcruntime:VCRUNTIME140.dll
 0002:00000104       \177VCRUNTIME140_NULL_THUNK_DATA 10072104     vcruntime:VCRUNTIME140.dll
 0002:00000108       __imp__atol                10072108     ucrt:api-ms-win-crt-convert-l1-1-0.dll
 0002:0000010c       \177api-ms-win-crt-convert-l1-1-0_NULL_THUNK_DATA 1007210c     ucrt:api-ms-win-crt-convert-l1-1-0.dll
 0002:00000110       __imp__getenv              10072110     ucrt:api-ms-win-crt-environment-l1-1-0.dll
 0002:00000114       \177api-ms-win-crt-environment-l1-1-0_NULL_THUNK_DATA 10072114     ucrt:api-ms-win-crt-environment-l1-1-0.dll
 0002:00000118       __imp__calloc              10072118     ucrt:api-ms-win-crt-heap-l1-1-0.dll
 0002:0000011c       __imp__free                1007211c     ucrt:api-ms-win-crt-heap-l1-1-0.dll
 0002:00000120       __imp___callnewh           10072120     ucrt:api-ms-win-crt-heap-l1-1-0.dll
 0002:00000124       __imp__realloc             10072124     ucrt:api-ms-win-crt-heap-l1-1-0.dll
 0002:00000128       __imp__malloc              10072128     ucrt:api-ms-win-crt-heap-l1-1-0.dll
 0002:0000012c       \177api-ms-win-crt-heap-l1-1-0_NULL_THUNK_DATA 1007212c     ucrt:api-ms-win-crt-heap-l1-1-0.dll
 0002:00000130       __imp__floor               10072130     ucrt:api-ms-win-crt-math-l1-1-0.dll
 0002:00000134       __imp___libm_sse2_pow_precise 10072134     ucrt:api-ms-win-crt-math-l1-1-0.dll
 0002:00000138       __imp___libm_sse2_sqrt_precise 10072138     ucrt:api-ms-win-crt-math-l1-1-0.dll
 0002:0000013c       \177api-ms-win-crt-math-l1-1-0_NULL_THUNK_DATA 1007213c     ucrt:api-ms-win-crt-math-l1-1-0.dll
 0002:00000140       __imp___cexit              10072140     ucrt:api-ms-win-crt-runtime-l1-1-0.dll
 0002:00000144       __imp___initialize_onexit_table 10072144     ucrt:api-ms-win-crt-runtime-l1-1-0.dll
 0002:00000148       __imp___configure_narrow_argv 10072148     ucrt:api-ms-win-crt-runtime-l1-1-0.dll
 0002:0000014c       __imp___seh_filter_dll     1007214c     ucrt:api-ms-win-crt-runtime-l1-1-0.dll
 0002:00000150       __imp___initterm_e         10072150     ucrt:api-ms-win-crt-runtime-l1-1-0.dll
 0002:00000154       __imp___initterm           10072154     ucrt:api-ms-win-crt-runtime-l1-1-0.dll
 0002:00000158       __imp___initialize_narrow_environment 10072158     ucrt:api-ms-win-crt-runtime-l1-1-0.dll
 0002:0000015c       __imp___execute_onexit_table 1007215c     ucrt:api-ms-win-crt-runtime-l1-1-0.dll
 0002:00000160       \177api-ms-win-crt-runtime-l1-1-0_NULL_THUNK_DATA 10072160     ucrt:api-ms-win-crt-runtime-l1-1-0.dll
 0002:00000164       __imp__fopen               10072164     ucrt:api-ms-win-crt-stdio-l1-1-0.dll
 0002:00000168       __imp__fread               10072168     ucrt:api-ms-win-crt-stdio-l1-1-0.dll
 0002:0000016c       __imp__fseek               1007216c     ucrt:api-ms-win-crt-stdio-l1-1-0.dll
 0002:00000170       __imp__ftell               10072170     ucrt:api-ms-win-crt-stdio-l1-1-0.dll
 0002:00000174       __imp__fclose              10072174     ucrt:api-ms-win-crt-stdio-l1-1-0.dll
 0002:00000178       __imp____stdio_common_vsprintf 10072178     ucrt:api-ms-win-crt-stdio-l1-1-0.dll
 0002:0000017c       \177api-ms-win-crt-stdio-l1-1-0_NULL_THUNK_DATA 1007217c     ucrt:api-ms-win-crt-stdio-l1-1-0.dll
 0002:00000180       __imp__strncpy             10072180     ucrt:api-ms-win-crt-string-l1-1-0.dll
 0002:00000184       __imp___stricmp            10072184     ucrt:api-ms-win-crt-string-l1-1-0.dll
 0002:00000184       __imp__stricmp             10072184     ucrt:api-ms-win-crt-string-l1-1-0.dll
 0002:00000188       __imp___wcsicmp            10072188     ucrt:api-ms-win-crt-string-l1-1-0.dll
 0002:00000188       __imp__wcsicmp             10072188     ucrt:api-ms-win-crt-string-l1-1-0.dll
 0002:0000018c       __imp__strncmp             1007218c     ucrt:api-ms-win-crt-string-l1-1-0.dll
 0002:00000190       \177api-ms-win-crt-string-l1-1-0_NULL_THUNK_DATA 10072190     ucrt:api-ms-win-crt-string-l1-1-0.dll
 0002:00000194       __imp__qsort               10072194     ucrt:api-ms-win-crt-utility-l1-1-0.dll
 0002:00000198       \177api-ms-win-crt-utility-l1-1-0_NULL_THUNK_DATA 10072198     ucrt:api-ms-win-crt-utility-l1-1-0.dll
 0002:0000019c       __imp__GrPrim_Sg2dGetCompInfo@16 1007219c     awt:awt.dll
 0002:000001a0       __imp__GetNativePrim@8     100721a0     awt:awt.dll
 0002:000001a4       __imp__SurfaceData_IntersectBounds@8 100721a4     awt:awt.dll
 0002:000001a8       __imp__AccelGlyphCache_RemoveAllCellInfos 100721a8     awt:awt.dll
 0002:000001ac       __imp__GrPrim_Sg2dGetClip@12 100721ac     awt:awt.dll
 0002:000001b0       __imp__GrPrim_Sg2dGetPixel@8 100721b0     awt:awt.dll
 0002:000001b4       __imp__SurfaceData_GetOps@8 100721b4     awt:awt.dll
 0002:000001b8       __imp__GrPrim_Sg2dGetEaRGB@8 100721b8     awt:awt.dll
 0002:000001bc       __imp__GrPrim_Sg2dGetLCDTextContrast@8 100721bc     awt:awt.dll
 0002:000001c0       \177awt_NULL_THUNK_DATA    100721c0     awt:awt.dll
 0002:000001c4       __imp__JNU_ThrowInternalError@8 100721c4     java:java.dll
 0002:000001c8       __imp__JNU_ThrowArrayIndexOutOfBoundsException@8 100721c8     java:java.dll
 0002:000001cc       __imp__JNU_NewStringPlatform@8 100721cc     java:java.dll
 0002:000001d0       \177java_NULL_THUNK_DATA   100721d0     java:java.dll
 0002:000001d4       ___guard_check_icall_fptr  100721d4     MSVCRT:guard_support.obj
 0002:000001d8       ___castguard_check_failure_os_handled_fptr 100721d8     MSVCRT:guard_support.obj
 0002:000001dc       ___xc_a                    100721dc     MSVCRT:initializers.obj
 0002:000001e0       ___xc_z                    100721e0     MSVCRT:initializers.obj
 0002:000001e4       ___xi_a                    100721e4     MSVCRT:initializers.obj
 0002:000001e8       ___xi_z                    100721e8     MSVCRT:initializers.obj
 0002:000001ec       ___xp_a                    100721ec     MSVCRT:initializers.obj
 0002:000001f0       ___xp_z                    100721f0     MSVCRT:initializers.obj
 0002:000001f4       ___xt_a                    100721f4     MSVCRT:initializers.obj
 0002:000001f8       ___xt_z                    100721f8     MSVCRT:initializers.obj
 0002:00000204       ??_7ArabicOpenTypeLayoutEngine@@6B@ 10072204     ArabicLayoutEngine.obj
 0002:00000244       ??_7UnicodeArabicOpenTypeLayoutEngine@@6B@ 10072244     ArabicLayoutEngine.obj
 0002:00000280       ?shapeTypes@ArabicShaping@@0QBJB 10072280     ArabicShaping.obj
 0002:00000310       ?glyphSubstitutionTable@CanonShaping@@2QBEB 10072310     CanonData.obj
 0002:0000ddf8       ?glyphSubstitutionTableLen@CanonShaping@@2IB 1007fdf8     CanonData.obj
 0002:0000ddfc       ?glyphDefinitionTableLen@CanonShaping@@2IB 1007fdfc     CanonData.obj
 0002:0000de00       ?glyphDefinitionTable@CanonShaping@@2QBEB 1007fe00     CanonData.obj
 0002:0000e3dc       ??_7ContextualGlyphInsertionProcessor2@@6B@ 100803dc     ContextualGlyphInsertionProc2.obj
 0002:0000e3f8       ??_7ContextualGlyphSubstitutionProcessor@@6B@ 100803f8     ContextualGlyphSubstProc.obj
 0002:0000e414       ??_7ContextualGlyphSubstitutionProcessor2@@6B@ 10080414     ContextualGlyphSubstProc2.obj
 0002:0000e42c       ?fieldMasks@DeviceTable@@0QBGB 1008042c     DeviceTables.obj
 0002:0000e434       ?fieldSignBits@DeviceTable@@0QBGB 10080434     DeviceTables.obj
 0002:0000e43c       ?fieldBits@DeviceTable@@0QBGB 1008043c     DeviceTables.obj
 0002:0000e444       __real@3e2aaaad            10080444     DrawGlyphList.obj
 0002:0000e448       __real@3f000000            10080448     DrawGlyphList.obj
 0002:0000e450       __real@3ff0000000000000    10080450     DrawGlyphList.obj
 0002:0000e458       __real@40400000            10080458     DrawGlyphList.obj
 0002:0000e460       __real@4059000000000000    10080460     DrawGlyphList.obj
 0002:0000e468       __real@406fe00000000000    10080468     DrawGlyphList.obj
 0002:0000e48c       ??_7LEFontInstance@@6B@    1008048c     FontInstanceAdapter.obj
 0002:0000e50c       ??_7FontInstanceAdapter@@6B@ 1008050c     FontInstanceAdapter.obj
 0002:0000e594       __real@3f800000            10080594     FontInstanceAdapter.obj
 0002:0000e598       __real@42900000            10080598     FontInstanceAdapter.obj
 0002:0000e5a0       __xmm@80000000800000008000000080000000 100805a0     FontInstanceAdapter.obj
 0002:0000e5b4       ??_7LEGlyphFilter@@6B@     100805b4     GDEFMarkFilter.obj
 0002:0000e5c0       ??_7GDEFMarkFilter@@6B@    100805c0     GDEFMarkFilter.obj
 0002:0000e5cc       ??_7GXLayoutEngine@@6B@    100805cc     GXLayoutEngine.obj
 0002:0000e600       ??_7GXLayoutEngine2@@6B@   10080600     GXLayoutEngine2.obj
 0002:0000e634       ??_7GlyphIterator@@6B@     10080634     GlyphIterator.obj
 0002:0000e63c       ??_7GlyphPositioningLookupProcessor@@6B@ 1008063c     GlyphPosnLookupProc.obj
 0002:0000e648       ??_7GlyphSubstitutionLookupProcessor@@6B@ 10080648     GlyphSubstLookupProc.obj
 0002:0000e66c       ??_7HanOpenTypeLayoutEngine@@6B@ 1008066c     HanLayoutEngine.obj
 0002:0000e7bc       ??_7HangulOpenTypeLayoutEngine@@6B@ 100807bc     HangulLayoutEngine.obj
 0002:0000fdc8       ??_7IndicOpenTypeLayoutEngine@@6B@ 10081dc8     IndicLayoutEngine.obj
 0002:0000fe08       ??_7IndicRearrangementProcessor@@6B@ 10081e08     IndicRearrangementProcessor.obj
 0002:0000fe24       ??_7IndicRearrangementProcessor2@@6B@ 10081e24     IndicRearrangementProcessor2.obj
 0002:00010044       ??_7KhmerOpenTypeLayoutEngine@@6B@ 10082044     KhmerLayoutEngine.obj
 0002:00010370       ??_7LECharMapper@@6B@      10082370     LEFontInstance.obj
 0002:0001037c       ??_7LEInsertionCallback@@6B@ 1008237c     LEGlyphStorage.obj
 0002:00010388       ??_7LEGlyphStorage@@6B@    10082388     LEGlyphStorage.obj
 0002:00010398       ??_7LEInsertionList@@6B@   10082398     LEInsertionList.obj
 0002:000103a0       ?controlChars@DefaultCharMapper@@0QBKB 100823a0     LayoutEngine.obj
 0002:000103e8       ?controlCharsCount@DefaultCharMapper@@0JB 100823e8     LayoutEngine.obj
 0002:000103ec       ?controlCharsZWJCount@DefaultCharMapper@@0JB 100823ec     LayoutEngine.obj
 0002:000103f0       ?controlCharsZWJ@DefaultCharMapper@@0QBKB 100823f0     LayoutEngine.obj
 0002:00010448       ?kTypoFlagKern@LayoutEngine@@2JB 10082448     LayoutEngine.obj
 0002:0001044c       ?kTypoFlagLiga@LayoutEngine@@2JB 1008244c     LayoutEngine.obj
 0002:00010454       ??_7LayoutEngine@@6B@      10082454     LayoutEngine.obj
 0002:00010488       ??_7CharSubstitutionFilter@@6B@ 10082488     LayoutEngine.obj
 0002:00010494       ??_7DefaultCharMapper@@6B@ 10082494     LayoutEngine.obj
 0002:000104a0       ??_7CanonMarkFilter@@6B@   100824a0     LayoutEngine.obj
 0002:000104ac       ??_7LigatureSubstitutionProcessor@@6B@ 100824ac     LigatureSubstProc.obj
 0002:000104c8       ??_7LigatureSubstitutionProcessor2@@6B@ 100824c8     LigatureSubstProc2.obj
 0002:000104e4       ??_7LookupProcessor@@6B@   100824e4     LookupProcessor.obj
 0002:000104f0       ?mirroredChars@DefaultCharMapper@@0QBKB 100824f0     MirroredCharData.obj
 0002:00010a20       ?srahCderorrim@DefaultCharMapper@@0QBKB 10082a20     MirroredCharData.obj
 0002:00010f50       ?mirroredCharsCount@DefaultCharMapper@@0JB 10082f50     MirroredCharData.obj
 0002:00010f58       ??_7NonContextualGlyphSubstitutionProcessor@@6B@ 10082f58     NonContextualGlyphSubstProc.obj
 0002:00010f64       ??_7NonContextualGlyphSubstitutionProcessor2@@6B@ 10082f64     NonContextualGlyphSubstProc2.obj
 0002:00011044       ??_7OpenTypeLayoutEngine@@6B@ 10083044     OpenTypeLayoutEngine.obj
 0002:00011080       ?languageTags@OpenTypeLayoutEngine@@2QBKB 10083080     ScriptAndLanguageTags.obj
 0002:000111a0       ?scriptTags@OpenTypeLayoutEngine@@0QBKB 100831a0     ScriptAndLanguageTags.obj
 0002:0001141c       ??_7SegmentArrayProcessor@@6B@ 1008341c     SegmentArrayProcessor.obj
 0002:0001142c       ??_7SegmentArrayProcessor2@@6B@ 1008342c     SegmentArrayProcessor2.obj
 0002:0001143c       ??_7SegmentSingleProcessor@@6B@ 1008343c     SegmentSingleProcessor.obj
 0002:0001144c       ??_7SegmentSingleProcessor2@@6B@ 1008344c     SegmentSingleProcessor2.obj
 0002:00011458       ?shapingTypeTable@ArabicShaping@@0QBEB 10083458     ShapingTypeData.obj
 0002:00011968       ?shapingTypeTableLen@ArabicShaping@@0IB 10083968     ShapingTypeData.obj
 0002:00011970       ??_7SimpleArrayProcessor@@6B@ 10083970     SimpleArrayProcessor.obj
 0002:00011980       ??_7SimpleArrayProcessor2@@6B@ 10083980     SimpleArrayProcessor2.obj
 0002:00011990       ??_7SingleTableProcessor@@6B@ 10083990     SingleTableProcessor.obj
 0002:000119a0       ??_7SingleTableProcessor2@@6B@ 100839a0     SingleTableProcessor2.obj
 0002:000119b0       ??_7StateTableProcessor@@6B@ 100839b0     StateTableProcessor.obj
 0002:000119c8       ??_7StateTableProcessor2@@6B@ 100839c8     StateTableProcessor2.obj
 0002:000119e0       ??_7SubtableProcessor@@6B@ 100839e0     SubtableProcessor.obj
 0002:000119ec       ??_7SubtableProcessor2@@6B@ 100839ec     SubtableProcessor2.obj
 0002:000119f4       ??_C@_0BM@DODCGPJL@sun?1font?1GlyphLayout$GVData@ 100839f4     SunLayoutEngine.obj
 0002:00011a10       ??_C@_01JPJNBJEM@I@        10083a10     SunLayoutEngine.obj
 0002:00011a14       ??_C@_06HHPHCOMB@_count@   10083a14     SunLayoutEngine.obj
 0002:00011a1c       ??_C@_06PPHBKICC@_flags@   10083a1c     SunLayoutEngine.obj
 0002:00011a24       ??_C@_02EBOMBDPA@?$FLI@    10083a24     SunLayoutEngine.obj
 0002:00011a28       ??_C@_07PKNHOODJ@_glyphs@  10083a28     SunLayoutEngine.obj
 0002:00011a30       ??_C@_02MGHEAPDP@?$FLF@    10083a30     SunLayoutEngine.obj
 0002:00011a34       ??_C@_0L@BHNDECPI@_positions@ 10083a34     SunLayoutEngine.obj
 0002:00011a40       ??_C@_08MEOKMKLN@_indices@ 10083a40     SunLayoutEngine.obj
 0002:00011a4c       ??_C@_0P@EFKBJFIG@count?5negative@ 10083a4c     SunLayoutEngine.obj
 0002:00011a5c       ??_C@_0BA@CNGMEPKA@glypharray?5null@ 10083a5c     SunLayoutEngine.obj
 0002:00011a6c       ??_C@_00CNPNBAHC@@         10083a6c     SunLayoutEngine.obj
 0002:00011a70       ??_C@_0BD@ODPDFFNE@indices?5array?5null@ 10083a70     SunLayoutEngine.obj
 0002:00011a88       ??_7ThaiLayoutEngine@@6B@  10083a88     ThaiLayoutEngine.obj
 0002:00011bd0       ?classTable@ThaiShaping@@0QBEB 10083bd0     ThaiStateTables.obj
 0002:00011c30       ?thaiStateTable@ThaiShaping@@0QAY0BD@$$CBUStateTransition@1@A 10083c30     ThaiStateTables.obj
 0002:000123ec       ??_7TibetanOpenTypeLayoutEngine@@6B@ 100843ec     TibetanLayoutEngine.obj
 0002:00012a1c       ??_7TrimmedArrayProcessor@@6B@ 10084a1c     TrimmedArrayProcessor.obj
 0002:00012a2c       ??_7TrimmedArrayProcessor2@@6B@ 10084a2c     TrimmedArrayProcessor2.obj
 0002:00012a7c       __real@00000000            10084a7c     ValueRecords.obj
 0002:00012b2c       ??_C@_11LOCGONAA@@         10084b2c     fontpath.obj
 0002:00012b30       ??_C@_07GCCENIMJ@?2System@ 10084b30     fontpath.obj
 0002:00012b38       ??_C@_09FJGNFLHN@?2System32@ 10084b38     fontpath.obj
 0002:00012b44       ??_C@_06MIJGMACG@?2Fonts@  10084b44     fontpath.obj
 0002:00012b4c       ??_C@_01ICJEACDI@?$DL@     10084b4c     fontpath.obj
 0002:00012b50       ??_C@_03NHMNJBCN@?5?$CG?5@ 10084b50     fontpath.obj
 0002:00012b54       ??_C@_17BCGMALNF@?$AA?5?$AA?$CG?$AA?5@ 10084b54     fontpath.obj
 0002:00012b5c       ??_C@_0BC@LEKPNIDO@java?1util?1HashMap@ 10084b5c     fontpath.obj
 0002:00012b70       ??_C@_0DJ@FLFJBGBN@?$CILjava?1lang?1Object?$DLLjava?1lang?1O@ 10084b70     fontpath.obj
 0002:00012bac       ??_C@_03KMONJGDG@put@      10084bac     fontpath.obj
 0002:00012bb0       ??_C@_0BG@DHOOFEJE@?$CILjava?1lang?1Object?$DL?$CJZ@ 10084bb0     fontpath.obj
 0002:00012bc8       ??_C@_0M@ILMAKOC@containsKey@ 10084bc8     fontpath.obj
 0002:00012bd4       ??_C@_0BE@GPOIDJOH@java?1util?1ArrayList@ 10084bd4     fontpath.obj
 0002:00012be8       ??_C@_04PFANPMCN@?$CII?$CJV@ 10084be8     fontpath.obj
 0002:00012bf0       ??_C@_06FALKBLGB@?$DMinit?$DO@ 10084bf0     fontpath.obj
 0002:00012bf8       ??_C@_03BDGOHNNK@add@      10084bf8     fontpath.obj
 0002:00012bfc       ??_C@_0BB@FLFAIHG@java?1lang?1String@ 10084bfc     fontpath.obj
 0002:00012c10       ??_C@_0CH@BHMNPKMP@?$CILjava?1util?1Locale?$DL?$CJLjava?1lang?1@ 10084c10     fontpath.obj
 0002:00012c38       ??_C@_0M@IMBDOEKL@toLowerCase@ 10084c38     fontpath.obj
 0002:00012c44       ??_C@_19OLAFNMII@?$AA?4?$AAt?$AAt?$AAf@ 10084c44     fontpath.obj
 0002:00012c50       ??_C@_19MKNEPBPF@?$AA?4?$AAo?$AAt?$AAf@ 10084c50     fontpath.obj
 0002:00012c74       ??_C@_03GAEACAIP@?$CI?$CJV@ 10084c74     freetypeScaler.obj
 0002:00012c78       ??_C@_0BB@NIMAMPFF@invalidateScaler@ 10084c78     freetypeScaler.obj
 0002:00012c8c       ??_C@_0BE@LLDKDDBI@FREETYPE_PROPERTIES@ 10084c8c     freetypeScaler.obj
 0002:00012ca0       ??_C@_08OKLLNAKL@truetype@ 10084ca0     freetypeScaler.obj
 0002:00012cac       ??_C@_0BE@OJJAFABD@interpreter?9version@ 10084cac     freetypeScaler.obj
 0002:00012cc0       __real@37800000            10084cc0     freetypeScaler.obj
 0002:00012cc4       __real@3c800000            10084cc4     freetypeScaler.obj
 0002:00012cc8       __real@3ef0000000000000    10084cc8     freetypeScaler.obj
 0002:00012cd0       __real@3f90000000000000    10084cd0     freetypeScaler.obj
 0002:00012cd8       __real@4050000000000000    10084cd8     freetypeScaler.obj
 0002:00012ce0       __real@40f0000000000000    10084ce0     freetypeScaler.obj
 0002:00012ce8       __real@42800000            10084ce8     freetypeScaler.obj
 0002:00012cf0       __real@c0f0000000000000    10084cf0     freetypeScaler.obj
 0002:00012d00       __xmm@00010000000000000000366a00010000 10084d00     freetypeScaler.obj
 0002:00012d10       __xmm@80000000000000008000000000000000 10084d10     freetypeScaler.obj
 0002:00012d20       ??_C@_0BG@NKHBBPH@sun?1font?1TrueTypeFont@ 10084d20     sunFont.obj
 0002:00012d38       ??_C@_0BL@GAAGJDLL@?$CILjava?1nio?1ByteBuffer?$DLII?$CJI@ 10084d38     sunFont.obj
 0002:00012d54       ??_C@_09CKAKNPHP@readBlock@ 10084d54     sunFont.obj
 0002:00012d60       ??_C@_06JMOJDKIE@?$CIII?$CJ?$FLB@ 10084d60     sunFont.obj
 0002:00012d68       ??_C@_09IDIEPDPI@readBytes@ 10084d68     sunFont.obj
 0002:00012d74       ??_C@_0BD@OPLCIPMH@sun?1font?1Type1Font@ 10084d74     sunFont.obj
 0002:00012d88       ??_C@_0BJ@LMHMPPKE@?$CILjava?1nio?1ByteBuffer?$DL?$CJV@ 10084d88     sunFont.obj
 0002:00012da4       ??_C@_08CJNGBMAG@readFile@ 10084da4     sunFont.obj
 0002:00012db0       ??_C@_0BM@DGICEJAA@java?1awt?1geom?1Point2D$Float@ 10084db0     sunFont.obj
 0002:00012dcc       ??_C@_05BHHDPELC@?$CIFF?$CJV@ 10084dcc     sunFont.obj
 0002:00012dd4       ??_C@_01BIAFAFID@F@        10084dd4     sunFont.obj
 0002:00012dd8       ??_C@_01FJMABOPO@x@        10084dd8     sunFont.obj
 0002:00012ddc       ??_C@_01EANLCPLP@y@        10084ddc     sunFont.obj
 0002:00012de0       ??_C@_0BH@ENELCGL@sun?1font?1StrikeMetrics@ 10084de0     sunFont.obj
 0002:00012df8       ??_C@_0O@LBAHCNJL@?$CIFFFFFFFFFF?$CJV@ 10084df8     sunFont.obj
 0002:00012e08       ??_C@_0CA@PDMBNICK@java?1awt?1geom?1Rectangle2D$Float@ 10084e08     sunFont.obj
 0002:00012e28       ??_C@_07PMCFNNPC@?$CIFFFF?$CJV@ 10084e28     sunFont.obj
 0002:00012e30       ??_C@_05IGKADHGO@width@    10084e30     sunFont.obj
 0002:00012e38       ??_C@_06LNLHEAAG@height@   10084e38     sunFont.obj
 0002:00012e40       ??_C@_0BK@COJNCHEM@java?1awt?1geom?1GeneralPath@ 10084e40     sunFont.obj
 0002:00012e5c       ??_C@_0L@MDPODKN@?$CII?$FLBI?$FLFI?$CJV@ 10084e5c     sunFont.obj
 0002:00012e68       ??_C@_0BA@OKNBFGCN@sun?1font?1Font2D@ 10084e68     sunFont.obj
 0002:00012e78       ??_C@_04DIFHPCLD@?$CII?$CJI@ 10084e78     sunFont.obj
 0002:00012e80       ??_C@_0M@NMGOHDEJ@charToGlyph@ 10084e80     sunFont.obj
 0002:00012e8c       ??_C@_0BP@CBNLOFNN@?$CI?$CJLsun?1font?1CharToGlyphMapper?$DL@ 10084e8c     sunFont.obj
 0002:00012eac       ??_C@_09DGCMEJKL@getMapper@ 10084eac     sunFont.obj
 0002:00012eb8       ??_C@_05IPLNOPFN@?$CII?$CJ?$FLB@ 10084eb8     sunFont.obj
 0002:00012ec0       ??_C@_0O@DBNIPDIH@getTableBytes@ 10084ec0     sunFont.obj
 0002:00012ed0       ??_C@_04DGAFFDEF@?$CIC?$CJZ@ 10084ed0     sunFont.obj
 0002:00012ed8       ??_C@_0L@PGEPPKMA@canDisplay@ 10084ed8     sunFont.obj
 0002:00012ee4       ??_C@_0BL@GAPGNAAC@sun?1font?1CharToGlyphMapper@ 10084ee4     sunFont.obj
 0002:00012f00       ??_C@_0BI@GDBHNKM@sun?1font?1PhysicalStrike@ 10084f00     sunFont.obj
 0002:00012f18       ??_C@_0CB@IBGFEOCM@?$CII?$CJLjava?1awt?1geom?1Point2D$Float@ 10084f18     sunFont.obj
 0002:00012f3c       ??_C@_0BA@FMKHNFIF@getGlyphMetrics@ 10084f3c     sunFont.obj
 0002:00012f4c       ??_C@_0CC@IBLMDHKA@?$CIII?$CJLjava?1awt?1geom?1Point2D$Floa@ 10084f4c     sunFont.obj
 0002:00012f70       ??_C@_0O@NHLNHECD@getGlyphPoint@ 10084f70     sunFont.obj
 0002:00012f80       ??_C@_0CB@CONGGNHA@?$CILjava?1awt?1geom?1Point2D$Float?$DL?$CJ@ 10084f80     sunFont.obj
 0002:00012fa4       ??_C@_0M@MJABIGBP@adjustPoint@ 10084fa4     sunFont.obj
 0002:00012fb0       ??_C@_01LELAEKIP@J@        10084fb0     sunFont.obj
 0002:00012fb4       ??_C@_0P@DPIICNJB@pScalerContext@ 10084fb4     sunFont.obj
 0002:00012fc4       ??_C@_0BD@LPHBDEDB@sun?1font?1GlyphList@ 10084fc4     sunFont.obj
 0002:00012fd8       ??_C@_03BKCJCHLK@len@      10084fd8     sunFont.obj
 0002:00012fdc       ??_C@_02GKMBEADD@?$FLJ@    10084fdc     sunFont.obj
 0002:00012fe0       ??_C@_06IAHKIHIK@images@   10084fe0     sunFont.obj
 0002:00012fe8       ??_C@_01POHCFINO@Z@        10084fe8     sunFont.obj
 0002:00012fec       ??_C@_0N@CLHDJEN@usePositions@ 10084fec     sunFont.obj
 0002:00012ffc       ??_C@_09HEJILCIA@positions@ 10084ffc     sunFont.obj
 0002:00013008       ??_C@_0M@IOGNPDID@lcdRGBOrder@ 10085008     sunFont.obj
 0002:00013014       ??_C@_0N@OIMCCICM@lcdSubPixPos@ 10085014     sunFont.obj
 0002:00013078       _ft_raccess_guess_table    10085078     freetype:ftbase.obj
 0002:0001312c       ??_C@_02PEOAMJM@?4_@       1008512c     freetype:ftbase.obj
 0002:00013130       ??_C@_05FLPKNBDI@?1rsrc@   10085130     freetype:ftbase.obj
 0002:00013138       ??_C@_0BC@OBHLCHMP@?1?4?4namedfork?1rsrc@ 10085138     freetype:ftbase.obj
 0002:0001314c       ??_C@_0O@FDMCFKOC@resource?4frk?1@ 1008514c     freetype:ftbase.obj
 0002:0001315c       ??_C@_0L@FGJFJHGF@?4resource?1@ 1008515c     freetype:ftbase.obj
 0002:00013168       ??_C@_01FGNFDNOH@?$CF@     10085168     freetype:ftbase.obj
 0002:0001316c       ??_C@_0O@KCDCBAF@?4AppleDouble?1@ 1008516c     freetype:ftbase.obj
 0002:0001317c       ??_C@_03LBLPCGAC@cid@      1008517c     freetype:ftbase.obj
 0002:00013180       ??_C@_05MJDCDNNA@type1@    10085180     freetype:ftbase.obj
 0002:00013188       ??_C@_03IINFADLN@cff@      10085188     freetype:ftbase.obj
 0002:0001318c       ??_C@_07IAOBDJBM@kerning@  1008518c     freetype:ftbase.obj
 0002:00013194       ??_C@_0L@POCJHJKN@glyph?9dict@ 10085194     freetype:ftbase.obj
 0002:000131a0       ??_C@_0BF@GDPJODJF@postscript?9font?9name@ 100851a0     freetype:ftbase.obj
 0002:000131b8       ??_C@_0L@MBBJBANC@sfnt?9table@ 100851b8     freetype:ftbase.obj
 0002:000131c4       ??_C@_08OHCKCLF@tt?9cmaps@ 100851c4     freetype:ftbase.obj
 0002:000131d0       ??_C@_0L@CIHKIEFA@properties@ 100851d0     freetype:ftbase.obj
 0002:000131dc       ??_C@_06GNKBHGHD@type42@   100851dc     freetype:ftbase.obj
 0002:000131e4       ??_C@_0BA@DHLLBDBB@truetype?9engine@ 100851e4     freetype:ftbase.obj
 0002:00013210       _af_blue_strings           10085210     freetype:autofit.obj
 0002:00013418       _af_blue_stringsets        10085418     freetype:autofit.obj
 0002:00013500       _autofit_module_class      10085500     freetype:autofit.obj
 0002:00013524       _af_writing_system_classes 10085524     freetype:autofit.obj
 0002:00013538       _af_cyrl_script_class      10085538     freetype:autofit.obj
 0002:0001354c       _af_grek_script_class      1008554c     freetype:autofit.obj
 0002:00013560       _af_hebr_script_class      10085560     freetype:autofit.obj
 0002:00013574       _af_latn_script_class      10085574     freetype:autofit.obj
 0002:00013588       _af_none_script_class      10085588     freetype:autofit.obj
 0002:0001359c       _af_beng_script_class      1008559c     freetype:autofit.obj
 0002:000135b0       _af_deva_script_class      100855b0     freetype:autofit.obj
 0002:000135c4       _af_gujr_script_class      100855c4     freetype:autofit.obj
 0002:000135d8       _af_guru_script_class      100855d8     freetype:autofit.obj
 0002:000135ec       _af_knda_script_class      100855ec     freetype:autofit.obj
 0002:00013600       _af_limb_script_class      10085600     freetype:autofit.obj
 0002:00013614       _af_mlym_script_class      10085614     freetype:autofit.obj
 0002:00013628       _af_orya_script_class      10085628     freetype:autofit.obj
 0002:0001363c       _af_sinh_script_class      1008563c     freetype:autofit.obj
 0002:00013650       _af_sund_script_class      10085650     freetype:autofit.obj
 0002:00013664       _af_sylo_script_class      10085664     freetype:autofit.obj
 0002:00013678       _af_taml_script_class      10085678     freetype:autofit.obj
 0002:0001368c       _af_telu_script_class      1008568c     freetype:autofit.obj
 0002:000136a0       _af_tibt_script_class      100856a0     freetype:autofit.obj
 0002:000136b4       _af_hani_script_class      100856b4     freetype:autofit.obj
 0002:000136c8       _af_script_classes         100856c8     freetype:autofit.obj
 0002:0001371c       _af_cyrl_c2cp_style_class  1008571c     freetype:autofit.obj
 0002:00013730       _af_cyrl_c2sc_style_class  10085730     freetype:autofit.obj
 0002:00013744       _af_cyrl_ordn_style_class  10085744     freetype:autofit.obj
 0002:00013758       _af_cyrl_pcap_style_class  10085758     freetype:autofit.obj
 0002:0001376c       _af_cyrl_sinf_style_class  1008576c     freetype:autofit.obj
 0002:00013780       _af_cyrl_smcp_style_class  10085780     freetype:autofit.obj
 0002:00013794       _af_cyrl_subs_style_class  10085794     freetype:autofit.obj
 0002:000137a8       _af_cyrl_sups_style_class  100857a8     freetype:autofit.obj
 0002:000137bc       _af_cyrl_titl_style_class  100857bc     freetype:autofit.obj
 0002:000137d0       _af_cyrl_dflt_style_class  100857d0     freetype:autofit.obj
 0002:000137e4       _af_grek_c2cp_style_class  100857e4     freetype:autofit.obj
 0002:000137f8       _af_grek_c2sc_style_class  100857f8     freetype:autofit.obj
 0002:0001380c       _af_grek_ordn_style_class  1008580c     freetype:autofit.obj
 0002:00013820       _af_grek_pcap_style_class  10085820     freetype:autofit.obj
 0002:00013834       _af_grek_sinf_style_class  10085834     freetype:autofit.obj
 0002:00013848       _af_grek_smcp_style_class  10085848     freetype:autofit.obj
 0002:0001385c       _af_grek_subs_style_class  1008585c     freetype:autofit.obj
 0002:00013870       _af_grek_sups_style_class  10085870     freetype:autofit.obj
 0002:00013884       _af_grek_titl_style_class  10085884     freetype:autofit.obj
 0002:00013898       _af_grek_dflt_style_class  10085898     freetype:autofit.obj
 0002:000138ac       _af_hebr_dflt_style_class  100858ac     freetype:autofit.obj
 0002:000138c0       _af_latn_c2cp_style_class  100858c0     freetype:autofit.obj
 0002:000138d4       _af_latn_c2sc_style_class  100858d4     freetype:autofit.obj
 0002:000138e8       _af_latn_ordn_style_class  100858e8     freetype:autofit.obj
 0002:000138fc       _af_latn_pcap_style_class  100858fc     freetype:autofit.obj
 0002:00013910       _af_latn_sinf_style_class  10085910     freetype:autofit.obj
 0002:00013924       _af_latn_smcp_style_class  10085924     freetype:autofit.obj
 0002:00013938       _af_latn_subs_style_class  10085938     freetype:autofit.obj
 0002:0001394c       _af_latn_sups_style_class  1008594c     freetype:autofit.obj
 0002:00013960       _af_latn_titl_style_class  10085960     freetype:autofit.obj
 0002:00013974       _af_latn_dflt_style_class  10085974     freetype:autofit.obj
 0002:00013988       _af_none_dflt_style_class  10085988     freetype:autofit.obj
 0002:0001399c       _af_beng_dflt_style_class  1008599c     freetype:autofit.obj
 0002:000139b0       _af_deva_dflt_style_class  100859b0     freetype:autofit.obj
 0002:000139c4       _af_gujr_dflt_style_class  100859c4     freetype:autofit.obj
 0002:000139d8       _af_guru_dflt_style_class  100859d8     freetype:autofit.obj
 0002:000139ec       _af_knda_dflt_style_class  100859ec     freetype:autofit.obj
 0002:00013a00       _af_limb_dflt_style_class  10085a00     freetype:autofit.obj
 0002:00013a14       _af_mlym_dflt_style_class  10085a14     freetype:autofit.obj
 0002:00013a28       _af_orya_dflt_style_class  10085a28     freetype:autofit.obj
 0002:00013a3c       _af_sinh_dflt_style_class  10085a3c     freetype:autofit.obj
 0002:00013a50       _af_sund_dflt_style_class  10085a50     freetype:autofit.obj
 0002:00013a64       _af_sylo_dflt_style_class  10085a64     freetype:autofit.obj
 0002:00013a78       _af_taml_dflt_style_class  10085a78     freetype:autofit.obj
 0002:00013a8c       _af_telu_dflt_style_class  10085a8c     freetype:autofit.obj
 0002:00013aa0       _af_tibt_dflt_style_class  10085aa0     freetype:autofit.obj
 0002:00013ab4       _af_hani_dflt_style_class  10085ab4     freetype:autofit.obj
 0002:00013ac8       _af_style_classes          10085ac8     freetype:autofit.obj
 0002:00013b88       _af_cyrl_uniranges         10085b88     freetype:autofit.obj
 0002:00013bb0       _af_grek_uniranges         10085bb0     freetype:autofit.obj
 0002:00013bc8       _af_hebr_uniranges         10085bc8     freetype:autofit.obj
 0002:00013be0       _af_latn_uniranges         10085be0     freetype:autofit.obj
 0002:00013c98       _af_none_uniranges         10085c98     freetype:autofit.obj
 0002:00013ca0       _af_beng_uniranges         10085ca0     freetype:autofit.obj
 0002:00013cb0       _af_deva_uniranges         10085cb0     freetype:autofit.obj
 0002:00013cc0       _af_gujr_uniranges         10085cc0     freetype:autofit.obj
 0002:00013cd0       _af_guru_uniranges         10085cd0     freetype:autofit.obj
 0002:00013ce0       _af_knda_uniranges         10085ce0     freetype:autofit.obj
 0002:00013cf0       _af_limb_uniranges         10085cf0     freetype:autofit.obj
 0002:00013d00       _af_mlym_uniranges         10085d00     freetype:autofit.obj
 0002:00013d10       _af_orya_uniranges         10085d10     freetype:autofit.obj
 0002:00013d20       _af_sinh_uniranges         10085d20     freetype:autofit.obj
 0002:00013d30       _af_sund_uniranges         10085d30     freetype:autofit.obj
 0002:00013d40       _af_sylo_uniranges         10085d40     freetype:autofit.obj
 0002:00013d50       _af_taml_uniranges         10085d50     freetype:autofit.obj
 0002:00013d60       _af_telu_uniranges         10085d60     freetype:autofit.obj
 0002:00013d70       _af_tibt_uniranges         10085d70     freetype:autofit.obj
 0002:00013d80       _af_hani_uniranges         10085d80     freetype:autofit.obj
 0002:00013e88       _af_dummy_writing_system_class 10085e88     freetype:autofit.obj
 0002:00013ea4       _af_latin_writing_system_class 10085ea4     freetype:autofit.obj
 0002:00013ec0       _af_cjk_writing_system_class 10085ec0     freetype:autofit.obj
 0002:00013edc       _af_indic_writing_system_class 10085edc     freetype:autofit.obj
 0002:00013f10       _af_autofitter_interface   10085f10     freetype:autofit.obj
 0002:00013f20       ??_C@_0BA@OKOILHEH@fallback?9script@ 10085f20     freetype:autofit.obj
 0002:00013f30       ??_C@_0P@PHBNIPOP@default?9script@ 10085f30     freetype:autofit.obj
 0002:00013f40       ??_C@_0BC@OOHNGIJD@increase?9x?9height@ 10085f40     freetype:autofit.obj
 0002:00013f54       ??_C@_0BE@CELKBFDM@glyph?9to?9script?9map@ 10085f54     freetype:autofit.obj
 0002:00013f68       ??_C@_0L@MNEBCNMP@autofitter@ 10085f68     freetype:autofit.obj
 0002:00013f80       __xmm@00000000000000000001000000010000 10085f80     freetype:autofit.obj
 0002:00013ff8       _tt_driver_class           10085ff8     freetype:truetype.obj
 0002:00014058       _tt_default_graphics_state 10086058     freetype:truetype.obj
 0002:00014540       ??_C@_06ODJMJFLN@Weight@   10086540     freetype:truetype.obj
 0002:00014548       ??_C@_05IBAMDCFI@Width@    10086548     freetype:truetype.obj
 0002:00014550       ??_C@_0M@EDHPABCB@OpticalSize@ 10086550     freetype:truetype.obj
 0002:0001455c       ??_C@_05BCGFHEPH@Slant@    1008655c     freetype:truetype.obj
 0002:00014564       ??_C@_0BB@PMIOOMFN@xf86?9driver?9name@ 10086564     freetype:truetype.obj
 0002:00014578       ??_C@_08KJILHNAM@TrueType@ 10086578     freetype:truetype.obj
 0002:00014584       ??_C@_0O@DHADKGAK@multi?9masters@ 10086584     freetype:truetype.obj
 0002:00014594       ??_C@_07CDLHCBDE@tt?9glyf@ 10086594     freetype:truetype.obj
 0002:0001459c       ??_C@_04JAPIGAPK@sfnt@     1008659c     freetype:truetype.obj
 0002:000145a4       ??_C@_07JBKHDJHE@?4notdef@ 100865a4     freetype:truetype.obj
 0002:000145ac       ??_C@_0P@EMKCEFJO@?$CF?$CBPS?9AdobeFont@ 100865ac     freetype:type1.obj
 0002:000145bc       ??_C@_0L@LLIKMEDC@?$CF?$CBFontType@ 100865bc     freetype:type1.obj
 0002:000145c8       ??_C@_05OJJBIBFE@eexec@    100865c8     freetype:type1.obj
 0002:000145d0       ??_C@_0BB@MLEHKAJM@StandardEncoding@ 100865d0     freetype:type1.obj
 0002:000145e4       ??_C@_0P@LHOFAKJ@ExpertEncoding@ 100865e4     freetype:type1.obj
 0002:000145f4       ??_C@_0BC@OHHLKLPP@ISOLatin1Encoding@ 100865f4     freetype:type1.obj
 0002:00014608       ??_C@_03BHPKJDPK@dup@      10086608     freetype:type1.obj
 0002:00014cb0       _t1_driver_class           10086cb0     freetype:type1.obj
 0002:00014d7c       ??_C@_07CPCPJPKL@version@  10086d7c     freetype:type1.obj
 0002:00014d84       ??_C@_06JHGCIHDH@Notice@   10086d84     freetype:type1.obj
 0002:00014d8c       ??_C@_08FPDCFGEH@FullName@ 10086d8c     freetype:type1.obj
 0002:00014d98       ??_C@_0L@KKMPOENF@FamilyName@ 10086d98     freetype:type1.obj
 0002:00014da4       ??_C@_0M@ILCDBHGP@ItalicAngle@ 10086da4     freetype:type1.obj
 0002:00014db0       ??_C@_0N@OPLNPOL@isFixedPitch@ 10086db0     freetype:type1.obj
 0002:00014dc0       ??_C@_0BC@CCIMILPE@UnderlinePosition@ 10086dc0     freetype:type1.obj
 0002:00014dd4       ??_C@_0BD@KBICJDLM@UnderlineThickness@ 10086dd4     freetype:type1.obj
 0002:00014de8       ??_C@_06FIINGLDE@FSType@   10086de8     freetype:type1.obj
 0002:00014df0       ??_C@_08OMJGNOHD@UniqueID@ 10086df0     freetype:type1.obj
 0002:00014dfc       ??_C@_05CIIKKFON@lenIV@    10086dfc     freetype:type1.obj
 0002:00014e04       ??_C@_0O@PJDGHDCK@LanguageGroup@ 10086e04     freetype:type1.obj
 0002:00014e14       ??_C@_08NLHBPEGP@password@ 10086e14     freetype:type1.obj
 0002:00014e20       ??_C@_09IPAGIEBG@BlueScale@ 10086e20     freetype:type1.obj
 0002:00014e2c       ??_C@_09GDCMDLCO@BlueShift@ 10086e2c     freetype:type1.obj
 0002:00014e38       ??_C@_08IPFLJFPM@BlueFuzz@ 10086e38     freetype:type1.obj
 0002:00014e44       ??_C@_0L@DKDIMLOI@BlueValues@ 10086e44     freetype:type1.obj
 0002:00014e50       ??_C@_0L@CCJAIIMC@OtherBlues@ 10086e50     freetype:type1.obj
 0002:00014e5c       ??_C@_0M@OIPOLIDA@FamilyBlues@ 10086e5c     freetype:type1.obj
 0002:00014e68       ??_C@_0BB@FMLCJJDP@FamilyOtherBlues@ 10086e68     freetype:type1.obj
 0002:00014e7c       ??_C@_05PHECBFLF@StdHW@    10086e7c     freetype:type1.obj
 0002:00014e84       ??_C@_05OBPKJLMP@StdVW@    10086e84     freetype:type1.obj
 0002:00014e8c       ??_C@_0L@NKGPCONN@MinFeature@ 10086e8c     freetype:type1.obj
 0002:00014e98       ??_C@_09NCKADFKP@StemSnapH@ 10086e98     freetype:type1.obj
 0002:00014ea4       ??_C@_09GOBAKHA@StemSnapV@ 10086ea4     freetype:type1.obj
 0002:00014eb0       ??_C@_0BA@PKGIFANC@ExpansionFactor@ 10086eb0     freetype:type1.obj
 0002:00014ec0       ??_C@_09BDDIAPM@ForceBold@ 10086ec0     freetype:type1.obj
 0002:00014ecc       ??_C@_08MKFDOKHL@FontName@ 10086ecc     freetype:type1.obj
 0002:00014ed8       ??_C@_09PNDIDGHG@PaintType@ 10086ed8     freetype:type1.obj
 0002:00014ee4       ??_C@_08GBFACKAL@FontType@ 10086ee4     freetype:type1.obj
 0002:00014ef0       ??_C@_0M@GLGMDIGG@StrokeWidth@ 10086ef0     freetype:type1.obj
 0002:00014efc       ??_C@_08EBMMLPNI@FontBBox@ 10086efc     freetype:type1.obj
 0002:00014f08       ??_C@_03DOACNACD@NDV@      10086f08     freetype:type1.obj
 0002:00014f0c       ??_C@_03MMGIAIPO@CDV@      10086f0c     freetype:type1.obj
 0002:00014f10       ??_C@_0N@PGGOPDKP@DesignVector@ 10086f10     freetype:type1.obj
 0002:00014f20       ??_C@_0L@LNCCOCBB@FontMatrix@ 10086f20     freetype:type1.obj
 0002:00014f2c       ??_C@_08EJAHIGCJ@Encoding@ 10086f2c     freetype:type1.obj
 0002:00014f38       ??_C@_05DHFNOCDJ@Subrs@    10086f38     freetype:type1.obj
 0002:00014f40       ??_C@_0M@EKIFGBLL@CharStrings@ 10086f40     freetype:type1.obj
 0002:00014f4c       ??_C@_07CFINJGKH@Private@  10086f4c     freetype:type1.obj
 0002:00014f54       ??_C@_0BF@BEKHBPMN@BlendDesignPositions@ 10086f54     freetype:type1.obj
 0002:00014f6c       ??_C@_0P@FPDIEJKK@BlendDesignMap@ 10086f6c     freetype:type1.obj
 0002:00014f7c       ??_C@_0P@LEAACMFJ@BlendAxisTypes@ 10086f7c     freetype:type1.obj
 0002:00014f8c       ??_C@_0N@JPPBHHHF@WeightVector@ 10086f8c     freetype:type1.obj
 0002:00014f9c       ??_C@_0P@KEOGGALI@BuildCharArray@ 10086f9c     freetype:type1.obj
 0002:00014fac       ??_C@_09BJJLCLMA@closefile@ 10086fac     freetype:type1.obj
 0002:00014fb8       ??_C@_0O@CJLBGMNG@FontDirectory@ 10086fb8     freetype:type1.obj
 0002:00014fc8       ??_C@_08MNGCAOLP@pshinter@ 10086fc8     freetype:type1.obj
 0002:00014fd4       ??_C@_0BB@JIMLNENF@postscript?9cmaps@ 10086fd4     freetype:type1.obj
 0002:00014fe8       ??_C@_05MNCLAAKB@psaux@    10086fe8     freetype:type1.obj
 0002:00014ff0       ??_C@_07FFHPBFOK@Regular@  10086ff0     freetype:type1.obj
 0002:00014ff8       ??_C@_04DIPHHIHJ@Bold@     10086ff8     freetype:type1.obj
 0002:00015000       ??_C@_05BPGNDIAE@Black@    10087000     freetype:type1.obj
 0002:00015008       ??_C@_06JCBOBHIA@Type?51@  10087008     freetype:type1.obj
 0002:00015010       ??_C@_0BA@EAOIOGJA@postscript?9info@ 10087010     freetype:type1.obj
 0002:00015050       _cff_cmap_encoding_class_rec 10087050     freetype:cff.obj
 0002:00015078       _cff_cmap_unicode_class_rec 10087078     freetype:cff.obj
 0002:000150a0       _cff_driver_class          100870a0     freetype:cff.obj
 0002:00015f38       ??_C@_0BF@GIDENNON@darkening?9parameters@ 10087f38     freetype:cff.obj
 0002:00015f50       ??_C@_0P@DGAAAJJA@hinting?9engine@ 10087f50     freetype:cff.obj
 0002:00015f60       ??_C@_0BC@GFOLLGHN@no?9stem?9darkening@ 10087f60     freetype:cff.obj
 0002:00015f74       ??_C@_03IFCOMOMB@CFF@      10087f74     freetype:cff.obj
 0002:00015f78       ??_C@_03LMEEOLHO@CID@      10087f78     freetype:cff.obj
 0002:00015f7c       ??_C@_0CA@JGHPJJJF@?$CF?$CBPS?9Adobe?93?40?5Resource?9CIDFont@ 10087f7c     freetype:type1cid.obj
 0002:00015f9c       ??_C@_09BFOLOCGO@StartData@ 10087f9c     freetype:type1cid.obj
 0002:00015fa8       ??_C@_06EMLBPOPP@?1sfnts@  10087fa8     freetype:type1cid.obj
 0002:00015fb0       ??_C@_05NPBNGLLN@?$CIHex?$CJ@ 10087fb0     freetype:type1cid.obj
 0002:000166e8       _t1cid_driver_class        100886e8     freetype:type1cid.obj
 0002:00016790       ??_C@_0M@CKCGNNAK@CIDFontName@ 10088790     freetype:type1cid.obj
 0002:0001679c       ??_C@_0P@FDOGBFAP@CIDFontVersion@ 1008879c     freetype:type1cid.obj
 0002:000167ac       ??_C@_0M@IBCFBNHK@CIDFontType@ 100887ac     freetype:type1cid.obj
 0002:000167b8       ??_C@_08EPBENDNC@Registry@ 100887b8     freetype:type1cid.obj
 0002:000167c4       ??_C@_08HMKBFHBJ@Ordering@ 100887c4     freetype:type1cid.obj
 0002:000167d0       ??_C@_0L@EJNILPMC@Supplement@ 100887d0     freetype:type1cid.obj
 0002:000167dc       ??_C@_07CNNFHHEA@UIDBase@  100887dc     freetype:type1cid.obj
 0002:000167e4       ??_C@_0N@LBMCPKAC@CIDMapOffset@ 100887e4     freetype:type1cid.obj
 0002:000167f4       ??_C@_07NNGKIHHK@FDBytes@  100887f4     freetype:type1cid.obj
 0002:000167fc       ??_C@_07BBMAIHOE@GDBytes@  100887fc     freetype:type1cid.obj
 0002:00016804       ??_C@_08LPCKMOBH@CIDCount@ 10088804     freetype:type1cid.obj
 0002:00016810       ??_C@_0O@DKIHOHFK@SubrMapOffset@ 10088810     freetype:type1cid.obj
 0002:00016820       ??_C@_07OJDBLIDF@SDBytes@  10088820     freetype:type1cid.obj
 0002:00016828       ??_C@_09NKAONILE@SubrCount@ 10088828     freetype:type1cid.obj
 0002:00016834       ??_C@_0BC@HBJENNOG@lenBuildCharArray@ 10088834     freetype:type1cid.obj
 0002:00016848       ??_C@_0BD@BGHMBBEO@ForceBoldThreshold@ 10088848     freetype:type1cid.obj
 0002:0001685c       ??_C@_07PEKDNLEP@FDArray@  1008885c     freetype:type1cid.obj
 0002:00016864       ??_C@_0BC@JBBEDJNJ@?$CFADOBeginFontDict@ 10088864     freetype:type1cid.obj
 0002:00016878       ??_C@_0L@DDPIBKML@CID?5Type?51@ 10088878     freetype:type1cid.obj
 0002:00016884       ??_C@_05CNMLIGFM@t1cid@    10088884     freetype:type1cid.obj
 0002:0001692c       _pfr_cmap_class_rec        1008892c     freetype:pfr.obj
 0002:00016958       _pfr_driver_class          10088958     freetype:pfr.obj
 0002:000169b8       _pfr_metrics_service_rec   100889b8     freetype:pfr.obj
 0002:000169dc       ??_C@_0M@BAGPBJNL@pfr?9metrics@ 100889dc     freetype:pfr.obj
 0002:000169e8       ??_C@_03OJCMOBOF@PFR@      100889e8     freetype:pfr.obj
 0002:000169ec       ??_C@_03OENHCMJJ@pfr@      100889ec     freetype:pfr.obj
 0002:00016cc0       _t42_driver_class          10088cc0     freetype:type42.obj
 0002:00016d68       ??_C@_05FJOKMJFH@sfnts@    10088d68     freetype:type42.obj
 0002:00016d70       ??_C@_0BC@IJJLOJBO@?$CF?$CBPS?9TrueTypeFont@ 10088d70     freetype:type42.obj
 0002:00016d84       ??_C@_05MDIJLHEA@known@    10088d84     freetype:type42.obj
 0002:00016d8c       ??_C@_07GJBALKN@Type?542@  10088d8c     freetype:type42.obj
 0002:00016d98       _winfnt_driver_class       10088d98     freetype:winfnt.obj
 0002:00016fa0       ??_C@_0M@DFCIIFPB@Bold?5Italic@ 10088fa0     freetype:winfnt.obj
 0002:00016fac       ??_C@_06PPMHIBHB@Italic@   10088fac     freetype:winfnt.obj
 0002:00016fb4       ??_C@_0M@FPCOPFGH@Windows?5FNT@ 10088fb4     freetype:winfnt.obj
 0002:00016fc0       ??_C@_08NAMFKPDH@winfonts@ 10088fc0     freetype:winfnt.obj
 0002:000170e8       _pcf_driver_class          100890e8     freetype:pcf.obj
 0002:00017148       _pcf_cmap_class            10089148     freetype:pcf.obj
 0002:00017190       ??_C@_05NOFPJGIP@SLANT@    10089190     freetype:pcf.obj
 0002:00017198       ??_C@_07EGOIFKG@Oblique@   10089198     freetype:pcf.obj
 0002:000171a0       ??_C@_0M@FCJHKPGH@WEIGHT_NAME@ 100891a0     freetype:pcf.obj
 0002:000171ac       ??_C@_0O@DANCJNNA@SETWIDTH_NAME@ 100891ac     freetype:pcf.obj
 0002:000171bc       ??_C@_0P@BLEODLOA@ADD_STYLE_NAME@ 100891bc     freetype:pcf.obj
 0002:000171cc       ??_C@_0M@FBEHGJKE@FAMILY_NAME@ 100891cc     freetype:pcf.obj
 0002:000171d8       ??_C@_0O@KPOPAFON@AVERAGE_WIDTH@ 100891d8     freetype:pcf.obj
 0002:000171e8       ??_C@_0L@JCJJGPJF@POINT_SIZE@ 100891e8     freetype:pcf.obj
 0002:000171f4       ??_C@_0L@CNGHIHBP@PIXEL_SIZE@ 100891f4     freetype:pcf.obj
 0002:00017200       ??_C@_0N@NBDHNJFJ@RESOLUTION_X@ 10089200     freetype:pcf.obj
 0002:00017210       ??_C@_0N@MICMOIBI@RESOLUTION_Y@ 10089210     freetype:pcf.obj
 0002:00017220       ??_C@_0BB@OHIDJKBJ@CHARSET_REGISTRY@ 10089220     freetype:pcf.obj
 0002:00017234       ??_C@_0BB@OBJAMPOC@CHARSET_ENCODING@ 10089234     freetype:pcf.obj
 0002:00017248       ??_C@_05FPAEEJJG@10646@    10089248     freetype:pcf.obj
 0002:00017250       ??_C@_04LBDHIBCK@8859@     10089250     freetype:pcf.obj
 0002:00017258       ??_C@_01HIHLOKLC@1@        10089258     freetype:pcf.obj
 0002:0001725c       ??_C@_03DDONLALG@bdf@      1008925c     freetype:pcf.obj
 0002:00017260       ??_C@_03MBEJPEFL@PCF@      10089260     freetype:pcf.obj
 0002:00017264       ??_C@_03MMLCDJCH@pcf@      10089264     freetype:pcf.obj
 0002:00017268       _ps_table_funcs            10089268     freetype:psaux.obj
 0002:00017278       _ps_parser_funcs           10089278     freetype:psaux.obj
 0002:000172ac       _t1_builder_funcs          100892ac     freetype:psaux.obj
 0002:000172cc       _t1_decoder_funcs          100892cc     freetype:psaux.obj
 0002:000172d8       _t1_cmap_standard_class_rec 100892d8     freetype:psaux.obj
 0002:00017300       _t1_cmap_expert_class_rec  10089300     freetype:psaux.obj
 0002:00017328       _t1_cmap_custom_class_rec  10089328     freetype:psaux.obj
 0002:00017350       _t1_cmap_unicode_class_rec 10089350     freetype:psaux.obj
 0002:00017378       _afm_parser_funcs          10089378     freetype:psaux.obj
 0002:00017384       _t1_cmap_classes           10089384     freetype:psaux.obj
 0002:000173b0       _psaux_module_class        100893b0     freetype:psaux.obj
 0002:000175f0       ??_C@_08NBPEBJDA@Ascender@ 100895f0     freetype:psaux.obj
 0002:000175fc       ??_C@_09POOBGNPO@AxisLabel@ 100895fc     freetype:psaux.obj
 0002:00017608       ??_C@_08KLONHBMG@AxisType@ 10089608     freetype:psaux.obj
 0002:00017614       ??_C@_01HMGJMAIH@B@        10089614     freetype:psaux.obj
 0002:00017618       ??_C@_01GFHCPBMG@C@        10089618     freetype:psaux.obj
 0002:0001761c       ??_C@_02KJDGAJLC@CC@       1008961c     freetype:psaux.obj
 0002:00017620       ??_C@_02EKMCNAHJ@CH@       10089620     freetype:psaux.obj
 0002:00017624       ??_C@_09JOCJHGEG@CapHeight@ 10089624     freetype:psaux.obj
 0002:00017630       ??_C@_09CGMEAFLF@CharWidth@ 10089630     freetype:psaux.obj
 0002:0001763c       ??_C@_0N@LHPDLMAH@CharacterSet@ 1008963c     freetype:psaux.obj
 0002:0001764c       ??_C@_0L@EMODJLOD@Characters@ 1008964c     freetype:psaux.obj
 0002:00017658       ??_C@_09JMDLBBJN@Descender@ 10089658     freetype:psaux.obj
 0002:00017664       ??_C@_0P@JNPLONMI@EncodingScheme@ 10089664     freetype:psaux.obj
 0002:00017674       ??_C@_07DLEALFPL@EndAxis@  10089674     freetype:psaux.obj
 0002:0001767c       ??_C@_0P@GFNMGKCM@EndCharMetrics@ 1008967c     freetype:psaux.obj
 0002:0001768c       ??_C@_0O@JABMALCH@EndComposites@ 1008968c     freetype:psaux.obj
 0002:0001769c       ??_C@_0N@FNMEONKF@EndDirection@ 1008969c     freetype:psaux.obj
 0002:000176ac       ??_C@_0P@FGFFCKLI@EndFontMetrics@ 100896ac     freetype:psaux.obj
 0002:000176bc       ??_C@_0M@HKHGIIOM@EndKernData@ 100896bc     freetype:psaux.obj
 0002:000176c8       ??_C@_0N@IJIACAAI@EndKernPairs@ 100896c8     freetype:psaux.obj
 0002:000176d8       ??_C@_0N@FEBBJBLC@EndTrackKern@ 100896d8     freetype:psaux.obj
 0002:000176e8       ??_C@_07BNJNBMEL@EscChar@  100896e8     freetype:psaux.obj
 0002:000176f0       ??_C@_0L@PAHDJIHN@IsBaseFont@ 100896f0     freetype:psaux.obj
 0002:000176fc       ??_C@_09OIFAOJEJ@IsCIDFont@ 100896fc     freetype:psaux.obj
 0002:00017708       ??_C@_0N@LNIFJEBO@IsFixedPitch@ 10089708     freetype:psaux.obj
 0002:00017718       ??_C@_08CHFNODLO@IsFixedV@ 10089718     freetype:psaux.obj
 0002:00017724       ??_C@_02MGMKBJJI@KP@       10089724     freetype:psaux.obj
 0002:00017728       ??_C@_03MGLCBEGC@KPH@      10089728     freetype:psaux.obj
 0002:0001772c       ??_C@_03IMHAAGDD@KPX@      1008972c     freetype:psaux.obj
 0002:00017730       ??_C@_03JFGLDHHC@KPY@      10089730     freetype:psaux.obj
 0002:00017734       ??_C@_01OCOKONAJ@L@        10089734     freetype:psaux.obj
 0002:00017738       ??_C@_0O@NDBFHPJC@MappingScheme@ 10089738     freetype:psaux.obj
 0002:00017748       ??_C@_0M@PGHPLBFB@MetricsSets@ 10089748     freetype:psaux.obj
 0002:00017754       ??_C@_01NANMIPIL@N@        10089754     freetype:psaux.obj
 0002:00017758       ??_C@_03LMDOAABO@PCC@      10089758     freetype:psaux.obj
 0002:0001775c       ??_C@_09JMBADFPL@StartAxis@ 1008975c     freetype:psaux.obj
 0002:00017768       ??_C@_0BB@JDMDJAID@StartCharMetrics@ 10089768     freetype:psaux.obj
 0002:0001777c       ??_C@_0BA@DGMAPPPC@StartComposites@ 1008977c     freetype:psaux.obj
 0002:0001778c       ??_C@_0P@DNGHFPAA@StartDirection@ 1008978c     freetype:psaux.obj
 0002:0001779c       ??_C@_0BB@KAEKNABH@StartFontMetrics@ 1008979c     freetype:psaux.obj
 0002:000177b0       ??_C@_0O@GJEKPIHD@StartKernData@ 100897b0     freetype:psaux.obj
 0002:000177c0       ??_C@_0P@OJCDJCKN@StartKernPairs@ 100897c0     freetype:psaux.obj
 0002:000177d0       ??_C@_0BA@HHMIMKDE@StartKernPairs0@ 100897d0     freetype:psaux.obj
 0002:000177e0       ??_C@_0BA@GONDPLHF@StartKernPairs1@ 100897e0     freetype:psaux.obj
 0002:000177f0       ??_C@_0P@DELCCDBH@StartTrackKern@ 100897f0     freetype:psaux.obj
 0002:00017800       ??_C@_09DJCDMHFC@TrackKern@ 10089800     freetype:psaux.obj
 0002:0001780c       ??_C@_02IEGOIODN@VV@       1008980c     freetype:psaux.obj
 0002:00017810       ??_C@_07HFOFDFIM@VVector@  10089810     freetype:psaux.obj
 0002:00017818       ??_C@_07NGFJPNPN@Version@  10089818     freetype:psaux.obj
 0002:00017820       ??_C@_01ELNMCGJD@W@        10089820     freetype:psaux.obj
 0002:00017824       ??_C@_02LGALCICL@W0@       10089824     freetype:psaux.obj
 0002:00017828       ??_C@_03NOGICFDE@W0X@      10089828     freetype:psaux.obj
 0002:0001782c       ??_C@_03MHHDBEHF@W0Y@      1008982c     freetype:psaux.obj
 0002:00017830       ??_C@_02KPBABJGK@W1@       10089830     freetype:psaux.obj
 0002:00017834       ??_C@_03NPKKEPAD@W1X@      10089834     freetype:psaux.obj
 0002:00017838       ??_C@_03MGLBHOEC@W1Y@      10089838     freetype:psaux.obj
 0002:0001783c       ??_C@_02BLCPMJIE@WX@       1008983c     freetype:psaux.obj
 0002:00017840       ??_C@_02CDEPIMF@WY@        10089840     freetype:psaux.obj
 0002:00017844       ??_C@_07MIHJBPO@XHeight@   10089844     freetype:psaux.obj
 0002:0001784c       ??_C@_04LOAJBDKD@true@     1008984c     freetype:psaux.obj
 0002:00017858       _psnames_module_class      10089858     freetype:psmodule.obj
 0002:00026ba0       ??_C@_07POODEHEH@psnames@  10098ba0     freetype:psmodule.obj
 0002:00026bb4       _pshinter_module_class     10098bb4     freetype:pshinter.obj
 0002:00026bd8       _ft_standard_raster        10098bd8     freetype:raster.obj
 0002:00026bf0       _ft_raster1_renderer_class 10098bf0     freetype:raster.obj
 0002:00026c2c       _ft_raster5_renderer_class 10098c2c     freetype:raster.obj
 0002:00026c68       ??_C@_07EFFNHEPH@raster1@  10098c68     freetype:raster.obj
 0002:00026c70       ??_C@_07CBDBLBPD@raster5@  10098c70     freetype:raster.obj
 0002:00026c78       _tt_cmap13_class_rec       10098c78     freetype:sfnt.obj
 0002:00026cac       _tt_cmap14_class_rec       10098cac     freetype:sfnt.obj
 0002:00026dd8       _sfnt_module_class         10098dd8     freetype:sfnt.obj
 0002:00027174       _tt_cmap0_class_rec        10099174     freetype:sfnt.obj
 0002:000271a8       _tt_cmap2_class_rec        100991a8     freetype:sfnt.obj
 0002:000271dc       _tt_cmap4_class_rec        100991dc     freetype:sfnt.obj
 0002:00027210       _tt_cmap6_class_rec        10099210     freetype:sfnt.obj
 0002:00027244       _tt_cmap8_class_rec        10099244     freetype:sfnt.obj
 0002:00027278       _tt_cmap10_class_rec       10099278     freetype:sfnt.obj
 0002:000272ac       _tt_cmap12_class_rec       100992ac     freetype:sfnt.obj
 0002:000272e0       _ft_grays_raster           100992e0     freetype:smooth.obj
 0002:00027310       _ft_smooth_renderer_class  10099310     freetype:smooth.obj
 0002:0002734c       _ft_smooth_lcd_renderer_class 1009934c     freetype:smooth.obj
 0002:00027388       _ft_smooth_lcdv_renderer_class 10099388     freetype:smooth.obj
 0002:000273c4       ??_C@_06INICNAFJ@smooth@   100993c4     freetype:smooth.obj
 0002:000273cc       ??_C@_0L@KCJBAIJI@smooth?9lcd@ 100993cc     freetype:smooth.obj
 0002:000273d8       ??_C@_0M@IHBDFEAO@smooth?9lcdv@ 100993d8     freetype:smooth.obj
 0002:00027a18       _bdf_driver_class          10099a18     freetype:bdf.obj
 0002:00027a78       _bdf_cmap_class            10099a78     freetype:bdf.obj
 0002:00027ac0       ??_C@_0BC@DEIBICAG@AVG_CAPITAL_WIDTH@ 10099ac0     freetype:bdf.obj
 0002:00027ad4       ??_C@_0BE@FDPIDJIH@AVG_LOWERCASE_WIDTH@ 10099ad4     freetype:bdf.obj
 0002:00027ae8       ??_C@_0L@IPPBEDCK@CAP_HEIGHT@ 10099ae8     freetype:bdf.obj
 0002:00027af4       ??_C@_0BE@KNHMGHPI@CHARSET_COLLECTIONS@ 10099af4     freetype:bdf.obj
 0002:00027b08       ??_C@_07JEDAPFNH@COMMENT@  10099b08     freetype:bdf.obj
 0002:00027b10       ??_C@_09DJIAAPDG@COPYRIGHT@ 10099b10     freetype:bdf.obj
 0002:00027b1c       ??_C@_0N@LOGJBDOF@DEFAULT_CHAR@ 10099b1c     freetype:bdf.obj
 0002:00027b2c       ??_C@_0M@LFJMPFGC@DESTINATION@ 10099b2c     freetype:bdf.obj
 0002:00027b38       ??_C@_0BB@PJMJCLEI@DEVICE_FONT_NAME@ 10099b38     freetype:bdf.obj
 0002:00027b4c       ??_C@_09GEIPNEKC@END_SPACE@ 10099b4c     freetype:bdf.obj
 0002:00027b58       ??_C@_09DLOGKOHL@FACE_NAME@ 10099b58     freetype:bdf.obj
 0002:00027b64       ??_C@_0N@LCIIJFB@FIGURE_WIDTH@ 10099b64     freetype:bdf.obj
 0002:00027b74       ??_C@_04IJMKNFPK@FONT@     10099b74     freetype:bdf.obj
 0002:00027b7c       ??_C@_0BC@LNICJLFI@FONTNAME_REGISTRY@ 10099b7c     freetype:bdf.obj
 0002:00027b90       ??_C@_0M@ECCDLGDC@FONT_ASCENT@ 10099b90     freetype:bdf.obj
 0002:00027b9c       ??_C@_0N@BAIKBLGK@FONT_DESCENT@ 10099b9c     freetype:bdf.obj
 0002:00027bac       ??_C@_07GMNLECKJ@FOUNDRY@  10099bac     freetype:bdf.obj
 0002:00027bb4       ??_C@_09IGHCOKHJ@FULL_NAME@ 10099bb4     freetype:bdf.obj
 0002:00027bc0       ??_C@_0N@LHJKBLMB@ITALIC_ANGLE@ 10099bc0     freetype:bdf.obj
 0002:00027bd0       ??_C@_09IDPFHPOD@MAX_SPACE@ 10099bd0     freetype:bdf.obj
 0002:00027bdc       ??_C@_09ICPJOFFH@MIN_SPACE@ 10099bdc     freetype:bdf.obj
 0002:00027be8       ??_C@_0L@CKCFAFFG@NORM_SPACE@ 10099be8     freetype:bdf.obj
 0002:00027bf4       ??_C@_06FMPEGAHJ@NOTICE@   10099bf4     freetype:bdf.obj
 0002:00027bfc       ??_C@_0L@MANNMNIK@QUAD_WIDTH@ 10099bfc     freetype:bdf.obj
 0002:00027c08       ??_C@_0L@CAMLDNCF@RAW_ASCENT@ 10099c08     freetype:bdf.obj
 0002:00027c14       ??_C@_0BC@LNOEENJF@RAW_AVERAGE_WIDTH@ 10099c14     freetype:bdf.obj
 0002:00027c28       ??_C@_0BG@PEMOHOIO@RAW_AVG_CAPITAL_WIDTH@ 10099c28     freetype:bdf.obj
 0002:00027c40       ??_C@_0BI@BEKJFFLM@RAW_AVG_LOWERCASE_WIDTH@ 10099c40     freetype:bdf.obj
 0002:00027c58       ??_C@_0P@PDBKEGFB@RAW_CAP_HEIGHT@ 10099c58     freetype:bdf.obj
 0002:00027c68       ??_C@_0M@JDDLHGCG@RAW_DESCENT@ 10099c68     freetype:bdf.obj
 0002:00027c74       ??_C@_0O@FDGFBIGM@RAW_END_SPACE@ 10099c74     freetype:bdf.obj
 0002:00027c84       ??_C@_0BB@LHIJKBAI@RAW_FIGURE_WIDTH@ 10099c84     freetype:bdf.obj
 0002:00027c98       ??_C@_0O@LEBPLDCN@RAW_MAX_SPACE@ 10099c98     freetype:bdf.obj
 0002:00027ca8       ??_C@_0O@LFBDCJJJ@RAW_MIN_SPACE@ 10099ca8     freetype:bdf.obj
 0002:00027cb8       ??_C@_0P@FGMOAACN@RAW_NORM_SPACE@ 10099cb8     freetype:bdf.obj
 0002:00027cc8       ??_C@_0P@FBIMICGE@RAW_PIXEL_SIZE@ 10099cc8     freetype:bdf.obj
 0002:00027cd8       ??_C@_0P@OOHCGKOO@RAW_POINT_SIZE@ 10099cd8     freetype:bdf.obj
 0002:00027ce8       ??_C@_0O@HNFKKCGD@RAW_PIXELSIZE@ 10099ce8     freetype:bdf.obj
 0002:00027cf8       ??_C@_0O@FDNDDOFA@RAW_POINTSIZE@ 10099cf8     freetype:bdf.obj
 0002:00027d08       ??_C@_0P@LMDGMIPB@RAW_QUAD_WIDTH@ 10099d08     freetype:bdf.obj
 0002:00027d18       ??_C@_0BD@HHNHPPKD@RAW_SMALL_CAP_SIZE@ 10099d18     freetype:bdf.obj
 0002:00027d2c       ??_C@_0BF@DLAIFMIE@RAW_STRIKEOUT_ASCENT@ 10099d2c     freetype:bdf.obj
 0002:00027d44       ??_C@_0BG@DCPBCGDJ@RAW_STRIKEOUT_DESCENT@ 10099d44     freetype:bdf.obj
 0002:00027d5c       ??_C@_0BD@FGAMCDPE@RAW_SUBSCRIPT_SIZE@ 10099d5c     freetype:bdf.obj
 0002:00027d70       ??_C@_0BA@ICOMKGEO@RAW_SUBSCRIPT_X@ 10099d70     freetype:bdf.obj
 0002:00027d80       ??_C@_0BA@JLPHJHAP@RAW_SUBSCRIPT_Y@ 10099d80     freetype:bdf.obj
 0002:00027d90       ??_C@_0BF@ILCJEECH@RAW_SUPERSCRIPT_SIZE@ 10099d90     freetype:bdf.obj
 0002:00027da8       ??_C@_0BC@EMCLOPNI@RAW_SUPERSCRIPT_X@ 10099da8     freetype:bdf.obj
 0002:00027dbc       ??_C@_0BC@FFDANOJJ@RAW_SUPERSCRIPT_Y@ 10099dbc     freetype:bdf.obj
 0002:00027dd0       ??_C@_0BH@LIHCGIBB@RAW_UNDERLINE_POSITION@ 10099dd0     freetype:bdf.obj
 0002:00027de8       ??_C@_0BI@OEPMFPAK@RAW_UNDERLINE_THICKNESS@ 10099de8     freetype:bdf.obj
 0002:00027e00       ??_C@_0N@LFICGJOL@RAW_X_HEIGHT@ 10099e00     freetype:bdf.obj
 0002:00027e10       ??_C@_0BC@JMGAMBDF@RELATIVE_SETWIDTH@ 10099e10     freetype:bdf.obj
 0002:00027e24       ??_C@_0BA@NKHOPHOP@RELATIVE_WEIGHT@ 10099e24     freetype:bdf.obj
 0002:00027e34       ??_C@_0L@JGAABLGD@RESOLUTION@ 10099e34     freetype:bdf.obj
 0002:00027e40       ??_C@_0P@CJBLANOF@SMALL_CAP_SIZE@ 10099e40     freetype:bdf.obj
 0002:00027e50       ??_C@_07JKNGKIOL@SPACING@  10099e50     freetype:bdf.obj
 0002:00027e58       ??_C@_0BB@MOJIHJPL@STRIKEOUT_ASCENT@ 10099e58     freetype:bdf.obj
 0002:00027e6c       ??_C@_0BC@PCLONKLB@STRIKEOUT_DESCENT@ 10099e6c     freetype:bdf.obj
 0002:00027e80       ??_C@_0P@IMANBLC@SUBSCRIPT_SIZE@ 10099e80     freetype:bdf.obj
 0002:00027e90       ??_C@_0M@EFEHOFPP@SUBSCRIPT_X@ 10099e90     freetype:bdf.obj
 0002:00027e9c       ??_C@_0M@FMFMNELO@SUBSCRIPT_Y@ 10099e9c     freetype:bdf.obj
 0002:00027ea8       ??_C@_0BB@HOLJGBFI@SUPERSCRIPT_SIZE@ 10099ea8     freetype:bdf.obj
 0002:00027ebc       ??_C@_0O@FOCAKHKA@SUPERSCRIPT_X@ 10099ebc     freetype:bdf.obj
 0002:00027ecc       ??_C@_0O@EHDLJGOB@SUPERSCRIPT_Y@ 10099ecc     freetype:bdf.obj
 0002:00027edc       ??_C@_0BD@FLNBCMPP@UNDERLINE_POSITION@ 10099edc     freetype:bdf.obj
 0002:00027ef0       ??_C@_0BE@KDKNDDDB@UNDERLINE_THICKNESS@ 10099ef0     freetype:bdf.obj
 0002:00027f04       ??_C@_06CIAKHCPD@WEIGHT@   10099f04     freetype:bdf.obj
 0002:00027f0c       ??_C@_08IHHFFHAA@X_HEIGHT@ 10099f0c     freetype:bdf.obj
 0002:00027f18       ??_C@_0BG@NJJHMBCE@_MULE_BASELINE_OFFSET@ 10099f18     freetype:bdf.obj
 0002:00027f30       ??_C@_0BH@EGBLCDE@_MULE_RELATIVE_COMPOSE@ 10099f30     freetype:bdf.obj
 0002:00027f48       ??_C@_01JOAMLHOP@?9@       10099f48     freetype:bdf.obj
 0002:00027f4c       ??_C@_05HCHEPOAH@CHARS@    10099f4c     freetype:bdf.obj
 0002:00027f54       ??_C@_02EOIDJNGE@?5?$CL@   10099f54     freetype:bdf.obj
 0002:00027f58       ??_C@_07MLEKHHFJ@ENDFONT@  10099f58     freetype:bdf.obj
 0002:00027f60       ??_C@_07MDHLCACL@ENDCHAR@  10099f60     freetype:bdf.obj
 0002:00027f68       ??_C@_09BPKMEANO@STARTCHAR@ 10099f68     freetype:bdf.obj
 0002:00027f74       ??_C@_08LEFKDKKN@ENCODING@ 10099f74     freetype:bdf.obj
 0002:00027f80       ??_C@_06HDKFFNNH@SWIDTH@   10099f80     freetype:bdf.obj
 0002:00027f88       ??_C@_06NBNMPPJH@DWIDTH@   10099f88     freetype:bdf.obj
 0002:00027f90       ??_C@_03OONKDOKH@BBX@      10099f90     freetype:bdf.obj
 0002:00027f94       ??_C@_06PGFOEMDN@BITMAP@   10099f94     freetype:bdf.obj
 0002:00027f9c       ??_C@_0O@JFDPHGFD@ENDPROPERTIES@ 10099f9c     freetype:bdf.obj
 0002:00027fac       ??_C@_03OACELNE@?$CFhd@    10099fac     freetype:bdf.obj
 0002:00027fb0       ??_C@_0BG@NDMEGDOA@_XFREE86_GLYPH_RANGES@ 10099fb0     freetype:bdf.obj
 0002:00027fc8       ??_C@_09BHJNBHKM@STARTFONT@ 10099fc8     freetype:bdf.obj
 0002:00027fd4       ??_C@_0BA@HGECMEMA@STARTPROPERTIES@ 10099fd4     freetype:bdf.obj
 0002:00027fe4       ??_C@_0BA@PIDAKDPC@FONTBOUNDINGBOX@ 10099fe4     freetype:bdf.obj
 0002:00027ff4       ??_C@_04EMFHLKGI@SIZE@     10099ff4     freetype:bdf.obj
 0002:00027ffc       ??_C@_03DOBGHNMK@BDF@      10099ffc     freetype:bdf.obj
 0002:00028000       __xmm@00000008000000000000000100000001 1009a000     freetype:bdf.obj
 0002:00028010       ??_C@_02JDPG@rb@           1009a010     freetype:ftsystem.obj
 0002:000293b4       ??_C@_0CI@CGMOPDPD@oversubscribed?5dynamic?5bit?5leng@ 1009b3b4     freetype:ftgzip.obj
 0002:000293dc       ??_C@_0CE@LOHAHEGK@incomplete?5dynamic?5bit?5lengths?5@ 1009b3dc     freetype:ftgzip.obj
 0002:00029400       ??_C@_0CD@GJIDGCKE@oversubscribed?5literal?1length?5t@ 1009b400     freetype:ftgzip.obj
 0002:00029424       ??_C@_0BP@NEEEJJNA@incomplete?5literal?1length?5tree@ 1009b424     freetype:ftgzip.obj
 0002:00029444       ??_C@_0BN@KBLCDIAI@oversubscribed?5distance?5tree@ 1009b444     freetype:ftgzip.obj
 0002:00029464       ??_C@_0BJ@CBCPDPJF@incomplete?5distance?5tree@ 1009b464     freetype:ftgzip.obj
 0002:00029480       ??_C@_0CB@KPKKKLFO@empty?5distance?5tree?5with?5length@ 1009b480     freetype:ftgzip.obj
 0002:000294a4       ??_C@_0BM@FFFLPBBC@invalid?5literal?1length?5code@ 1009b4a4     freetype:ftgzip.obj
 0002:000294c0       ??_C@_0BG@LBKINIKP@invalid?5distance?5code@ 1009b4c0     freetype:ftgzip.obj
 0002:000294d8       ??_C@_0BD@PJCBIDD@invalid?5block?5type@ 1009b4d8     freetype:ftgzip.obj
 0002:000294ec       ??_C@_0BN@LGAADGOK@invalid?5stored?5block?5lengths@ 1009b4ec     freetype:ftgzip.obj
 0002:0002950c       ??_C@_0CE@GMIGFPBB@too?5many?5length?5or?5distance?5sym@ 1009b50c     freetype:ftgzip.obj
 0002:00029530       ??_C@_0BK@BMMPFBBH@invalid?5bit?5length?5repeat@ 1009b530     freetype:ftgzip.obj
 0002:0002954c       ??_C@_05DOIEBMOI@1?41?44@  1009b54c     freetype:ftgzip.obj
 0002:00029554       ??_C@_0BL@IHKGDAEE@unknown?5compression?5method@ 1009b554     freetype:ftgzip.obj
 0002:00029570       ??_C@_0BE@EMOGCLGO@invalid?5window?5size@ 1009b570     freetype:ftgzip.obj
 0002:00029584       ??_C@_0BH@LIBMMIGA@incorrect?5header?5check@ 1009b584     freetype:ftgzip.obj
 0002:0002959c       ??_C@_0BA@MOKMMFOD@need?5dictionary@ 1009b59c     freetype:ftgzip.obj
 0002:000295ac       ??_C@_0BF@MEIGEHBE@incorrect?5data?5check@ 1009b5ac     freetype:ftgzip.obj
 0002:000295e0       ??_7type_info@@6B@         1009b5e0     MSVCRT:std_type_info_static.obj
 0002:00029620       __pDefaultRawDllMain       1009b620     MSVCRT:dll_dllmain.obj
 0002:00029620       __pRawDllMain              1009b620     MSVCRT:dll_dllmain.obj
 0002:00029628       ??_7exception@std@@6B@     1009b628     MSVCRT:throw_bad_alloc.obj
 0002:00029630       ??_C@_0BC@EOODALEL@Unknown?5exception@ 1009b630     MSVCRT:throw_bad_alloc.obj
 0002:00029648       ??_7bad_alloc@std@@6B@     1009b648     MSVCRT:throw_bad_alloc.obj
 0002:00029650       ??_C@_0P@GHFPNOJB@bad?5allocation@ 1009b650     MSVCRT:throw_bad_alloc.obj
 0002:00029664       ??_7bad_array_new_length@std@@6B@ 1009b664     MSVCRT:throw_bad_alloc.obj
 0002:0002966c       ??_C@_0BF@KINCDENJ@bad?5array?5new?5length@ 1009b66c     MSVCRT:throw_bad_alloc.obj
 0002:00029690       __load_config_used         1009b690     MSVCRT:loadcfg.obj
 0002:000297c0       ??_R4ArabicOpenTypeLayoutEngine@@6B@ 1009b7c0     ArabicLayoutEngine.obj
 0002:000297d4       ??_R3ArabicOpenTypeLayoutEngine@@8 1009b7d4     ArabicLayoutEngine.obj
 0002:000297e4       ??_R2ArabicOpenTypeLayoutEngine@@8 1009b7e4     ArabicLayoutEngine.obj
 0002:000297f8       ??_R1A@?0A@EA@ArabicOpenTypeLayoutEngine@@8 1009b7f8     ArabicLayoutEngine.obj
 0002:00029814       ??_R1A@?0A@EA@OpenTypeLayoutEngine@@8 1009b814     ArabicLayoutEngine.obj
 0002:00029830       ??_R3OpenTypeLayoutEngine@@8 1009b830     ArabicLayoutEngine.obj
 0002:00029840       ??_R2OpenTypeLayoutEngine@@8 1009b840     ArabicLayoutEngine.obj
 0002:00029850       ??_R1A@?0A@EA@LayoutEngine@@8 1009b850     ArabicLayoutEngine.obj
 0002:0002986c       ??_R3LayoutEngine@@8       1009b86c     ArabicLayoutEngine.obj
 0002:0002987c       ??_R2LayoutEngine@@8       1009b87c     ArabicLayoutEngine.obj
 0002:00029888       ??_R13?0A@EA@UObject@@8    1009b888     ArabicLayoutEngine.obj
 0002:000298a4       ??_R3UObject@@8            1009b8a4     ArabicLayoutEngine.obj
 0002:000298b4       ??_R2UObject@@8            1009b8b4     ArabicLayoutEngine.obj
 0002:000298bc       ??_R1A@?0A@EA@UObject@@8   1009b8bc     ArabicLayoutEngine.obj
 0002:000298d8       ??_R4UnicodeArabicOpenTypeLayoutEngine@@6B@ 1009b8d8     ArabicLayoutEngine.obj
 0002:000298ec       ??_R3UnicodeArabicOpenTypeLayoutEngine@@8 1009b8ec     ArabicLayoutEngine.obj
 0002:000298fc       ??_R2UnicodeArabicOpenTypeLayoutEngine@@8 1009b8fc     ArabicLayoutEngine.obj
 0002:00029914       ??_R1A@?0A@EA@UnicodeArabicOpenTypeLayoutEngine@@8 1009b914     ArabicLayoutEngine.obj
 0002:00029930       ??_R4ContextualGlyphInsertionProcessor2@@6B@ 1009b930     ContextualGlyphInsertionProc2.obj
 0002:00029944       ??_R3ContextualGlyphInsertionProcessor2@@8 1009b944     ContextualGlyphInsertionProc2.obj
 0002:00029954       ??_R2ContextualGlyphInsertionProcessor2@@8 1009b954     ContextualGlyphInsertionProc2.obj
 0002:00029968       ??_R1A@?0A@EA@ContextualGlyphInsertionProcessor2@@8 1009b968     ContextualGlyphInsertionProc2.obj
 0002:00029984       ??_R1A@?0A@EA@StateTableProcessor2@@8 1009b984     ContextualGlyphInsertionProc2.obj
 0002:000299a0       ??_R3StateTableProcessor2@@8 1009b9a0     ContextualGlyphInsertionProc2.obj
 0002:000299b0       ??_R2StateTableProcessor2@@8 1009b9b0     ContextualGlyphInsertionProc2.obj
 0002:000299c0       ??_R1A@?0A@EA@SubtableProcessor2@@8 1009b9c0     ContextualGlyphInsertionProc2.obj
 0002:000299dc       ??_R3SubtableProcessor2@@8 1009b9dc     ContextualGlyphInsertionProc2.obj
 0002:000299ec       ??_R2SubtableProcessor2@@8 1009b9ec     ContextualGlyphInsertionProc2.obj
 0002:000299f8       ??_R13?0A@EA@UMemory@@8    1009b9f8     ContextualGlyphInsertionProc2.obj
 0002:00029a14       ??_R3UMemory@@8            1009ba14     ContextualGlyphInsertionProc2.obj
 0002:00029a24       ??_R2UMemory@@8            1009ba24     ContextualGlyphInsertionProc2.obj
 0002:00029a2c       ??_R1A@?0A@EA@UMemory@@8   1009ba2c     ContextualGlyphInsertionProc2.obj
 0002:00029a48       ??_R4ContextualGlyphSubstitutionProcessor@@6B@ 1009ba48     ContextualGlyphSubstProc.obj
 0002:00029a5c       ??_R3ContextualGlyphSubstitutionProcessor@@8 1009ba5c     ContextualGlyphSubstProc.obj
 0002:00029a6c       ??_R2ContextualGlyphSubstitutionProcessor@@8 1009ba6c     ContextualGlyphSubstProc.obj
 0002:00029a80       ??_R1A@?0A@EA@ContextualGlyphSubstitutionProcessor@@8 1009ba80     ContextualGlyphSubstProc.obj
 0002:00029a9c       ??_R1A@?0A@EA@StateTableProcessor@@8 1009ba9c     ContextualGlyphSubstProc.obj
 0002:00029ab8       ??_R3StateTableProcessor@@8 1009bab8     ContextualGlyphSubstProc.obj
 0002:00029ac8       ??_R2StateTableProcessor@@8 1009bac8     ContextualGlyphSubstProc.obj
 0002:00029ad8       ??_R1A@?0A@EA@SubtableProcessor@@8 1009bad8     ContextualGlyphSubstProc.obj
 0002:00029af4       ??_R3SubtableProcessor@@8  1009baf4     ContextualGlyphSubstProc.obj
 0002:00029b04       ??_R2SubtableProcessor@@8  1009bb04     ContextualGlyphSubstProc.obj
 0002:00029b10       ??_R4ContextualGlyphSubstitutionProcessor2@@6B@ 1009bb10     ContextualGlyphSubstProc2.obj
 0002:00029b24       ??_R3ContextualGlyphSubstitutionProcessor2@@8 1009bb24     ContextualGlyphSubstProc2.obj
 0002:00029b34       ??_R2ContextualGlyphSubstitutionProcessor2@@8 1009bb34     ContextualGlyphSubstProc2.obj
 0002:00029b48       ??_R1A@?0A@EA@ContextualGlyphSubstitutionProcessor2@@8 1009bb48     ContextualGlyphSubstProc2.obj
 0002:00029b64       ??_R4LEFontInstance@@6B@   1009bb64     FontInstanceAdapter.obj
 0002:00029b78       ??_R3LEFontInstance@@8     1009bb78     FontInstanceAdapter.obj
 0002:00029b88       ??_R2LEFontInstance@@8     1009bb88     FontInstanceAdapter.obj
 0002:00029b94       ??_R1A@?0A@EA@LEFontInstance@@8 1009bb94     FontInstanceAdapter.obj
 0002:00029bb0       ??_R4FontInstanceAdapter@@6B@ 1009bbb0     FontInstanceAdapter.obj
 0002:00029bc4       ??_R3FontInstanceAdapter@@8 1009bbc4     FontInstanceAdapter.obj
 0002:00029bd4       ??_R2FontInstanceAdapter@@8 1009bbd4     FontInstanceAdapter.obj
 0002:00029be4       ??_R1A@?0A@EA@FontInstanceAdapter@@8 1009bbe4     FontInstanceAdapter.obj
 0002:00029c00       ??_R4LEGlyphFilter@@6B@    1009bc00     GDEFMarkFilter.obj
 0002:00029c14       ??_R3LEGlyphFilter@@8      1009bc14     GDEFMarkFilter.obj
 0002:00029c24       ??_R2LEGlyphFilter@@8      1009bc24     GDEFMarkFilter.obj
 0002:00029c2c       ??_R1A@?0A@EA@LEGlyphFilter@@8 1009bc2c     GDEFMarkFilter.obj
 0002:00029c48       ??_R4GDEFMarkFilter@@6B@   1009bc48     GDEFMarkFilter.obj
 0002:00029c5c       ??_R3GDEFMarkFilter@@8     1009bc5c     GDEFMarkFilter.obj
 0002:00029c6c       ??_R2GDEFMarkFilter@@8     1009bc6c     GDEFMarkFilter.obj
 0002:00029c7c       ??_R1A@?0A@EA@GDEFMarkFilter@@8 1009bc7c     GDEFMarkFilter.obj
 0002:00029c98       ??_R4GXLayoutEngine@@6B@   1009bc98     GXLayoutEngine.obj
 0002:00029cac       ??_R3GXLayoutEngine@@8     1009bcac     GXLayoutEngine.obj
 0002:00029cbc       ??_R2GXLayoutEngine@@8     1009bcbc     GXLayoutEngine.obj
 0002:00029ccc       ??_R1A@?0A@EA@GXLayoutEngine@@8 1009bccc     GXLayoutEngine.obj
 0002:00029ce8       ??_R4GXLayoutEngine2@@6B@  1009bce8     GXLayoutEngine2.obj
 0002:00029cfc       ??_R3GXLayoutEngine2@@8    1009bcfc     GXLayoutEngine2.obj
 0002:00029d0c       ??_R2GXLayoutEngine2@@8    1009bd0c     GXLayoutEngine2.obj
 0002:00029d1c       ??_R1A@?0A@EA@GXLayoutEngine2@@8 1009bd1c     GXLayoutEngine2.obj
 0002:00029d38       ??_R4GlyphIterator@@6B@    1009bd38     GlyphIterator.obj
 0002:00029d4c       ??_R3GlyphIterator@@8      1009bd4c     GlyphIterator.obj
 0002:00029d5c       ??_R2GlyphIterator@@8      1009bd5c     GlyphIterator.obj
 0002:00029d68       ??_R1A@?0A@EA@GlyphIterator@@8 1009bd68     GlyphIterator.obj
 0002:00029d84       ??_R4GlyphPositioningLookupProcessor@@6B@ 1009bd84     GlyphPosnLookupProc.obj
 0002:00029d98       ??_R3GlyphPositioningLookupProcessor@@8 1009bd98     GlyphPosnLookupProc.obj
 0002:00029da8       ??_R2GlyphPositioningLookupProcessor@@8 1009bda8     GlyphPosnLookupProc.obj
 0002:00029db8       ??_R1A@?0A@EA@GlyphPositioningLookupProcessor@@8 1009bdb8     GlyphPosnLookupProc.obj
 0002:00029dd4       ??_R1A@?0A@EA@LookupProcessor@@8 1009bdd4     GlyphPosnLookupProc.obj
 0002:00029df0       ??_R3LookupProcessor@@8    1009bdf0     GlyphPosnLookupProc.obj
 0002:00029e00       ??_R2LookupProcessor@@8    1009be00     GlyphPosnLookupProc.obj
 0002:00029e0c       ??_R4GlyphSubstitutionLookupProcessor@@6B@ 1009be0c     GlyphSubstLookupProc.obj
 0002:00029e20       ??_R3GlyphSubstitutionLookupProcessor@@8 1009be20     GlyphSubstLookupProc.obj
 0002:00029e30       ??_R2GlyphSubstitutionLookupProcessor@@8 1009be30     GlyphSubstLookupProc.obj
 0002:00029e40       ??_R1A@?0A@EA@GlyphSubstitutionLookupProcessor@@8 1009be40     GlyphSubstLookupProc.obj
 0002:00029e5c       ??_R4HanOpenTypeLayoutEngine@@6B@ 1009be5c     HanLayoutEngine.obj
 0002:00029e70       ??_R3HanOpenTypeLayoutEngine@@8 1009be70     HanLayoutEngine.obj
 0002:00029e80       ??_R2HanOpenTypeLayoutEngine@@8 1009be80     HanLayoutEngine.obj
 0002:00029e94       ??_R1A@?0A@EA@HanOpenTypeLayoutEngine@@8 1009be94     HanLayoutEngine.obj
 0002:00029eb0       ??_R4HangulOpenTypeLayoutEngine@@6B@ 1009beb0     HangulLayoutEngine.obj
 0002:00029ec4       ??_R3HangulOpenTypeLayoutEngine@@8 1009bec4     HangulLayoutEngine.obj
 0002:00029ed4       ??_R2HangulOpenTypeLayoutEngine@@8 1009bed4     HangulLayoutEngine.obj
 0002:00029ee8       ??_R1A@?0A@EA@HangulOpenTypeLayoutEngine@@8 1009bee8     HangulLayoutEngine.obj
 0002:00029f04       ??_R4IndicOpenTypeLayoutEngine@@6B@ 1009bf04     IndicLayoutEngine.obj
 0002:00029f18       ??_R3IndicOpenTypeLayoutEngine@@8 1009bf18     IndicLayoutEngine.obj
 0002:00029f28       ??_R2IndicOpenTypeLayoutEngine@@8 1009bf28     IndicLayoutEngine.obj
 0002:00029f3c       ??_R1A@?0A@EA@IndicOpenTypeLayoutEngine@@8 1009bf3c     IndicLayoutEngine.obj
 0002:00029f58       ??_R4IndicRearrangementProcessor@@6B@ 1009bf58     IndicRearrangementProcessor.obj
 0002:00029f6c       ??_R3IndicRearrangementProcessor@@8 1009bf6c     IndicRearrangementProcessor.obj
 0002:00029f7c       ??_R2IndicRearrangementProcessor@@8 1009bf7c     IndicRearrangementProcessor.obj
 0002:00029f90       ??_R1A@?0A@EA@IndicRearrangementProcessor@@8 1009bf90     IndicRearrangementProcessor.obj
 0002:00029fac       ??_R4IndicRearrangementProcessor2@@6B@ 1009bfac     IndicRearrangementProcessor2.obj
 0002:00029fc0       ??_R3IndicRearrangementProcessor2@@8 1009bfc0     IndicRearrangementProcessor2.obj
 0002:00029fd0       ??_R2IndicRearrangementProcessor2@@8 1009bfd0     IndicRearrangementProcessor2.obj
 0002:00029fe4       ??_R1A@?0A@EA@IndicRearrangementProcessor2@@8 1009bfe4     IndicRearrangementProcessor2.obj
 0002:0002a000       ??_R4KhmerOpenTypeLayoutEngine@@6B@ 1009c000     KhmerLayoutEngine.obj
 0002:0002a014       ??_R3KhmerOpenTypeLayoutEngine@@8 1009c014     KhmerLayoutEngine.obj
 0002:0002a024       ??_R2KhmerOpenTypeLayoutEngine@@8 1009c024     KhmerLayoutEngine.obj
 0002:0002a038       ??_R1A@?0A@EA@KhmerOpenTypeLayoutEngine@@8 1009c038     KhmerLayoutEngine.obj
 0002:0002a054       ??_R4LECharMapper@@6B@     1009c054     LEFontInstance.obj
 0002:0002a068       ??_R3LECharMapper@@8       1009c068     LEFontInstance.obj
 0002:0002a078       ??_R2LECharMapper@@8       1009c078     LEFontInstance.obj
 0002:0002a080       ??_R1A@?0A@EA@LECharMapper@@8 1009c080     LEFontInstance.obj
 0002:0002a09c       ??_R4LEInsertionCallback@@6B@ 1009c09c     LEGlyphStorage.obj
 0002:0002a0b0       ??_R3LEInsertionCallback@@8 1009c0b0     LEGlyphStorage.obj
 0002:0002a0c0       ??_R2LEInsertionCallback@@8 1009c0c0     LEGlyphStorage.obj
 0002:0002a0c8       ??_R1A@?0A@EA@LEInsertionCallback@@8 1009c0c8     LEGlyphStorage.obj
 0002:0002a0e4       ??_R4LEGlyphStorage@@6B@   1009c0e4     LEGlyphStorage.obj
 0002:0002a0f8       ??_R3LEGlyphStorage@@8     1009c0f8     LEGlyphStorage.obj
 0002:0002a108       ??_R2LEGlyphStorage@@8     1009c108     LEGlyphStorage.obj
 0002:0002a118       ??_R1A@?0A@EA@LEGlyphStorage@@8 1009c118     LEGlyphStorage.obj
 0002:0002a134       ??_R1A@?0A@EN@LEInsertionCallback@@8 1009c134     LEGlyphStorage.obj
 0002:0002a150       ??_R4LEInsertionList@@6B@  1009c150     LEInsertionList.obj
 0002:0002a164       ??_R3LEInsertionList@@8    1009c164     LEInsertionList.obj
 0002:0002a174       ??_R2LEInsertionList@@8    1009c174     LEInsertionList.obj
 0002:0002a180       ??_R1A@?0A@EA@LEInsertionList@@8 1009c180     LEInsertionList.obj
 0002:0002a19c       ??_R4LayoutEngine@@6B@     1009c19c     LayoutEngine.obj
 0002:0002a1b0       ??_R4CharSubstitutionFilter@@6B@ 1009c1b0     LayoutEngine.obj
 0002:0002a1c4       ??_R3CharSubstitutionFilter@@8 1009c1c4     LayoutEngine.obj
 0002:0002a1d4       ??_R2CharSubstitutionFilter@@8 1009c1d4     LayoutEngine.obj
 0002:0002a1e4       ??_R1A@?0A@EA@CharSubstitutionFilter@@8 1009c1e4     LayoutEngine.obj
 0002:0002a200       ??_R4DefaultCharMapper@@6B@ 1009c200     LayoutEngine.obj
 0002:0002a214       ??_R3DefaultCharMapper@@8  1009c214     LayoutEngine.obj
 0002:0002a224       ??_R2DefaultCharMapper@@8  1009c224     LayoutEngine.obj
 0002:0002a234       ??_R1A@?0A@EA@DefaultCharMapper@@8 1009c234     LayoutEngine.obj
 0002:0002a250       ??_R4CanonMarkFilter@@6B@  1009c250     LayoutEngine.obj
 0002:0002a264       ??_R3CanonMarkFilter@@8    1009c264     LayoutEngine.obj
 0002:0002a274       ??_R2CanonMarkFilter@@8    1009c274     LayoutEngine.obj
 0002:0002a284       ??_R1A@?0A@EA@CanonMarkFilter@@8 1009c284     LayoutEngine.obj
 0002:0002a2a0       ??_R4LigatureSubstitutionProcessor@@6B@ 1009c2a0     LigatureSubstProc.obj
 0002:0002a2b4       ??_R3LigatureSubstitutionProcessor@@8 1009c2b4     LigatureSubstProc.obj
 0002:0002a2c4       ??_R2LigatureSubstitutionProcessor@@8 1009c2c4     LigatureSubstProc.obj
 0002:0002a2d8       ??_R1A@?0A@EA@LigatureSubstitutionProcessor@@8 1009c2d8     LigatureSubstProc.obj
 0002:0002a2f4       ??_R4LigatureSubstitutionProcessor2@@6B@ 1009c2f4     LigatureSubstProc2.obj
 0002:0002a308       ??_R3LigatureSubstitutionProcessor2@@8 1009c308     LigatureSubstProc2.obj
 0002:0002a318       ??_R2LigatureSubstitutionProcessor2@@8 1009c318     LigatureSubstProc2.obj
 0002:0002a32c       ??_R1A@?0A@EA@LigatureSubstitutionProcessor2@@8 1009c32c     LigatureSubstProc2.obj
 0002:0002a348       ??_R4LookupProcessor@@6B@  1009c348     LookupProcessor.obj
 0002:0002a35c       ??_R4NonContextualGlyphSubstitutionProcessor@@6B@ 1009c35c     NonContextualGlyphSubstProc.obj
 0002:0002a370       ??_R3NonContextualGlyphSubstitutionProcessor@@8 1009c370     NonContextualGlyphSubstProc.obj
 0002:0002a380       ??_R2NonContextualGlyphSubstitutionProcessor@@8 1009c380     NonContextualGlyphSubstProc.obj
 0002:0002a390       ??_R1A@?0A@EA@NonContextualGlyphSubstitutionProcessor@@8 1009c390     NonContextualGlyphSubstProc.obj
 0002:0002a3ac       ??_R4NonContextualGlyphSubstitutionProcessor2@@6B@ 1009c3ac     NonContextualGlyphSubstProc2.obj
 0002:0002a3c0       ??_R3NonContextualGlyphSubstitutionProcessor2@@8 1009c3c0     NonContextualGlyphSubstProc2.obj
 0002:0002a3d0       ??_R2NonContextualGlyphSubstitutionProcessor2@@8 1009c3d0     NonContextualGlyphSubstProc2.obj
 0002:0002a3e0       ??_R1A@?0A@EA@NonContextualGlyphSubstitutionProcessor2@@8 1009c3e0     NonContextualGlyphSubstProc2.obj
 0002:0002a3fc       ??_R4OpenTypeLayoutEngine@@6B@ 1009c3fc     OpenTypeLayoutEngine.obj
 0002:0002a410       ??_R4SegmentArrayProcessor@@6B@ 1009c410     SegmentArrayProcessor.obj
 0002:0002a424       ??_R3SegmentArrayProcessor@@8 1009c424     SegmentArrayProcessor.obj
 0002:0002a434       ??_R2SegmentArrayProcessor@@8 1009c434     SegmentArrayProcessor.obj
 0002:0002a448       ??_R1A@?0A@EA@SegmentArrayProcessor@@8 1009c448     SegmentArrayProcessor.obj
 0002:0002a464       ??_R4SegmentArrayProcessor2@@6B@ 1009c464     SegmentArrayProcessor2.obj
 0002:0002a478       ??_R3SegmentArrayProcessor2@@8 1009c478     SegmentArrayProcessor2.obj
 0002:0002a488       ??_R2SegmentArrayProcessor2@@8 1009c488     SegmentArrayProcessor2.obj
 0002:0002a49c       ??_R1A@?0A@EA@SegmentArrayProcessor2@@8 1009c49c     SegmentArrayProcessor2.obj
 0002:0002a4b8       ??_R4SegmentSingleProcessor@@6B@ 1009c4b8     SegmentSingleProcessor.obj
 0002:0002a4cc       ??_R3SegmentSingleProcessor@@8 1009c4cc     SegmentSingleProcessor.obj
 0002:0002a4dc       ??_R2SegmentSingleProcessor@@8 1009c4dc     SegmentSingleProcessor.obj
 0002:0002a4f0       ??_R1A@?0A@EA@SegmentSingleProcessor@@8 1009c4f0     SegmentSingleProcessor.obj
 0002:0002a50c       ??_R4SegmentSingleProcessor2@@6B@ 1009c50c     SegmentSingleProcessor2.obj
 0002:0002a520       ??_R3SegmentSingleProcessor2@@8 1009c520     SegmentSingleProcessor2.obj
 0002:0002a530       ??_R2SegmentSingleProcessor2@@8 1009c530     SegmentSingleProcessor2.obj
 0002:0002a544       ??_R1A@?0A@EA@SegmentSingleProcessor2@@8 1009c544     SegmentSingleProcessor2.obj
 0002:0002a560       ??_R4SimpleArrayProcessor@@6B@ 1009c560     SimpleArrayProcessor.obj
 0002:0002a574       ??_R3SimpleArrayProcessor@@8 1009c574     SimpleArrayProcessor.obj
 0002:0002a584       ??_R2SimpleArrayProcessor@@8 1009c584     SimpleArrayProcessor.obj
 0002:0002a598       ??_R1A@?0A@EA@SimpleArrayProcessor@@8 1009c598     SimpleArrayProcessor.obj
 0002:0002a5b4       ??_R4SimpleArrayProcessor2@@6B@ 1009c5b4     SimpleArrayProcessor2.obj
 0002:0002a5c8       ??_R3SimpleArrayProcessor2@@8 1009c5c8     SimpleArrayProcessor2.obj
 0002:0002a5d8       ??_R2SimpleArrayProcessor2@@8 1009c5d8     SimpleArrayProcessor2.obj
 0002:0002a5ec       ??_R1A@?0A@EA@SimpleArrayProcessor2@@8 1009c5ec     SimpleArrayProcessor2.obj
 0002:0002a608       ??_R4SingleTableProcessor@@6B@ 1009c608     SingleTableProcessor.obj
 0002:0002a61c       ??_R3SingleTableProcessor@@8 1009c61c     SingleTableProcessor.obj
 0002:0002a62c       ??_R2SingleTableProcessor@@8 1009c62c     SingleTableProcessor.obj
 0002:0002a640       ??_R1A@?0A@EA@SingleTableProcessor@@8 1009c640     SingleTableProcessor.obj
 0002:0002a65c       ??_R4SingleTableProcessor2@@6B@ 1009c65c     SingleTableProcessor2.obj
 0002:0002a670       ??_R3SingleTableProcessor2@@8 1009c670     SingleTableProcessor2.obj
 0002:0002a680       ??_R2SingleTableProcessor2@@8 1009c680     SingleTableProcessor2.obj
 0002:0002a694       ??_R1A@?0A@EA@SingleTableProcessor2@@8 1009c694     SingleTableProcessor2.obj
 0002:0002a6b0       ??_R4StateTableProcessor@@6B@ 1009c6b0     StateTableProcessor.obj
 0002:0002a6c4       ??_R4StateTableProcessor2@@6B@ 1009c6c4     StateTableProcessor2.obj
 0002:0002a6d8       ??_R4SubtableProcessor@@6B@ 1009c6d8     SubtableProcessor.obj
 0002:0002a6ec       ??_R4SubtableProcessor2@@6B@ 1009c6ec     SubtableProcessor2.obj
 0002:0002a700       ??_R4ThaiLayoutEngine@@6B@ 1009c700     ThaiLayoutEngine.obj
 0002:0002a714       ??_R3ThaiLayoutEngine@@8   1009c714     ThaiLayoutEngine.obj
 0002:0002a724       ??_R2ThaiLayoutEngine@@8   1009c724     ThaiLayoutEngine.obj
 0002:0002a734       ??_R1A@?0A@EA@ThaiLayoutEngine@@8 1009c734     ThaiLayoutEngine.obj
 0002:0002a750       ??_R4TibetanOpenTypeLayoutEngine@@6B@ 1009c750     TibetanLayoutEngine.obj
 0002:0002a764       ??_R3TibetanOpenTypeLayoutEngine@@8 1009c764     TibetanLayoutEngine.obj
 0002:0002a774       ??_R2TibetanOpenTypeLayoutEngine@@8 1009c774     TibetanLayoutEngine.obj
 0002:0002a788       ??_R1A@?0A@EA@TibetanOpenTypeLayoutEngine@@8 1009c788     TibetanLayoutEngine.obj
 0002:0002a7a4       ??_R4TrimmedArrayProcessor@@6B@ 1009c7a4     TrimmedArrayProcessor.obj
 0002:0002a7b8       ??_R3TrimmedArrayProcessor@@8 1009c7b8     TrimmedArrayProcessor.obj
 0002:0002a7c8       ??_R2TrimmedArrayProcessor@@8 1009c7c8     TrimmedArrayProcessor.obj
 0002:0002a7dc       ??_R1A@?0A@EA@TrimmedArrayProcessor@@8 1009c7dc     TrimmedArrayProcessor.obj
 0002:0002a7f8       ??_R4TrimmedArrayProcessor2@@6B@ 1009c7f8     TrimmedArrayProcessor2.obj
 0002:0002a80c       ??_R3TrimmedArrayProcessor2@@8 1009c80c     TrimmedArrayProcessor2.obj
 0002:0002a81c       ??_R2TrimmedArrayProcessor2@@8 1009c81c     TrimmedArrayProcessor2.obj
 0002:0002a830       ??_R1A@?0A@EA@TrimmedArrayProcessor2@@8 1009c830     TrimmedArrayProcessor2.obj
 0002:0002a84c       ??_R4type_info@@6B@        1009c84c     MSVCRT:std_type_info_static.obj
 0002:0002a860       ??_R3type_info@@8          1009c860     MSVCRT:std_type_info_static.obj
 0002:0002a870       ??_R2type_info@@8          1009c870     MSVCRT:std_type_info_static.obj
 0002:0002a878       ??_R1A@?0A@EA@type_info@@8 1009c878     MSVCRT:std_type_info_static.obj
 0002:0002a894       ??_R4exception@std@@6B@    1009c894     MSVCRT:throw_bad_alloc.obj
 0002:0002a8a8       ??_R3exception@std@@8      1009c8a8     MSVCRT:throw_bad_alloc.obj
 0002:0002a8b8       ??_R2exception@std@@8      1009c8b8     MSVCRT:throw_bad_alloc.obj
 0002:0002a8c0       ??_R1A@?0A@EA@exception@std@@8 1009c8c0     MSVCRT:throw_bad_alloc.obj
 0002:0002a8dc       ??_R4bad_alloc@std@@6B@    1009c8dc     MSVCRT:throw_bad_alloc.obj
 0002:0002a8f0       ??_R3bad_alloc@std@@8      1009c8f0     MSVCRT:throw_bad_alloc.obj
 0002:0002a900       ??_R2bad_alloc@std@@8      1009c900     MSVCRT:throw_bad_alloc.obj
 0002:0002a90c       ??_R1A@?0A@EA@bad_alloc@std@@8 1009c90c     MSVCRT:throw_bad_alloc.obj
 0002:0002a928       ??_R4bad_array_new_length@std@@6B@ 1009c928     MSVCRT:throw_bad_alloc.obj
 0002:0002a93c       ??_R3bad_array_new_length@std@@8 1009c93c     MSVCRT:throw_bad_alloc.obj
 0002:0002a94c       ??_R2bad_array_new_length@std@@8 1009c94c     MSVCRT:throw_bad_alloc.obj
 0002:0002a95c       ??_R1A@?0A@EA@bad_array_new_length@std@@8 1009c95c     MSVCRT:throw_bad_alloc.obj
 0002:0002a978       ___safe_se_handler_table   1009c978     <linker-defined>
 0002:0002a97c       ___volatile_metadata       1009c97c     <linker-defined>
 0002:0002af7c       ___rtc_iaa                 1009cf7c     MSVCRT:initsect.obj
 0002:0002af80       ___rtc_izz                 1009cf80     MSVCRT:initsect.obj
 0002:0002af84       ___rtc_taa                 1009cf84     MSVCRT:initsect.obj
 0002:0002af88       ___rtc_tzz                 1009cf88     MSVCRT:initsect.obj
 0002:0002aff4       __TI2?AVbad_alloc@std@@    1009cff4     MSVCRT:throw_bad_alloc.obj
 0002:0002b004       __CTA2?AVbad_alloc@std@@   1009d004     MSVCRT:throw_bad_alloc.obj
 0002:0002b010       __CT??_R0?AVbad_alloc@std@@@8??0bad_alloc@std@@QAE@ABV01@@Z12 1009d010     MSVCRT:throw_bad_alloc.obj
 0002:0002b02c       __CT??_R0?AVexception@std@@@8??0exception@std@@QAE@ABV01@@Z12 1009d02c     MSVCRT:throw_bad_alloc.obj
 0002:0002b048       __TI3?AVbad_array_new_length@std@@ 1009d048     MSVCRT:throw_bad_alloc.obj
 0002:0002b058       __CTA3?AVbad_array_new_length@std@@ 1009d058     MSVCRT:throw_bad_alloc.obj
 0002:0002b068       __CT??_R0?AVbad_array_new_length@std@@@8??0bad_array_new_length@std@@QAE@ABV01@@Z12 1009d068     MSVCRT:throw_bad_alloc.obj
 0002:0002b9e0       __IMPORT_DESCRIPTOR_java   1009d9e0     java:java.dll
 0002:0002b9f4       __IMPORT_DESCRIPTOR_ADVAPI32 1009d9f4     advapi32:ADVAPI32.dll
 0002:0002ba08       __IMPORT_DESCRIPTOR_USER32 1009da08     user32:USER32.dll
 0002:0002ba1c       __IMPORT_DESCRIPTOR_GDI32  1009da1c     gdi32:GDI32.dll
 0002:0002ba30       __IMPORT_DESCRIPTOR_awt    1009da30     awt:awt.dll
 0002:0002ba44       __IMPORT_DESCRIPTOR_KERNEL32 1009da44     kernel32:KERNEL32.dll
 0002:0002ba58       __IMPORT_DESCRIPTOR_VCRUNTIME140 1009da58     vcruntime:VCRUNTIME140.dll
 0002:0002ba6c       __IMPORT_DESCRIPTOR_api-ms-win-crt-heap-l1-1-0 1009da6c     ucrt:api-ms-win-crt-heap-l1-1-0.dll
 0002:0002ba80       __IMPORT_DESCRIPTOR_api-ms-win-crt-math-l1-1-0 1009da80     ucrt:api-ms-win-crt-math-l1-1-0.dll
 0002:0002ba94       __IMPORT_DESCRIPTOR_api-ms-win-crt-environment-l1-1-0 1009da94     ucrt:api-ms-win-crt-environment-l1-1-0.dll
 0002:0002baa8       __IMPORT_DESCRIPTOR_api-ms-win-crt-string-l1-1-0 1009daa8     ucrt:api-ms-win-crt-string-l1-1-0.dll
 0002:0002babc       __IMPORT_DESCRIPTOR_api-ms-win-crt-utility-l1-1-0 1009dabc     ucrt:api-ms-win-crt-utility-l1-1-0.dll
 0002:0002bad0       __IMPORT_DESCRIPTOR_api-ms-win-crt-convert-l1-1-0 1009dad0     ucrt:api-ms-win-crt-convert-l1-1-0.dll
 0002:0002bae4       __IMPORT_DESCRIPTOR_api-ms-win-crt-stdio-l1-1-0 1009dae4     ucrt:api-ms-win-crt-stdio-l1-1-0.dll
 0002:0002baf8       __IMPORT_DESCRIPTOR_api-ms-win-crt-runtime-l1-1-0 1009daf8     ucrt:api-ms-win-crt-runtime-l1-1-0.dll
 0002:0002bb0c       __NULL_IMPORT_DESCRIPTOR   1009db0c     java:java.dll
 0003:00000000       _defaultGammaLUT           1009f000     DrawGlyphList.obj
 0003:00000100       _defaultInvGammaLUT        1009f100     DrawGlyphList.obj
 0003:00000210       __fltused                  1009f210     MSVCRT:fltused.obj
 0003:00000214       ___security_cookie_complement 1009f214     MSVCRT:gs_cookie.obj
 0003:00000218       ___security_cookie         1009f218     MSVCRT:gs_cookie.obj
 0003:00000220       ___isa_enabled             1009f220     MSVCRT:cpu_disp.obj
 0003:00000224       ___scrt_native_dllmain_reason 1009f224     MSVCRT:utility.obj
 0003:00000230       ___scrt_ucrt_dll_is_in_use 1009f230     MSVCRT:ucrt_stubs.obj
 0003:00000234       ??_R0?AVbad_alloc@std@@@8  1009f234     MSVCRT:throw_bad_alloc.obj
 0003:00000250       ??_R0?AVexception@std@@@8  1009f250     MSVCRT:throw_bad_alloc.obj
 0003:0000026c       ??_R0?AVbad_array_new_length@std@@@8 1009f26c     MSVCRT:throw_bad_alloc.obj
 0003:00000294       ??_R0?AVArabicOpenTypeLayoutEngine@@@8 1009f294     ArabicLayoutEngine.obj
 0003:000002c0       ??_R0?AVOpenTypeLayoutEngine@@@8 1009f2c0     ArabicLayoutEngine.obj
 0003:000002e4       ??_R0?AVLayoutEngine@@@8   1009f2e4     ArabicLayoutEngine.obj
 0003:00000300       ??_R0?AUUObject@@@8        1009f300     ArabicLayoutEngine.obj
 0003:00000318       ??_R0?AVUnicodeArabicOpenTypeLayoutEngine@@@8 1009f318     ArabicLayoutEngine.obj
 0003:00000348       ??_R0?AVContextualGlyphInsertionProcessor2@@@8 1009f348     ContextualGlyphInsertionProc2.obj
 0003:0000037c       ??_R0?AVStateTableProcessor2@@@8 1009f37c     ContextualGlyphInsertionProc2.obj
 0003:000003a0       ??_R0?AVSubtableProcessor2@@@8 1009f3a0     ContextualGlyphInsertionProc2.obj
 0003:000003c4       ??_R0?AUUMemory@@@8        1009f3c4     ContextualGlyphInsertionProc2.obj
 0003:000003dc       ??_R0?AVContextualGlyphSubstitutionProcessor@@@8 1009f3dc     ContextualGlyphSubstProc.obj
 0003:00000410       ??_R0?AVStateTableProcessor@@@8 1009f410     ContextualGlyphSubstProc.obj
 0003:00000434       ??_R0?AVSubtableProcessor@@@8 1009f434     ContextualGlyphSubstProc.obj
 0003:00000454       ??_R0?AVContextualGlyphSubstitutionProcessor2@@@8 1009f454     ContextualGlyphSubstProc2.obj
 0003:00000488       ??_R0?AVLEFontInstance@@@8 1009f488     FontInstanceAdapter.obj
 0003:000004a8       ??_R0?AVFontInstanceAdapter@@@8 1009f4a8     FontInstanceAdapter.obj
 0003:000004cc       ??_R0?AVLEGlyphFilter@@@8  1009f4cc     GDEFMarkFilter.obj
 0003:000004e8       ??_R0?AVGDEFMarkFilter@@@8 1009f4e8     GDEFMarkFilter.obj
 0003:00000508       ??_R0?AVGXLayoutEngine@@@8 1009f508     GXLayoutEngine.obj
 0003:00000528       ??_R0?AVGXLayoutEngine2@@@8 1009f528     GXLayoutEngine2.obj
 0003:00000548       ??_R0?AVGlyphIterator@@@8  1009f548     GlyphIterator.obj
 0003:00000564       ??_R0?AVGlyphPositioningLookupProcessor@@@8 1009f564     GlyphPosnLookupProc.obj
 0003:00000594       ??_R0?AVLookupProcessor@@@8 1009f594     GlyphPosnLookupProc.obj
 0003:000005b4       ??_R0?AVGlyphSubstitutionLookupProcessor@@@8 1009f5b4     GlyphSubstLookupProc.obj
 0003:000005e4       ??_R0?AVHanOpenTypeLayoutEngine@@@8 1009f5e4     HanLayoutEngine.obj
 0003:0000060c       ??_R0?AVHangulOpenTypeLayoutEngine@@@8 1009f60c     HangulLayoutEngine.obj
 0003:00000638       ??_R0?AVIndicOpenTypeLayoutEngine@@@8 1009f638     IndicLayoutEngine.obj
 0003:00000660       ??_R0?AVIndicRearrangementProcessor@@@8 1009f660     IndicRearrangementProcessor.obj
 0003:0000068c       ??_R0?AVIndicRearrangementProcessor2@@@8 1009f68c     IndicRearrangementProcessor2.obj
 0003:000006b8       ??_R0?AVKhmerOpenTypeLayoutEngine@@@8 1009f6b8     KhmerLayoutEngine.obj
 0003:000006e0       ??_R0?AVLECharMapper@@@8   1009f6e0     LEFontInstance.obj
 0003:000006fc       ??_R0?AVLEInsertionCallback@@@8 1009f6fc     LEGlyphStorage.obj
 0003:00000720       ??_R0?AVLEGlyphStorage@@@8 1009f720     LEGlyphStorage.obj
 0003:00000740       ??_R0?AVLEInsertionList@@@8 1009f740     LEInsertionList.obj
 0003:00000760       ??_R0?AVCharSubstitutionFilter@@@8 1009f760     LayoutEngine.obj
 0003:00000788       ??_R0?AVDefaultCharMapper@@@8 1009f788     LayoutEngine.obj
 0003:000007a8       ??_R0?AVCanonMarkFilter@@@8 1009f7a8     LayoutEngine.obj
 0003:000007c8       ??_R0?AVLigatureSubstitutionProcessor@@@8 1009f7c8     LigatureSubstProc.obj
 0003:000007f4       ??_R0?AVLigatureSubstitutionProcessor2@@@8 1009f7f4     LigatureSubstProc2.obj
 0003:00000824       ??_R0?AVNonContextualGlyphSubstitutionProcessor@@@8 1009f824     NonContextualGlyphSubstProc.obj
 0003:0000085c       ??_R0?AVNonContextualGlyphSubstitutionProcessor2@@@8 1009f85c     NonContextualGlyphSubstProc2.obj
 0003:00000894       ??_R0?AVSegmentArrayProcessor@@@8 1009f894     SegmentArrayProcessor.obj
 0003:000008b8       ??_R0?AVSegmentArrayProcessor2@@@8 1009f8b8     SegmentArrayProcessor2.obj
 0003:000008e0       ??_R0?AVSegmentSingleProcessor@@@8 1009f8e0     SegmentSingleProcessor.obj
 0003:00000908       ??_R0?AVSegmentSingleProcessor2@@@8 1009f908     SegmentSingleProcessor2.obj
 0003:00000930       ??_R0?AVSimpleArrayProcessor@@@8 1009f930     SimpleArrayProcessor.obj
 0003:00000954       ??_R0?AVSimpleArrayProcessor2@@@8 1009f954     SimpleArrayProcessor2.obj
 0003:00000978       ??_R0?AVSingleTableProcessor@@@8 1009f978     SingleTableProcessor.obj
 0003:0000099c       ??_R0?AVSingleTableProcessor2@@@8 1009f99c     SingleTableProcessor2.obj
 0003:000009c0       ??_R0?AVThaiLayoutEngine@@@8 1009f9c0     ThaiLayoutEngine.obj
 0003:000009e0       ??_R0?AVTibetanOpenTypeLayoutEngine@@@8 1009f9e0     TibetanLayoutEngine.obj
 0003:00000a0c       ??_R0?AVTrimmedArrayProcessor@@@8 1009fa0c     TrimmedArrayProcessor.obj
 0003:00000a30       ??_R0?AVTrimmedArrayProcessor2@@@8 1009fa30     TrimmedArrayProcessor2.obj
 0003:00000a58       ??_R0?AVtype_info@@@8      1009fa58     MSVCRT:std_type_info_static.obj
 0003:00000cb8       ___isa_available           1009fcb8     MSVCRT:cpu_disp.obj
 0003:00000cbc       ___favor                   1009fcbc     MSVCRT:cpu_disp.obj
 0003:00000fe0       ?__type_info_root_node@@3U__type_info_node@@A 1009ffe0     MSVCRT:tncleanup.obj
 0003:00000fe8       ?_OptionsStorage@?1??__local_stdio_scanf_options@@9@4_KA 1009ffe8     MSVCRT:default_local_stdio_options.obj
 0003:00000ff0       ___scrt_current_native_startup_state 1009fff0     MSVCRT:utility.obj
 0003:00000ff4       ___scrt_native_startup_lock 1009fff4     MSVCRT:utility.obj
 0003:00001014       ___scrt_debugger_hook_flag 100a0014     MSVCRT:utility_desktop.obj
 0003:00001020       _sunFontIDs                100a0020     <common>
 0003:000010c0       _lcdInvGammaLUT            100a00c0     <common>
 0003:00001320       _lcdGammaLUT               100a0320     <common>
 0003:00001580       ?_OptionsStorage@?1??__local_stdio_printf_options@@9@9 100a0580     <common>
 0003:00001588       ___dyn_tls_init_callback   100a0588     <common>

 entry point at        0001:0006f4ac

 Static symbols

 0000:fff5b000       .debug$S                   10000000     fontmanager.exp
 0000:fff5b000       .debug$S                   10000000     vcruntime:VCRUNTIME140.dll
 0000:fff5b000       .debug$S                   10000000     vcruntime:VCRUNTIME140.dll
 0000:fff5b000       .debug$S                   10000000     vcruntime:VCRUNTIME140.dll
 0000:fff5b000       .debug$S                   10000000     vcruntime:VCRUNTIME140.dll
 0000:fff5b000       .debug$S                   10000000     vcruntime:VCRUNTIME140.dll
 0000:fff5b000       .debug$S                   10000000     vcruntime:VCRUNTIME140.dll
 0000:fff5b000       .debug$S                   10000000     vcruntime:VCRUNTIME140.dll
 0000:fff5b000       .debug$S                   10000000     vcruntime:VCRUNTIME140.dll
 0000:fff5b000       .debug$S                   10000000     vcruntime:VCRUNTIME140.dll
 0000:fff5b000       .debug$S                   10000000     vcruntime:VCRUNTIME140.dll
 0000:fff5b000       .debug$S                   10000000     vcruntime:VCRUNTIME140.dll
 0000:fff5b000       .debug$S                   10000000     vcruntime:VCRUNTIME140.dll
 0000:fff5b000       .debug$S                   10000000     vcruntime:VCRUNTIME140.dll
 0000:fff5b000       .debug$S                   10000000     vcruntime:VCRUNTIME140.dll
 0000:fff5b000       .debug$S                   10000000     vcruntime:VCRUNTIME140.dll
 0000:fff5b000       .debug$S                   10000000     vcruntime:VCRUNTIME140.dll
 0000:fff5b000       .debug$S                   10000000     vcruntime:VCRUNTIME140.dll
 0000:fff5b000       .debug$S                   10000000     vcruntime:VCRUNTIME140.dll
 0000:fff5b000       .debug$S                   10000000     ucrt:api-ms-win-crt-convert-l1-1-0.dll
 0000:fff5b000       .debug$S                   10000000     ucrt:api-ms-win-crt-environment-l1-1-0.dll
 0000:fff5b000       .debug$S                   10000000     ucrt:api-ms-win-crt-heap-l1-1-0.dll
 0000:fff5b000       .debug$S                   10000000     ucrt:api-ms-win-crt-heap-l1-1-0.dll
 0000:fff5b000       .debug$S                   10000000     ucrt:api-ms-win-crt-heap-l1-1-0.dll
 0000:fff5b000       .debug$S                   10000000     ucrt:api-ms-win-crt-heap-l1-1-0.dll
 0000:fff5b000       .debug$S                   10000000     ucrt:api-ms-win-crt-heap-l1-1-0.dll
 0000:fff5b000       .debug$S                   10000000     ucrt:api-ms-win-crt-math-l1-1-0.dll
 0000:fff5b000       .debug$S                   10000000     ucrt:api-ms-win-crt-math-l1-1-0.dll
 0000:fff5b000       .debug$S                   10000000     ucrt:api-ms-win-crt-math-l1-1-0.dll
 0000:fff5b000       .debug$S                   10000000     ucrt:api-ms-win-crt-math-l1-1-0.dll
 0000:fff5b000       .debug$S                   10000000     ucrt:api-ms-win-crt-runtime-l1-1-0.dll
 0000:fff5b000       .debug$S                   10000000     ucrt:api-ms-win-crt-runtime-l1-1-0.dll
 0000:fff5b000       .debug$S                   10000000     ucrt:api-ms-win-crt-runtime-l1-1-0.dll
 0000:fff5b000       .debug$S                   10000000     ucrt:api-ms-win-crt-runtime-l1-1-0.dll
 0000:fff5b000       .debug$S                   10000000     ucrt:api-ms-win-crt-runtime-l1-1-0.dll
 0000:fff5b000       .debug$S                   10000000     ucrt:api-ms-win-crt-runtime-l1-1-0.dll
 0000:fff5b000       .debug$S                   10000000     ucrt:api-ms-win-crt-runtime-l1-1-0.dll
 0000:fff5b000       .debug$S                   10000000     ucrt:api-ms-win-crt-runtime-l1-1-0.dll
 0000:fff5b000       .debug$S                   10000000     ucrt:api-ms-win-crt-runtime-l1-1-0.dll
 0000:fff5b000       .debug$S                   10000000     ucrt:api-ms-win-crt-runtime-l1-1-0.dll
 0000:fff5b000       .debug$S                   10000000     ucrt:api-ms-win-crt-runtime-l1-1-0.dll
 0000:fff5b000       .debug$S                   10000000     ucrt:api-ms-win-crt-runtime-l1-1-0.dll
 0000:fff5b000       .debug$S                   10000000     ucrt:api-ms-win-crt-stdio-l1-1-0.dll
 0000:fff5b000       .debug$S                   10000000     ucrt:api-ms-win-crt-stdio-l1-1-0.dll
 0000:fff5b000       .debug$S                   10000000     ucrt:api-ms-win-crt-stdio-l1-1-0.dll
 0000:fff5b000       .debug$S                   10000000     ucrt:api-ms-win-crt-stdio-l1-1-0.dll
 0000:fff5b000       .debug$S                   10000000     ucrt:api-ms-win-crt-stdio-l1-1-0.dll
 0000:fff5b000       .debug$S                   10000000     ucrt:api-ms-win-crt-stdio-l1-1-0.dll
 0000:fff5b000       .debug$S                   10000000     ucrt:api-ms-win-crt-string-l1-1-0.dll
 0000:fff5b000       .debug$S                   10000000     ucrt:api-ms-win-crt-string-l1-1-0.dll
 0000:fff5b000       .debug$S                   10000000     ucrt:api-ms-win-crt-string-l1-1-0.dll
 0000:fff5b000       .debug$S                   10000000     ucrt:api-ms-win-crt-string-l1-1-0.dll
 0000:fff5b000       .debug$S                   10000000     ucrt:api-ms-win-crt-utility-l1-1-0.dll
 0000:fff5b000       .debug$S                   10000000     advapi32:ADVAPI32.dll
 0000:fff5b000       .debug$S                   10000000     advapi32:ADVAPI32.dll
 0000:fff5b000       .debug$S                   10000000     advapi32:ADVAPI32.dll
 0000:fff5b000       .debug$S                   10000000     advapi32:ADVAPI32.dll
 0000:fff5b000       .debug$S                   10000000     advapi32:ADVAPI32.dll
 0000:fff5b000       .debug$S                   10000000     advapi32:ADVAPI32.dll
 0000:fff5b000       .debug$S                   10000000     gdi32:GDI32.dll
 0000:fff5b000       .debug$S                   10000000     gdi32:GDI32.dll
 0000:fff5b000       .debug$S                   10000000     gdi32:GDI32.dll
 0000:fff5b000       .debug$S                   10000000     gdi32:GDI32.dll
 0000:fff5b000       .debug$S                   10000000     gdi32:GDI32.dll
 0000:fff5b000       .debug$S                   10000000     gdi32:GDI32.dll
 0000:fff5b000       .debug$S                   10000000     gdi32:GDI32.dll
 0000:fff5b000       .debug$S                   10000000     gdi32:GDI32.dll
 0000:fff5b000       .debug$S                   10000000     gdi32:GDI32.dll
 0000:fff5b000       .debug$S                   10000000     gdi32:GDI32.dll
 0000:fff5b000       .debug$S                   10000000     gdi32:GDI32.dll
 0000:fff5b000       .debug$S                   10000000     gdi32:GDI32.dll
 0000:fff5b000       .debug$S                   10000000     gdi32:GDI32.dll
 0000:fff5b000       .debug$S                   10000000     gdi32:GDI32.dll
 0000:fff5b000       .debug$S                   10000000     gdi32:GDI32.dll
 0000:fff5b000       .debug$S                   10000000     gdi32:GDI32.dll
 0000:fff5b000       .debug$S                   10000000     gdi32:GDI32.dll
 0000:fff5b000       .debug$S                   10000000     kernel32:KERNEL32.dll
 0000:fff5b000       .debug$S                   10000000     kernel32:KERNEL32.dll
 0000:fff5b000       .debug$S                   10000000     kernel32:KERNEL32.dll
 0000:fff5b000       .debug$S                   10000000     kernel32:KERNEL32.dll
 0000:fff5b000       .debug$S                   10000000     kernel32:KERNEL32.dll
 0000:fff5b000       .debug$S                   10000000     kernel32:KERNEL32.dll
 0000:fff5b000       .debug$S                   10000000     kernel32:KERNEL32.dll
 0000:fff5b000       .debug$S                   10000000     kernel32:KERNEL32.dll
 0000:fff5b000       .debug$S                   10000000     kernel32:KERNEL32.dll
 0000:fff5b000       .debug$S                   10000000     kernel32:KERNEL32.dll
 0000:fff5b000       .debug$S                   10000000     kernel32:KERNEL32.dll
 0000:fff5b000       .debug$S                   10000000     kernel32:KERNEL32.dll
 0000:fff5b000       .debug$S                   10000000     kernel32:KERNEL32.dll
 0000:fff5b000       .debug$S                   10000000     kernel32:KERNEL32.dll
 0000:fff5b000       .debug$S                   10000000     kernel32:KERNEL32.dll
 0000:fff5b000       .debug$S                   10000000     kernel32:KERNEL32.dll
 0000:fff5b000       .debug$S                   10000000     kernel32:KERNEL32.dll
 0000:fff5b000       .debug$S                   10000000     kernel32:KERNEL32.dll
 0000:fff5b000       .debug$S                   10000000     user32:USER32.dll
 0000:fff5b000       .debug$S                   10000000     user32:USER32.dll
 0000:fff5b000       .debug$S                   10000000     user32:USER32.dll
 0000:fff5b000       .debug$S                   10000000     user32:USER32.dll
 0000:fff5b000       .debug$S                   10000000     user32:USER32.dll
 0000:fff5b000       .debug$S                   10000000     user32:USER32.dll
 0000:fff5b000       .debug$S                   10000000     awt:awt.dll
 0000:fff5b000       .debug$S                   10000000     awt:awt.dll
 0000:fff5b000       .debug$S                   10000000     awt:awt.dll
 0000:fff5b000       .debug$S                   10000000     awt:awt.dll
 0000:fff5b000       .debug$S                   10000000     awt:awt.dll
 0000:fff5b000       .debug$S                   10000000     awt:awt.dll
 0000:fff5b000       .debug$S                   10000000     awt:awt.dll
 0000:fff5b000       .debug$S                   10000000     awt:awt.dll
 0000:fff5b000       .debug$S                   10000000     awt:awt.dll
 0000:fff5b000       .debug$S                   10000000     java:java.dll
 0000:fff5b000       .debug$S                   10000000     java:java.dll
 0000:fff5b000       .debug$S                   10000000     java:java.dll
 0001:00002220       _cf2_free_instance         10003220 f   freetype:cff.obj
 0001:00002220       _cff_driver_done           10003220 f   freetype:cff.obj
 0001:00002220       _ps_parser_done            10003220 f   freetype:psaux.obj
 0001:00002220       _Horizontal_Sweep_Init     10003220 f   freetype:raster.obj
 0001:00002220       _Horizontal_Sweep_Step     10003220 f   freetype:raster.obj
 0001:00002220       _ft_black_set_mode         10003220 f   freetype:raster.obj
 0001:00002220       _T1_Driver_Done            10003220 f   freetype:type1.obj
 0001:00002220       _cid_driver_done           10003220 f   freetype:type1cid.obj
 0001:00002220       _T42_Driver_Done           10003220 f   freetype:type42.obj
 0001:00005b30       $LN179                     10006b30     ContextualSubstSubtables.obj
 0001:00007018       $LN325                     10008018     ContextualSubstSubtables.obj
 0001:00007b50       _drawGlyphList             10008b50 f   DrawGlyphList.obj
 0001:00007cc0       _drawGlyphListLCD          10008cc0 f   DrawGlyphList.obj
 0001:00009030       _tt_cmap14_char_index      1000a030 f i freetype:sfnt.obj
 0001:00009030       _T1_Driver_Init            1000a030 f i freetype:type1.obj
 0001:00009030       _cid_driver_init           1000a030 f i freetype:type1cid.obj
 0001:0000a12c       $LN42                      1000b12c     GlyphIterator.obj
 0001:0000a394       $LN46                      1000b394     GlyphIterator.obj
 0001:0000a534       $LN46                      1000b534     GlyphIterator.obj
 0001:0000b57c       $LN413                     1000c57c     GlyphPosnLookupProc.obj
 0001:0000bab8       $LN323                     1000cab8     GlyphSubstLookupProc.obj
 0001:0000d474       $LN315                     1000e474     IndicRearrangementProcessor.obj
 0001:0000e358       $LN315                     1000f358     IndicRearrangementProcessor2.obj
 0001:000101f0       $LN449                     100111f0     IndicReordering.obj
 0001:00010208       $LN448                     10011208     IndicReordering.obj
 0001:00013c24       $LN208                     10014c24     LayoutEngine.obj
 0001:00013c44       $LN207                     10014c44     LayoutEngine.obj
 0001:00013c6c       $LN210                     10014c6c     LayoutEngine.obj
 0001:00013c74       $LN209                     10014c74     LayoutEngine.obj
 0001:00013c8c       $LN212                     10014c8c     LayoutEngine.obj
 0001:00013ca0       $LN211                     10014ca0     LayoutEngine.obj
 0001:00019b50       $LN268                     1001ab50     MorphTables.obj
 0001:0001a43c       $LN383                     1001b43c     MorphTables2.obj
 0001:0001a460       $LN382                     1001b460     MorphTables2.obj
 0001:0001a47c       $LN384                     1001b47c     MorphTables2.obj
 0001:0001aa68       $LN74                      1001ba68     NonContextualGlyphSubstProc.obj
 0001:0001ac08       $LN74                      1001bc08     NonContextualGlyphSubstProc2.obj
 0001:0001b744       $LN16                      1001c744     OpenTypeLayoutEngine.obj
 0001:0001b76c       $LN15                      1001c76c     OpenTypeLayoutEngine.obj
 0001:0001ba20       $LN26                      1001ca20     OpenTypeLayoutEngine.obj
 0001:0001ba48       $LN25                      1001ca48     OpenTypeLayoutEngine.obj
 0001:00020b14       $LN63                      10021b14     ThaiShaping.obj
 0001:00020b1c       $LN62                      10021b1c     ThaiShaping.obj
 0001:00020e94       $LN38                      10021e94     ThaiShaping.obj
 0001:00022390       _CheckFontFamilyProcW@16   10023390 f   fontpath.obj
 0001:000223e0       _EnumFamilyNamesA@16       100233e0 f   fontpath.obj
 0001:00022510       _EnumFamilyNamesW@16       10023510 f   fontpath.obj
 0001:00022680       _EnumFontFacesInFamilyProcA@16 10023680 f   fontpath.obj
 0001:00022710       _EnumFontFacesInFamilyProcW@16 10023710 f   fontpath.obj
 0001:00022890       _GetOSVersion              10023890 f   fontpath.obj
 0001:00023300       _registerFontW             10024300 f   fontpath.obj
 0001:00023480       _moveTo                    10024480 f   freetypeScaler.obj
 0001:000234f0       _lineTo                    100244f0 f   freetypeScaler.obj
 0001:00023550       _conicTo                   10024550 f   freetypeScaler.obj
 0001:000235f0       _cubicTo                   100245f0 f   freetypeScaler.obj
 0001:00024720       _ReadTTFontFileFunc        10025720 f   freetypeScaler.obj
 0001:00024880       _getFTOutline              10025880 f   freetypeScaler.obj
 0001:00024940       _getGlyphGeneralPath       10025940 f   freetypeScaler.obj
 0001:00024b00       _getGlyphImageNativeInternal 10025b00 f   freetypeScaler.obj
 0001:00025140       _invalidateJavaScaler      10026140 f   freetypeScaler.obj
 0001:000251c0       _setupFTContext            100261c0 f   freetypeScaler.obj
 0001:00025fe0       _initFontIDs               10026fe0 f   sunFont.obj
 0001:000266b0       _raccess_guess_apple_double 100276b0 f   freetype:ftbase.obj
 0001:000266e0       _raccess_guess_apple_single 100276e0 f   freetype:ftbase.obj
 0001:00026710       _raccess_guess_darwin_ufs_export 10027710 f   freetype:ftbase.obj
 0001:00026770       _raccess_guess_darwin_newvfs 10027770 f   freetype:ftbase.obj
 0001:000267e0       _raccess_guess_darwin_hfsplus 100277e0 f   freetype:ftbase.obj
 0001:00026850       _raccess_guess_vfat        10027850 f   freetype:ftbase.obj
 0001:00026890       _raccess_guess_linux_cap   10027890 f   freetype:ftbase.obj
 0001:000268d0       _raccess_guess_linux_double 100278d0 f   freetype:ftbase.obj
 0001:00026930       _raccess_guess_linux_netatalk 10027930 f   freetype:ftbase.obj
 0001:00026990       _Destroy_Driver            10027990 f   freetype:ftbase.obj
 0001:000269d0       _Destroy_Module            100279d0 f   freetype:ftbase.obj
 0001:00026a70       _FT_Add64                  10027a70 f   freetype:ftbase.obj
 0001:00027560       _FT_GlyphLoader_Adjust_Points 10028560 f   freetype:ftbase.obj
 0001:000275b0       _FT_GlyphLoader_Adjust_Subglyphs 100285b0 f   freetype:ftbase.obj
 0001:00029c54       $LN57                      1002ac54     freetype:ftbase.obj
 0001:0002a784       $LN47                      1002b784     freetype:ftbase.obj
 0001:0002a7ac       $LN46                      1002b7ac     freetype:ftbase.obj
 0001:0002aca0       _IsMacBinary               1002bca0 f   freetype:ftbase.obj
 0001:0002ada0       _IsMacResource             1002bda0 f   freetype:ftbase.obj
 0001:0002aea0       _Mac_Read_POST_Resource    1002bea0 f   freetype:ftbase.obj
 0001:0002b130       _Mac_Read_sfnt_Resource    1002c130 f   freetype:ftbase.obj
 0001:0002b250       __ft_face_scale_advances   1002c250 f   freetype:ftbase.obj
 0001:0002b2b0       _destroy_charmaps          1002c2b0 f   freetype:ftbase.obj
 0001:0002b310       _destroy_face              1002c310 f   freetype:ftbase.obj
 0001:0002b3d0       _destroy_size              1002c3d0 f   freetype:ftbase.obj
 0001:0002b420       _find_unicode_charmap      1002c420 f   freetype:ftbase.obj
 0001:0002b4a0       _ft_add_renderer           1002c4a0 f   freetype:ftbase.obj
 0001:0002b550       _ft_cmap_done_internal     1002c550 f   freetype:ftbase.obj
 0001:0002b6b0       _ft_div64by32              1002c6b0 f   freetype:ftbase.obj
 0001:0002b760       _ft_glyphslot_clear        1002c760 f   freetype:ftbase.obj
 0001:0002b810       _ft_glyphslot_done         1002c810 f   freetype:ftbase.obj
 0001:0002b8e0       _ft_glyphslot_grid_fit_metrics 1002c8e0 f   freetype:ftbase.obj
 0001:0002b990       _ft_glyphslot_init         1002c990 f   freetype:ftbase.obj
 0001:0002ba60       _ft_lookup_PS_in_sfnt_stream 1002ca60 f   freetype:ftbase.obj
 0001:0002bbe0       _ft_lookup_glyph_renderer  1002cbe0 f   freetype:ftbase.obj
 0001:0002bf90       _ft_multo64                1002cf90 f   freetype:ftbase.obj
 0001:0002bff0       _ft_property_do            1002cff0 f   freetype:ftbase.obj
 0001:0002c0f0       _ft_raccess_rule_by_darwin_vfs 1002d0f0 f   freetype:ftbase.obj
 0001:0002c120       _ft_raccess_sort_ref_by_id 1002d120 f   freetype:ftbase.obj
 0001:0002c140       _ft_recompute_scaled_metrics 1002d140 f   freetype:ftbase.obj
 0001:0002c1b0       _ft_remove_renderer        1002d1b0 f   freetype:ftbase.obj
 0001:0002c290       _ft_set_current_renderer   1002d290 f   freetype:ftbase.obj
 0001:0002c320       _ft_trig_downscale         1002d320 f   freetype:ftbase.obj
 0001:0002c380       _ft_trig_prenorm           1002d380 f   freetype:ftbase.obj
 0001:0002c3e0       _ft_trig_pseudo_polarize   1002d3e0 f   freetype:ftbase.obj
 0001:0002c500       _load_face_in_embedded_rfork 1002d500 f   freetype:ftbase.obj
 0001:0002c670       _load_mac_face             1002d670 f   freetype:ftbase.obj
 0001:0002c6d0       _memory_stream_close       1002d6d0 f   freetype:ftbase.obj
 0001:0002c6d0       _sfnt_stream_close         1002d6d0 f   freetype:sfnt.obj
 0001:0002c700       _new_memory_stream         1002d700 f   freetype:ftbase.obj
 0001:0002c760       _open_face                 1002d760 f   freetype:ftbase.obj
 0001:0002c8b0       _open_face_PS_from_sfnt_stream 1002d8b0 f   freetype:ftbase.obj
 0001:0002c980       _open_face_from_buffer     1002d980 f   freetype:ftbase.obj
 0001:0002ca40       _raccess_get_rule_type_from_rule_index 1002da40 f   freetype:ftbase.obj
 0001:0002ca60       _raccess_guess_apple_generic 1002da60 f   freetype:ftbase.obj
 0001:0002cb60       _raccess_guess_linux_double_from_file_name 1002db60 f   freetype:ftbase.obj
 0001:0002cbc0       _raccess_make_file_name    1002dbc0 f   freetype:ftbase.obj
 0001:0002ccb0       _BBox_Move_To              1002dcb0 f   freetype:ftbbox.obj
 0001:0002ccd0       _BBox_Conic_To             1002dcd0 f   freetype:ftbbox.obj
 0001:0002cd40       _BBox_Cubic_To             1002dd40 f   freetype:ftbbox.obj
 0001:0002cdd0       _BBox_Conic_Check          1002ddd0 f   freetype:ftbbox.obj
 0001:0002ce10       _BBox_Cubic_Check          1002de10 f   freetype:ftbbox.obj
 0001:0002d110       _update_cubic_max          1002e110 f   freetype:ftbbox.obj
 0001:0002d2d0       _af_latin_metrics_init     1002e2d0 f   freetype:autofit.obj
 0001:0002d330       _af_latin_metrics_scale    1002e330 f   freetype:autofit.obj
 0001:0002d370       _af_cjk_metrics_init       1002e370 f   freetype:autofit.obj
 0001:0002d3d0       _af_cjk_metrics_scale      1002e3d0 f   freetype:autofit.obj
 0001:0002d410       _af_cjk_hints_init         1002e410 f   freetype:autofit.obj
 0001:0002d490       _af_cjk_hints_apply        1002e490 f   freetype:autofit.obj
 0001:0002d550       _af_dummy_hints_init       1002e550 f   freetype:autofit.obj
 0001:0002d590       _af_dummy_hints_apply      1002e590 f   freetype:autofit.obj
 0001:0002d5c0       _af_latin_hints_init       1002e5c0 f   freetype:autofit.obj
 0001:0002d650       _af_latin_hints_apply      1002e650 f   freetype:autofit.obj
 0001:0002d700       _af_indic_metrics_init     1002e700 f   freetype:autofit.obj
 0001:0002d770       _af_indic_metrics_scale    1002e770 f   freetype:autofit.obj
 0001:0002d780       _af_indic_hints_init       1002e780 f   freetype:autofit.obj
 0001:0002d790       _af_indic_hints_apply      1002e790 f   freetype:autofit.obj
 0001:0002d7a0       _af_property_set           1002e7a0 f   freetype:autofit.obj
 0001:0002d8d0       _af_property_get           1002e8d0 f   freetype:autofit.obj
 0001:0002da30       _af_get_interface          1002ea30 f   freetype:autofit.obj
 0001:0002da40       _af_autofitter_init        1002ea40 f   freetype:autofit.obj
 0001:0002da60       _af_autofitter_done        1002ea60 f   freetype:autofit.obj
 0001:0002da70       _af_autofitter_load_glyph  1002ea70 f   freetype:autofit.obj
 0001:0002da90       _af_axis_hints_new_edge    1002ea90 f   freetype:autofit.obj
 0001:0002db90       _af_axis_hints_new_segment 1002eb90 f   freetype:autofit.obj
 0001:0002dc20       _af_cjk_align_edge_points  1002ec20 f   freetype:autofit.obj
 0001:0002dd30       _af_cjk_align_linked_edge  1002ed30 f   freetype:autofit.obj
 0001:0002dd70       _af_cjk_align_serif_edge   1002ed70 f   freetype:autofit.obj
 0001:0002dd70       _af_latin_align_serif_edge 1002ed70 f   freetype:autofit.obj
 0001:0002dd90       _af_cjk_compute_stem_width 1002ed90 f   freetype:autofit.obj
 0001:0002df30       _af_cjk_hint_edges         1002ef30 f   freetype:autofit.obj
 0001:0002e2d0       _af_cjk_hints_compute_blue_edges 1002f2d0 f   freetype:autofit.obj
 0001:0002e480       _af_cjk_hints_compute_edges 1002f480 f   freetype:autofit.obj
 0001:0002e840       _af_cjk_hints_compute_segments 1002f840 f   freetype:autofit.obj
 0001:0002e8d0       _af_cjk_hints_detect_features 1002f8d0 f   freetype:autofit.obj
 0001:0002e900       _af_cjk_hints_link_segments 1002f900 f   freetype:autofit.obj
 0001:0002ec10       _af_cjk_metrics_check_digits 1002fc10 f   freetype:autofit.obj
 0001:0002ec10       _af_latin_metrics_check_digits 1002fc10 f   freetype:autofit.obj
 0001:0002ec90       _af_cjk_metrics_init_blues 1002fc90 f   freetype:autofit.obj
 0001:0002f060       _af_cjk_metrics_init_widths 10030060 f   freetype:autofit.obj
 0001:0002f060       _af_latin_metrics_init_widths 10030060 f   freetype:autofit.obj
 0001:0002f370       _af_cjk_metrics_scale_dim  10030370 f   freetype:autofit.obj
 0001:0002f520       _af_cjk_snap_width         10030520 f   freetype:autofit.obj
 0001:0002f520       _af_latin_snap_width       10030520 f   freetype:autofit.obj
 0001:0002f5a0       _af_direction_compute      100305a0 f   freetype:autofit.obj
 0001:0002f610       _af_face_globals_compute_style_coverage 10030610 f   freetype:autofit.obj
 0001:0002f7b0       _af_face_globals_free      100307b0 f   freetype:autofit.obj
 0001:0002f840       _af_face_globals_get_metrics 10030840 f   freetype:autofit.obj
 0001:0002f940       _af_face_globals_is_digit  10030940 f   freetype:autofit.obj
 0001:0002f960       _af_face_globals_new       10030960 f   freetype:autofit.obj
 0001:0002fa20       _af_glyph_hints_align_edge_points 10030a20 f   freetype:autofit.obj
 0001:0002fb00       _af_glyph_hints_align_strong_points 10030b00 f   freetype:autofit.obj
 0001:0002fd00       _af_glyph_hints_align_weak_points 10030d00 f   freetype:autofit.obj
 0001:0002fed0       _af_glyph_hints_done       10030ed0 f   freetype:autofit.obj
 0001:0002ff90       _af_glyph_hints_init       10030f90 f   freetype:autofit.obj
 0001:0002ffb0       _af_glyph_hints_reload     10030fb0 f   freetype:autofit.obj
 0001:00030400       _af_glyph_hints_rescale    10031400 f   freetype:autofit.obj
 0001:00030420       _af_glyph_hints_save       10031420 f   freetype:autofit.obj
 0001:00030480       _af_hint_normal_stem       10031480 f   freetype:autofit.obj
 0001:00030620       _af_iup_interp             10031620 f   freetype:autofit.obj
 0001:00030740       _af_iup_shift              10031740 f   freetype:autofit.obj
 0001:000307b0       _af_latin_align_linked_edge 100317b0 f   freetype:autofit.obj
 0001:000307f0       _af_latin_compute_stem_width 100317f0 f   freetype:autofit.obj
 0001:000309f0       _af_latin_hint_edges       100319f0 f   freetype:autofit.obj
 0001:00030f80       _af_latin_hints_compute_blue_edges 10031f80 f   freetype:autofit.obj
 0001:00031140       _af_latin_hints_compute_edges 10032140 f   freetype:autofit.obj
 0001:00031470       _af_latin_hints_compute_segments 10032470 f   freetype:autofit.obj
 0001:00031770       _af_latin_hints_detect_features 10032770 f   freetype:autofit.obj
 0001:000317a0       _af_latin_hints_link_segments 100327a0 f   freetype:autofit.obj
 0001:00031950       _af_latin_metrics_init_blues 10032950 f   freetype:autofit.obj
 0001:00032200       _af_latin_metrics_scale_dim 10033200 f   freetype:autofit.obj
 0001:000324c0       _af_loader_done            100334c0 f   freetype:autofit.obj
 0001:00032500       _af_loader_init            10033500 f   freetype:autofit.obj
 0001:00032540       _af_loader_load_g          10033540 f   freetype:autofit.obj
 0001:00032dc0       _af_loader_load_glyph      10033dc0 f   freetype:autofit.obj
 0001:00032ec0       _af_loader_reset           10033ec0 f   freetype:autofit.obj
 0001:00032f20       _af_property_get_face_globals 10033f20 f   freetype:autofit.obj
 0001:00032f70       _af_sort_and_quantize_widths 10033f70 f   freetype:autofit.obj
 0001:00033260       _af_sort_pos               10034260 f   freetype:autofit.obj
 0001:000332a0       _tt_face_init              100342a0 f   freetype:truetype.obj
 0001:00033420       _tt_face_done              10034420 f   freetype:truetype.obj
 0001:000334e0       _tt_size_init              100344e0 f   freetype:truetype.obj
 0001:00033500       _tt_size_done              10034500 f   freetype:truetype.obj
 0001:00033520       _tt_driver_init            10034520 f   freetype:truetype.obj
 0001:00033550       _tt_driver_done            10034550 f   freetype:truetype.obj
 0001:00033580       _tt_slot_init              10034580 f   freetype:truetype.obj
 0001:000335a0       _tt_face_get_location      100345a0 f   freetype:truetype.obj
 0001:000336a0       _TT_Set_MM_Blend           100346a0 f   freetype:truetype.obj
 0001:00033810       _TT_Set_Var_Design         10034810 f   freetype:truetype.obj
 0001:000339e0       _TT_Get_MM_Var             100349e0 f   freetype:truetype.obj
 0001:00033e10       _tt_property_set           10034e10 f   freetype:truetype.obj
 0001:00033e80       _tt_property_get           10034e80 f   freetype:truetype.obj
 0001:00033ed0       _cff_get_kerning           10034ed0 f   freetype:cff.obj
 0001:00033ed0       _tt_get_kerning            10034ed0 f   freetype:truetype.obj
 0001:00033f10       _tt_get_advances           10034f10 f   freetype:truetype.obj
 0001:00033fa0       _tt_size_select            10034fa0 f   freetype:truetype.obj
 0001:00033ff0       _tt_size_request           10034ff0 f   freetype:truetype.obj
 0001:00034080       _tt_glyph_load             10035080 f   freetype:truetype.obj
 0001:00034110       _tt_get_interface          10035110 f   freetype:truetype.obj
 0001:00034170       _Compute_Funcs             10035170 f   freetype:truetype.obj
 0001:000342b0       _Compute_Point_Displacement 100352b0 f   freetype:truetype.obj
 0001:00034390       _Compute_Round             10035390 f   freetype:truetype.obj
 0001:0003441c       $LN13                      1003541c     freetype:truetype.obj
 0001:00034440       _Current_Ppem              10035440 f   freetype:truetype.obj
 0001:00034490       _Current_Ratio             10035490 f   freetype:truetype.obj
 0001:00034510       _Direct_Move               10035510 f   freetype:truetype.obj
 0001:00034590       _Direct_Move_Orig          10035590 f   freetype:truetype.obj
 0001:00034600       _Direct_Move_Orig_X        10035600 f   freetype:truetype.obj
 0001:00034620       _Direct_Move_Orig_Y        10035620 f   freetype:truetype.obj
 0001:00034640       _Direct_Move_X             10035640 f   freetype:truetype.obj
 0001:00034660       _Direct_Move_Y             10035660 f   freetype:truetype.obj
 0001:00034690       _Dual_Project              10035690 f   freetype:truetype.obj
 0001:000346c0       _GetShortIns               100356c0 f   freetype:truetype.obj
 0001:00034700       _Init_Context              10035700 f   freetype:truetype.obj
 0001:00034770       _Ins_ALIGNPTS              10035770 f   freetype:truetype.obj
 0001:00034800       _Ins_ALIGNRP               10035800 f   freetype:truetype.obj
 0001:000348e0       _Ins_CALL                  100358e0 f   freetype:truetype.obj
 0001:000349b0       _Ins_DELTAC                100359b0 f   freetype:truetype.obj
 0001:00034ac0       _Ins_DELTAP                10035ac0 f   freetype:truetype.obj
 0001:00034bd0       _Ins_ELSE                  10035bd0 f   freetype:truetype.obj
 0001:00034c10       _Ins_ENDF                  10035c10 f   freetype:truetype.obj
 0001:00034c70       _Ins_FDEF                  10035c70 f   freetype:truetype.obj
 0001:00034d60       _Ins_FLIPPT                10035d60 f   freetype:truetype.obj
 0001:00034df0       _Ins_FLIPRGOFF             10035df0 f   freetype:truetype.obj
 0001:00034e50       _Ins_FLIPRGON              10035e50 f   freetype:truetype.obj
 0001:00034eb0       _Ins_GC                    10035eb0 f   freetype:truetype.obj
 0001:00034f20       _Ins_GETINFO               10035f20 f   freetype:truetype.obj
 0001:00034f80       _Ins_Goto_CodeRange        10035f80 f   freetype:truetype.obj
 0001:00035000       _Ins_IDEF                  10036000 f   freetype:truetype.obj
 0001:000350d0       _Ins_IF                    100360d0 f   freetype:truetype.obj
 0001:00035130       _Ins_INSTCTRL              10036130 f   freetype:truetype.obj
 0001:00035190       _Ins_IP                    10036190 f   freetype:truetype.obj
 0001:000354b0       _Ins_ISECT                 100364b0 f   freetype:truetype.obj
 0001:000356e0       _Ins_IUP                   100366e0 f   freetype:truetype.obj
 0001:00035850       _Ins_LOOPCALL              10036850 f   freetype:truetype.obj
 0001:00035930       _Ins_MD                    10036930 f   freetype:truetype.obj
 0001:00035b00       _Ins_MDAP                  10036b00 f   freetype:truetype.obj
 0001:00035b90       _Ins_MDRP                  10036b90 f   freetype:truetype.obj
 0001:00035de0       _Ins_MIAP                  10036de0 f   freetype:truetype.obj
 0001:00035f20       _Ins_MINDEX                10036f20 f   freetype:truetype.obj
 0001:00035f80       _Ins_MIRP                  10036f80 f   freetype:truetype.obj
 0001:000361d0       _Ins_MSIRP                 100371d0 f   freetype:truetype.obj
 0001:000362e0       _Ins_NPUSHB                100372e0 f   freetype:truetype.obj
 0001:00036350       _Ins_NPUSHW                10037350 f   freetype:truetype.obj
 0001:000363c0       _Ins_PUSHB                 100373c0 f   freetype:truetype.obj
 0001:00036430       _Ins_PUSHW                 10037430 f   freetype:truetype.obj
 0001:000364a0       _Ins_ROLL                  100374a0 f   freetype:truetype.obj
 0001:000364c0       _Ins_SCANCTRL              100374c0 f   freetype:truetype.obj
 0001:00036590       _Ins_SCANTYPE              10037590 f   freetype:truetype.obj
 0001:000365b0       _Ins_SCFS                  100375b0 f   freetype:truetype.obj
 0001:00036630       _Ins_SDPVTL                10037630 f   freetype:truetype.obj
 0001:00036740       _Ins_SHC                   10037740 f   freetype:truetype.obj
 0001:00036830       _Ins_SHP                   10037830 f   freetype:truetype.obj
 0001:000368f0       _Ins_SHPIX                 100378f0 f   freetype:truetype.obj
 0001:000369c0       _Ins_SHZ                   100379c0 f   freetype:truetype.obj
 0001:00036a80       _Ins_SZP0                  10037a80 f   freetype:truetype.obj
 0001:00036b10       _Ins_SZP1                  10037b10 f   freetype:truetype.obj
 0001:00036ba0       _Ins_SZP2                  10037ba0 f   freetype:truetype.obj
 0001:00036c20       _Ins_SZPS                  10037c20 f   freetype:truetype.obj
 0001:00036ce0       _Ins_SxVTL                 10037ce0 f   freetype:truetype.obj
 0001:00036d70       _Ins_UNKNOWN               10037d70 f   freetype:truetype.obj
 0001:00036e10       _Ins_UTP                   10037e10 f   freetype:truetype.obj
 0001:00036e70       _Move_CVT                  10037e70 f   freetype:truetype.obj
 0001:00036e90       _Move_CVT_Stretched        10037e90 f   freetype:truetype.obj
 0001:00036ec0       _Move_Zp2_Point            10037ec0 f   freetype:truetype.obj
 0001:00036f30       _Normalize                 10037f30 f   freetype:truetype.obj
 0001:00036fa0       _Project                   10037fa0 f   freetype:truetype.obj
 0001:00036fd0       _Project_x                 10037fd0 f   freetype:truetype.obj
 0001:00036fe0       _Project_y                 10037fe0 f   freetype:truetype.obj
 0001:00036ff0       _Read_CVT                  10037ff0 f   freetype:truetype.obj
 0001:00037010       _Read_CVT_Stretched        10038010 f   freetype:truetype.obj
 0001:00037060       _Round_Down_To_Grid        10038060 f   freetype:truetype.obj
 0001:00037090       _Round_None                10038090 f   freetype:truetype.obj
 0001:000370c0       _Round_Super               100380c0 f   freetype:truetype.obj
 0001:00037120       _Round_Super_45            10038120 f   freetype:truetype.obj
 0001:00037180       _Round_To_Double_Grid      10038180 f   freetype:truetype.obj
 0001:000371c0       _Round_To_Grid             100381c0 f   freetype:truetype.obj
 0001:00037200       _Round_To_Half_Grid        10038200 f   freetype:truetype.obj
 0001:00037240       _Round_Up_To_Grid          10038240 f   freetype:truetype.obj
 0001:00037280       _SetSuperRound             10038280 f   freetype:truetype.obj
 0001:0003736c       $LN18                      1003836c     freetype:truetype.obj
 0001:0003737c       $LN17                      1003837c     freetype:truetype.obj
 0001:00037440       $LN20                      10038440     freetype:truetype.obj
 0001:00037454       $LN19                      10038454     freetype:truetype.obj
 0001:00037490       _SkipCode                  10038490 f   freetype:truetype.obj
 0001:00037510       _TT_Access_Glyph_Frame     10038510 f   freetype:truetype.obj
 0001:00037560       _TT_Clear_CodeRange        10038560 f   freetype:truetype.obj
 0001:00037590       _TT_Done_Context           10038590 f   freetype:truetype.obj
 0001:00037630       _TT_DotFix14               10038630 f   freetype:truetype.obj
 0001:000376d0       _TT_Forget_Glyph_Frame     100386d0 f   freetype:truetype.obj
 0001:000376f0       _TT_Get_HMetrics           100386f0 f   freetype:truetype.obj
 0001:00037720       _TT_Get_VMetrics           10038720 f   freetype:truetype.obj
 0001:000377b0       _TT_Goto_CodeRange         100387b0 f   freetype:truetype.obj
 0001:000377f0       _TT_Hint_Glyph             100387f0 f   freetype:truetype.obj
 0001:00037a70       _TT_Init_Glyph_Loading     10038a70 f   freetype:truetype.obj
 0001:00037ab0       _TT_Load_Composite_Glyph   10038ab0 f   freetype:truetype.obj
 0001:00037cd0       _TT_Load_Context           10038cd0 f   freetype:truetype.obj
 0001:00037f80       _TT_Load_Glyph             10038f80 f   freetype:truetype.obj
 0001:000381d8       $LN30                      100391d8     freetype:truetype.obj
 0001:000381f0       _TT_Load_Glyph_Header      100391f0 f   freetype:truetype.obj
 0001:00038290       _TT_Load_Simple_Glyph      10039290 f   freetype:truetype.obj
 0001:000386c0       _TT_MulFix14               100396c0 f   freetype:truetype.obj
 0001:00038770       _TT_Process_Composite_Component 10039770 f   freetype:truetype.obj
 0001:00038950       _TT_Process_Composite_Glyph 10039950 f   freetype:truetype.obj
 0001:00038b70       _TT_Process_Simple_Glyph   10039b70 f   freetype:truetype.obj
 0001:00039a08       $LN282                     1003aa08     freetype:truetype.obj
 0001:00039c50       _TT_Run_Context            1003ac50 f   freetype:truetype.obj
 0001:00039d30       _TT_Save_Context           1003ad30 f   freetype:truetype.obj
 0001:00039dc0       _TT_Set_CodeRange          1003adc0 f   freetype:truetype.obj
 0001:00039df0       _TT_Vary_Get_Glyph_Deltas  1003adf0 f   freetype:truetype.obj
 0001:0003a310       _Update_Max                1003b310 f   freetype:truetype.obj
 0001:0003a360       _Write_CVT                 1003b360 f   freetype:truetype.obj
 0001:0003a380       _Write_CVT_Stretched       1003b380 f   freetype:truetype.obj
 0001:0003a3b0       __iup_worker_interpolate   1003b3b0 f   freetype:truetype.obj
 0001:0003a500       __iup_worker_shift         1003b500 f   freetype:truetype.obj
 0001:0003a550       _compute_glyph_metrics     1003b550 f   freetype:truetype.obj
 0001:0003a7a0       _ft_var_apply_tuple        1003b7a0 f   freetype:truetype.obj
 0001:0003a8b0       _ft_var_load_avar          1003b8b0 f   freetype:truetype.obj
 0001:0003aa50       _ft_var_load_gvar          1003ba50 f   freetype:truetype.obj
 0001:0003ac90       _ft_var_readpackeddeltas   1003bc90 f   freetype:truetype.obj
 0001:0003ad90       _ft_var_readpackedpoints   1003bd90 f   freetype:truetype.obj
 0001:0003aed0       _load_sbit_image           1003bed0 f   freetype:truetype.obj
 0001:0003afc0       _load_truetype_glyph       1003bfc0 f   freetype:truetype.obj
 0001:0003b870       _translate_array           1003c870 f   freetype:truetype.obj
 0001:0003b8b0       _tt_check_single_notdef    1003c8b0 f   freetype:truetype.obj
 0001:0003b9a0       _tt_check_trickyness       1003c9a0 f   freetype:truetype.obj
 0001:0003b9e0       _tt_check_trickyness_family 1003c9e0 f   freetype:truetype.obj
 0001:0003ba20       _tt_check_trickyness_sfnt_ids 1003ca20 f   freetype:truetype.obj
 0001:0003bb80       _tt_done_blend             1003cb80 f   freetype:truetype.obj
 0001:0003bc30       _tt_face_done_loca         1003cc30 f   freetype:truetype.obj
 0001:0003bc60       _tt_face_free_hdmx         1003cc60 f   freetype:truetype.obj
 0001:0003bca0       _tt_face_get_device_metrics 1003cca0 f   freetype:truetype.obj
 0001:0003bd10       _tt_face_load_cvt          1003cd10 f   freetype:truetype.obj
 0001:0003be00       _tt_face_load_fpgm         1003ce00 f   freetype:truetype.obj
 0001:0003be60       _tt_face_load_hdmx         1003ce60 f   freetype:truetype.obj
 0001:0003bfd0       _tt_face_load_loca         1003cfd0 f   freetype:truetype.obj
 0001:0003c120       _tt_face_load_prep         1003d120 f   freetype:truetype.obj
 0001:0003c180       _tt_face_vary_cvt          1003d180 f   freetype:truetype.obj
 0001:0003c540       _tt_get_metrics            1003d540 f   freetype:truetype.obj
 0001:0003c5f0       _tt_get_metrics_incr_overrides 1003d5f0 f   freetype:truetype.obj
 0001:0003c690       _tt_get_sfnt_checksum      1003d690 f   freetype:truetype.obj
 0001:0003c6e0       _tt_glyphzone_done         1003d6e0 f   freetype:truetype.obj
 0001:0003c750       _tt_glyphzone_new          1003d750 f   freetype:truetype.obj
 0001:0003c860       _tt_loader_init            1003d860 f   freetype:truetype.obj
 0001:0003caa0       _tt_prepare_zone           1003daa0 f   freetype:truetype.obj
 0001:0003cb10       _tt_size_done_bytecode     1003db10 f   freetype:truetype.obj
 0001:0003cbf0       _tt_size_init_bytecode     1003dbf0 f   freetype:truetype.obj
 0001:0003cde0       _tt_size_ready_bytecode    1003dde0 f   freetype:truetype.obj
 0001:0003cf50       _tt_size_reset             1003df50 f   freetype:truetype.obj
 0001:0003d130       _tt_size_run_fpgm          1003e130 f   freetype:truetype.obj
 0001:0003d260       _tt_size_run_prep          1003e260 f   freetype:truetype.obj
 0001:0003d3c0       _tt_synth_sfnt_checksum    1003e3c0 f   freetype:truetype.obj
 0001:0003d450       _T1_Get_Multi_Master       1003e450 f   freetype:type1.obj
 0001:0003d4d0       _T1_Get_MM_Var             1003e4d0 f   freetype:type1.obj
 0001:0003d710       _T1_Set_MM_Blend           1003e710 f   freetype:type1.obj
 0001:0003d7e0       _T1_Set_MM_Design          1003e7e0 f   freetype:type1.obj
 0001:0003d920       _T1_Set_Var_Design         1003e920 f   freetype:type1.obj
 0001:0003d9a0       _parse_blend_axis_types    1003e9a0 f   freetype:type1.obj
 0001:0003dae0       _parse_blend_design_positions 1003eae0 f   freetype:type1.obj
 0001:0003dcf0       _parse_blend_design_map    1003ecf0 f   freetype:type1.obj
 0001:0003df00       _parse_weight_vector       1003ef00 f   freetype:type1.obj
 0001:0003e050       _parse_buildchar           1003f050 f   freetype:type1.obj
 0001:0003e070       _parse_private             1003f070 f   freetype:type1.obj
 0001:0003e080       _t1_parse_font_matrix      1003f080 f   freetype:type1.obj
 0001:0003e080       _t42_parse_font_matrix     1003f080 f   freetype:type42.obj
 0001:0003e1a0       _parse_encoding            1003f1a0 f   freetype:type1.obj
 0001:0003e590       _parse_subrs               1003f590 f   freetype:type1.obj
 0001:0003e7d0       _parse_charstrings         1003f7d0 f   freetype:type1.obj
 0001:0003edb0       _T1_Size_Done              1003fdb0 f   freetype:type1.obj
 0001:0003ede0       _T1_Size_Request           1003fde0 f   freetype:type1.obj
 0001:0003ee20       _T1_Size_Init              1003fe20 f   freetype:type1.obj
 0001:0003ee70       _T1_Face_Init              1003fe70 f   freetype:type1.obj
 0001:0003f210       $LN72                      10040210     freetype:type1.obj
 0001:0003f220       _T1_Face_Done              10040220 f   freetype:type1.obj
 0001:0003f400       _T1_GlyphSlot_Init         10040400 f   freetype:type1.obj
 0001:0003f450       _cff_slot_done             10040450 f   freetype:cff.obj
 0001:0003f450       _T1_GlyphSlot_Done         10040450 f   freetype:type1.obj
 0001:0003f450       _cid_slot_done             10040450 f   freetype:type1cid.obj
 0001:0003f470       _T1_Get_Advances           10040470 f   freetype:type1.obj
 0001:0003f590       _T1_Load_Glyph             10040590 f   freetype:type1.obj
 0001:0003fb10       _T1_Read_Metrics           10040b10 f   freetype:type1.obj
 0001:0003fcc0       _T1_Get_Track_Kerning      10040cc0 f   freetype:type1.obj
 0001:0003fd50       _t1_get_glyph_name         10040d50 f   freetype:type1.obj
 0001:0003fd50       _t42_get_glyph_name        10040d50 f   freetype:type42.obj
 0001:0003fd80       _t1_get_name_index         10040d80 f   freetype:type1.obj
 0001:0003fdf0       _t1_get_ps_name            10040df0 f   freetype:type1.obj
 0001:0003fdf0       _t42_get_ps_font_name      10040df0 f   freetype:type42.obj
 0001:0003fe00       _t1_ps_get_font_info       10040e00 f   freetype:type1.obj
 0001:0003fe00       _t42_ps_get_font_info      10040e00 f   freetype:type42.obj
 0001:0003fe30       _t1_ps_get_font_extra      10040e30 f   freetype:type1.obj
 0001:0003fe30       _t42_ps_get_font_extra     10040e30 f   freetype:type42.obj
 0001:0003fe50       _t1_ps_has_glyph_names     10040e50 f   freetype:type1.obj
 0001:0003fe50       _t42_ps_has_glyph_names    10040e50 f   freetype:type42.obj
 0001:0003fe60       _t1_ps_get_font_private    10040e60 f   freetype:type1.obj
 0001:0003fe60       _t42_ps_get_font_private   10040e60 f   freetype:type42.obj
 0001:0003fe80       _t1_ps_get_font_value      10040e80 f   freetype:type1.obj
 0001:000406e8       $LN123                     100416e8     freetype:type1.obj
 0001:000407a0       $LN124                     100417a0     freetype:type1.obj
 0001:000407b0       $LN125                     100417b0     freetype:type1.obj
 0001:000407c0       _Get_Interface             100417c0 f   freetype:type1.obj
 0001:000407d0       _Get_Kerning               100417d0 f   freetype:type1.obj
 0001:00040810       _T1_Compute_Max_Advance    10041810 f   freetype:type1.obj
 0001:00040920       _T1_Done_Blend             10041920 f   freetype:type1.obj
 0001:00040a80       _T1_Done_Metrics           10041a80 f   freetype:type1.obj
 0001:00040ad0       _T1_Finalize_Parser        10041ad0 f   freetype:type1.obj
 0001:00040b20       _T1_Get_Kerning            10041b20 f   freetype:type1.obj
 0001:00040ba0       _T1_Get_Private_Dict       10041ba0 f   freetype:type1.obj
 0001:00040f60       _T1_New_Parser             10041f60 f   freetype:type1.obj
 0001:000410e0       _T1_Open_Face              100420e0 f   freetype:type1.obj
 0001:000414e0       _T1_Parse_Glyph            100424e0 f   freetype:type1.obj
 0001:00041530       _T1_Parse_Glyph_And_Get_Char_String 10042530 f   freetype:type1.obj
 0001:00041660       _T1_Read_PFM               10042660 f   freetype:type1.obj
 0001:00041870       _T1_Size_Get_Globals_Funcs 10042870 f   freetype:type1.obj
 0001:000418b0       _check_type1_format        100428b0 f   freetype:type1.obj
 0001:00041980       _afm_compare_kern_pairs    10042980 f   freetype:psaux.obj
 0001:00041980       _compare_kern_pairs        10042980 f   freetype:type1.obj
 0001:000419b0       _mm_axis_unmap             100429b0 f   freetype:type1.obj
 0001:00041a40       _mm_weights_unmap          10042a40 f   freetype:type1.obj
 0001:00041b20       _parse_dict                10042b20 f   freetype:type1.obj
 0001:00041f20       _read_binary_data          10042f20 f   freetype:type1.obj
 0001:00041fa0       _read_pfb_tag              10042fa0 f   freetype:type1.obj
 0001:00042010       _t1_allocate_blend         10043010 f   freetype:type1.obj
 0001:00042210       _t1_done_loader            10043210 f   freetype:type1.obj
 0001:00042290       _t1_get_index              10043290 f   freetype:type1.obj
 0001:00042310       _t1_init_loader            10043310 f   freetype:type1.obj
 0001:00042330       _t1_load_keyword           10043330 f   freetype:type1.obj
 0001:00042450       $LN26                      10043450     freetype:type1.obj
 0001:00042470       _cff_cmap_encoding_init    10043470 f   freetype:cff.obj
 0001:00042490       _cff_cmap_encoding_done    10043490 f   freetype:cff.obj
 0001:000424a0       _cff_cmap_encoding_char_index 100434a0 f   freetype:cff.obj
 0001:000424c0       _cff_cmap_encoding_char_next 100434c0 f   freetype:cff.obj
 0001:00042520       _cff_cmap_unicode_init     10043520 f   freetype:cff.obj
 0001:00042560       _cff_cmap_unicode_done     10043560 f   freetype:cff.obj
 0001:00042560       _t1_cmap_unicode_done      10043560 f   freetype:psaux.obj
 0001:00042590       _cff_cmap_unicode_char_index 10043590 f   freetype:cff.obj
 0001:000425b0       _cff_cmap_unicode_char_next 100435b0 f   freetype:cff.obj
 0001:000425d0       _cff_size_init             100435d0 f   freetype:cff.obj
 0001:00042720       _cff_size_done             10043720 f   freetype:cff.obj
 0001:00042780       _cff_size_request          10043780 f   freetype:cff.obj
 0001:00042890       _cff_size_select           10043890 f   freetype:cff.obj
 0001:00042970       _cff_slot_init             10043970 f   freetype:cff.obj
 0001:000429d0       _cff_face_init             100439d0 f   freetype:cff.obj
 0001:000431d0       _cff_face_done             100441d0 f   freetype:cff.obj
 0001:00043220       _cff_driver_init           10044220 f   freetype:cff.obj
 0001:00043270       _cff_glyph_load            10044270 f   freetype:cff.obj
 0001:000432d0       _cff_get_advances          100442d0 f   freetype:cff.obj
 0001:00043340       _cff_get_glyph_name        10044340 f   freetype:cff.obj
 0001:00043390       _cff_get_name_index        10044390 f   freetype:cff.obj
 0001:00043440       _cff_ps_has_glyph_names    10044440 f   freetype:cff.obj
 0001:00043460       _cff_ps_get_font_info      10044460 f   freetype:cff.obj
 0001:00043540       _cff_get_ps_name           10044540 f   freetype:cff.obj
 0001:00043560       _cff_get_cmap_info         10044560 f   freetype:cff.obj
 0001:000435d0       _cff_get_ros               100445d0 f   freetype:cff.obj
 0001:00043660       _cff_get_is_cid            10044660 f   freetype:cff.obj
 0001:00043690       _cff_get_cid_from_glyph_index 10044690 f   freetype:cff.obj
 0001:000436e0       _cff_property_set          100446e0 f   freetype:cff.obj
 0001:00043890       _cff_property_get          10044890 f   freetype:cff.obj
 0001:00043990       _cff_get_interface         10044990 f   freetype:cff.obj
 0001:000439e0       _cff_parse_font_matrix     100449e0 f   freetype:cff.obj
 0001:00043ac0       _cff_parse_font_bbox       10044ac0 f   freetype:cff.obj
 0001:00043b40       _cff_parse_private_dict    10044b40 f   freetype:cff.obj
 0001:00043b90       _cff_parse_cid_ros         10044b90 f   freetype:cff.obj
 0001:00043bf0       _CFF_Done_FD_Select        10044bf0 f   freetype:cff.obj
 0001:00043c20       _CFF_Load_FD_Select        10044c20 f   freetype:cff.obj
 0001:00043cc0       _cf2_arrstack_clear        10044cc0 f   freetype:cff.obj
 0001:00043cd0       _cf2_arrstack_finalize     10044cd0 f   freetype:cff.obj
 0001:00043d10       _cf2_arrstack_getBuffer    10044d10 f   freetype:cff.obj
 0001:00043d20       _cf2_arrstack_getPointer   10044d20 f   freetype:cff.obj
 0001:00043d50       _cf2_arrstack_init         10044d50 f   freetype:cff.obj
 0001:00043d90       _cf2_arrstack_push         10044d90 f   freetype:cff.obj
 0001:00043de0       _cf2_arrstack_setCount     10044de0 f   freetype:cff.obj
 0001:00043e10       _cf2_arrstack_setNumElements 10044e10 f   freetype:cff.obj
 0001:00043ea0       _cf2_arrstack_size         10044ea0 f   freetype:cff.obj
 0001:00043eb0       _cf2_blues_capture         10044eb0 f   freetype:cff.obj
 0001:00044070       _cf2_blues_init            10045070 f   freetype:cff.obj
 0001:00044560       _cf2_buf_isEnd             10045560 f   freetype:cff.obj
 0001:00044580       _cf2_buf_readByte          10045580 f   freetype:cff.obj
 0001:000445b0       _cf2_builder_cubeTo        100455b0 f   freetype:cff.obj
 0001:00044610       _cf2_builder_lineTo        10045610 f   freetype:cff.obj
 0001:00044650       _cf2_builder_moveTo        10045650 f   freetype:cff.obj
 0001:00044670       _cf2_checkTransform        10045670 f   freetype:cff.obj
 0001:000446d0       _cf2_computeDarkening      100456d0 f   freetype:cff.obj
 0001:00044930       _cf2_decoder_parse_charstrings 10045930 f   freetype:cff.obj
 0001:00044af0       _cf2_doFlex                10045af0 f   freetype:cff.obj
 0001:00044c90       _cf2_doStems               10045c90 f   freetype:cff.obj
 0001:00044d70       _cf2_font_setup            10045d70 f   freetype:cff.obj
 0001:00044fb0       _cf2_freeSeacComponent     10045fb0 f   freetype:cff.obj
 0001:00044fd0       _cf2_getBlueMetrics        10045fd0 f   freetype:cff.obj
 0001:00045020       _cf2_getBlueValues         10046020 f   freetype:cff.obj
 0001:00045050       _cf2_getDefaultWidthX      10046050 f   freetype:cff.obj
 0001:00045070       _cf2_getFamilyBlues        10046070 f   freetype:cff.obj
 0001:000450a0       _cf2_getFamilyOtherBlues   100460a0 f   freetype:cff.obj
 0001:000450d0       _cf2_getGlyphOutline       100460d0 f   freetype:cff.obj
 0001:000451a0       _cf2_getLanguageGroup      100461a0 f   freetype:cff.obj
 0001:000451c0       _cf2_getNominalWidthX      100461c0 f   freetype:cff.obj
 0001:000451e0       _cf2_getOtherBlues         100461e0 f   freetype:cff.obj
 0001:00045210       _cf2_getPpemY              10046210 f   freetype:cff.obj
 0001:00045230       _cf2_getScaleAndHintFlag   10046230 f   freetype:cff.obj
 0001:000452b0       _cf2_getSeacComponent      100462b0 f   freetype:cff.obj
 0001:00045310       _cf2_getStdHW              10046310 f   freetype:cff.obj
 0001:00045330       _cf2_getStdVW              10046330 f   freetype:cff.obj
 0001:00045350       _cf2_getSubfont            10046350 f   freetype:cff.obj
 0001:00045360       _cf2_getUnitsPerEm         10046360 f   freetype:cff.obj
 0001:00045370       _cf2_getWindingMomentum    10046370 f   freetype:cff.obj
 0001:000453a0       _cf2_glyphpath_closeOpenPath 100463a0 f   freetype:cff.obj
 0001:00045420       _cf2_glyphpath_computeIntersection 10046420 f   freetype:cff.obj
 0001:000456a0       _cf2_glyphpath_computeOffset 100466a0 f   freetype:cff.obj
 0001:000459a0       _cf2_glyphpath_curveTo     100469a0 f   freetype:cff.obj
 0001:00045b60       _cf2_glyphpath_finalize    10046b60 f   freetype:cff.obj
 0001:00045b70       _cf2_glyphpath_hintPoint   10046b70 f   freetype:cff.obj
 0001:00045cd0       _cf2_glyphpath_init        10046cd0 f   freetype:cff.obj
 0001:00045e10       _cf2_glyphpath_lineTo      10046e10 f   freetype:cff.obj
 0001:00045f80       _cf2_glyphpath_moveTo      10046f80 f   freetype:cff.obj
 0001:00046010       _cf2_glyphpath_pushMove    10047010 f   freetype:cff.obj
 0001:000460c0       _cf2_glyphpath_pushPrevElem 100470c0 f   freetype:cff.obj
 0001:00046310       _cf2_hint_init             10047310 f   freetype:cff.obj
 0001:00046450       _cf2_hint_initZero         10047450 f   freetype:cff.obj
 0001:00046470       _cf2_hint_isBottom         10047470 f   freetype:cff.obj
 0001:00046480       _cf2_hint_isLocked         10047480 f   freetype:cff.obj
 0001:00046490       _cf2_hint_isPair           10047490 f   freetype:cff.obj
 0001:000464a0       _cf2_hint_isPairTop        100474a0 f   freetype:cff.obj
 0001:000464b0       _cf2_hint_isSynthetic      100474b0 f   freetype:cff.obj
 0001:000464c0       _cf2_hint_isTop            100474c0 f   freetype:cff.obj
 0001:000464d0       _cf2_hint_isValid          100474d0 f   freetype:cff.obj
 0001:000464e0       _cf2_hint_lock             100474e0 f   freetype:cff.obj
 0001:000464f0       _cf2_hintmap_adjustHints   100474f0 f   freetype:cff.obj
 0001:00046740       _cf2_hintmap_build         10047740 f   freetype:cff.obj
 0001:00046a80       _cf2_hintmap_init          10047a80 f   freetype:cff.obj
 0001:00046ac0       _cf2_hintmap_insertHint    10047ac0 f   freetype:cff.obj
 0001:00046cf0       _cf2_hintmap_isValid       10047cf0 f   freetype:cff.obj
 0001:00046d00       _cf2_hintmap_map           10047d00 f   freetype:cff.obj
 0001:00046e20       _cf2_hintmask_getMaskPtr   10047e20 f   freetype:cff.obj
 0001:00046e30       _cf2_hintmask_init         10047e30 f   freetype:cff.obj
 0001:00046e70       _cf2_hintmask_isNew        10047e70 f   freetype:cff.obj
 0001:00046e80       _cf2_hintmask_isValid      10047e80 f   freetype:cff.obj
 0001:00046e90       _cf2_hintmask_read         10047e90 f   freetype:cff.obj
 0001:00046ed0       _cf2_hintmask_setAll       10047ed0 f   freetype:cff.obj
 0001:00046f20       _cf2_hintmask_setCounts    10047f20 f   freetype:cff.obj
 0001:00046f60       _cf2_hintmask_setNew       10047f60 f   freetype:cff.obj
 0001:00046f70       _cf2_initGlobalRegionBuffer 10047f70 f   freetype:cff.obj
 0001:00046fc0       _cf2_initLocalRegionBuffer 10047fc0 f   freetype:cff.obj
 0001:00047010       _cf2_interpT2CharString    10048010 f   freetype:cff.obj
 0001:000480f8       $LN445                     100490f8     freetype:cff.obj
 0001:00048144       $LN444                     10049144     freetype:cff.obj
 0001:00048164       $LN447                     10049164     freetype:cff.obj
 0001:00048178       $LN446                     10049178     freetype:cff.obj
 0001:000481a0       _cf2_outline_close         100491a0 f   freetype:cff.obj
 0001:000481c0       _cf2_outline_init          100491c0 f   freetype:cff.obj
 0001:00048200       _cf2_outline_reset         10049200 f   freetype:cff.obj
 0001:00048220       _cf2_setError              10049220 f   freetype:cff.obj
 0001:00048240       _cf2_setGlyphWidth         10049240 f   freetype:cff.obj
 0001:00048260       _cf2_stack_clear           10049260 f   freetype:cff.obj
 0001:00048280       _cf2_stack_count           10049280 f   freetype:cff.obj
 0001:000482a0       _cf2_stack_free            100492a0 f   freetype:cff.obj
 0001:000482c0       _cf2_stack_getReal         100492c0 f   freetype:cff.obj
 0001:00048330       _cf2_stack_init            10049330 f   freetype:cff.obj
 0001:00048370       _cf2_stack_popFixed        10049370 f   freetype:cff.obj
 0001:000483e0       _cf2_stack_popInt          100493e0 f   freetype:cff.obj
 0001:00048430       _cf2_stack_pushFixed       10049430 f   freetype:cff.obj
 0001:00048470       _cf2_stack_pushInt         10049470 f   freetype:cff.obj
 0001:000484b0       _cff_builder_add_contour   100494b0 f   freetype:cff.obj
 0001:00048520       _cff_builder_add_point     10049520 f   freetype:cff.obj
 0001:00048570       _cff_builder_add_point1    10049570 f   freetype:cff.obj
 0001:000485a0       _cff_builder_close_contour 100495a0 f   freetype:cff.obj
 0001:000485a0       _t1_builder_close_contour  100495a0 f   freetype:psaux.obj
 0001:00048670       _cff_builder_done          10049670 f   freetype:cff.obj
 0001:00048670       _t1_builder_done           10049670 f   freetype:psaux.obj
 0001:00048690       _cff_builder_init          10049690 f   freetype:cff.obj
 0001:00048730       _cff_builder_start_point   10049730 f   freetype:cff.obj
 0001:00048770       _cff_charset_cid_to_gindex 10049770 f   freetype:cff.obj
 0001:00048790       _cff_charset_compute_cids  10049790 f   freetype:cff.obj
 0001:000488c0       _cff_charset_done          100498c0 f   freetype:cff.obj
 0001:00048900       _cff_charset_free_cids     10049900 f   freetype:cff.obj
 0001:00048930       _cff_charset_load          10049930 f   freetype:cff.obj
 0001:00048c10       _cff_check_points          10049c10 f   freetype:cff.obj
 0001:00048c10       _t1_builder_check_points   10049c10 f   freetype:psaux.obj
 0001:00048c50       _cff_compute_bias          10049c50 f   freetype:cff.obj
 0001:00048c90       _cff_decoder_init          10049c90 f   freetype:cff.obj
 0001:00048d00       _cff_decoder_prepare       10049d00 f   freetype:cff.obj
 0001:00048dc0       _cff_encoding_done         10049dc0 f   freetype:cff.obj
 0001:00048de0       _cff_encoding_load         10049de0 f   freetype:cff.obj
 0001:00049140       _cff_fd_select_get         1004a140 f   freetype:cff.obj
 0001:000491f0       _cff_font_done             1004a1f0 f   freetype:cff.obj
 0001:00049350       _cff_font_load             1004a350 f   freetype:cff.obj
 0001:00049720       _cff_free_glyph_data       1004a720 f   freetype:cff.obj
 0001:00049780       _cff_get_glyph_data        1004a780 f   freetype:cff.obj
 0001:000497e0       _cff_get_standard_encoding 1004a7e0 f   freetype:cff.obj
 0001:00049800       _cff_index_access_element  1004a800 f   freetype:cff.obj
 0001:00049950       _cff_index_done            1004a950 f   freetype:cff.obj
 0001:00049990       _cff_index_forget_element  1004a990 f   freetype:cff.obj
 0001:000499b0       _cff_index_get_name        1004a9b0 f   freetype:cff.obj
 0001:00049a30       _cff_index_get_pointers    1004aa30 f   freetype:cff.obj
 0001:00049b90       _cff_index_get_sid_string  1004ab90 f   freetype:cff.obj
 0001:00049be0       _cff_index_get_string      1004abe0 f   freetype:cff.obj
 0001:00049c00       _cff_index_init            1004ac00 f   freetype:cff.obj
 0001:00049d30       _cff_index_load_offsets    1004ad30 f   freetype:cff.obj
 0001:00049ec0       _cff_index_read_offset     1004aec0 f   freetype:cff.obj
 0001:00049f20       _cff_lookup_glyph_by_stdcharcode 1004af20 f   freetype:cff.obj
 0001:00049f70       _cff_make_private_dict     1004af70 f   freetype:cff.obj
 0001:0004a100       _cff_parse_fixed           1004b100 f   freetype:cff.obj
 0001:0004a120       _cff_parse_fixed_dynamic   1004b120 f   freetype:cff.obj
 0001:0004a1d0       _cff_parse_fixed_scaled    1004b1d0 f   freetype:cff.obj
 0001:0004a1e0       _cff_parse_integer         1004b1e0 f   freetype:cff.obj
 0001:0004a280       _cff_parse_num             1004b280 f   freetype:cff.obj
 0001:0004a2b0       _cff_parse_real            1004b2b0 f   freetype:cff.obj
 0001:0004a650       _cff_parser_init           1004b650 f   freetype:cff.obj
 0001:0004a690       _cff_parser_run            1004b690 f   freetype:cff.obj
 0001:0004a8bc       $LN86                      1004b8bc     freetype:cff.obj
 0001:0004a8e0       _cff_sid_to_glyph_name     1004b8e0 f   freetype:cff.obj
 0001:0004a910       _cff_size_get_globals_funcs 1004b910 f   freetype:cff.obj
 0001:0004a960       _cff_slot_load             1004b960 f   freetype:cff.obj
 0001:0004b360       _cff_strcpy                1004c360 f   freetype:cff.obj
 0001:0004b380       _cff_subfont_done          1004c380 f   freetype:cff.obj
 0001:0004b3c0       _cff_subfont_load          1004c3c0 f   freetype:cff.obj
 0001:0004b600       _do_fixed                  1004c600 f   freetype:cff.obj
 0001:0004b660       _remove_style              1004c660 f   freetype:cff.obj
 0001:0004b6f0       _remove_subset_prefix      1004c6f0 f   freetype:cff.obj
 0001:0004b7a0       _cid_parse_font_matrix     1004c7a0 f   freetype:type1cid.obj
 0001:0004b8e0       _parse_fd_array            1004c8e0 f   freetype:type1cid.obj
 0001:0004b970       _parse_expansion_factor    1004c970 f   freetype:type1cid.obj
 0001:0004b9c0       _cid_slot_init             1004c9c0 f   freetype:type1cid.obj
 0001:0004ba10       _cid_size_done             1004ca10 f   freetype:type1cid.obj
 0001:0004ba40       _cid_size_init             1004ca40 f   freetype:type1cid.obj
 0001:0004ba90       _cid_size_request          1004ca90 f   freetype:type1cid.obj
 0001:0004bad0       _cid_face_init             1004cad0 f   freetype:type1cid.obj
 0001:0004bd50       _cid_face_done             1004cd50 f   freetype:type1cid.obj
 0001:0004bf00       _cid_slot_load_glyph       1004cf00 f   freetype:type1cid.obj
 0001:0004c370       _cid_get_postscript_name   1004d370 f   freetype:type1cid.obj
 0001:0004c390       _cid_ps_get_font_info      1004d390 f   freetype:type1cid.obj
 0001:0004c3c0       _cid_ps_get_font_extra     1004d3c0 f   freetype:type1cid.obj
 0001:0004c3e0       _cid_get_ros               1004d3e0 f   freetype:type1cid.obj
 0001:0004c420       _cid_get_is_cid            1004d420 f   freetype:type1cid.obj
 0001:0004c440       _cid_get_cid_from_glyph_index 1004d440 f   freetype:type1cid.obj
 0001:0004c460       _cid_get_interface         1004d460 f   freetype:type1cid.obj
 0001:0004c470       _cid_done_loader           1004d470 f   freetype:type1cid.obj
 0001:0004c480       _cid_face_open             1004d480 f   freetype:type1cid.obj
 0001:0004c5a0       _cid_get_offset            1004d5a0 f   freetype:type1cid.obj
 0001:0004c5d0       _cid_hex_to_binary         1004d5d0 f   freetype:type1cid.obj
 0001:0004c770       _cid_init_loader           1004d770 f   freetype:type1cid.obj
 0001:0004c790       _cid_load_glyph            1004d790 f   freetype:type1cid.obj
 0001:0004cae0       _cid_load_keyword          1004dae0 f   freetype:type1cid.obj
 0001:0004cb94       $LN23                      1004db94     freetype:type1cid.obj
 0001:0004cbb0       _cid_parse_dict            1004dbb0 f   freetype:type1cid.obj
 0001:0004cd10       _cid_parser_done           1004dd10 f   freetype:type1cid.obj
 0001:0004cd40       _cid_parser_new            1004dd40 f   freetype:type1cid.obj
 0001:0004d0d0       _cid_read_subrs            1004e0d0 f   freetype:type1cid.obj
 0001:0004d420       _cid_size_get_globals_funcs 1004e420 f   freetype:type1cid.obj
 0001:0004d460       _pfr_face_init             1004e460 f   freetype:pfr.obj
 0001:0004d7c0       _pfr_face_done             1004e7c0 f   freetype:pfr.obj
 0001:0004d810       _pfr_face_get_kerning      1004e810 f   freetype:pfr.obj
 0001:0004da20       _pfr_slot_init             1004ea20 f   freetype:pfr.obj
 0001:0004da50       _pfr_slot_done             1004ea50 f   freetype:pfr.obj
 0001:0004da60       _pfr_slot_load             1004ea60 f   freetype:pfr.obj
 0001:0004dd10       _pfr_extra_item_load_bitmap_info 1004ed10 f   freetype:pfr.obj
 0001:0004def0       _pfr_extra_item_load_font_id 1004eef0 f   freetype:pfr.obj
 0001:0004df50       _pfr_extra_item_load_stem_snaps 1004ef50 f   freetype:pfr.obj
 0001:0004e010       _pfr_extra_item_load_kerning_pairs 1004f010 f   freetype:pfr.obj
 0001:0004e190       _pfr_cmap_init             1004f190 f   freetype:pfr.obj
 0001:0004e1f0       _bdf_cmap_done             1004f1f0 f   freetype:bdf.obj
 0001:0004e1f0       _pcf_cmap_done             1004f1f0 f   freetype:pcf.obj
 0001:0004e1f0       _pfr_cmap_done             1004f1f0 f   freetype:pfr.obj
 0001:0004e210       _pfr_cmap_char_index       1004f210 f   freetype:pfr.obj
 0001:0004e260       _pfr_cmap_char_next        1004f260 f   freetype:pfr.obj
 0001:0004e300       _pfr_get_kerning           1004f300 f   freetype:pfr.obj
 0001:0004e370       _pfr_get_advance           1004f370 f   freetype:pfr.obj
 0001:0004e3b0       _pfr_get_metrics           1004f3b0 f   freetype:pfr.obj
 0001:0004e430       _pfr_get_service           1004f430 f   freetype:pfr.obj
 0001:0004e440       _pfr_aux_name_load         1004f440 f   freetype:pfr.obj
 0001:0004e4e0       _pfr_bitwriter_decode_bytes 1004f4e0 f   freetype:pfr.obj
 0001:0004e5a0       _pfr_bitwriter_decode_rle1 1004f5a0 f   freetype:pfr.obj
 0001:0004e690       _pfr_bitwriter_decode_rle2 1004f690 f   freetype:pfr.obj
 0001:0004e770       _pfr_bitwriter_init        1004f770 f   freetype:pfr.obj
 0001:0004e7c0       _pfr_extra_items_parse     1004f7c0 f   freetype:pfr.obj
 0001:0004e870       _pfr_extra_items_skip      1004f870 f   freetype:pfr.obj
 0001:0004e890       _pfr_glyph_close_contour   1004f890 f   freetype:pfr.obj
 0001:0004e930       _pfr_glyph_curve_to        1004f930 f   freetype:pfr.obj
 0001:0004e9d0       _pfr_glyph_done            1004f9d0 f   freetype:pfr.obj
 0001:0004ea30       _pfr_glyph_end             1004fa30 f   freetype:pfr.obj
 0001:0004ea50       _pfr_glyph_init            1004fa50 f   freetype:pfr.obj
 0001:0004ea80       _pfr_glyph_line_to         1004fa80 f   freetype:pfr.obj
 0001:0004eaf0       _pfr_glyph_load            1004faf0 f   freetype:pfr.obj
 0001:0004eb20       _pfr_glyph_load_compound   1004fb20 f   freetype:pfr.obj
 0001:0004ee00       _pfr_glyph_load_rec        1004fe00 f   freetype:pfr.obj
 0001:0004eff0       _pfr_glyph_load_simple     1004fff0 f   freetype:pfr.obj
 0001:0004f490       $LN215                     10050490     freetype:pfr.obj
 0001:0004f4b0       $LN216                     100504b0     freetype:pfr.obj
 0001:0004f4d0       _pfr_glyph_move_to         100504d0 f   freetype:pfr.obj
 0001:0004f530       _pfr_glyph_start           10050530 f   freetype:pfr.obj
 0001:0004f540       _pfr_header_check          10050540 f   freetype:pfr.obj
 0001:0004f570       _pfr_header_load           10050570 f   freetype:pfr.obj
 0001:0004f5b0       _pfr_load_bitmap_bits      100505b0 f   freetype:pfr.obj
 0001:0004f640       _pfr_load_bitmap_metrics   10050640 f   freetype:pfr.obj
 0001:0004f85c       $LN71                      1005085c     freetype:pfr.obj
 0001:0004f86c       $LN72                      1005086c     freetype:pfr.obj
 0001:0004f87c       $LN73                      1005087c     freetype:pfr.obj
 0001:0004f890       _pfr_log_font_count        10050890 f   freetype:pfr.obj
 0001:0004f8e0       _pfr_log_font_load         100508e0 f   freetype:pfr.obj
 0001:0004fba0       _pfr_lookup_bitmap_data    10050ba0 f   freetype:pfr.obj
 0001:0004fca0       _pfr_phy_font_done         10050ca0 f   freetype:pfr.obj
 0001:0004fda0       _pfr_phy_font_load         10050da0 f   freetype:pfr.obj
 0001:00050280       _pfr_slot_load_bitmap      10051280 f   freetype:pfr.obj
 0001:00050550       _T42_Face_Init             10051550 f   freetype:type42.obj
 0001:0005082c       $LN54                      1005182c     freetype:type42.obj
 0001:00050840       _T42_Face_Done             10051840 f   freetype:type42.obj
 0001:000509e0       _T42_Size_Init             100519e0 f   freetype:type42.obj
 0001:00050a10       _T42_Size_Request          10051a10 f   freetype:type42.obj
 0001:00050a60       _T42_Size_Select           10051a60 f   freetype:type42.obj
 0001:00050ab0       _T42_Size_Done             10051ab0 f   freetype:type42.obj
 0001:00050af0       _T42_GlyphSlot_Init        10051af0 f   freetype:type42.obj
 0001:00050b30       _T42_GlyphSlot_Load        10051b30 f   freetype:type42.obj
 0001:00050c00       _T42_GlyphSlot_Done        10051c00 f   freetype:type42.obj
 0001:00050c20       _T42_Driver_Init           10051c20 f   freetype:type42.obj
 0001:00050c50       _t42_parse_encoding        10051c50 f   freetype:type42.obj
 0001:00050fc0       _t42_parse_charstrings     10051fc0 f   freetype:type42.obj
 0001:00051400       _t42_parse_sfnts           10052400 f   freetype:type42.obj
 0001:00051740       _t42_get_name_index        10052740 f   freetype:type42.obj
 0001:000517c0       _T42_Get_Interface         100527c0 f   freetype:type42.obj
 0001:000517d0       _T42_Open_Face             100527d0 f   freetype:type42.obj
 0001:00051a60       _t42_glyphslot_clear       10052a60 f   freetype:type42.obj
 0001:00051af0       _t42_is_space              10052af0 f   freetype:type42.obj
 0001:00051b20       _t42_load_keyword          10052b20 f   freetype:type42.obj
 0001:00051bb0       _t42_loader_done           10052bb0 f   freetype:type42.obj
 0001:00051c20       _t42_loader_init           10052c20 f   freetype:type42.obj
 0001:00051c40       _t42_parse_dict            10052c40 f   freetype:type42.obj
 0001:00051e70       _t42_parser_done           10052e70 f   freetype:type42.obj
 0001:00051ea0       _t42_parser_init           10052ea0 f   freetype:type42.obj
 0001:00052000       _fnt_cmap_init             10053000 f   freetype:winfnt.obj
 0001:00052030       _fnt_cmap_char_index       10053030 f   freetype:winfnt.obj
 0001:00052050       _fnt_cmap_char_next        10053050 f   freetype:winfnt.obj
 0001:00052090       _FNT_Face_Done             10053090 f   freetype:winfnt.obj
 0001:000520d0       _FNT_Face_Init             100530d0 f   freetype:winfnt.obj
 0001:000523d0       _FNT_Size_Select           100533d0 f   freetype:winfnt.obj
 0001:00052420       _FNT_Size_Request          10053420 f   freetype:winfnt.obj
 0001:000524c0       _FNT_Load_Glyph            100534c0 f   freetype:winfnt.obj
 0001:000526d0       _winfnt_get_header         100536d0 f   freetype:winfnt.obj
 0001:00052700       _winfnt_get_service        10053700 f   freetype:winfnt.obj
 0001:00052710       _fnt_face_get_dll_font     10053710 f   freetype:winfnt.obj
 0001:00052e20       _fnt_font_done             10053e20 f   freetype:winfnt.obj
 0001:00052e80       _fnt_font_load             10053e80 f   freetype:winfnt.obj
 0001:00052f50       _pcf_cmap_init             10053f50 f   freetype:pcf.obj
 0001:00052f70       _pcf_cmap_char_index       10053f70 f   freetype:pcf.obj
 0001:00052fd0       _pcf_cmap_char_next        10053fd0 f   freetype:pcf.obj
 0001:00053060       _PCF_Face_Done             10054060 f   freetype:pcf.obj
 0001:000531c0       _PCF_Face_Init             100541c0 f   freetype:pcf.obj
 0001:00053370       _PCF_Size_Select           10054370 f   freetype:pcf.obj
 0001:000533c0       _PCF_Size_Request          100543c0 f   freetype:pcf.obj
 0001:00053460       _PCF_Glyph_Load            10054460 f   freetype:pcf.obj
 0001:00053644       $LN29                      10054644     freetype:pcf.obj
 0001:00053670       _pcf_get_bdf_property      10054670 f   freetype:pcf.obj
 0001:000536b0       _pcf_get_charset_id        100546b0 f   freetype:pcf.obj
 0001:000536d0       _pcf_driver_requester      100546d0 f   freetype:pcf.obj
 0001:000536e0       _BitOrderInvert            100546e0 f   freetype:pcf.obj
 0001:00053730       _FourByteSwap              10054730 f   freetype:pcf.obj
 0001:00053770       _TwoByteSwap               10054770 f   freetype:pcf.obj
 0001:000537a0       _pcf_find_property         100547a0 f   freetype:pcf.obj
 0001:00053830       _pcf_get_accel             10054830 f   freetype:pcf.obj
 0001:00053950       _pcf_get_bitmaps           10054950 f   freetype:pcf.obj
 0001:00053b00       _pcf_get_encodings         10054b00 f   freetype:pcf.obj
 0001:00053d50       _pcf_get_metric            10054d50 f   freetype:pcf.obj
 0001:00053df0       _pcf_get_metrics           10054df0 f   freetype:pcf.obj
 0001:00053f90       _pcf_get_properties        10054f90 f   freetype:pcf.obj
 0001:00054250       _pcf_has_table_type        10055250 f   freetype:pcf.obj
 0001:00054280       _pcf_interpret_style       10055280 f   freetype:pcf.obj
 0001:000544e0       _pcf_load_font             100554e0 f   freetype:pcf.obj
 0001:00054810       _pcf_read_TOC              10055810 f   freetype:pcf.obj
 0001:000549b0       _pcf_seek_to_table_type    100559b0 f   freetype:pcf.obj
 0001:00054a40       _ps_table_new              10055a40 f   freetype:psaux.obj
 0001:00054ad0       _ps_table_add              10055ad0 f   freetype:psaux.obj
 0001:00054b80       _ps_table_done             10055b80 f   freetype:psaux.obj
 0001:00054bd0       _ps_table_release          10055bd0 f   freetype:psaux.obj
 0001:00054c20       _ps_parser_skip_spaces     10055c20 f   freetype:psaux.obj
 0001:00054c40       _ps_parser_skip_PS_token   10055c40 f   freetype:psaux.obj
 0001:00054d70       _ps_parser_to_token        10055d70 f   freetype:psaux.obj
 0001:00054ea0       _ps_parser_to_token_array  10055ea0 f   freetype:psaux.obj
 0001:00054f60       _ps_parser_load_field      10055f60 f   freetype:psaux.obj
 0001:00055308       $LN84                      10056308     freetype:psaux.obj
 0001:00055330       _ps_parser_load_field_table 10056330 f   freetype:psaux.obj
 0001:00055470       _ps_parser_to_int          10056470 f   freetype:psaux.obj
 0001:00055490       _ps_parser_to_bytes        10056490 f   freetype:psaux.obj
 0001:00055520       _ps_parser_to_fixed        10056520 f   freetype:psaux.obj
 0001:00055540       _ps_parser_to_coord_array  10056540 f   freetype:psaux.obj
 0001:00055570       _ps_parser_to_fixed_array  10056570 f   freetype:psaux.obj
 0001:000555a0       _ps_parser_init            100565a0 f   freetype:psaux.obj
 0001:000555f0       _t1_builder_init           100565f0 f   freetype:psaux.obj
 0001:000556a0       _t1_builder_add_point      100566a0 f   freetype:psaux.obj
 0001:00055700       _t1_builder_add_point1     10056700 f   freetype:psaux.obj
 0001:00055730       _t1_builder_add_contour    10056730 f   freetype:psaux.obj
 0001:000557b0       _t1_builder_start_point    100567b0 f   freetype:psaux.obj
 0001:000557f0       _t1_decrypt                100567f0 f   freetype:psaux.obj
 0001:00055810       _t1_decoder_parse_charstrings 10056810 f   freetype:psaux.obj
 0001:00056618       $LN422                     10057618     freetype:psaux.obj
 0001:00056668       $LN421                     10057668     freetype:psaux.obj
 0001:00056768       $LN424                     10057768     freetype:psaux.obj
 0001:00056790       $LN423                     10057790     freetype:psaux.obj
 0001:000567b4       $LN426                     100577b4     freetype:psaux.obj
 0001:000567bc       $LN425                     100577bc     freetype:psaux.obj
 0001:000567d8       $LN428                     100577d8     freetype:psaux.obj
 0001:00056818       $LN427                     10057818     freetype:psaux.obj
 0001:00056838       $LN429                     10057838     freetype:psaux.obj
 0001:000568a0       _t1_decoder_init           100578a0 f   freetype:psaux.obj
 0001:00056940       _t1_decoder_done           10057940 f   freetype:psaux.obj
 0001:00056950       _afm_parser_init           10057950 f   freetype:psaux.obj
 0001:000569b0       _afm_parser_done           100579b0 f   freetype:psaux.obj
 0001:000569d0       _afm_parser_parse          100579d0 f   freetype:psaux.obj
 0001:00056c48       $LN57                      10057c48     freetype:psaux.obj
 0001:00056c6c       $LN56                      10057c6c     freetype:psaux.obj
 0001:00056ca0       _t1_cmap_std_done          10057ca0 f   freetype:psaux.obj
 0001:00056cd0       _t1_cmap_std_char_index    10057cd0 f   freetype:psaux.obj
 0001:00056d60       _t1_cmap_std_char_next     10057d60 f   freetype:psaux.obj
 0001:00056db0       _t1_cmap_standard_init     10057db0 f   freetype:psaux.obj
 0001:00056dd0       _t1_cmap_expert_init       10057dd0 f   freetype:psaux.obj
 0001:00056df0       _t1_cmap_custom_init       10057df0 f   freetype:psaux.obj
 0001:00056e20       _t1_cmap_custom_done       10057e20 f   freetype:psaux.obj
 0001:00056e40       _t1_cmap_custom_char_index 10057e40 f   freetype:psaux.obj
 0001:00056e70       _t1_cmap_custom_char_next  10057e70 f   freetype:psaux.obj
 0001:00056ed0       _t1_cmap_unicode_init      10057ed0 f   freetype:psaux.obj
 0001:00056f00       _t1_cmap_unicode_char_index 10057f00 f   freetype:psaux.obj
 0001:00056f20       _t1_cmap_unicode_char_next 10057f20 f   freetype:psaux.obj
 0001:00056f40       _PS_Conv_ASCIIHexDecode    10057f40 f   freetype:psaux.obj
 0001:00056ff0       _PS_Conv_EexecDecode       10057ff0 f   freetype:psaux.obj
 0001:00057080       _PS_Conv_Strtol            10058080 f   freetype:psaux.obj
 0001:00057170       _PS_Conv_ToFixed           10058170 f   freetype:psaux.obj
 0001:000573d0       _PS_Conv_ToInt             100583d0 f   freetype:psaux.obj
 0001:00057430       _afm_parse_kern_data       10058430 f   freetype:psaux.obj
 0001:000574ac       $LN23                      100584ac     freetype:psaux.obj
 0001:000574c0       $LN22                      100584c0     freetype:psaux.obj
 0001:00057500       _afm_parse_kern_pairs      10058500 f   freetype:psaux.obj
 0001:000576a0       $LN34                      100586a0     freetype:psaux.obj
 0001:000576b0       $LN33                      100586b0     freetype:psaux.obj
 0001:000576f0       _afm_parse_track_kern      100586f0 f   freetype:psaux.obj
 0001:0005784c       $LN38                      1005884c     freetype:psaux.obj
 0001:0005785c       $LN37                      1005885c     freetype:psaux.obj
 0001:000578a0       _afm_parser_next_key       100588a0 f   freetype:psaux.obj
 0001:00057940       _afm_parser_read_int       10058940 f   freetype:psaux.obj
 0001:00057980       _afm_parser_read_vals      10058980 f   freetype:psaux.obj
 0001:00057aa4       $LN28                      10058aa4     freetype:psaux.obj
 0001:00057ac0       _afm_parser_skip_section   10058ac0 f   freetype:psaux.obj
 0001:00057b40       _afm_stream_read_one       10058b40 f   freetype:psaux.obj
 0001:00057bc0       _afm_stream_read_string    10058bc0 f   freetype:psaux.obj
 0001:00057c20       _afm_stream_skip_spaces    10058c20 f   freetype:psaux.obj
 0001:00057ca0       _afm_tokenize              10058ca0 f   freetype:psaux.obj
 0001:00057d00       _ps_tobool                 10058d00 f   freetype:psaux.obj
 0001:00057d70       _ps_tocoordarray           10058d70 f   freetype:psaux.obj
 0001:00057e50       _ps_tofixedarray           10058e50 f   freetype:psaux.obj
 0001:00057f30       _psaux_get_glyph_name      10058f30 f   freetype:psaux.obj
 0001:00057f50       _reallocate_t1_table       10058f50 f   freetype:psaux.obj
 0001:00057fc0       _shift_elements            10058fc0 f   freetype:psaux.obj
 0001:00058000       _skip_comment              10059000 f   freetype:psaux.obj
 0001:00058030       _skip_literal_string       10059030 f   freetype:psaux.obj
 0001:000580b8       $LN41                      100590b8     freetype:psaux.obj
 0001:000580c0       $LN40                      100590c0     freetype:psaux.obj
 0001:00058110       _skip_procedure            10059110 f   freetype:psaux.obj
 0001:000581b8       $LN25                      100591b8     freetype:psaux.obj
 0001:000581d0       $LN24                      100591d0     freetype:psaux.obj
 0001:00058230       _skip_spaces               10059230 f   freetype:psaux.obj
 0001:00058280       _skip_string               10059280 f   freetype:psaux.obj
 0001:000582f0       _t1_cmap_std_init          100592f0 f   freetype:psaux.obj
 0001:00058330       _t1_decoder_parse_glyph    10059330 f   freetype:psaux.obj
 0001:00058350       _t1_lookup_glyph_by_stdcharcode 10059350 f   freetype:psaux.obj
 0001:000583f0       _t1operator_seac           100593f0 f   freetype:psaux.obj
 0001:000585b0       _ps_unicode_value          100595b0 f   freetype:psmodule.obj
 0001:000586b0       _ps_unicodes_init          100596b0 f   freetype:psmodule.obj
 0001:00058990       _ps_unicodes_char_index    10059990 f   freetype:psmodule.obj
 0001:00058a00       _ps_unicodes_char_next     10059a00 f   freetype:psmodule.obj
 0001:00058ab0       _ps_get_macintosh_name     10059ab0 f   freetype:psmodule.obj
 0001:00058ad0       _ps_get_standard_strings   10059ad0 f   freetype:psmodule.obj
 0001:00058af0       _psnames_get_service       10059af0 f   freetype:psmodule.obj
 0001:00058b00       _compare_uni_maps          10059b00 f   freetype:psmodule.obj
 0001:00058b50       _ft_get_adobe_glyph_index  10059b50 f   freetype:psmodule.obj
 0001:00058c30       _ps_check_extra_glyph_name 10059c30 f   freetype:psmodule.obj
 0001:00058cb0       _ps_check_extra_glyph_unicode 10059cb0 f   freetype:psmodule.obj
 0001:00058cf0       _ps_hinter_done            10059cf0 f   freetype:pshinter.obj
 0001:00058d20       _ps_hinter_init            10059d20 f   freetype:pshinter.obj
 0001:00058d60       _pshinter_get_globals_funcs 10059d60 f   freetype:pshinter.obj
 0001:00058d70       _pshinter_get_t1_funcs     10059d70 f   freetype:pshinter.obj
 0001:00058d80       _pshinter_get_t2_funcs     10059d80 f   freetype:pshinter.obj
 0001:00058d90       _ps_dimension_add_counter  10059d90 f   freetype:pshinter.obj
 0001:00058e50       _ps_dimension_add_t1stem   10059e50 f   freetype:pshinter.obj
 0001:00058f50       _ps_dimension_done         10059f50 f   freetype:pshinter.obj
 0001:00058f80       _ps_dimension_end          10059f80 f   freetype:pshinter.obj
 0001:00058fb0       _ps_dimension_end_mask     10059fb0 f   freetype:pshinter.obj
 0001:00058fd0       _ps_dimension_init         10059fd0 f   freetype:pshinter.obj
 0001:00058ff0       _ps_dimension_reset_mask   10059ff0 f   freetype:pshinter.obj
 0001:00059020       _ps_dimension_set_mask_bits 1005a020 f   freetype:pshinter.obj
 0001:00059060       _ps_hint_table_alloc       1005a060 f   freetype:pshinter.obj
 0001:000590d0       _ps_hint_table_done        1005a0d0 f   freetype:pshinter.obj
 0001:00059100       _ps_hint_table_ensure      1005a100 f   freetype:pshinter.obj
 0001:000593a0       _ps_hints_close            1005a3a0 f   freetype:pshinter.obj
 0001:000593e0       _ps_hints_done             1005a3e0 f   freetype:pshinter.obj
 0001:00059420       _ps_hints_init             1005a420 f   freetype:pshinter.obj
 0001:00059450       _ps_hints_open             1005a450 f   freetype:pshinter.obj
 0001:000594a0       _ps_hints_stem             1005a4a0 f   freetype:pshinter.obj
 0001:00059520       _ps_hints_t1reset          1005a520 f   freetype:pshinter.obj
 0001:00059580       _ps_hints_t1stem3          1005a580 f   freetype:pshinter.obj
 0001:00059670       _ps_hints_t2counter        1005a670 f   freetype:pshinter.obj
 0001:000596e0       _ps_hints_t2mask           1005a6e0 f   freetype:pshinter.obj
 0001:00059740       _ps_mask_clear_bit         1005a740 f   freetype:pshinter.obj
 0001:00059770       _ps_mask_done              1005a770 f   freetype:pshinter.obj
 0001:000597b0       _ps_mask_ensure            1005a7b0 f   freetype:pshinter.obj
 0001:00059810       _ps_mask_set_bit           1005a810 f   freetype:pshinter.obj
 0001:00059870       _ps_mask_table_alloc       1005a870 f   freetype:pshinter.obj
 0001:000598d0       _ps_mask_table_done        1005a8d0 f   freetype:pshinter.obj
 0001:00059920       _ps_mask_table_ensure      1005a920 f   freetype:pshinter.obj
 0001:00059970       _ps_mask_table_last        1005a970 f   freetype:pshinter.obj
 0001:000599b0       _ps_mask_table_merge       1005a9b0 f   freetype:pshinter.obj
 0001:00059aa0       _ps_mask_table_merge_all   1005aaa0 f   freetype:pshinter.obj
 0001:00059b00       _ps_mask_table_set_bits    1005ab00 f   freetype:pshinter.obj
 0001:00059be0       _ps_mask_table_test_intersect 1005abe0 f   freetype:pshinter.obj
 0001:00059c50       _ps_mask_test_bit          1005ac50 f   freetype:pshinter.obj
 0001:00059c80       _psh_blues_scale_zones     1005ac80 f   freetype:pshinter.obj
 0001:00059f20       _psh_blues_set_zones       1005af20 f   freetype:pshinter.obj
 0001:0005a080       _psh_blues_set_zones_0     1005b080 f   freetype:pshinter.obj
 0001:0005a180       _psh_blues_snap_stem       1005b180 f   freetype:pshinter.obj
 0001:0005a260       _psh_calc_max_height       1005b260 f   freetype:pshinter.obj
 0001:0005a2b0       _psh_compute_dir           1005b2b0 f   freetype:pshinter.obj
 0001:0005a310       _psh_dimension_quantize_len 1005b310 f   freetype:pshinter.obj
 0001:0005a3a0       _psh_globals_destroy       1005b3a0 f   freetype:pshinter.obj
 0001:0005a3f0       _psh_globals_funcs_init    1005b3f0 f   freetype:pshinter.obj
 0001:0005a410       _psh_globals_new           1005b410 f   freetype:pshinter.obj
 0001:0005a5c0       _psh_globals_scale_widths  1005b5c0 f   freetype:pshinter.obj
 0001:0005a690       _psh_globals_set_scale     1005b690 f   freetype:pshinter.obj
 0001:0005a710       _psh_glyph_compute_extrema 1005b710 f   freetype:pshinter.obj
 0001:0005a820       _psh_glyph_compute_inflections 1005b820 f   freetype:pshinter.obj
 0001:0005a970       _psh_glyph_done            1005b970 f   freetype:pshinter.obj
 0001:0005a9d0       _psh_glyph_find_blue_points 1005b9d0 f   freetype:pshinter.obj
 0001:0005aae0       _psh_glyph_find_strong_points 1005bae0 f   freetype:pshinter.obj
 0001:0005ac10       _psh_glyph_init            1005bc10 f   freetype:pshinter.obj
 0001:0005ae70       _psh_glyph_interpolate_normal_points 1005be70 f   freetype:pshinter.obj
 0001:0005b0e0       _psh_glyph_interpolate_other_points 1005c0e0 f   freetype:pshinter.obj
 0001:0005b320       _psh_glyph_interpolate_strong_points 1005c320 f   freetype:pshinter.obj
 0001:0005b420       _psh_glyph_load_points     1005c420 f   freetype:pshinter.obj
 0001:0005b4a0       _psh_glyph_save_points     1005c4a0 f   freetype:pshinter.obj
 0001:0005b510       _psh_hint_align            1005c510 f   freetype:pshinter.obj
 0001:0005b820       _psh_hint_overlap          1005c820 f   freetype:pshinter.obj
 0001:0005b850       _psh_hint_snap_stem_side_delta 1005c850 f   freetype:pshinter.obj
 0001:0005b890       _psh_hint_table_activate_mask 1005c890 f   freetype:pshinter.obj
 0001:0005b980       _psh_hint_table_align_hints 1005c980 f   freetype:pshinter.obj
 0001:0005b9c0       _psh_hint_table_deactivate 1005c9c0 f   freetype:pshinter.obj
 0001:0005b9f0       _psh_hint_table_done       1005c9f0 f   freetype:pshinter.obj
 0001:0005ba60       _psh_hint_table_find_strong_points 1005ca60 f   freetype:pshinter.obj
 0001:0005bc40       _psh_hint_table_init       1005cc40 f   freetype:pshinter.obj
 0001:0005bd60       _psh_hint_table_record     1005cd60 f   freetype:pshinter.obj
 0001:0005bde0       _psh_hint_table_record_mask 1005cde0 f   freetype:pshinter.obj
 0001:0005be40       _t1_hints_funcs_init       1005ce40 f   freetype:pshinter.obj
 0001:0005be80       _t1_hints_open             1005ce80 f   freetype:pshinter.obj
 0001:0005bea0       _t1_hints_stem             1005cea0 f   freetype:pshinter.obj
 0001:0005bee0       _t2_hints_funcs_init       1005cee0 f   freetype:pshinter.obj
 0001:0005bf20       _t2_hints_open             1005cf20 f   freetype:pshinter.obj
 0001:0005bf40       _t2_hints_stems            1005cf40 f   freetype:pshinter.obj
 0001:0005c030       _ft_black_new              1005d030 f   freetype:raster.obj
 0001:0005c070       _ft_black_done             1005d070 f   freetype:raster.obj
 0001:0005c090       _ft_black_reset            1005d090 f   freetype:raster.obj
 0001:0005c0e0       _ft_black_render           1005d0e0 f   freetype:raster.obj
 0001:0005c200       _ft_raster1_init           1005d200 f   freetype:raster.obj
 0001:0005c200       _ft_smooth_init            1005d200 f   freetype:smooth.obj
 0001:0005c230       _ft_raster1_set_mode       1005d230 f   freetype:raster.obj
 0001:0005c230       _ft_smooth_set_mode        1005d230 f   freetype:smooth.obj
 0001:0005c250       _ft_raster1_transform      1005d250 f   freetype:raster.obj
 0001:0005c250       _ft_smooth_transform       1005d250 f   freetype:smooth.obj
 0001:0005c2a0       _ft_raster1_get_cbox       1005d2a0 f   freetype:raster.obj
 0001:0005c2a0       _ft_smooth_get_cbox        1005d2a0 f   freetype:smooth.obj
 0001:0005c2d0       _ft_raster1_render         1005d2d0 f   freetype:raster.obj
 0001:0005c4e0       _Bezier_Down               1005d4e0 f   freetype:raster.obj
 0001:0005c560       _Bezier_Up                 1005d560 f   freetype:raster.obj
 0001:0005c700       _Conic_To                  1005d700 f   freetype:raster.obj
 0001:0005c840       _Convert_Glyph             1005d840 f   freetype:raster.obj
 0001:0005c990       _Cubic_To                  1005d990 f   freetype:raster.obj
 0001:0005cb00       _Decompose_Curve           1005db00 f   freetype:raster.obj
 0001:0005ce60       _DelOld                    1005de60 f   freetype:raster.obj
 0001:0005ce90       _Draw_Sweep                1005de90 f   freetype:raster.obj
 0001:0005d1e0       _End_Profile               1005e1e0 f   freetype:raster.obj
 0001:0005d270       _Finalize_Profile_Table    1005e270 f   freetype:raster.obj
 0001:0005d330       _Horizontal_Sweep_Drop     1005e330 f   freetype:raster.obj
 0001:0005d4d0       $LN29                      1005e4d0     freetype:raster.obj
 0001:0005d4f0       _Horizontal_Sweep_Span     1005e4f0 f   freetype:raster.obj
 0001:0005d560       _Init_Linked               1005e560 f   freetype:raster.obj
 0001:0005d570       _InsNew                    1005e570 f   freetype:raster.obj
 0001:0005d5a0       _Insert_Y_Turn             1005e5a0 f   freetype:raster.obj
 0001:0005d620       _Line_Down                 1005e620 f   freetype:raster.obj
 0001:0005d670       _Line_To                   1005e670 f   freetype:raster.obj
 0001:0005d7c0       _Line_Up                   1005e7c0 f   freetype:raster.obj
 0001:0005d970       _New_Profile               1005e970 f   freetype:raster.obj
 0001:0005da50       _Render_Glyph              1005ea50 f   freetype:raster.obj
 0001:0005db80       _Render_Gray_Glyph         1005eb80 f   freetype:raster.obj
 0001:0005db90       _Render_Single_Pass        1005eb90 f   freetype:raster.obj
 0001:0005dcd0       _Set_High_Precision        1005ecd0 f   freetype:raster.obj
 0001:0005dd30       _Sort                      1005ed30 f   freetype:raster.obj
 0001:0005ddb0       _Split_Conic               1005edb0 f   freetype:raster.obj
 0001:0005ddb0       _gray_split_conic          1005edb0 f   freetype:smooth.obj
 0001:0005de20       _Split_Cubic               1005ee20 f   freetype:raster.obj
 0001:0005deb0       _Vertical_Sweep_Drop       1005eeb0 f   freetype:raster.obj
 0001:0005e050       $LN28                      1005f050     freetype:raster.obj
 0001:0005e070       _Vertical_Sweep_Init       1005f070 f   freetype:raster.obj
 0001:0005e0c0       _Vertical_Sweep_Span       1005f0c0 f   freetype:raster.obj
 0001:0005e1c0       _Vertical_Sweep_Step       1005f1c0 f   freetype:raster.obj
 0001:0005e1e0       _tt_cmap13_char_index      1005f1e0 f   freetype:sfnt.obj
 0001:0005e200       _tt_cmap13_char_next       1005f200 f   freetype:sfnt.obj
 0001:0005e260       _tt_cmap13_get_info        1005f260 f   freetype:sfnt.obj
 0001:0005e2a0       _tt_cmap14_done            1005f2a0 f   freetype:sfnt.obj
 0001:0005e2d0       _tt_cmap14_init            1005f2d0 f   freetype:sfnt.obj
 0001:0005e320       _tt_cmap14_validate        1005f320 f   freetype:sfnt.obj
 0001:0005e5f0       _tt_cmap14_char_next       1005f5f0 f   freetype:sfnt.obj
 0001:0005e600       _tt_cmap14_get_info        1005f600 f   freetype:sfnt.obj
 0001:0005e620       _tt_cmap14_char_var_index  1005f620 f   freetype:sfnt.obj
 0001:0005e6d0       _tt_cmap14_char_var_isdefault 1005f6d0 f   freetype:sfnt.obj
 0001:0005e780       _tt_cmap14_variants        1005f780 f   freetype:sfnt.obj
 0001:0005e7f0       _tt_cmap14_char_variants   1005f7f0 f   freetype:sfnt.obj
 0001:0005e8f0       _tt_cmap14_variant_chars   1005f8f0 f   freetype:sfnt.obj
 0001:0005ebf0       _tt_face_load_kern         1005fbf0 f   freetype:sfnt.obj
 0001:0005edf0       _tt_face_get_kerning       1005fdf0 f   freetype:sfnt.obj
 0001:0005efb0       _sfnt_init_face            1005ffb0 f   freetype:sfnt.obj
 0001:0005f070       _sfnt_load_face            10060070 f   freetype:sfnt.obj
 0001:0005f820       _sfnt_done_face            10060820 f   freetype:sfnt.obj
 0001:0005f9d0       _tt_face_find_bdf_prop     100609d0 f   freetype:sfnt.obj
 0001:0005fbc8       $LN37                      10060bc8     freetype:sfnt.obj
 0001:0005fbe0       _tt_face_load_sbit         10060be0 f   freetype:sfnt.obj
 0001:0005fe90       _tt_face_free_sbit         10060e90 f   freetype:sfnt.obj
 0001:0005fed0       _tt_face_set_sbit_strike   10060ed0 f   freetype:sfnt.obj
 0001:0005fef0       _tt_face_load_strike_metrics 10060ef0 f   freetype:sfnt.obj
 0001:000600c0       _tt_face_load_sbit_image   100610c0 f   freetype:sfnt.obj
 0001:000601d0       _tt_face_get_ps_name       100611d0 f   freetype:sfnt.obj
 0001:00060300       _tt_face_free_ps_names     10061300 f   freetype:sfnt.obj
 0001:00060400       _get_sfnt_table            10061400 f   freetype:sfnt.obj
 0001:00060480       $LN19                      10061480     freetype:sfnt.obj
 0001:000604a0       _sfnt_table_info           100614a0 f   freetype:sfnt.obj
 0001:00060510       _sfnt_get_glyph_name       10061510 f   freetype:sfnt.obj
 0001:00060550       _sfnt_get_name_index       10061550 f   freetype:sfnt.obj
 0001:000605d0       _sfnt_get_ps_name          100615d0 f   freetype:sfnt.obj
 0001:00060830       _sfnt_get_charset_id       10061830 f   freetype:sfnt.obj
 0001:000608a0       _sfnt_get_interface        100618a0 f   freetype:sfnt.obj
 0001:000608b0       _tt_face_goto_table        100618b0 f   freetype:sfnt.obj
 0001:000608f0       _tt_face_load_font_dir     100618f0 f   freetype:sfnt.obj
 0001:00060a60       _tt_face_load_any          10061a60 f   freetype:sfnt.obj
 0001:00060ac0       _tt_face_load_head         10061ac0 f   freetype:sfnt.obj
 0001:00060ae0       _tt_face_load_cmap         10061ae0 f   freetype:sfnt.obj
 0001:00060b30       _tt_face_load_maxp         10061b30 f   freetype:sfnt.obj
 0001:00060be0       _tt_face_load_name         10061be0 f   freetype:sfnt.obj
 0001:00060d60       _tt_face_load_os2          10061d60 f   freetype:sfnt.obj
 0001:00060e10       _tt_face_load_post         10061e10 f   freetype:sfnt.obj
 0001:00060e50       _tt_face_load_pclt         10061e50 f   freetype:sfnt.obj
 0001:00060e90       _tt_face_free_name         10061e90 f   freetype:sfnt.obj
 0001:00060f20       _tt_face_load_gasp         10061f20 f   freetype:sfnt.obj
 0001:00061040       _tt_face_load_bhed         10062040 f   freetype:sfnt.obj
 0001:00061060       _tt_face_load_hhea         10062060 f   freetype:sfnt.obj
 0001:000610d0       _tt_face_load_hmtx         100620d0 f   freetype:sfnt.obj
 0001:00061140       _tt_face_get_metrics       10062140 f   freetype:sfnt.obj
 0001:00061280       _tt_get_cmap_info          10062280 f   freetype:sfnt.obj
 0001:000612a0       _tt_cmap_init              100622a0 f   freetype:sfnt.obj
 0001:000612b0       _tt_cmap0_validate         100622b0 f   freetype:sfnt.obj
 0001:00061330       _tt_cmap0_char_index       10062330 f   freetype:sfnt.obj
 0001:00061350       _tt_cmap0_char_next        10062350 f   freetype:sfnt.obj
 0001:00061390       _tt_cmap0_get_info         10062390 f   freetype:sfnt.obj
 0001:000613c0       _tt_cmap2_validate         100623c0 f   freetype:sfnt.obj
 0001:00061580       _tt_cmap2_char_index       10062580 f   freetype:sfnt.obj
 0001:00061620       _tt_cmap2_char_next        10062620 f   freetype:sfnt.obj
 0001:00061750       _tt_cmap2_get_info         10062750 f   freetype:sfnt.obj
 0001:00061780       _tt_cmap4_init             10062780 f   freetype:sfnt.obj
 0001:000617c0       _tt_cmap4_validate         100627c0 f   freetype:sfnt.obj
 0001:00061b40       _tt_cmap4_char_index       10062b40 f   freetype:sfnt.obj
 0001:00061b80       _tt_cmap4_char_next        10062b80 f   freetype:sfnt.obj
 0001:00061bf0       _tt_cmap4_get_info         10062bf0 f   freetype:sfnt.obj
 0001:00061c20       _tt_cmap6_validate         10062c20 f   freetype:sfnt.obj
 0001:00061cc0       _tt_cmap6_char_index       10062cc0 f   freetype:sfnt.obj
 0001:00061d10       _tt_cmap6_char_next        10062d10 f   freetype:sfnt.obj
 0001:00061db0       _tt_cmap6_get_info         10062db0 f   freetype:sfnt.obj
 0001:00061de0       _tt_cmap8_validate         10062de0 f   freetype:sfnt.obj
 0001:00062040       _tt_cmap8_char_index       10063040 f   freetype:sfnt.obj
 0001:00062120       _tt_cmap8_char_next        10063120 f   freetype:sfnt.obj
 0001:00062230       _tt_cmap8_get_info         10063230 f   freetype:sfnt.obj
 0001:00062270       _tt_cmap10_validate        10063270 f   freetype:sfnt.obj
 0001:00062330       _tt_cmap10_char_index      10063330 f   freetype:sfnt.obj
 0001:000623a0       _tt_cmap10_char_next       100633a0 f   freetype:sfnt.obj
 0001:00062440       _tt_cmap10_get_info        10063440 f   freetype:sfnt.obj
 0001:00062480       _tt_cmap12_init            10063480 f   freetype:sfnt.obj
 0001:00062480       _tt_cmap13_init            10063480 f   freetype:sfnt.obj
 0001:000624c0       _tt_cmap12_validate        100634c0 f   freetype:sfnt.obj
 0001:00062630       _tt_cmap12_char_index      10063630 f   freetype:sfnt.obj
 0001:00062650       _tt_cmap12_char_next       10063650 f   freetype:sfnt.obj
 0001:000626b0       _tt_cmap12_get_info        100636b0 f   freetype:sfnt.obj
 0001:000626f0       _tt_cmap13_validate        100636f0 f   freetype:sfnt.obj
 0001:00062860       _check_table_dir           10063860 f   freetype:sfnt.obj
 0001:000629e0       _compare_offsets           100639e0 f   freetype:sfnt.obj
 0001:00062a00       _load_format_20            10063a00 f   freetype:sfnt.obj
 0001:00062cb0       _load_format_25            10063cb0 f   freetype:sfnt.obj
 0001:00062d90       _load_post_names           10063d90 f   freetype:sfnt.obj
 0001:00062e30       _sfnt_find_encoding        10063e30 f   freetype:sfnt.obj
 0001:00062e70       _sfnt_open_font            10063e70 f   freetype:sfnt.obj
 0001:00063070       _tt_cmap12_char_map_binary 10064070 f   freetype:sfnt.obj
 0001:000631f0       _tt_cmap12_next            100641f0 f   freetype:sfnt.obj
 0001:000632e0       _tt_cmap13_char_map_binary 100642e0 f   freetype:sfnt.obj
 0001:00063450       _tt_cmap13_next            10064450 f   freetype:sfnt.obj
 0001:00063520       _tt_cmap14_char_map_def_binary 10064520 f   freetype:sfnt.obj
 0001:000635b0       _tt_cmap14_char_map_nondef_binary 100645b0 f   freetype:sfnt.obj
 0001:00063630       _tt_cmap14_def_char_count  10064630 f   freetype:sfnt.obj
 0001:00063680       _tt_cmap14_ensure          10064680 f   freetype:sfnt.obj
 0001:000636d0       _tt_cmap14_find_variant    100646d0 f   freetype:sfnt.obj
 0001:00063750       _tt_cmap14_get_def_chars   10064750 f   freetype:sfnt.obj
 0001:000637f0       _tt_cmap14_get_nondef_chars 100647f0 f   freetype:sfnt.obj
 0001:00063880       _tt_cmap2_get_subheader    10064880 f   freetype:sfnt.obj
 0001:000638f0       _tt_cmap4_char_map_binary  100648f0 f   freetype:sfnt.obj
 0001:00063d50       _tt_cmap4_char_map_linear  10064d50 f   freetype:sfnt.obj
 0001:00063f50       _tt_cmap4_next             10064f50 f   freetype:sfnt.obj
 0001:00064000       _tt_cmap4_set_range        10065000 f   freetype:sfnt.obj
 0001:00064140       _tt_face_build_cmaps       10065140 f   freetype:sfnt.obj
 0001:000643c0       _tt_face_done_kern         100653c0 f   freetype:sfnt.obj
 0001:00064410       _tt_face_free_bdf_props    10065410 f   freetype:sfnt.obj
 0001:00064450       _tt_face_get_name          10065450 f   freetype:sfnt.obj
 0001:00064680       $LN55                      10065680     freetype:sfnt.obj
 0001:00064690       _tt_face_load_bdf_props    10065690 f   freetype:sfnt.obj
 0001:00064860       _tt_face_load_generic_header 10065860 f   freetype:sfnt.obj
 0001:000648a0       _tt_face_load_sbix_image   100658a0 f   freetype:sfnt.obj
 0001:00064ac0       _tt_face_lookup_table      10065ac0 f   freetype:sfnt.obj
 0001:00064b00       _tt_name_entry_ascii_from_other 10065b00 f   freetype:sfnt.obj
 0001:00064b70       _tt_name_entry_ascii_from_utf16 10065b70 f   freetype:sfnt.obj
 0001:00064bf0       _tt_sbit_decoder_alloc_bitmap 10065bf0 f   freetype:sfnt.obj
 0001:00064cac       $LN15                      10065cac     freetype:sfnt.obj
 0001:00064cc4       $LN14                      10065cc4     freetype:sfnt.obj
 0001:00064cf0       _tt_sbit_decoder_init      10065cf0 f   freetype:sfnt.obj
 0001:00064e50       _tt_sbit_decoder_load_bit_aligned 10065e50 f   freetype:sfnt.obj
 0001:00065090       _tt_sbit_decoder_load_bitmap 10066090 f   freetype:sfnt.obj
 0001:000651f8       $LN38                      100661f8     freetype:sfnt.obj
 0001:00065204       $LN37                      10066204     freetype:sfnt.obj
 0001:00065218       $LN40                      10066218     freetype:sfnt.obj
 0001:00065234       $LN39                      10066234     freetype:sfnt.obj
 0001:00065250       _tt_sbit_decoder_load_byte_aligned 10066250 f   freetype:sfnt.obj
 0001:000653e0       _tt_sbit_decoder_load_compound 100663e0 f   freetype:sfnt.obj
 0001:00065510       _tt_sbit_decoder_load_image 10066510 f   freetype:sfnt.obj
 0001:000658b8       $LN63                      100668b8     freetype:sfnt.obj
 0001:000658d0       $LN62                      100668d0     freetype:sfnt.obj
 0001:000658f0       _tt_sbit_decoder_load_metrics 100668f0 f   freetype:sfnt.obj
 0001:00065970       _woff_open_font            10066970 f   freetype:sfnt.obj
 0001:00065ed0       _gray_move_to              10066ed0 f   freetype:smooth.obj
 0001:00065f20       _gray_line_to              10066f20 f   freetype:smooth.obj
 0001:00065f50       _gray_conic_to             10066f50 f   freetype:smooth.obj
 0001:00065f70       _gray_cubic_to             10066f70 f   freetype:smooth.obj
 0001:00065f90       _gray_raster_render        10066f90 f   freetype:smooth.obj
 0001:00066180       _gray_raster_new           10067180 f   freetype:smooth.obj
 0001:000661c0       _gray_raster_done          100671c0 f   freetype:smooth.obj
 0001:000661e0       _gray_raster_reset         100671e0 f   freetype:smooth.obj
 0001:00066230       _ft_smooth_render          10067230 f   freetype:smooth.obj
 0001:00066260       _ft_smooth_render_lcd      10067260 f   freetype:smooth.obj
 0001:00066290       _ft_smooth_render_lcd_v    10067290 f   freetype:smooth.obj
 0001:000662c0       _ft_smooth_render_generic  100672c0 f   freetype:smooth.obj
 0001:00066630       _gray_compute_cbox         10067630 f   freetype:smooth.obj
 0001:00066710       _gray_convert_glyph        10067710 f   freetype:smooth.obj
 0001:00066aa0       _gray_convert_glyph_inner  10067aa0 f   freetype:smooth.obj
 0001:00066b10       _gray_find_cell            10067b10 f   freetype:smooth.obj
 0001:00066b80       _gray_hline                10067b80 f   freetype:smooth.obj
 0001:00066cb0       _gray_init_cells           10067cb0 f   freetype:smooth.obj
 0001:00066d00       _gray_record_cell          10067d00 f   freetype:smooth.obj
 0001:00066d30       _gray_render_conic         10067d30 f   freetype:smooth.obj
 0001:00066e70       _gray_render_cubic         10067e70 f   freetype:smooth.obj
 0001:00067040       _gray_render_line          10068040 f   freetype:smooth.obj
 0001:000672d0       _gray_render_scanline      100682d0 f   freetype:smooth.obj
 0001:00067470       _gray_render_span          10068470 f   freetype:smooth.obj
 0001:00067508       $LN24                      10068508     freetype:smooth.obj
 0001:00067530       _gray_set_cell             10068530 f   freetype:smooth.obj
 0001:000675b0       _gray_split_cubic          100685b0 f   freetype:smooth.obj
 0001:00067690       _gray_start_cell           10068690 f   freetype:smooth.obj
 0001:000676f0       _gray_sweep                100686f0 f   freetype:smooth.obj
 0001:000677f0       _bdf_cmap_init             100687f0 f   freetype:bdf.obj
 0001:00067820       _bdf_cmap_char_index       10068820 f   freetype:bdf.obj
 0001:00067890       _bdf_cmap_char_next        10068890 f   freetype:bdf.obj
 0001:00067930       _BDF_Face_Done             10068930 f   freetype:bdf.obj
 0001:000679e0       _BDF_Face_Init             100689e0 f   freetype:bdf.obj
 0001:00067f20       _BDF_Size_Select           10068f20 f   freetype:bdf.obj
 0001:00067f60       _BDF_Size_Request          10068f60 f   freetype:bdf.obj
 0001:00068000       _BDF_Glyph_Load            10069000 f   freetype:bdf.obj
 0001:00068120       $LN20                      10069120     freetype:bdf.obj
 0001:00068140       _bdf_get_bdf_property      10069140 f   freetype:bdf.obj
 0001:000681b0       _bdf_get_charset_id        100691b0 f   freetype:bdf.obj
 0001:000681d0       _bdf_driver_requester      100691d0 f   freetype:bdf.obj
 0001:000681f0       __bdf_add_comment          100691f0 f   freetype:bdf.obj
 0001:00068260       __bdf_add_property         10069260 f   freetype:bdf.obj
 0001:00068580       __bdf_atol                 10069580 f   freetype:bdf.obj
 0001:00068690       __bdf_atos                 10069690 f   freetype:bdf.obj
 0001:000687b0       __bdf_atoul                100697b0 f   freetype:bdf.obj
 0001:00068890       __bdf_is_atom              10069890 f   freetype:bdf.obj
 0001:00068980       __bdf_list_done            10069980 f   freetype:bdf.obj
 0001:000689b0       __bdf_list_ensure          100699b0 f   freetype:bdf.obj
 0001:00068a30       __bdf_list_init            10069a30 f   freetype:bdf.obj
 0001:00068a50       __bdf_list_join            10069a50 f   freetype:bdf.obj
 0001:00068ae0       __bdf_list_shift           10069ae0 f   freetype:bdf.obj
 0001:00068b30       __bdf_list_split           10069b30 f   freetype:bdf.obj
 0001:00068d60       __bdf_parse_glyphs         10069d60 f   freetype:bdf.obj
 0001:000696a0       __bdf_parse_properties     1006a6a0 f   freetype:bdf.obj
 0001:000698d0       __bdf_parse_start          1006a8d0 f   freetype:bdf.obj
 0001:0006a010       __bdf_readstream           1006b010 f   freetype:bdf.obj
 0001:0006a220       __bdf_set_default_spacing  1006b220 f   freetype:bdf.obj
 0001:0006a38c       $LN21                      1006b38c     freetype:bdf.obj
 0001:0006a39c       $LN20                      1006b39c     freetype:bdf.obj
 0001:0006a3d0       _bdf_create_property       1006b3d0 f   freetype:bdf.obj
 0001:0006a4d0       _bdf_free_font             1006b4d0 f   freetype:bdf.obj
 0001:0006a700       _bdf_get_font_property     1006b700 f   freetype:bdf.obj
 0001:0006a750       _bdf_get_property          1006b750 f   freetype:bdf.obj
 0001:0006a7a0       _bdf_interpret_style       1006b7a0 f   freetype:bdf.obj
 0001:0006aa20       _bdf_load_font             1006ba20 f   freetype:bdf.obj
 0001:0006ac70       _by_encoding               1006bc70 f   freetype:bdf.obj
 0001:0006aca0       _hash_bucket               1006bca0 f   freetype:bdf.obj
 0001:0006ad50       _hash_free                 1006bd50 f   freetype:bdf.obj
 0001:0006adb0       _hash_init                 1006bdb0 f   freetype:bdf.obj
 0001:0006ae00       _hash_insert               1006be00 f   freetype:bdf.obj
 0001:0006ae90       _hash_lookup               1006be90 f   freetype:bdf.obj
 0001:0006aeb0       _hash_rehash               1006beb0 f   freetype:bdf.obj
 0001:0006b070       _ft_alloc                  1006c070 f   freetype:ftsystem.obj
 0001:0006b080       _ft_ansi_stream_close      1006c080 f   freetype:ftsystem.obj
 0001:0006b0b0       _ft_ansi_stream_io         1006c0b0 f   freetype:ftsystem.obj
 0001:0006b100       _ft_free                   1006c100 f   freetype:ftsystem.obj
 0001:0006b110       _ft_realloc                1006c110 f   freetype:ftsystem.obj
 0001:0006b520       $LN115                     1006c520     freetype:ftbitmap.obj
 0001:0006b524       $LN114                     1006c524     freetype:ftbitmap.obj
 0001:0006b52c       $LN116                     1006c52c     freetype:ftbitmap.obj
 0001:0006b910       $LN75                      1006c910     freetype:ftbitmap.obj
 0001:0006b9c0       _ft_bitmap_assure_buffer   1006c9c0 f   freetype:ftbitmap.obj
 0001:0006bbc8       $LN64                      1006cbc8     freetype:ftbitmap.obj
 0001:0006bbe0       _ft_gray_for_premultiplied_srgb_bgra 1006cbe0 f   freetype:ftbitmap.obj
 0001:0006bf80       _adler32                   1006cf80 f   freetype:ftgzip.obj
 0001:0006c0b0       _ft_gzip_alloc             1006d0b0 f   freetype:ftgzip.obj
 0001:0006c0d0       _ft_gzip_check_header      1006d0d0 f   freetype:ftgzip.obj
 0001:0006c220       _ft_gzip_file_done         1006d220 f   freetype:ftgzip.obj
 0001:0006c280       _ft_gzip_file_fill_input   1006d280 f   freetype:ftgzip.obj
 0001:0006c310       _ft_gzip_file_fill_output  1006d310 f   freetype:ftgzip.obj
 0001:0006c3a0       _ft_gzip_file_init         1006d3a0 f   freetype:ftgzip.obj
 0001:0006c440       _ft_gzip_file_io           1006d440 f   freetype:ftgzip.obj
 0001:0006c4e0       _ft_gzip_file_reset        1006d4e0 f   freetype:ftgzip.obj
 0001:0006c540       _ft_gzip_file_skip_output  1006d540 f   freetype:ftgzip.obj
 0001:0006c590       _ft_gzip_free              1006d590 f   freetype:ftgzip.obj
 0001:0006c5a0       _ft_gzip_get_uncompressed_size 1006d5a0 f   freetype:ftgzip.obj
 0001:0006c5f0       _ft_gzip_stream_close      1006d5f0 f   freetype:ftgzip.obj
 0001:0006c620       _ft_gzip_stream_io         1006d620 f   freetype:ftgzip.obj
 0001:0006c640       _huft_build                1006d640 f   freetype:ftgzip.obj
 0001:0006cb80       _inflate                   1006db80 f   freetype:ftgzip.obj
 0001:0006cee8       $LN54                      1006dee8     freetype:ftgzip.obj
 0001:0006cf20       _inflateEnd                1006df20 f   freetype:ftgzip.obj
 0001:0006cf70       _inflateInit2_             1006df70 f   freetype:ftgzip.obj
 0001:0006d080       _inflateReset              1006e080 f   freetype:ftgzip.obj
 0001:0006d0d0       _inflate_blocks            1006e0d0 f   freetype:ftgzip.obj
 0001:0006da6c       $LN169                     1006ea6c     freetype:ftgzip.obj
 0001:0006da94       $LN170                     1006ea94     freetype:ftgzip.obj
 0001:0006dab0       _inflate_blocks_free       1006eab0 f   freetype:ftgzip.obj
 0001:0006daf0       _inflate_blocks_new        1006eaf0 f   freetype:ftgzip.obj
 0001:0006dba0       _inflate_blocks_reset      1006eba0 f   freetype:ftgzip.obj
 0001:0006dc20       _inflate_codes             1006ec20 f   freetype:ftgzip.obj
 0001:0006e224       $LN107                     1006f224     freetype:ftgzip.obj
 0001:0006e250       _inflate_codes_free        1006f250 f   freetype:ftgzip.obj
 0001:0006e270       _inflate_codes_new         1006f270 f   freetype:ftgzip.obj
 0001:0006e2b0       _inflate_flush             1006f2b0 f   freetype:ftgzip.obj
 0001:0006e3e0       _inflate_trees_bits        1006f3e0 f   freetype:ftgzip.obj
 0001:0006e470       _inflate_trees_dynamic     1006f470 f   freetype:ftgzip.obj
 0001:0006e5a0       _inflate_trees_fixed       1006f5a0 f   freetype:ftgzip.obj
 0001:0006e5d0       _zcalloc                   1006f5d0 f   freetype:ftgzip.obj
 0001:0006e5e0       _zcfree                    1006f5e0 f   freetype:ftgzip.obj
 0001:0006e6a0       _ft_lzw_check_header       1006f6a0 f   freetype:ftlzw.obj
 0001:0006e6f0       _ft_lzw_file_done          1006f6f0 f   freetype:ftlzw.obj
 0001:0006e720       _ft_lzw_file_fill_output   1006f720 f   freetype:ftlzw.obj
 0001:0006e770       _ft_lzw_file_init          1006f770 f   freetype:ftlzw.obj
 0001:0006e7d0       _ft_lzw_file_io            1006f7d0 f   freetype:ftlzw.obj
 0001:0006e8a0       _ft_lzw_file_reset         1006f8a0 f   freetype:ftlzw.obj
 0001:0006e8e0       _ft_lzw_file_skip_output   1006f8e0 f   freetype:ftlzw.obj
 0001:0006e960       _ft_lzw_stream_close       1006f960 f   freetype:ftlzw.obj
 0001:0006e990       _ft_lzw_stream_io          1006f990 f   freetype:ftlzw.obj
 0001:0006ea00       _ft_lzwstate_get_code      1006fa00 f   freetype:ftlzw.obj
 0001:0006ede0       _ft_lzwstate_prefix_grow   1006fde0 f   freetype:ftlzw.obj
 0001:0006ee50       _ft_lzwstate_refill        1006fe50 f   freetype:ftlzw.obj
 0001:0006eef0       _ft_lzwstate_stack_grow    1006fef0 f   freetype:ftlzw.obj
 0001:0006efe0       $$000000                   1006ffe0     MSVCRT:ftol2.obj
 0001:0006eff0       $$000000                   1006fff0     MSVCRT:ftol2.obj
 0001:0006f001       L3B                        10070001     MSVCRT:ftol2.obj
 0001:0006f044       L3F                        10070044     MSVCRT:ftol2.obj
 0001:0006f04c       L40                        1007004c     MSVCRT:ftol2.obj
 0001:0006f05f       L41                        1007005f     MSVCRT:ftol2.obj
 0001:0006f0d0       $$000000                   100700d0     MSVCRT:ftol3.obj
 0001:0006f0ef       _ftol3_default             100700ef     MSVCRT:ftol3.obj
 0001:0006f103       _ftol3_notsafe             10070103     MSVCRT:ftol3.obj
 0001:0006f123       _ftol3_mincheck            10070123     MSVCRT:ftol3.obj
 0001:0006f129       _ftol3_NaN                 10070129     MSVCRT:ftol3.obj
 0001:0006f131       _ftol3_retmin              10070131     MSVCRT:ftol3.obj
 0001:0006f140       $$000000                   10070140     MSVCRT:alloca16.obj
 0001:0006f156       alloca_8                   10070156     MSVCRT:alloca16.obj
 0001:0006f16c       ?dllmain_crt_dispatch@@YGHQAUHINSTANCE__@@KQAX@Z 1007016c f   MSVCRT:dll_dllmain.obj
 0001:0006f1bf       ?dllmain_crt_process_attach@@YAHQAUHINSTANCE__@@QAX@Z 100701bf f   MSVCRT:dll_dllmain.obj
 0001:0006f2c6       ?dllmain_crt_process_detach@@YAH_N@Z 100702c6 f   MSVCRT:dll_dllmain.obj
 0001:0006f376       ?dllmain_dispatch@@YAHQAUHINSTANCE__@@KQAX@Z 10070376 f   MSVCRT:dll_dllmain.obj
 0001:0006f481       ?dllmain_raw@@YGHQAUHINSTANCE__@@KQAX@Z 10070481 f   MSVCRT:dll_dllmain.obj
 0001:0006f4d0       $$000000                   100704d0     MSVCRT:chkstk.obj
 0001:0006f4e4       cs10                       100704e4     MSVCRT:chkstk.obj
 0001:0006f4f2       cs20                       100704f2     MSVCRT:chkstk.obj
 0001:0006f912       ___get_entropy             10070912 f   MSVCRT:gs_support.obj
 0001:0006fa07       ?find_pe_section@@YAPAU_IMAGE_SECTION_HEADER@@QAEI@Z 10070a07 f   MSVCRT:utility.obj
 0001:0006fe60       $$000000                   10070e60     MSVCRT:sehprolg4.obj
 0002:00000298       ?featureMap@@3QBUFeatureMap@@B 10072298     ArabicShaping.obj
 0002:0000e470       ?cacheMap@@3QBKB           10080470     FontInstanceAdapter.obj
 0002:0000e650       ?featureMap@@3QBUFeatureMap@@B 10080650     HanLayoutEngine.obj
 0002:0000e6a8       ?stateTable@@3QAY05$$CBUStateTransition@@A 100806a8     HangulLayoutEngine.obj
 0002:0000e798       ?featureMap@@3QBUFeatureMap@@B 10080798     HangulLayoutEngine.obj
 0002:0000e7f8       ?devaCharClasses@@3QBKB    100807f8     IndicClassTables.obj
 0002:0000e9c0       ?bengCharClasses@@3QBKB    100809c0     IndicClassTables.obj
 0002:0000ebb0       ?punjCharClasses@@3QBKB    10080bb0     IndicClassTables.obj
 0002:0000ed88       ?gujrCharClasses@@3QBKB    10080d88     IndicClassTables.obj
 0002:0000ef48       ?oryaCharClasses@@3QBKB    10080f48     IndicClassTables.obj
 0002:0000f110       ?tamlCharClasses@@3QBKB    10081110     IndicClassTables.obj
 0002:0000f2e0       ?teluCharClasses@@3QBKB    100812e0     IndicClassTables.obj
 0002:0000f4a0       ?kndaCharClasses@@3QBKB    100814a0     IndicClassTables.obj
 0002:0000f660       ?mlymCharClasses@@3QBKB    10081660     IndicClassTables.obj
 0002:0000f820       ?sinhCharClasses@@3QBKB    10081820     IndicClassTables.obj
 0002:0000f9f4       ?bengSplitTable@@3QAY02$$CBGA 100819f4     IndicClassTables.obj
 0002:0000fa00       ?oryaSplitTable@@3QAY02$$CBGA 10081a00     IndicClassTables.obj
 0002:0000fa14       ?tamlSplitTable@@3QAY02$$CBGA 10081a14     IndicClassTables.obj
 0002:0000fa28       ?teluSplitTable@@3QAY02$$CBGA 10081a28     IndicClassTables.obj
 0002:0000fa30       ?kndaSplitTable@@3QAY02$$CBGA 10081a30     IndicClassTables.obj
 0002:0000fa50       ?mlymSplitTable@@3QAY02$$CBGA 10081a50     IndicClassTables.obj
 0002:0000fa64       ?sinhSplitTable@@3QAY02$$CBGA 10081a64     IndicClassTables.obj
 0002:0000fa7c       ?devaClassTable@@3UIndicClassTable@@B 10081a7c     IndicClassTables.obj
 0002:0000fa90       ?bengClassTable@@3UIndicClassTable@@B 10081a90     IndicClassTables.obj
 0002:0000faa4       ?punjClassTable@@3UIndicClassTable@@B 10081aa4     IndicClassTables.obj
 0002:0000fab8       ?gujrClassTable@@3UIndicClassTable@@B 10081ab8     IndicClassTables.obj
 0002:0000facc       ?oryaClassTable@@3UIndicClassTable@@B 10081acc     IndicClassTables.obj
 0002:0000fae0       ?tamlClassTable@@3UIndicClassTable@@B 10081ae0     IndicClassTables.obj
 0002:0000faf4       ?teluClassTable@@3UIndicClassTable@@B 10081af4     IndicClassTables.obj
 0002:0000fb08       ?kndaClassTable@@3UIndicClassTable@@B 10081b08     IndicClassTables.obj
 0002:0000fb1c       ?mlymClassTable@@3UIndicClassTable@@B 10081b1c     IndicClassTables.obj
 0002:0000fb30       ?sinhClassTable@@3UIndicClassTable@@B 10081b30     IndicClassTables.obj
 0002:0000fb48       ?indicClassTables@@3QBQBUIndicClassTable@@B 10081b48     IndicClassTables.obj
 0002:0000fe40       ?featureMap@@3QBUFeatureMap@@B 10081e40     IndicReordering.obj
 0002:0000fec8       ?v2FeatureMap@@3QBUFeatureMap@@B 10081ec8     IndicReordering.obj
 0002:0000ff60       ?stateTable@@3QAY0BA@$$CBCA 10081f60     IndicReordering.obj
 0002:00010080       ?khmerCharClasses@@3QBKB   10082080     KhmerReordering.obj
 0002:00010200       ?khmerClassTable@@3UKhmerClassTable@@B 10082200     KhmerReordering.obj
 0002:00010208       ?featureMap@@3QBUFeatureMap@@B 10082208     KhmerReordering.obj
 0002:00010270       ?khmerStateTable@@3QAY0M@$$CBCA 10082270     KhmerReordering.obj
 0002:00010440       ?canonFeatureMap@@3QBUFeatureMap@@B 10082440     LayoutEngine.obj
 0002:00010f70       ?featureMap@@3QBUFeatureMap@@B 10082f70     OpenTypeLayoutEngine.obj
 0002:00011ab8       ?leftAboveVowels@?1??leftAboveVowel@ThaiShaping@@CAGGE@Z@4QAY06$$CBGA 10083ab8     ThaiShaping.obj
 0002:00011af0       ?lowerRightTones@?1??lowerRightTone@ThaiShaping@@CAGGE@Z@4QAY06$$CBGA 10083af0     ThaiShaping.obj
 0002:00011b28       ?lowerLeftTones@?1??lowerLeftTone@ThaiShaping@@CAGGE@Z@4QAY06$$CBGA 10083b28     ThaiShaping.obj
 0002:00011b60       ?upperLeftTones@?1??upperLeftTone@ThaiShaping@@CAGGE@Z@4QAY06$$CBGA 10083b60     ThaiShaping.obj
 0002:00011b98       ?lowerBelowVowels@?1??lowerBelowVowel@ThaiShaping@@CAGGE@Z@4QAY02$$CBGA 10083b98     ThaiShaping.obj
 0002:00011bb0       ?noDescenderCODs@?1??noDescenderCOD@ThaiShaping@@CAGGE@Z@4QAY03$$CBGA 10083bb0     ThaiShaping.obj
 0002:00012428       ?tibetanCharClasses@@3QBKB 10084428     TibetanReordering.obj
 0002:00012828       ?tibetanClassTable@@3UTibetanClassTable@@B 10084828     TibetanReordering.obj
 0002:00012830       ?featureMap@@3QBUFeatureMap@@B 10084830     TibetanReordering.obj
 0002:000128a0       ?tibetanStateTable@@3QAY0BB@$$CBCA 100848a0     TibetanReordering.obj
 0002:00012a38       ?bitsInNibble@?1??getFieldCount@ValueRecord@@CAFG@Z@4QBFB 10084a38     ValueRecords.obj
 0002:00012a58       ?beforeMasks@?1??getFieldIndex@ValueRecord@@CAFGF@Z@4QBGB 10084a58     ValueRecords.obj
 0002:00012a80       _FONTKEY_NT                10084a80     fontpath.obj
 0002:00012ab4       _FONTKEY_WIN               10084ab4     fontpath.obj
 0002:00012ae4       ?TTSUFFIX@?1??RegistryToBaseTTNameA@@9@9 10084ae4     fontpath.obj
 0002:00012af0       ?OTSUFFIX@?1??RegistryToBaseTTNameA@@9@9 10084af0     fontpath.obj
 0002:00012afc       ?TTSUFFIX@?1??RegistryToBaseTTNameW@@9@9 10084afc     fontpath.obj
 0002:00012b14       ?OTSUFFIX@?1??RegistryToBaseTTNameW@@9@9 10084b14     fontpath.obj
 0002:00012c5c       ?outline_funcs@?1??addToGP@@9@9 10084c5c     freetypeScaler.obj
 0002:00013028       _ft_default_modules        10085028     freetype:ftinit.obj
 0002:000130c0       _ft_trig_arctan_table      100850c0     freetype:ftbase.obj
 0002:00013118       _null_outline              10085118     freetype:ftbase.obj
 0002:000131f4       _bbox_interface            100851f4     freetype:ftbbox.obj
 0002:00013ef8       _af_service_properties     10085ef8     freetype:autofit.obj
 0002:00013f00       _af_services               10085f00     freetype:autofit.obj
 0002:00013f90       ?gvar_fields@?1??ft_var_load_gvar@@9@9 10085f90     freetype:truetype.obj
 0002:00013fb4       ?fvar_fields@?1??TT_Get_MM_Var@@9@9 10085fb4     freetype:truetype.obj
 0002:00013fd8       ?fvaraxis_fields@?1??TT_Get_MM_Var@@9@9 10085fd8     freetype:truetype.obj
 0002:0001409c       _tt_service_properties     1008609c     freetype:truetype.obj
 0002:000140a4       _tt_service_gx_multi_masters 100860a4     freetype:truetype.obj
 0002:000140b8       _tt_service_truetype_engine 100860b8     freetype:truetype.obj
 0002:000140bc       _tt_service_truetype_glyf  100860bc     freetype:truetype.obj
 0002:000140c0       _tt_services               100860c0     freetype:truetype.obj
 0002:000140f0       ?trick_names@?1??tt_check_trickyness_family@@9@9 100860f0     freetype:truetype.obj
 0002:000141a8       ?sfnt_id@?1??tt_check_trickyness_sfnt_ids@@9@9 100861a8     freetype:truetype.obj
 0002:00014340       _Pop_Push_Count            10086340     freetype:truetype.obj
 0002:00014440       _opcode_length             10086440     freetype:truetype.obj
 0002:00014610       _t1_keywords               10086610     freetype:type1.obj
 0002:00014cac       _t1_service_ps_name        10086cac     freetype:type1.obj
 0002:00014d10       _t1_service_glyph_dict     10086d10     freetype:type1.obj
 0002:00014d18       _t1_service_multi_masters  10086d18     freetype:type1.obj
 0002:00014d2c       _t1_service_ps_info        10086d2c     freetype:type1.obj
 0002:00014d40       _t1_service_kerning        10086d40     freetype:type1.obj
 0002:00014d44       _t1_services               10086d44     freetype:type1.obj
 0002:00015020       ?readFromStack@?EP@??cf2_interpT2CharString@@9@9 10087020     freetype:cff.obj
 0002:0001502c       ?readFromStack@?FB@??cf2_interpT2CharString@@9@9 1008702c     freetype:cff.obj
 0002:00015038       ?readFromStack@?FD@??cf2_interpT2CharString@@9@9 10087038     freetype:cff.obj
 0002:00015044       ?readFromStack@?FF@??cf2_interpT2CharString@@9@9 10087044     freetype:cff.obj
 0002:00015100       _cff_service_glyph_dict    10087100     freetype:cff.obj
 0002:00015108       _cff_service_ps_info       10087108     freetype:cff.obj
 0002:0001511c       _cff_service_ps_name       1008711c     freetype:cff.obj
 0002:00015120       _cff_service_get_cmap_info 10087120     freetype:cff.obj
 0002:00015124       _cff_service_cid_info      10087124     freetype:cff.obj
 0002:00015130       _cff_service_properties    10087130     freetype:cff.obj
 0002:00015138       _cff_services              10087138     freetype:cff.obj
 0002:00015178       _power_tens                10087178     freetype:cff.obj
 0002:000151a0       _cff_field_handlers        100871a0     freetype:cff.obj
 0002:00015750       _cff_isoadobe_charset      10087750     freetype:cff.obj
 0002:00015920       _cff_expert_charset        10087920     freetype:cff.obj
 0002:00015a70       _cff_expertsubset_charset  10087a70     freetype:cff.obj
 0002:00015b20       _cff_standard_encoding     10087b20     freetype:cff.obj
 0002:00015d20       _cff_expert_encoding       10087d20     freetype:cff.obj
 0002:00015f20       ?cff_header_fields@?1??cff_font_load@@9@9 10087f20     freetype:cff.obj
 0002:00015fb8       _cid_field_records         10087fb8     freetype:type1cid.obj
 0002:000166e4       _cid_service_ps_name       100886e4     freetype:type1cid.obj
 0002:00016748       _cid_service_ps_info       10088748     freetype:type1cid.obj
 0002:0001675c       _cid_service_cid_info      1008875c     freetype:type1cid.obj
 0002:00016768       _cid_services              10088768     freetype:type1cid.obj
 0002:00016890       _pfr_header_fields         10088890     freetype:pfr.obj
 0002:00016904       _pfr_phy_font_extra_items  10088904     freetype:pfr.obj
 0002:000169c4       _pfr_services              100889c4     freetype:pfr.obj
 0002:000169f0       _t42_keywords              100889f0     freetype:type42.obj
 0002:00016d20       _t42_service_glyph_dict    10088d20     freetype:type42.obj
 0002:00016d28       _t42_service_ps_font_name  10088d28     freetype:type42.obj
 0002:00016d2c       _t42_service_ps_info       10088d2c     freetype:type42.obj
 0002:00016d40       _t42_services              10088d40     freetype:type42.obj
 0002:00016df8       _winmz_header_fields       10088df8     freetype:winfnt.obj
 0002:00016e0c       _winne_header_fields       10088e0c     freetype:winfnt.obj
 0002:00016e24       _winpe32_header_fields     10088e24     freetype:winfnt.obj
 0002:00016e58       _winpe32_section_fields    10088e58     freetype:winfnt.obj
 0002:00016e78       _winpe_rsrc_dir_fields     10088e78     freetype:winfnt.obj
 0002:00016e98       _winpe_rsrc_dir_entry_fields 10088e98     freetype:winfnt.obj
 0002:00016ea8       _winpe_rsrc_data_entry_fields 10088ea8     freetype:winfnt.obj
 0002:00016ec0       _winfnt_header_fields      10088ec0     freetype:winfnt.obj
 0002:00016f58       _fnt_cmap_class_rec        10088f58     freetype:winfnt.obj
 0002:00016f80       _fnt_cmap_class            10088f80     freetype:winfnt.obj
 0002:00016f84       _winfnt_service_rec        10088f84     freetype:winfnt.obj
 0002:00016f88       _winfnt_services           10088f88     freetype:winfnt.obj
 0002:00016fd0       _pcf_toc_header            10088fd0     freetype:pcf.obj
 0002:00016fe0       _pcf_table_header          10088fe0     freetype:pcf.obj
 0002:00016ff8       _pcf_metric_header         10088ff8     freetype:pcf.obj
 0002:00017018       _pcf_metric_msb_header     10089018     freetype:pcf.obj
 0002:00017038       _pcf_compressed_metric_header 10089038     freetype:pcf.obj
 0002:00017054       _pcf_property_header       10089054     freetype:pcf.obj
 0002:00017068       _pcf_property_msb_header   10089068     freetype:pcf.obj
 0002:0001707c       _pcf_accel_header          1008907c     freetype:pcf.obj
 0002:000170b0       _pcf_accel_msb_header      100890b0     freetype:pcf.obj
 0002:00017170       _pcf_service_bdf           10089170     freetype:pcf.obj
 0002:00017178       _pcf_services              10089178     freetype:pcf.obj
 0002:00017394       _psaux_interface           10089394     freetype:psaux.obj
 0002:000173d8       _t1_args_count             100893d8     freetype:psaux.obj
 0002:00017448       _afm_key_table             10089448     freetype:psaux.obj
 0002:00017570       _ft_char_table             10089570     freetype:psaux.obj
 0002:00017880       _ft_standard_glyph_names   10089880     freetype:psmodule.obj
 0002:000186f0       _ft_mac_names              1008a6f0     freetype:psmodule.obj
 0002:000188f8       _ft_sid_names              1008a8f8     freetype:psmodule.obj
 0002:00018c08       _t1_standard_encoding      1008ac08     freetype:psmodule.obj
 0002:00018e08       _t1_expert_encoding        1008ae08     freetype:psmodule.obj
 0002:00019008       _ft_adobe_glyph_list       1008b008     freetype:psmodule.obj
 0002:00026ac8       _ft_extra_glyph_unicodes   10098ac8     freetype:psmodule.obj
 0002:00026af0       _ft_extra_glyph_names      10098af0     freetype:psmodule.obj
 0002:00026b48       _ft_extra_glyph_name_offsets 10098b48     freetype:psmodule.obj
 0002:00026b70       _pscmaps_interface         10098b70     freetype:psmodule.obj
 0002:00026b90       _pscmaps_services          10098b90     freetype:psmodule.obj
 0002:00026ba8       _pshinter_interface        10098ba8     freetype:pshinter.obj
 0002:00026ce0       _tt_cmap_classes           10098ce0     freetype:sfnt.obj
 0002:00026d08       ?tt_encodings@?1??sfnt_find_encoding@@9@9 10098d08     freetype:sfnt.obj
 0002:00026d8c       ?woff_header_fields@?1??woff_open_font@@9@9 10098d8c     freetype:sfnt.obj
 0002:00026dc8       ?ttc_header_fields@?1??sfnt_open_font@@9@9 10098dc8     freetype:sfnt.obj
 0002:00026dfc       _sfnt_service_sfnt_table   10098dfc     freetype:sfnt.obj
 0002:00026e08       _sfnt_service_glyph_dict   10098e08     freetype:sfnt.obj
 0002:00026e10       _sfnt_service_ps_name      10098e10     freetype:sfnt.obj
 0002:00026e14       _tt_service_get_cmap_info  10098e14     freetype:sfnt.obj
 0002:00026e18       _sfnt_service_bdf          10098e18     freetype:sfnt.obj
 0002:00026e20       _sfnt_services             10098e20     freetype:sfnt.obj
 0002:00026e50       _sfnt_interface            10098e50     freetype:sfnt.obj
 0002:00026ec4       ?table_dir_entry_fields@?1??check_table_dir@@9@9 10098ec4     freetype:sfnt.obj
 0002:00026edc       ?offset_table_fields@?1??tt_face_load_font_dir@@9@9 10098edc     freetype:sfnt.obj
 0002:00026ef8       ?header_fields@?1??tt_face_load_generic_header@@9@9 10098ef8     freetype:sfnt.obj
 0002:00026f4c       ?maxp_fields@?1??tt_face_load_maxp@@9@9 10098f4c     freetype:sfnt.obj
 0002:00026f5c       ?maxp_fields_extra@?1??tt_face_load_maxp@@9@9 10098f5c     freetype:sfnt.obj
 0002:00026f98       ?name_table_fields@?1??tt_face_load_name@@9@9 10098f98     freetype:sfnt.obj
 0002:00026fac       ?name_record_fields@?1??tt_face_load_name@@9@9 10098fac     freetype:sfnt.obj
 0002:00026fc8       ?os2_fields@?1??tt_face_load_os2@@9@9 10098fc8     freetype:sfnt.obj
 0002:00027078       ?os2_fields_extra1@?1??tt_face_load_os2@@9@9 10099078     freetype:sfnt.obj
 0002:00027088       ?os2_fields_extra2@?1??tt_face_load_os2@@9@9 10099088     freetype:sfnt.obj
 0002:000270a4       ?os2_fields_extra5@?1??tt_face_load_os2@@9@9 100990a4     freetype:sfnt.obj
 0002:000270b4       ?post_fields@?1??tt_face_load_post@@9@9 100990b4     freetype:sfnt.obj
 0002:000270e0       ?pclt_fields@?1??tt_face_load_pclt@@9@9 100990e0     freetype:sfnt.obj
 0002:00027128       ?metrics_header_fields@?1??tt_face_load_hhea@@9@9 10099128     freetype:sfnt.obj
 0002:000272f8       _func_interface            100992f8     freetype:smooth.obj
 0002:000273e8       __bdf_opts                 100993e8     freetype:bdf.obj
 0002:000273f8       __bdf_properties           100993f8     freetype:bdf.obj
 0002:00027928       __num_bdf_properties       10099928     freetype:bdf.obj
 0002:0002792c       _empty                     1009992c     freetype:bdf.obj
 0002:00027930       _a2i                       10099930     freetype:bdf.obj
 0002:000279b0       _odigits                   100999b0     freetype:bdf.obj
 0002:000279d0       _ddigits                   100999d0     freetype:bdf.obj
 0002:000279f0       _hdigits                   100999f0     freetype:bdf.obj
 0002:00027a10       _nibble_mask               10099a10     freetype:bdf.obj
 0002:00027aa0       _bdf_service_bdf           10099aa0     freetype:bdf.obj
 0002:00027aa8       _bdf_services              10099aa8     freetype:bdf.obj
 0002:00028014       _null_bitmap               1009a014     freetype:ftbitmap.obj
 0002:00028030       _cplens                    1009a030     freetype:ftgzip.obj
 0002:000280b0       _cplext                    1009a0b0     freetype:ftgzip.obj
 0002:00028130       _cpdist                    1009a130     freetype:ftgzip.obj
 0002:000281a8       _cpdext                    1009a1a8     freetype:ftgzip.obj
 0002:00028220       _fixed_tl                  1009a220     freetype:ftgzip.obj
 0002:00029220       _fixed_td                  1009b220     freetype:ftgzip.obj
 0002:00029320       _inflate_mask              1009b320     freetype:ftgzip.obj
 0002:00029368       _border                    1009b368     freetype:ftgzip.obj
 0002:000295d0       two32                      1009b5d0     MSVCRT:ftol2.obj
 0002:000295d4       two63                      1009b5d4     MSVCRT:ftol2.obj
 0002:000295d8       _NaN                       1009b5d8     MSVCRT:ftol2.obj
 0002:000295f0       _bias_low                  1009b5f0     MSVCRT:ftol3.obj
 0002:00029600       _bias_high                 1009b600     MSVCRT:ftol3.obj
 0002:00029610       _DP2to32                   1009b610     MSVCRT:ftol3.obj
 0002:00029618       _NaN                       1009b618     MSVCRT:ftol3.obj
 0002:0002961c       _onept5                    1009b61c     MSVCRT:ftol3.obj
 0002:00029684       _GS_ExceptionPointers      1009b684     MSVCRT:gs_report.obj
 0002:0002af90       __sehtable$?dllmain_crt_process_attach@@YAHQAUHINSTANCE__@@QAX@Z 1009cf90     MSVCRT:dll_dllmain.obj
 0002:0002afb0       __sehtable$?dllmain_crt_process_detach@@YAH_N@Z 1009cfb0     MSVCRT:dll_dllmain.obj
 0002:0002afd8       __sehtable$?dllmain_dispatch@@YAHQAUHINSTANCE__@@KQAX@Z 1009cfd8     MSVCRT:dll_dllmain.obj
 0002:0002b088       __sehtable$___scrt_is_nonwritable_in_current_image 1009d088     MSVCRT:utility.obj
 0002:0002b0b0       .edata                     1009d0b0     fontmanager.exp
 0002:0002b0d8       rgpv                       1009d0d8     fontmanager.exp
 0002:0002b170       rgszName                   1009d170     fontmanager.exp
 0002:0002b208       rgwOrd                     1009d208     fontmanager.exp
 0002:0002b254       szName                     1009d254     fontmanager.exp
 0002:0002b264       $N00001                    1009d264     fontmanager.exp
 0002:0002b292       $N00002                    1009d292     fontmanager.exp
 0002:0002b2cd       $N00003                    1009d2cd     fontmanager.exp
 0002:0002b309       $N00004                    1009d309     fontmanager.exp
 0002:0002b334       $N00005                    1009d334     fontmanager.exp
 0002:0002b373       $N00006                    1009d373     fontmanager.exp
 0002:0002b3ac       $N00007                    1009d3ac     fontmanager.exp
 0002:0002b3e6       $N00008                    1009d3e6     fontmanager.exp
 0002:0002b421       $N00009                    1009d421     fontmanager.exp
 0002:0002b459       $N00010                    1009d459     fontmanager.exp
 0002:0002b492       $N00011                    1009d492     fontmanager.exp
 0002:0002b4cd       $N00012                    1009d4cd     fontmanager.exp
 0002:0002b50e       $N00013                    1009d50e     fontmanager.exp
 0002:0002b549       $N00014                    1009d549     fontmanager.exp
 0002:0002b582       $N00015                    1009d582     fontmanager.exp
 0002:0002b5c3       $N00016                    1009d5c3     fontmanager.exp
 0002:0002b602       $N00017                    1009d602     fontmanager.exp
 0002:0002b641       $N00018                    1009d641     fontmanager.exp
 0002:0002b679       $N00019                    1009d679     fontmanager.exp
 0002:0002b6b2       $N00020                    1009d6b2     fontmanager.exp
 0002:0002b6df       $N00021                    1009d6df     fontmanager.exp
 0002:0002b715       $N00022                    1009d715     fontmanager.exp
 0002:0002b744       $N00023                    1009d744     fontmanager.exp
 0002:0002b779       $N00024                    1009d779     fontmanager.exp
 0002:0002b7a5       $N00025                    1009d7a5     fontmanager.exp
 0002:0002b7d2       $N00026                    1009d7d2     fontmanager.exp
 0002:0002b7ff       $N00027                    1009d7ff     fontmanager.exp
 0002:0002b82d       $N00028                    1009d82d     fontmanager.exp
 0002:0002b864       $N00029                    1009d864     fontmanager.exp
 0002:0002b88c       $N00030                    1009d88c     fontmanager.exp
 0002:0002b8b7       $N00031                    1009d8b7     fontmanager.exp
 0002:0002b8e6       $N00032                    1009d8e6     fontmanager.exp
 0002:0002b920       $N00033                    1009d920     fontmanager.exp
 0002:0002b95c       $N00034                    1009d95c     fontmanager.exp
 0002:0002b992       $N00035                    1009d992     fontmanager.exp
 0002:0002b9a7       $N00036                    1009d9a7     fontmanager.exp
 0002:0002b9b5       $N00037                    1009d9b5     fontmanager.exp
 0002:0002b9c9       $N00038                    1009d9c9     fontmanager.exp
 0002:0002bd5a       .idata$6                   1009dd5a     java:java.dll
 0002:0002bdca       .idata$6                   1009ddca     advapi32:ADVAPI32.dll
 0002:0002be32       .idata$6                   1009de32     user32:USER32.dll
 0002:0002bf6c       .idata$6                   1009df6c     gdi32:GDI32.dll
 0002:0002c07a       .idata$6                   1009e07a     awt:awt.dll
 0002:0002c1f2       .idata$6                   1009e1f2     kernel32:KERNEL32.dll
 0002:0002c2f4       .idata$6                   1009e2f4     vcruntime:VCRUNTIME140.dll
 0002:0002c4a4       .idata$6                   1009e4a4     ucrt:api-ms-win-crt-heap-l1-1-0.dll
 0002:0002c4c4       .idata$6                   1009e4c4     ucrt:api-ms-win-crt-math-l1-1-0.dll
 0002:0002c4e4       .idata$6                   1009e4e4     ucrt:api-ms-win-crt-environment-l1-1-0.dll
 0002:0002c50a       .idata$6                   1009e50a     ucrt:api-ms-win-crt-string-l1-1-0.dll
 0002:0002c52c       .idata$6                   1009e52c     ucrt:api-ms-win-crt-utility-l1-1-0.dll
 0002:0002c54e       .idata$6                   1009e54e     ucrt:api-ms-win-crt-convert-l1-1-0.dll
 0002:0002c570       .idata$6                   1009e570     ucrt:api-ms-win-crt-stdio-l1-1-0.dll
 0002:0002c590       .idata$6                   1009e590     ucrt:api-ms-win-crt-runtime-l1-1-0.dll
 0003:00000200       ?gvdClassName@@3PBDB       1009f200     SunLayoutEngine.obj
 0003:00000a80       ?z@?1??getStaticClassID@ArabicOpenTypeLayoutEngine@@SAPBDXZ@4DA 1009fa80     ArabicLayoutEngine.obj
 0003:00000a81       ?z@?1??getStaticClassID@ContextualGlyphInsertionProcessor2@@SAPBDXZ@4DA 1009fa81     ContextualGlyphInsertionProc2.obj
 0003:00000a82       ?z@?1??getStaticClassID@ContextualGlyphSubstitutionProcessor@@SAPBDXZ@4DA 1009fa82     ContextualGlyphSubstProc.obj
 0003:00000a83       ?z@?1??getStaticClassID@ContextualGlyphSubstitutionProcessor2@@SAPBDXZ@4DA 1009fa83     ContextualGlyphSubstProc2.obj
 0003:00000a84       ?z@?1??getStaticClassID@GXLayoutEngine@@SAPBDXZ@4DA 1009fa84     GXLayoutEngine.obj
 0003:00000a85       ?z@?1??getStaticClassID@GXLayoutEngine2@@SAPBDXZ@4DA 1009fa85     GXLayoutEngine2.obj
 0003:00000a86       ?z@?1??getStaticClassID@HanOpenTypeLayoutEngine@@SAPBDXZ@4DA 1009fa86     HanLayoutEngine.obj
 0003:00000a87       ?z@?1??getStaticClassID@HangulOpenTypeLayoutEngine@@SAPBDXZ@4DA 1009fa87     HangulLayoutEngine.obj
 0003:00000a88       ?z@?1??getStaticClassID@IndicOpenTypeLayoutEngine@@SAPBDXZ@4DA 1009fa88     IndicLayoutEngine.obj
 0003:00000a89       ?z@?1??getStaticClassID@IndicRearrangementProcessor@@SAPBDXZ@4DA 1009fa89     IndicRearrangementProcessor.obj
 0003:00000a8a       ?z@?1??getStaticClassID@IndicRearrangementProcessor2@@SAPBDXZ@4DA 1009fa8a     IndicRearrangementProcessor2.obj
 0003:00000a8b       ?z@?1??getStaticClassID@KhmerOpenTypeLayoutEngine@@SAPBDXZ@4DA 1009fa8b     KhmerLayoutEngine.obj
 0003:00000a8c       ?z@?1??getStaticClassID@LEFontInstance@@SAPBDXZ@4DA 1009fa8c     LEFontInstance.obj
 0003:00000a8d       ?z@?1??getStaticClassID@LEGlyphStorage@@SAPBDXZ@4DA 1009fa8d     LEGlyphStorage.obj
 0003:00000a8e       ?z@?1??getStaticClassID@LEInsertionList@@SAPBDXZ@4DA 1009fa8e     LEInsertionList.obj
 0003:00000a8f       ?z@?1??getStaticClassID@LayoutEngine@@SAPBDXZ@4DA 1009fa8f     LayoutEngine.obj
 0003:00000a90       ?z@?1??getStaticClassID@LigatureSubstitutionProcessor@@SAPBDXZ@4DA 1009fa90     LigatureSubstProc.obj
 0003:00000a91       ?z@?1??getStaticClassID@LigatureSubstitutionProcessor2@@SAPBDXZ@4DA 1009fa91     LigatureSubstProc2.obj
 0003:00000a92       ?z@?1??getStaticClassID@OpenTypeLayoutEngine@@SAPBDXZ@4DA 1009fa92     OpenTypeLayoutEngine.obj
 0003:00000a93       ?z@?1??getStaticClassID@SegmentArrayProcessor@@SAPBDXZ@4DA 1009fa93     SegmentArrayProcessor.obj
 0003:00000a94       ?z@?1??getStaticClassID@SegmentArrayProcessor2@@SAPBDXZ@4DA 1009fa94     SegmentArrayProcessor2.obj
 0003:00000a95       ?z@?1??getStaticClassID@SegmentSingleProcessor@@SAPBDXZ@4DA 1009fa95     SegmentSingleProcessor.obj
 0003:00000a96       ?z@?1??getStaticClassID@SegmentSingleProcessor2@@SAPBDXZ@4DA 1009fa96     SegmentSingleProcessor2.obj
 0003:00000a97       ?z@?1??getStaticClassID@SimpleArrayProcessor@@SAPBDXZ@4DA 1009fa97     SimpleArrayProcessor.obj
 0003:00000a98       ?z@?1??getStaticClassID@SimpleArrayProcessor2@@SAPBDXZ@4DA 1009fa98     SimpleArrayProcessor2.obj
 0003:00000a99       ?z@?1??getStaticClassID@SingleTableProcessor@@SAPBDXZ@4DA 1009fa99     SingleTableProcessor.obj
 0003:00000a9a       ?z@?1??getStaticClassID@SingleTableProcessor2@@SAPBDXZ@4DA 1009fa9a     SingleTableProcessor2.obj
 0003:00000a9c       ?gvdClass@@3PAV_jclass@@A  1009fa9c     SunLayoutEngine.obj
 0003:00000aa0       ?gvdCountFID@@3PAU_jfieldID@@A 1009faa0     SunLayoutEngine.obj
 0003:00000aa4       ?gvdFlagsFID@@3PAU_jfieldID@@A 1009faa4     SunLayoutEngine.obj
 0003:00000aa8       ?gvdGlyphsFID@@3PAU_jfieldID@@A 1009faa8     SunLayoutEngine.obj
 0003:00000aac       ?gvdPositionsFID@@3PAU_jfieldID@@A 1009faac     SunLayoutEngine.obj
 0003:00000ab0       ?gvdIndicesFID@@3PAU_jfieldID@@A 1009fab0     SunLayoutEngine.obj
 0003:00000ab4       ?z@?1??getStaticClassID@ThaiLayoutEngine@@SAPBDXZ@4DA 1009fab4     ThaiLayoutEngine.obj
 0003:00000ab5       ?z@?1??getStaticClassID@TibetanOpenTypeLayoutEngine@@SAPBDXZ@4DA 1009fab5     TibetanLayoutEngine.obj
 0003:00000ab6       ?z@?1??getStaticClassID@TrimmedArrayProcessor@@SAPBDXZ@4DA 1009fab6     TrimmedArrayProcessor.obj
 0003:00000ab7       ?z@?1??getStaticClassID@TrimmedArrayProcessor2@@SAPBDXZ@4DA 1009fab7     TrimmedArrayProcessor2.obj
 0003:00000ab8       _UNICODE_OS                1009fab8     fontpath.obj
 0003:00000abc       _screenDC                  1009fabc     fontpath.obj
 0003:00000ac0       _invalidateScalerMID       1009fac0     freetypeScaler.obj
 0003:00000ac8       _igLUTable                 1009fac8     lcdglyph.obj
 0003:00000cac       _theNullScalerContext      1009fcac     sunFont.obj
 0003:00000cb0       _initialisedFontIDs        1009fcb0     sunFont.obj
 0003:00000cb4       ?__proc_attached@@3HA      1009fcb4     MSVCRT:dll_dllmain.obj
 0003:00000cc0       _GS_ExceptionRecord        1009fcc0     MSVCRT:gs_report.obj
 0003:00000d10       _GS_ContextRecord          1009fd10     MSVCRT:gs_report.obj
 0003:00000ff8       ?is_initialized_as_dll@@3_NA 1009fff8     MSVCRT:utility.obj
 0003:00000ff9       ?module_local_atexit_table_initialized@@3_NA 1009fff9     MSVCRT:utility.obj
 0003:00000ffc       ?module_local_atexit_table@@3U_onexit_table_t@@A 1009fffc     MSVCRT:utility.obj
 0003:00001008       ?module_local_at_quick_exit_table@@3U_onexit_table_t@@A 100a0008     MSVCRT:utility.obj
 0004:00000060       $R000000                   100a1060     fontmanager.dll.res
